 EMenu

 Timestamp is 57a0e2bb (Tue Aug  2 21:13:15 2016)

 Preferred load address is 0000000180000000

 Start         Length     Name                   Class
 0001:00000000 00000010H .00cfg                  CODE
 0001:00000010 00000008H .CRT$XCA                CODE
 0001:00000018 00000008H .CRT$XCZ                CODE
 0001:00000020 00000008H .CRT$XIA                CODE
 0001:00000028 00000018H .CRT$XIC                CODE
 0001:00000040 00000008H .CRT$XIZ                CODE
 0001:00000048 00000008H .CRT$XPA                CODE
 0001:00000050 00000010H .CRT$XPX                CODE
 0001:00000060 00000008H .CRT$XPXA               CODE
 0001:00000068 00000008H .CRT$XPZ                CODE
 0001:00000070 00000008H .CRT$XTA                CODE
 0001:00000078 00000008H .CRT$XTZ                CODE
 0001:00000080 000075e8H .rdata                  CODE
 0001:00007668 000001f8H .rdata$r                CODE
 0001:00007860 00000010H .rdata$zETW0            CODE
 0001:00007870 00000077H .rdata$zETW1            CODE
 0001:000078e7 0000002cH .rdata$zETW2            CODE
 0001:00007913 00000001H .rdata$zETW9            CODE
 0001:00007914 0000034cH .rdata$zzzdbg           CODE
 0001:00007c60 00000008H .rtc$IAA                CODE
 0001:00007c68 00000008H .rtc$IZZ                CODE
 0001:00007c70 00000008H .rtc$TAA                CODE
 0001:00007c78 00000008H .rtc$TZZ                CODE
 0001:00007c80 000001e0H .text                   CODE
 0001:00007e60 00010dd0H .text$mn                CODE
 0001:00018c30 00000020H .text$mn$00             CODE
 0001:00018c50 00000260H .text$x                 CODE
 0001:00018eb0 00001050H .xdata                  CODE
 0001:00019f00 00000150H .xdata$x                CODE
 0001:0001a050 000000b6H .edata                  CODE
 0002:00000000 00000980H .data                   DATA
 0002:00000980 000000d0H .data$r                 DATA
 0002:00000a50 00001a38H .bss                    DATA
 0003:00000000 000013b0H .pdata                  DATA
 0004:00000000 000003c0H .idata$5                DATA
 0004:000003c0 00000064H .idata$2                DATA
 0004:00000424 00000014H .idata$3                DATA
 0004:00000438 000003c0H .idata$4                DATA
 0004:000007f8 00000872H .idata$6                DATA
 0005:00000000 00000080H .gfids$x                DATA
 0005:00000080 00000040H .gfids$y                DATA
 0006:00000000 000000a0H .rsrc$01                DATA
 0006:000000a0 000003a0H .rsrc$02                DATA

  Address         Publics by Value              Rva+Base               Lib:Object

 0000:00000000       __guard_iat_count          0000000000000000     <absolute>
 0000:00000000       __dynamic_value_reloc_table 0000000000000000     <absolute>
 0000:00000000       __guard_iat_table          0000000000000000     <absolute>
 0000:00000000       __guard_longjmp_table      0000000000000000     <absolute>
 0000:00000000       __guard_longjmp_count      0000000000000000     <absolute>
 0000:00000000       __guard_fids_count         0000000000000000     <absolute>
 0000:00000000       ___safe_se_handler_table   0000000000000000     <absolute>
 0000:00000000       ___safe_se_handler_count   0000000000000000     <absolute>
 0000:00000000       __guard_fids_table         0000000000000000     <absolute>
 0000:00000100       __guard_flags              0000000000000100     <absolute>
 0000:00000000       __ImageBase                0000000180000000     <linker-defined>
 0001:00000000       __guard_check_icall_fptr   0000000180001000     LIBCMT:guard_support.obj
 0001:00000008       __guard_dispatch_icall_fptr 0000000180001008     LIBCMT:guard_support.obj
 0001:00000010       __xc_a                     0000000180001010     LIBCMT:initializers.obj
 0001:00000018       __xc_z                     0000000180001018     LIBCMT:initializers.obj
 0001:00000020       __xi_a                     0000000180001020     LIBCMT:initializers.obj
 0001:00000028       __acrt_multibyte_initializer 0000000180001028     libucrt:multibyte_initializer.obj
 0001:00000030       __acrt_stdio_initializer   0000000180001030     libucrt:stdio_initializer.obj
 0001:00000038       __acrt_tran_fma3_initializer 0000000180001038     libucrt:fma3_initializer.obj
 0001:00000040       __xi_z                     0000000180001040     LIBCMT:initializers.obj
 0001:00000048       __xp_a                     0000000180001048     LIBCMT:initializers.obj
 0001:00000050       __acrt_locale_terminator   0000000180001050     libucrt:locale_initializer.obj
 0001:00000058       __dcrt_console_output_terminator 0000000180001058     libucrt:console_output_initializer.obj
 0001:00000060       __acrt_stdio_terminator    0000000180001060     libucrt:stdio_initializer.obj
 0001:00000068       __xp_z                     0000000180001068     LIBCMT:initializers.obj
 0001:00000070       __xt_a                     0000000180001070     LIBCMT:initializers.obj
 0001:00000078       __xt_z                     0000000180001078     LIBCMT:initializers.obj
 0001:00000080       MainGuid                   0000000180001080     EMenu.obj
 0001:00000090       MenuGuid                   0000000180001090     EMenu.obj
 0001:000000a0       DialogGuid                 00000001800010a0     EMenu.obj
 0001:000000b0       GuiTextMenuGuid            00000001800010b0     EMenu.obj
 0001:000000c0       ??_C@_1M@LBLKOFDL@?$AAE?$AAM?$AAe?$AAn?$AAu?$AA?$AA@ 00000001800010c0     EMenu.obj
 0001:000000d0       ??_C@_1DK@JMMNGKID@?$AAE?$AAM?$AAe?$AAn?$AAu?$AA?5?$AAP?$AAl?$AAu?$AAg?$AAi?$AAn?$AA?5?$AAf?$AAo?$AAr?$AA?5?$AAF?$AAa?$AAr?$AA?5?$AAM?$AAa?$AAn?$AAa?$AAg?$AAe?$AAr?$AA?$AA@ 00000001800010d0     EMenu.obj
 0001:00000110       ??_C@_1DE@BGKMIKPD@?$AAE?$AAu?$AAg?$AAe?$AAn?$AAe?$AA?5?$AAR?$AAo?$AAs?$AAh?$AAa?$AAl?$AA?5?$AA?$CG?$AA?5?$AAF?$AAa?$AAr?$AA?5?$AAG?$AAr?$AAo?$AAu?$AAp?$AA?$AA@ 0000000180001110     EMenu.obj
 0001:00000148       ??_C@_17CIEOGNAD@?$AA?5?$AA?5?$CF?$LK?$AA?$AA@ 0000000180001148     FarMenu.obj
 0001:00000150       ??_C@_13HOIJIPNN@?$AA?5?$AA?$AA@ 0000000180001150     FarMenu.obj
 0001:00000158       ??_C@_19JPHCGFBO@?$AAM?$AAa?$AAi?$AAn?$AA?$AA@ 0000000180001158     Plugin.obj
 0001:00000168       ??_C@_1O@BJPKKLLM@?$AAC?$AAo?$AAn?$AAf?$AAi?$AAg?$AA?$AA@ 0000000180001168     Plugin.obj
 0001:00000178       ??_C@_1BO@CLHFIDDE@?$AAC?$AAh?$AAo?$AAo?$AAs?$AAe?$AAM?$AAe?$AAn?$AAu?$AAT?$AAy?$AAp?$AAe?$AA?$AA@ 0000000180001178     Plugin.obj
 0001:00000198       ??_C@_1BI@GILJGMBA@?$AAC?$AAo?$AAn?$AAt?$AAe?$AAx?$AAt?$AAM?$AAe?$AAn?$AAu?$AA?$AA@ 0000000180001198     Plugin.obj
 0001:000001b0       ??_C@_1O@MCPHAIFL@?$AAM?$AAy?$AAC?$AAo?$AAm?$AAp?$AA?$AA@ 00000001800011b0     Plugin.obj
 0001:000001c0       ??_C@_1O@GOJJLDBG@?$AAE?$AAr?$AAr?$AAo?$AAr?$AA0?$AA?$AA@ 00000001800011c0     Plugin.obj
 0001:000001d0       ??_C@_1O@NGCFNEHD@?$AAE?$AAr?$AAr?$AAo?$AAr?$AA1?$AA?$AA@ 00000001800011d0     Plugin.obj
 0001:000001e0       ??_C@_1O@MEJAHLJN@?$AAE?$AAr?$AAr?$AAo?$AAr?$AA2?$AA?$AA@ 00000001800011e0     Plugin.obj
 0001:000001f0       ??_C@_1M@IAIJHCCH@?$AAC?$AAl?$AAo?$AAs?$AAe?$AA?$AA@ 00000001800011f0     Plugin.obj
 0001:00000200       ??_7?$DialogItemBinding@UFarDialogItem@@@@6B@ 0000000180001200     Plugin.obj
 0001:00000210       ??_7PluginCheckBoxBinding@@6B@ 0000000180001210     Plugin.obj
 0001:00000220       ??_7PluginRadioButtonBinding@@6B@ 0000000180001220     Plugin.obj
 0001:00000230       ??_7PluginIntEditFieldBinding@@6B@ 0000000180001230     Plugin.obj
 0001:00000240       ??_C@_15EFLNJKHH@?$AA?$CF?$AAu?$AA?$AA@ 0000000180001240     Plugin.obj
 0001:00000248       ??_7PluginUIntEditFieldBinding@@6B@ 0000000180001248     Plugin.obj
 0001:00000258       ??_7?$DialogBuilderBase@UFarDialogItem@@@@6B@ 0000000180001258     Plugin.obj
 0001:000002a0       ??_7PluginDialogBuilder@@6B@ 00000001800012a0     Plugin.obj
 0001:000002e8       ??_C@_11LOCGONAA@?$AA?$AA@ 00000001800012e8     Plugin.obj
 0001:000002f0       _GUID_000214f4_0000_0000_c000_000000000046 00000001800012f0     Plugin.obj
 0001:00000300       _GUID_bcfce0a0_ec17_11d0_8d10_00a0c90f2719 0000000180001300     Plugin.obj
 0001:00000310       ??_C@_1BO@BLHAFJIH@?$AAW?$AAa?$AAi?$AAt?$AAT?$AAo?$AAC?$AAo?$AAn?$AAt?$AAi?$AAn?$AAu?$AAe?$AA?$AA@ 0000000180001310     Plugin.obj
 0001:00000330       ??_C@_1O@HAPBPKPP@?$AAU?$AAs?$AAe?$AAG?$AAU?$AAI?$AA?$AA@ 0000000180001330     Plugin.obj
 0001:00000340       ??_C@_1BI@FNELDPIH@?$AAD?$AAe?$AAl?$AAU?$AAs?$AAi?$AAn?$AAg?$AAF?$AAa?$AAr?$AA?$AA@ 0000000180001340     Plugin.obj
 0001:00000358       ??_C@_1BO@ELNGBDOB@?$AAC?$AAl?$AAe?$AAa?$AAr?$AAS?$AAe?$AAl?$AAe?$AAc?$AAt?$AAi?$AAo?$AAn?$AA?$AA@ 0000000180001358     Plugin.obj
 0001:00000378       ??_C@_1O@EFKGCNCH@?$AAS?$AAi?$AAl?$AAe?$AAn?$AAt?$AA?$AA@ 0000000180001378     Plugin.obj
 0001:00000388       ??_C@_1BC@JAMHBCOF@?$AAH?$AAe?$AAl?$AAp?$AAt?$AAe?$AAx?$AAt?$AA?$AA@ 0000000180001388     Plugin.obj
 0001:000003a0       ??_C@_1BM@JNPKPLGJ@?$AAD?$AAi?$AAf?$AAf?$AAe?$AAr?$AAe?$AAn?$AAt?$AAO?$AAn?$AAl?$AAy?$AA?$AA@ 00000001800013a0     Plugin.obj
 0001:000003c0       ??_C@_1O@EOCFEDGM@?$AAG?$AAu?$AAi?$AAP?$AAo?$AAs?$AA?$AA@ 00000001800013c0     Plugin.obj
 0001:000003d0       ??_C@_1FE@DFGJMLLI@?$AAr?$AAc?$AAl?$AAk?$AA?3?$AAr?$AAc?$AAl?$AAk?$AA_?$AAt?$AAx?$AAt?$AA?3?$AAr?$AAc?$AAl?$AAk?$AA_?$AAg?$AAu?$AAi?$AA?3?$AAr?$AAc?$AAl?$AAk?$AA_?$AAc?$AAm?$AAd?$AA?3@ 00000001800013d0     Plugin.obj
 0001:00000428       ??_C@_1M@MGKMLCA@?$AAr?$AAc?$AAl?$AAk?$AA?3?$AA?$AA@ 0000000180001428     Plugin.obj
 0001:00000438       ??_C@_1BE@GEDAILNH@?$AAr?$AAc?$AAl?$AAk?$AA_?$AAt?$AAx?$AAt?$AA?3?$AA?$AA@ 0000000180001438     Plugin.obj
 0001:00000450       ??_C@_1BE@IMOELFKI@?$AAr?$AAc?$AAl?$AAk?$AA_?$AAg?$AAu?$AAi?$AA?3?$AA?$AA@ 0000000180001450     Plugin.obj
 0001:00000468       ??_C@_1BE@JGMPCMJC@?$AAr?$AAc?$AAl?$AAk?$AA_?$AAc?$AAm?$AAd?$AA?3?$AA?$AA@ 0000000180001468     Plugin.obj
 0001:00000480       ??_C@_1BG@CJEHAOD@?$AAr?$AAc?$AAl?$AAk?$AA_?$AAi?$AAt?$AAe?$AAm?$AA?3?$AA?$AA@ 0000000180001480     Plugin.obj
 0001:00000498       ??_C@_13FPGAJAPJ@?$AA?2?$AA?$AA@ 0000000180001498     Plugin.obj
 0001:0000049c       ??_C@_15DDHGOCBH@?$AA?4?$AA?4?$AA?$AA@ 000000018000149c     Plugin.obj
 0001:000004a8       ??_C@_1M@MDEFCCAF@?$AA?$CF?$AAu?$AA?5?$AA?$CF?$AAs?$AA?$AA@ 00000001800014a8     Plugin.obj
 0001:000004b4       ??_C@_15JOGBDECP@?$AA?0?$AA?5?$AA?$AA@ 00000001800014b4     Plugin.obj
 0001:000004bc       ??_C@_06LMEAOBLB@rename?$AA@ 00000001800014bc     Plugin.obj
 0001:000004c8       ??_C@_1BC@CGPONMNI@?$AAK?$AAe?$AAy?$AAs?$AA?8?$AAF?$AA6?$AA?8?$AA?$AA@ 00000001800014c8     Plugin.obj
 0001:000004dc       ??_C@_06FOBLBEIN@delete?$AA@ 00000001800014dc     Plugin.obj
 0001:000004e8       ??_C@_1BC@BMPELNKI@?$AAK?$AAe?$AAy?$AAs?$AA?8?$AAF?$AA8?$AA?8?$AA?$AA@ 00000001800014e8     Plugin.obj
 0001:00000500       ??_C@_1BO@PGPCBEEA@?$AAK?$AAe?$AAy?$AAs?$AA?8?$AAS?$AAh?$AAi?$AAf?$AAt?$AAD?$AAe?$AAl?$AA?8?$AA?$AA@ 0000000180001500     Plugin.obj
 0001:00000520       ??_C@_1BK@NGCLJGHJ@?$AAK?$AAe?$AAy?$AAs?$AA?8?$AAA?$AAl?$AAt?$AAD?$AAe?$AAl?$AA?8?$AA?$AA@ 0000000180001520     Plugin.obj
 0001:0000053c       ??_C@_15CMBHNMLL@?$AA?5?$AA?$CI?$AA?$AA@ 000000018000153c     Plugin.obj
 0001:00000544       ??_C@_13DIBMAFH@?$AA?$CJ?$AA?$AA@ 0000000180001544     Plugin.obj
 0001:00000550       __xmm@ffffffffffffffff0000000000000002 0000000180001550     Plugin.obj
 0001:00000560       __xmm@ffffffffffffffffffffffffffffffff 0000000180001560     Plugin.obj
 0001:00000570       IID_IContextMenu           0000000180001570     shell32:shguid.obj
 0001:00000580       IID_IShellFolder           0000000180001580     shell32:shguid.obj
 0001:00000590       IID_IDataObject            0000000180001590     uuid:objidl_i.obj
 0001:000005a0       IID_IDropTarget            00000001800015a0     uuid:oleidl_i.obj
 0001:000005b0       _pRawDllMain               00000001800015b0     LIBCMT:dll_dllmain.obj
 0001:000005b0       _pDefaultRawDllMain        00000001800015b0     LIBCMT:dll_dllmain.obj
 0001:000005c0       ??_7exception@std@@6B@     00000001800015c0     LIBCMT:throw_bad_alloc.obj
 0001:000005d0       ??_C@_0BC@EOODALEL@Unknown?5exception?$AA@ 00000001800015d0     LIBCMT:throw_bad_alloc.obj
 0001:000005f0       ??_7bad_alloc@std@@6B@     00000001800015f0     LIBCMT:throw_bad_alloc.obj
 0001:00000600       ??_C@_0P@GHFPNOJB@bad?5allocation?$AA@ 0000000180001600     LIBCMT:throw_bad_alloc.obj
 0001:00000618       ??_7bad_array_new_length@std@@6B@ 0000000180001618     LIBCMT:throw_bad_alloc.obj
 0001:00000628       ??_C@_0BF@KINCDENJ@bad?5array?5new?5length?$AA@ 0000000180001628     LIBCMT:throw_bad_alloc.obj
 0001:00000648       ??_7type_info@@6B@         0000000180001648     LIBCMT:std_type_info_static.obj
 0001:00000650       ??_7_com_error@@6B@        0000000180001650     comsuppw:comraise.obj
 0001:00000658       _Microsoft_CRTProvider     0000000180001658     libvcruntime:telemetry.obj
 0001:00000660       ??_C@_00CNPNBAHC@?$AA@     0000000180001660     libvcruntime:telemetry.obj
 0001:00000668       ??_C@_0O@JEOPJOMI@Main?5Invoked?4?$AA@ 0000000180001668     libvcruntime:telemetry.obj
 0001:00000678       ??_C@_0P@NEAEIBDO@Main?5Returned?4?$AA@ 0000000180001678     libvcruntime:telemetry.obj
 0001:000006f0       ??_C@_1BC@DNHGCMLG@?$AAa?$AAd?$AAv?$AAa?$AAp?$AAi?$AA3?$AA2?$AA?$AA@ 00000001800016f0     libvcruntime:winapi_downlevel.obj
 0001:00000708       ??_C@_1DM@KHCHBNEB@?$AAa?$AAp?$AAi?$AA?9?$AAm?$AAs?$AA?9?$AAw?$AAi?$AAn?$AA?9?$AAc?$AAo?$AAr?$AAe?$AA?9?$AAf?$AAi?$AAb?$AAe?$AAr?$AAs?$AA?9?$AAl?$AA1?$AA?9?$AA1?$AA?9?$AA1?$AA?$AA@ 0000000180001708     libvcruntime:winapi_downlevel.obj
 0001:00000748       ??_C@_1DK@LPPGFMPP@?$AAa?$AAp?$AAi?$AA?9?$AAm?$AAs?$AA?9?$AAw?$AAi?$AAn?$AA?9?$AAc?$AAo?$AAr?$AAe?$AA?9?$AAs?$AAy?$AAn?$AAc?$AAh?$AA?9?$AAl?$AA1?$AA?9?$AA2?$AA?9?$AA0?$AA?$AA@ 0000000180001748     libvcruntime:winapi_downlevel.obj
 0001:00000788       ??_C@_1BC@GDMECMAK@?$AAk?$AAe?$AAr?$AAn?$AAe?$AAl?$AA3?$AA2?$AA?$AA@ 0000000180001788     libvcruntime:winapi_downlevel.obj
 0001:000007a0       ??_C@_0O@BAMBGLIE@EventRegister?$AA@ 00000001800017a0     libvcruntime:winapi_downlevel.obj
 0001:000007b8       ??_C@_0BE@BJEEGHGK@EventSetInformation?$AA@ 00000001800017b8     libvcruntime:winapi_downlevel.obj
 0001:000007d0       ??_C@_0BA@FAKLIPIC@EventUnregister?$AA@ 00000001800017d0     libvcruntime:winapi_downlevel.obj
 0001:000007e8       ??_C@_0BD@PKLHJPHD@EventWriteTransfer?$AA@ 00000001800017e8     libvcruntime:winapi_downlevel.obj
 0001:00000808       ??_C@_08KNHFBNJ@FlsAlloc?$AA@ 0000000180001808     libvcruntime:winapi_downlevel.obj
 0001:00000820       ??_C@_07PEJMOBNF@FlsFree?$AA@ 0000000180001820     libvcruntime:winapi_downlevel.obj
 0001:00000830       ??_C@_0M@GDNOONDI@FlsGetValue?$AA@ 0000000180001830     libvcruntime:winapi_downlevel.obj
 0001:00000848       ??_C@_0M@JCPCPOEF@FlsSetValue?$AA@ 0000000180001848     libvcruntime:winapi_downlevel.obj
 0001:00000860       ??_C@_0BM@HCFOFFN@InitializeCriticalSectionEx?$AA@ 0000000180001860     libvcruntime:winapi_downlevel.obj
 0001:00000ba0       ??_C@_08EHJDFFNH@__based?$CI?$AA@ 0000000180001ba0     libvcruntime:undname.obj
 0001:00000bb0       ??_C@_07KOLFKCDI@__cdecl?$AA@ 0000000180001bb0     libvcruntime:undname.obj
 0001:00000bb8       ??_C@_08GHMPAG@__pascal?$AA@ 0000000180001bb8     libvcruntime:undname.obj
 0001:00000bc8       ??_C@_09IFJBGAPI@__stdcall?$AA@ 0000000180001bc8     libvcruntime:undname.obj
 0001:00000bd8       ??_C@_0L@NPHFGOKO@__thiscall?$AA@ 0000000180001bd8     libvcruntime:undname.obj
 0001:00000be8       ??_C@_0L@JMKHOMEK@__fastcall?$AA@ 0000000180001be8     libvcruntime:undname.obj
 0001:00000bf8       ??_C@_0N@BCKKPABJ@__vectorcall?$AA@ 0000000180001bf8     libvcruntime:undname.obj
 0001:00000c08       ??_C@_09HIJEGCPM@__clrcall?$AA@ 0000000180001c08     libvcruntime:undname.obj
 0001:00000c14       ??_C@_06GHPCKEAG@__eabi?$AA@ 0000000180001c14     libvcruntime:undname.obj
 0001:00000c20       ??_C@_07JOMMBBKO@__ptr64?$AA@ 0000000180001c20     libvcruntime:undname.obj
 0001:00000c28       ??_C@_0L@PILCLIHE@__restrict?$AA@ 0000000180001c28     libvcruntime:undname.obj
 0001:00000c38       ??_C@_0M@GFIIJFMG@__unaligned?$AA@ 0000000180001c38     libvcruntime:undname.obj
 0001:00000c48       ??_C@_09DHDLOLLB@restrict?$CI?$AA@ 0000000180001c48     libvcruntime:undname.obj
 0001:00000c54       ??_C@_04NIHEBCM@?5new?$AA@ 0000000180001c54     libvcruntime:undname.obj
 0001:00000c60       ??_C@_07FPCDHGMM@?5delete?$AA@ 0000000180001c60     libvcruntime:undname.obj
 0001:00000c68       ??_C@_01NEMOKFLO@?$DN?$AA@ 0000000180001c68     libvcruntime:undname.obj
 0001:00000c6c       ??_C@_02GPIOPFAK@?$DO?$DO?$AA@ 0000000180001c6c     libvcruntime:undname.obj
 0001:00000c70       ??_C@_02FODMEDOG@?$DM?$DM?$AA@ 0000000180001c70     libvcruntime:undname.obj
 0001:00000c74       ??_C@_01DCLJPIOD@?$CB?$AA@ 0000000180001c74     libvcruntime:undname.obj
 0001:00000c78       ??_C@_02EGOFBIJA@?$DN?$DN?$AA@ 0000000180001c78     libvcruntime:undname.obj
 0001:00000c7c       ??_C@_02FDNJECIE@?$CB?$DN?$AA@ 0000000180001c7c     libvcruntime:undname.obj
 0001:00000c80       ??_C@_02GPECMEKF@?$FL?$FN?$AA@ 0000000180001c80     libvcruntime:undname.obj
 0001:00000c88       ??_C@_08LHJFAFGD@operator?$AA@ 0000000180001c88     libvcruntime:undname.obj
 0001:00000c94       ??_C@_02HBOOOICD@?9?$DO?$AA@ 0000000180001c94     libvcruntime:undname.obj
 0001:00000c98       ??_C@_01NBENCBCI@?$CK?$AA@ 0000000180001c98     libvcruntime:undname.obj
 0001:00000c9c       ??_C@_02ECNGHCIF@?$CL?$CL?$AA@ 0000000180001c9c     libvcruntime:undname.obj
 0001:00000ca0       ??_C@_02BAABKJLB@?9?9?$AA@ 0000000180001ca0     libvcruntime:undname.obj
 0001:00000ca4       ??_C@_01JOAMLHOP@?9?$AA@   0000000180001ca4     libvcruntime:undname.obj
 0001:00000ca8       ??_C@_01MIFGBAGJ@?$CL?$AA@ 0000000180001ca8     libvcruntime:undname.obj
 0001:00000cac       ??_C@_01HNPIGOCE@?$CG?$AA@ 0000000180001cac     libvcruntime:undname.obj
 0001:00000cb0       ??_C@_03MNHNFDLC@?9?$DO?$CK?$AA@ 0000000180001cb0     libvcruntime:undname.obj
 0001:00000cb4       ??_C@_01KMDKNFGN@?1?$AA@   0000000180001cb4     libvcruntime:undname.obj
 0001:00000cb8       ??_C@_01FGNFDNOH@?$CF?$AA@ 0000000180001cb8     libvcruntime:undname.obj
 0001:00000cbc       ??_C@_01MNNFJEPP@?$DM?$AA@ 0000000180001cbc     libvcruntime:undname.obj
 0001:00000cc0       ??_C@_02EHCHHCKH@?$DM?$DN?$AA@ 0000000180001cc0     libvcruntime:undname.obj
 0001:00000cc4       ??_C@_01PPODPGHN@?$DO?$AA@ 0000000180001cc4     libvcruntime:undname.obj
 0001:00000cc8       ??_C@_02EEKDKGMJ@?$DO?$DN?$AA@ 0000000180001cc8     libvcruntime:undname.obj
 0001:00000ccc       ??_C@_01IHBHIGKO@?0?$AA@   0000000180001ccc     libvcruntime:undname.obj
 0001:00000cd0       ??_C@_02HCKGKOFO@?$CI?$CJ?$AA@ 0000000180001cd0     libvcruntime:undname.obj
 0001:00000cd4       ??_C@_01PJKLJHI@?$HO?$AA@  0000000180001cd4     libvcruntime:undname.obj
 0001:00000cd8       ??_C@_01JKBOJNNK@?$FO?$AA@ 0000000180001cd8     libvcruntime:undname.obj
 0001:00000cdc       ??_C@_01DNKMNLPK@?$HM?$AA@ 0000000180001cdc     libvcruntime:undname.obj
 0001:00000ce0       ??_C@_02PPKAJPJL@?$CG?$CG?$AA@ 0000000180001ce0     libvcruntime:undname.obj
 0001:00000ce4       ??_C@_02NONPIBCD@?$HM?$HM?$AA@ 0000000180001ce4     libvcruntime:undname.obj
 0001:00000ce8       ??_C@_02FPIMKNGF@?$CK?$DN?$AA@ 0000000180001ce8     libvcruntime:undname.obj
 0001:00000cec       ??_C@_02FOEOMHFC@?$CL?$DN?$AA@ 0000000180001cec     libvcruntime:undname.obj
 0001:00000cf0       ??_C@_02FKMDLLOA@?9?$DN?$AA@ 0000000180001cf0     libvcruntime:undname.obj
 0001:00000cf4       ??_C@_02FJEHGPIO@?1?$DN?$AA@ 0000000180001cf4     libvcruntime:undname.obj
 0001:00000cf8       ??_C@_02FENAOKFI@?$CF?$DN?$AA@ 0000000180001cf8     libvcruntime:undname.obj
 0001:00000cfc       ??_C@_03IKFCCPFF@?$DO?$DO?$DN?$AA@ 0000000180001cfc     libvcruntime:undname.obj
 0001:00000d00       ??_C@_03CDNPDDLA@?$DM?$DM?$DN?$AA@ 0000000180001d00     libvcruntime:undname.obj
 0001:00000d04       ??_C@_02FGJGFEAB@?$CG?$DN?$AA@ 0000000180001d04     libvcruntime:undname.obj
 0001:00000d08       ??_C@_02DHLNPPGH@?$HM?$DN?$AA@ 0000000180001d08     libvcruntime:undname.obj
 0001:00000d0c       ??_C@_02MHEGNOJ@?$FO?$DN?$AA@ 0000000180001d0c     libvcruntime:undname.obj
 0001:00000d10       ??_C@_09IFPLHPGF@?$GAvftable?8?$AA@ 0000000180001d10     libvcruntime:undname.obj
 0001:00000d20       ??_C@_09BLBHBJP@?$GAvbtable?8?$AA@ 0000000180001d20     libvcruntime:undname.obj
 0001:00000d30       ??_C@_07FEEIOKP@?$GAvcall?8?$AA@ 0000000180001d30     libvcruntime:undname.obj
 0001:00000d38       ??_C@_08LLFFHHDJ@?$GAtypeof?8?$AA@ 0000000180001d38     libvcruntime:undname.obj
 0001:00000d48       ??_C@_0BF@KDPPACIK@?$GAlocal?5static?5guard?8?$AA@ 0000000180001d48     libvcruntime:undname.obj
 0001:00000d60       ??_C@_08OBABFOLI@?$GAstring?8?$AA@ 0000000180001d60     libvcruntime:undname.obj
 0001:00000d70       ??_C@_0BD@JDLKDPAB@?$GAvbase?5destructor?8?$AA@ 0000000180001d70     libvcruntime:undname.obj
 0001:00000d88       ??_C@_0BN@DEGPLNFK@?$GAvector?5deleting?5destructor?8?$AA@ 0000000180001d88     libvcruntime:undname.obj
 0001:00000da8       ??_C@_0BO@OBMKPJIG@?$GAdefault?5constructor?5closure?8?$AA@ 0000000180001da8     libvcruntime:undname.obj
 0001:00000dc8       ??_C@_0BN@IMDCHIKM@?$GAscalar?5deleting?5destructor?8?$AA@ 0000000180001dc8     libvcruntime:undname.obj
 0001:00000de8       ??_C@_0BO@PFGOCPJJ@?$GAvector?5constructor?5iterator?8?$AA@ 0000000180001de8     libvcruntime:undname.obj
 0001:00000e08       ??_C@_0BN@LFPFMEDL@?$GAvector?5destructor?5iterator?8?$AA@ 0000000180001e08     libvcruntime:undname.obj
 0001:00000e28       ??_C@_0CE@IKBNEHA@?$GAvector?5vbase?5constructor?5iterat@ 0000000180001e28     libvcruntime:undname.obj
 0001:00000e50       ??_C@_0BL@NILFHHPC@?$GAvirtual?5displacement?5map?8?$AA@ 0000000180001e50     libvcruntime:undname.obj
 0001:00000e70       ??_C@_0CB@JONCMFFK@?$GAeh?5vector?5constructor?5iterator?8@ 0000000180001e70     libvcruntime:undname.obj
 0001:00000e98       ??_C@_0CA@GCEOPDGL@?$GAeh?5vector?5destructor?5iterator?8?$AA@ 0000000180001e98     libvcruntime:undname.obj
 0001:00000eb8       ??_C@_0CH@OOJPLCPH@?$GAeh?5vector?5vbase?5constructor?5ite@ 0000000180001eb8     libvcruntime:undname.obj
 0001:00000ee0       ??_C@_0BL@LLKPOHJI@?$GAcopy?5constructor?5closure?8?$AA@ 0000000180001ee0     libvcruntime:undname.obj
 0001:00000f00       ??_C@_0BA@KBCDOMBN@?$GAudt?5returning?8?$AA@ 0000000180001f00     libvcruntime:undname.obj
 0001:00000f10       ??_C@_03KLGMFNMG@?$GAEH?$AA@ 0000000180001f10     libvcruntime:undname.obj
 0001:00000f14       ??_C@_05KHLCHHI@?$GARTTI?$AA@ 0000000180001f14     libvcruntime:undname.obj
 0001:00000f20       ??_C@_0BA@KKLDJDLB@?$GAlocal?5vftable?8?$AA@ 0000000180001f20     libvcruntime:undname.obj
 0001:00000f30       ??_C@_0CE@IIHCMGGL@?$GAlocal?5vftable?5constructor?5closu@ 0000000180001f30     libvcruntime:undname.obj
 0001:00000f54       ??_C@_06FHBGPFGH@?5new?$FL?$FN?$AA@ 0000000180001f54     libvcruntime:undname.obj
 0001:00000f60       ??_C@_09LBNFPBCA@?5delete?$FL?$FN?$AA@ 0000000180001f60     libvcruntime:undname.obj
 0001:00000f70       ??_C@_0P@HJKNJFNN@?$GAomni?5callsig?8?$AA@ 0000000180001f70     libvcruntime:undname.obj
 0001:00000f80       ??_C@_0BL@CNOONJFP@?$GAplacement?5delete?5closure?8?$AA@ 0000000180001f80     libvcruntime:undname.obj
 0001:00000fa0       ??_C@_0BN@CKNJLHMB@?$GAplacement?5delete?$FL?$FN?5closure?8?$AA@ 0000000180001fa0     libvcruntime:undname.obj
 0001:00000fc0       ??_C@_0CG@CFDHKGGD@?$GAmanaged?5vector?5constructor?5iter@ 0000000180001fc0     libvcruntime:undname.obj
 0001:00000fe8       ??_C@_0CF@IMGKMJNO@?$GAmanaged?5vector?5destructor?5itera@ 0000000180001fe8     libvcruntime:undname.obj
 0001:00001010       ??_C@_0CG@HLDDJMAG@?$GAeh?5vector?5copy?5constructor?5iter@ 0000000180002010     libvcruntime:undname.obj
 0001:00001038       ??_C@_0CM@FCBBDIGB@?$GAeh?5vector?5vbase?5copy?5constructo@ 0000000180002038     libvcruntime:undname.obj
 0001:00001068       ??_C@_0BL@CLIPGLGB@?$GAdynamic?5initializer?5for?5?8?$AA@ 0000000180002068     libvcruntime:undname.obj
 0001:00001088       ??_C@_0CB@PDBIFEP@?$GAdynamic?5atexit?5destructor?5for?5?8@ 0000000180002088     libvcruntime:undname.obj
 0001:000010b0       ??_C@_0CD@CGAJBKEJ@?$GAvector?5copy?5constructor?5iterato@ 00000001800020b0     libvcruntime:undname.obj
 0001:000010d8       ??_C@_0CJ@GJELGAMM@?$GAvector?5vbase?5copy?5constructor?5i@ 00000001800020d8     libvcruntime:undname.obj
 0001:00001108       ??_C@_0CL@FGIJHLCE@?$GAmanaged?5vector?5copy?5constructor@ 0000000180002108     libvcruntime:undname.obj
 0001:00001138       ??_C@_0BM@PMGGMLDN@?$GAlocal?5static?5thread?5guard?8?$AA@ 0000000180002138     libvcruntime:undname.obj
 0001:00001158       ??_C@_0N@BDNMDMOL@operator?5?$CC?$CC?5?$AA@ 0000000180002158     libvcruntime:undname.obj
 0001:00001168       ??_C@_0BC@DAFEJGAK@?5Type?5Descriptor?8?$AA@ 0000000180002168     libvcruntime:undname.obj
 0001:00001180       ??_C@_0BM@LDKODKLH@?5Base?5Class?5Descriptor?5at?5?$CI?$AA@ 0000000180002180     libvcruntime:undname.obj
 0001:000011a0       ??_C@_0BD@LGICGFMM@?5Base?5Class?5Array?8?$AA@ 00000001800021a0     libvcruntime:undname.obj
 0001:000011b8       ??_C@_0BN@MECKDCOJ@?5Class?5Hierarchy?5Descriptor?8?$AA@ 00000001800021b8     libvcruntime:undname.obj
 0001:000011d8       ??_C@_0BK@CFCOFLF@?5Complete?5Object?5Locator?8?$AA@ 00000001800021d8     libvcruntime:undname.obj
 0001:00001200       __acrt_exception_action_table 0000000180002200     libucrt:exception_filter.obj
 0001:000012c0       __acrt_signal_action_table_count 00000001800022c0     libucrt:exception_filter.obj
 0001:000012c8       __acrt_signal_action_first_fpe_index 00000001800022c8     libucrt:exception_filter.obj
 0001:000012d0       __acrt_signal_action_fpe_count 00000001800022d0     libucrt:exception_filter.obj
 0001:000012d8       ??_C@_1BI@BGOHAHKC@?$AAm?$AAs?$AAc?$AAo?$AAr?$AAe?$AAe?$AA?4?$AAd?$AAl?$AAl?$AA?$AA@ 00000001800022d8     libucrt:exit.obj
 0001:000012f0       ??_C@_0P@MIGLKIOC@CorExitProcess?$AA@ 00000001800022f0     libucrt:exit.obj
 0001:00001490       ??_C@_1EG@CNNIPFIM@?$AAa?$AAp?$AAi?$AA?9?$AAm?$AAs?$AA?9?$AAw?$AAi?$AAn?$AA?9?$AAa?$AAp?$AAp?$AAm?$AAo?$AAd?$AAe?$AAl?$AA?9?$AAr?$AAu?$AAn?$AAt?$AAi?$AAm?$AAe?$AA?9?$AAl?$AA1?$AA?9?$AA1@ 0000000180002490     libucrt:winapi_thunks.obj
 0001:000014e0       ??_C@_1EA@JGEFHKEI@?$AAa?$AAp?$AAi?$AA?9?$AAm?$AAs?$AA?9?$AAw?$AAi?$AAn?$AA?9?$AAc?$AAo?$AAr?$AAe?$AA?9?$AAd?$AAa?$AAt?$AAe?$AAt?$AAi?$AAm?$AAe?$AA?9?$AAl?$AA1?$AA?9?$AA1?$AA?9?$AA1?$AA?$AA@ 00000001800024e0     libucrt:winapi_thunks.obj
 0001:00001520       ??_C@_1DI@GCIAAENM@?$AAa?$AAp?$AAi?$AA?9?$AAm?$AAs?$AA?9?$AAw?$AAi?$AAn?$AA?9?$AAc?$AAo?$AAr?$AAe?$AA?9?$AAf?$AAi?$AAl?$AAe?$AA?9?$AAl?$AA2?$AA?9?$AA1?$AA?9?$AA1?$AA?$AA@ 0000000180002520     libucrt:winapi_thunks.obj
 0001:00001560       ??_C@_1EI@MPIAOHOC@?$AAa?$AAp?$AAi?$AA?9?$AAm?$AAs?$AA?9?$AAw?$AAi?$AAn?$AA?9?$AAc?$AAo?$AAr?$AAe?$AA?9?$AAl?$AAo?$AAc?$AAa?$AAl?$AAi?$AAz?$AAa?$AAt?$AAi?$AAo?$AAn?$AA?9?$AAl?$AA1?$AA?9@ 0000000180002560     libucrt:winapi_thunks.obj
 0001:000015b0       ??_C@_1FK@FPHCKFIE@?$AAa?$AAp?$AAi?$AA?9?$AAm?$AAs?$AA?9?$AAw?$AAi?$AAn?$AA?9?$AAc?$AAo?$AAr?$AAe?$AA?9?$AAl?$AAo?$AAc?$AAa?$AAl?$AAi?$AAz?$AAa?$AAt?$AAi?$AAo?$AAn?$AA?9?$AAo?$AAb?$AAs@ 00000001800025b0     libucrt:winapi_thunks.obj
 0001:00001610       ??_C@_1EM@DILCGIIO@?$AAa?$AAp?$AAi?$AA?9?$AAm?$AAs?$AA?9?$AAw?$AAi?$AAn?$AA?9?$AAc?$AAo?$AAr?$AAe?$AA?9?$AAp?$AAr?$AAo?$AAc?$AAe?$AAs?$AAs?$AAt?$AAh?$AAr?$AAe?$AAa?$AAd?$AAs?$AA?9?$AAl@ 0000000180002610     libucrt:winapi_thunks.obj
 0001:00001660       ??_C@_1DM@LNCGDDPN@?$AAa?$AAp?$AAi?$AA?9?$AAm?$AAs?$AA?9?$AAw?$AAi?$AAn?$AA?9?$AAc?$AAo?$AAr?$AAe?$AA?9?$AAs?$AAt?$AAr?$AAi?$AAn?$AAg?$AA?9?$AAl?$AA1?$AA?9?$AA1?$AA?9?$AA0?$AA?$AA@ 0000000180002660     libucrt:winapi_thunks.obj
 0001:000016a0       ??_C@_1DO@FPAPJEMD@?$AAa?$AAp?$AAi?$AA?9?$AAm?$AAs?$AA?9?$AAw?$AAi?$AAn?$AA?9?$AAc?$AAo?$AAr?$AAe?$AA?9?$AAs?$AAy?$AAs?$AAi?$AAn?$AAf?$AAo?$AA?9?$AAl?$AA1?$AA?9?$AA2?$AA?9?$AA1?$AA?$AA@ 00000001800026a0     libucrt:winapi_thunks.obj
 0001:000016e0       ??_C@_1DK@NDHNAHIO@?$AAa?$AAp?$AAi?$AA?9?$AAm?$AAs?$AA?9?$AAw?$AAi?$AAn?$AA?9?$AAc?$AAo?$AAr?$AAe?$AA?9?$AAw?$AAi?$AAn?$AAr?$AAt?$AA?9?$AAl?$AA1?$AA?9?$AA1?$AA?9?$AA0?$AA?$AA@ 00000001800026e0     libucrt:winapi_thunks.obj
 0001:00001720       ??_C@_1DM@KGHDGBCM@?$AAa?$AAp?$AAi?$AA?9?$AAm?$AAs?$AA?9?$AAw?$AAi?$AAn?$AA?9?$AAc?$AAo?$AAr?$AAe?$AA?9?$AAx?$AAs?$AAt?$AAa?$AAt?$AAe?$AA?9?$AAl?$AA2?$AA?9?$AA1?$AA?9?$AA0?$AA?$AA@ 0000000180002720     libucrt:winapi_thunks.obj
 0001:00001760       ??_C@_1EO@IJIOEFOH@?$AAa?$AAp?$AAi?$AA?9?$AAm?$AAs?$AA?9?$AAw?$AAi?$AAn?$AA?9?$AAr?$AAt?$AAc?$AAo?$AAr?$AAe?$AA?9?$AAn?$AAt?$AAu?$AAs?$AAe?$AAr?$AA?9?$AAw?$AAi?$AAn?$AAd?$AAo?$AAw?$AA?9@ 0000000180002760     libucrt:winapi_thunks.obj
 0001:000017b0       ??_C@_1FG@HHGEKANL@?$AAa?$AAp?$AAi?$AA?9?$AAm?$AAs?$AA?9?$AAw?$AAi?$AAn?$AA?9?$AAs?$AAe?$AAc?$AAu?$AAr?$AAi?$AAt?$AAy?$AA?9?$AAs?$AAy?$AAs?$AAt?$AAe?$AAm?$AAf?$AAu?$AAn?$AAc?$AAt?$AAi@ 00000001800027b0     libucrt:winapi_thunks.obj
 0001:00001810       ??_C@_1FG@NCKKOLKO@?$AAe?$AAx?$AAt?$AA?9?$AAm?$AAs?$AA?9?$AAw?$AAi?$AAn?$AA?9?$AAk?$AAe?$AAr?$AAn?$AAe?$AAl?$AA3?$AA2?$AA?9?$AAp?$AAa?$AAc?$AAk?$AAa?$AAg?$AAe?$AA?9?$AAc?$AAu?$AAr?$AAr@ 0000000180002810     libucrt:winapi_thunks.obj
 0001:00001870       ??_C@_1EG@DBIOJECG@?$AAe?$AAx?$AAt?$AA?9?$AAm?$AAs?$AA?9?$AAw?$AAi?$AAn?$AA?9?$AAn?$AAt?$AAu?$AAs?$AAe?$AAr?$AA?9?$AAd?$AAi?$AAa?$AAl?$AAo?$AAg?$AAb?$AAo?$AAx?$AA?9?$AAl?$AA1?$AA?9?$AA1@ 0000000180002870     libucrt:winapi_thunks.obj
 0001:000018c0       ??_C@_1EO@FIHMJCLF@?$AAe?$AAx?$AAt?$AA?9?$AAm?$AAs?$AA?9?$AAw?$AAi?$AAn?$AA?9?$AAn?$AAt?$AAu?$AAs?$AAe?$AAr?$AA?9?$AAw?$AAi?$AAn?$AAd?$AAo?$AAw?$AAs?$AAt?$AAa?$AAt?$AAi?$AAo?$AAn?$AA?9@ 00000001800028c0     libucrt:winapi_thunks.obj
 0001:00001910       ??_C@_1O@BCCLBEOE@?$AAu?$AAs?$AAe?$AAr?$AA3?$AA2?$AA?$AA@ 0000000180002910     libucrt:winapi_thunks.obj
 0001:00001948       ??_C@_0BE@JOGNEJCI@GetCurrentPackageId?$AA@ 0000000180002948     libucrt:winapi_thunks.obj
 0001:00001970       ??_C@_0O@KKBNKAPF@LCMapStringEx?$AA@ 0000000180002970     libucrt:winapi_thunks.obj
 0001:00001988       ??_C@_0BB@HBDEELFH@LocaleNameToLCID?$AA@ 0000000180002988     libucrt:winapi_thunks.obj
 0001:00001b28       ??_C@_1M@HPNHIDJI@?$AAj?$AAa?$AA?9?$AAJ?$AAP?$AA?$AA@ 0000000180002b28     libucrt:mbctype.obj
 0001:00001b38       ??_C@_1M@BIBDDEMK@?$AAz?$AAh?$AA?9?$AAC?$AAN?$AA?$AA@ 0000000180002b38     libucrt:mbctype.obj
 0001:00001b48       ??_C@_1M@JLOOOEGK@?$AAk?$AAo?$AA?9?$AAK?$AAR?$AA?$AA@ 0000000180002b48     libucrt:mbctype.obj
 0001:00001b58       ??_C@_1M@CLNBBOPM@?$AAz?$AAh?$AA?9?$AAT?$AAW?$AA?$AA@ 0000000180002b58     libucrt:mbctype.obj
 0001:00001b70       __lc_time_c                0000000180002b70     libucrt:nlsdata.obj
 0001:00001e30       ??_C@_03KOEHGMDN@Sun?$AA@  0000000180002e30     libucrt:nlsdata.obj
 0001:00001e34       ??_C@_03PDAGKDH@Mon?$AA@   0000000180002e34     libucrt:nlsdata.obj
 0001:00001e38       ??_C@_03NAGEINEP@Tue?$AA@  0000000180002e38     libucrt:nlsdata.obj
 0001:00001e3c       ??_C@_03MHOMLAJA@Wed?$AA@  0000000180002e3c     libucrt:nlsdata.obj
 0001:00001e40       ??_C@_03IOFIKPDN@Thu?$AA@  0000000180002e40     libucrt:nlsdata.obj
 0001:00001e44       ??_C@_03IDIOELNC@Fri?$AA@  0000000180002e44     libucrt:nlsdata.obj
 0001:00001e48       ??_C@_03FEFJNEK@Sat?$AA@   0000000180002e48     libucrt:nlsdata.obj
 0001:00001e4c       ??_C@_06OOPIFAJ@Sunday?$AA@ 0000000180002e4c     libucrt:nlsdata.obj
 0001:00001e54       ??_C@_06JLEDEDGH@Monday?$AA@ 0000000180002e54     libucrt:nlsdata.obj
 0001:00001e60       ??_C@_07BAAGCFCM@Tuesday?$AA@ 0000000180002e60     libucrt:nlsdata.obj
 0001:00001e68       ??_C@_09DLIGFAKA@Wednesday?$AA@ 0000000180002e68     libucrt:nlsdata.obj
 0001:00001e78       ??_C@_08HACCIKIA@Thursday?$AA@ 0000000180002e78     libucrt:nlsdata.obj
 0001:00001e84       ??_C@_06JECMNKMI@Friday?$AA@ 0000000180002e84     libucrt:nlsdata.obj
 0001:00001e90       ??_C@_08INBOOONO@Saturday?$AA@ 0000000180002e90     libucrt:nlsdata.obj
 0001:00001e9c       ??_C@_03JIHJHPIE@Jan?$AA@  0000000180002e9c     libucrt:nlsdata.obj
 0001:00001ea0       ??_C@_03HJBDCHOM@Feb?$AA@  0000000180002ea0     libucrt:nlsdata.obj
 0001:00001ea4       ??_C@_03ODNJBKGA@Mar?$AA@  0000000180002ea4     libucrt:nlsdata.obj
 0001:00001ea8       ??_C@_03LEOLGMJP@Apr?$AA@  0000000180002ea8     libucrt:nlsdata.obj
 0001:00001eac       ??_C@_03CNMDKL@May?$AA@    0000000180002eac     libucrt:nlsdata.obj
 0001:00001eb0       ??_C@_03IDFGHECI@Jun?$AA@  0000000180002eb0     libucrt:nlsdata.obj
 0001:00001eb4       ??_C@_03LBGABGKK@Jul?$AA@  0000000180002eb4     libucrt:nlsdata.obj
 0001:00001eb8       ??_C@_03IFJFEIGA@Aug?$AA@  0000000180002eb8     libucrt:nlsdata.obj
 0001:00001ebc       ??_C@_03GGCAPAJC@Sep?$AA@  0000000180002ebc     libucrt:nlsdata.obj
 0001:00001ec0       ??_C@_03BMAOKBAD@Oct?$AA@  0000000180002ec0     libucrt:nlsdata.obj
 0001:00001ec4       ??_C@_03JPJOFNIA@Nov?$AA@  0000000180002ec4     libucrt:nlsdata.obj
 0001:00001ec8       ??_C@_03MKABNOCG@Dec?$AA@  0000000180002ec8     libucrt:nlsdata.obj
 0001:00001ed0       ??_C@_07CGJPFGJA@January?$AA@ 0000000180002ed0     libucrt:nlsdata.obj
 0001:00001ed8       ??_C@_08GNJGEPFN@February?$AA@ 0000000180002ed8     libucrt:nlsdata.obj
 0001:00001ee4       ??_C@_05HPCKOFNC@March?$AA@ 0000000180002ee4     libucrt:nlsdata.obj
 0001:00001eec       ??_C@_05DMJDNLEJ@April?$AA@ 0000000180002eec     libucrt:nlsdata.obj
 0001:00001ef4       ??_C@_04CNLMGBGM@June?$AA@ 0000000180002ef4     libucrt:nlsdata.obj
 0001:00001efc       ??_C@_04MIEPOIFP@July?$AA@ 0000000180002efc     libucrt:nlsdata.obj
 0001:00001f04       ??_C@_06LBBHFDDG@August?$AA@ 0000000180002f04     libucrt:nlsdata.obj
 0001:00001f10       ??_C@_09BHHEALKD@September?$AA@ 0000000180002f10     libucrt:nlsdata.obj
 0001:00001f20       ??_C@_07JJNFCEND@October?$AA@ 0000000180002f20     libucrt:nlsdata.obj
 0001:00001f28       ??_C@_08HCHEGEOA@November?$AA@ 0000000180002f28     libucrt:nlsdata.obj
 0001:00001f38       ??_C@_08EDHMEBNP@December?$AA@ 0000000180002f38     libucrt:nlsdata.obj
 0001:00001f44       ??_C@_02DEDBPAFC@AM?$AA@   0000000180002f44     libucrt:nlsdata.obj
 0001:00001f48       ??_C@_02CJNFDJBF@PM?$AA@   0000000180002f48     libucrt:nlsdata.obj
 0001:00001f50       ??_C@_08BPBNCDIB@MM?1dd?1yy?$AA@ 0000000180002f50     libucrt:nlsdata.obj
 0001:00001f60       ??_C@_0BE@CKGJFCPC@dddd?0?5MMMM?5dd?0?5yyyy?$AA@ 0000000180002f60     libucrt:nlsdata.obj
 0001:00001f78       ??_C@_08JCCMCCIL@HH?3mm?3ss?$AA@ 0000000180002f78     libucrt:nlsdata.obj
 0001:00001f88       ??_C@_17MBGCMIPB@?$AAS?$AAu?$AAn?$AA?$AA@ 0000000180002f88     libucrt:nlsdata.obj
 0001:00001f90       ??_C@_17KBOMKBF@?$AAM?$AAo?$AAn?$AA?$AA@ 0000000180002f90     libucrt:nlsdata.obj
 0001:00001f98       ??_C@_17BMKGEGOJ@?$AAT?$AAu?$AAe?$AA?$AA@ 0000000180002f98     libucrt:nlsdata.obj
 0001:00001fa0       ??_C@_17CJEDCEPE@?$AAW?$AAe?$AAd?$AA?$AA@ 0000000180002fa0     libucrt:nlsdata.obj
 0001:00001fa8       ??_C@_17PDPHAADD@?$AAT?$AAh?$AAu?$AA?$AA@ 0000000180002fa8     libucrt:nlsdata.obj
 0001:00001fb0       ??_C@_17HFOLPPLP@?$AAF?$AAr?$AAi?$AA?$AA@ 0000000180002fb0     libucrt:nlsdata.obj
 0001:00001fb8       ??_C@_17GGIBDPIH@?$AAS?$AAa?$AAt?$AA?$AA@ 0000000180002fb8     libucrt:nlsdata.obj
 0001:00001fc0       ??_C@_1O@IHNHDHPB@?$AAS?$AAu?$AAn?$AAd?$AAa?$AAy?$AA?$AA@ 0000000180002fc0     libucrt:nlsdata.obj
 0001:00001fd0       ??_C@_1O@MMNBFLIA@?$AAM?$AAo?$AAn?$AAd?$AAa?$AAy?$AA?$AA@ 0000000180002fd0     libucrt:nlsdata.obj
 0001:00001fe0       ??_C@_1BA@ENFBFFEK@?$AAT?$AAu?$AAe?$AAs?$AAd?$AAa?$AAy?$AA?$AA@ 0000000180002fe0     libucrt:nlsdata.obj
 0001:00001ff0       ??_C@_1BE@EBOGMDOH@?$AAW?$AAe?$AAd?$AAn?$AAe?$AAs?$AAd?$AAa?$AAy?$AA?$AA@ 0000000180002ff0     libucrt:nlsdata.obj
 0001:00002008       ??_C@_1BC@HHMNLIHE@?$AAT?$AAh?$AAu?$AAr?$AAs?$AAd?$AAa?$AAy?$AA?$AA@ 0000000180003008     libucrt:nlsdata.obj
 0001:00002020       ??_C@_1O@PDICJHAG@?$AAF?$AAr?$AAi?$AAd?$AAa?$AAy?$AA?$AA@ 0000000180003020     libucrt:nlsdata.obj
 0001:00002030       ??_C@_1BC@ENMNNPAJ@?$AAS?$AAa?$AAt?$AAu?$AAr?$AAd?$AAa?$AAy?$AA?$AA@ 0000000180003030     libucrt:nlsdata.obj
 0001:00002048       ??_C@_17DKNBKCHM@?$AAJ?$AAa?$AAn?$AA?$AA@ 0000000180003048     libucrt:nlsdata.obj
 0001:00002050       ??_C@_17LMDJEKJN@?$AAF?$AAe?$AAb?$AA?$AA@ 0000000180003050     libucrt:nlsdata.obj
 0001:00002058       ??_C@_17CKNLEDEC@?$AAM?$AAa?$AAr?$AA?$AA@ 0000000180003058     libucrt:nlsdata.obj
 0001:00002060       ??_C@_17LFPOIHDD@?$AAA?$AAp?$AAr?$AA?$AA@ 0000000180003060     libucrt:nlsdata.obj
 0001:00002068       ??_C@_17PNNKMEED@?$AAM?$AAa?$AAy?$AA?$AA@ 0000000180003068     libucrt:nlsdata.obj
 0001:00002070       ??_C@_17KCJGOCPB@?$AAJ?$AAu?$AAn?$AA?$AA@ 0000000180003070     libucrt:nlsdata.obj
 0001:00002078       ??_C@_17IJPCKHK@?$AAJ?$AAu?$AAl?$AA?$AA@ 0000000180003078     libucrt:nlsdata.obj
 0001:00002080       ??_C@_17ICPELBCN@?$AAA?$AAu?$AAg?$AA?$AA@ 0000000180003080     libucrt:nlsdata.obj
 0001:00002088       ??_C@_17HCHCOKMG@?$AAS?$AAe?$AAp?$AA?$AA@ 0000000180003088     libucrt:nlsdata.obj
 0001:00002090       ??_C@_17FNLKOI@?$AAO?$AAc?$AAt?$AA?$AA@ 0000000180003090     libucrt:nlsdata.obj
 0001:00002098       ??_C@_17BBDMLCIG@?$AAN?$AAo?$AAv?$AA?$AA@ 0000000180003098     libucrt:nlsdata.obj
 0001:000020a0       ??_C@_17EGKACKIF@?$AAD?$AAe?$AAc?$AA?$AA@ 00000001800030a0     libucrt:nlsdata.obj
 0001:000020a8       ??_C@_1BA@EFMEIEBA@?$AAJ?$AAa?$AAn?$AAu?$AAa?$AAr?$AAy?$AA?$AA@ 00000001800030a8     libucrt:nlsdata.obj
 0001:000020b8       ??_C@_1BC@JGDDFFAM@?$AAF?$AAe?$AAb?$AAr?$AAu?$AAa?$AAr?$AAy?$AA?$AA@ 00000001800030b8     libucrt:nlsdata.obj
 0001:000020d0       ??_C@_1M@IKEENEDF@?$AAM?$AAa?$AAr?$AAc?$AAh?$AA?$AA@ 00000001800030d0     libucrt:nlsdata.obj
 0001:000020e0       ??_C@_1M@GJNLMHFD@?$AAA?$AAp?$AAr?$AAi?$AAl?$AA?$AA@ 00000001800030e0     libucrt:nlsdata.obj
 0001:000020f0       ??_C@_19EPFLPGAP@?$AAJ?$AAu?$AAn?$AAe?$AA?$AA@ 00000001800030f0     libucrt:nlsdata.obj
 0001:00002100       ??_C@_19BIFMLPCD@?$AAJ?$AAu?$AAl?$AAy?$AA?$AA@ 0000000180003100     libucrt:nlsdata.obj
 0001:00002110       ??_C@_1O@PAHLKOAC@?$AAA?$AAu?$AAg?$AAu?$AAs?$AAt?$AA?$AA@ 0000000180003110     libucrt:nlsdata.obj
 0001:00002120       ??_C@_1BE@DKAAMBJL@?$AAS?$AAe?$AAp?$AAt?$AAe?$AAm?$AAb?$AAe?$AAr?$AA?$AA@ 0000000180003120     libucrt:nlsdata.obj
 0001:00002138       ??_C@_1BA@EPANDLNG@?$AAO?$AAc?$AAt?$AAo?$AAb?$AAe?$AAr?$AA?$AA@ 0000000180003138     libucrt:nlsdata.obj
 0001:00002148       ??_C@_1BC@BGLIFPF@?$AAN?$AAo?$AAv?$AAe?$AAm?$AAb?$AAe?$AAr?$AA?$AA@ 0000000180003148     libucrt:nlsdata.obj
 0001:00002160       ??_C@_1BC@FEMKIFH@?$AAD?$AAe?$AAc?$AAe?$AAm?$AAb?$AAe?$AAr?$AA?$AA@ 0000000180003160     libucrt:nlsdata.obj
 0001:00002174       ??_C@_15ODEHAHHF@?$AAA?$AAM?$AA?$AA@ 0000000180003174     libucrt:nlsdata.obj
 0001:0000217c       ??_C@_15CLMNNGEL@?$AAP?$AAM?$AA?$AA@ 000000018000317c     libucrt:nlsdata.obj
 0001:00002188       ??_C@_1BC@IEBCMHCM@?$AAM?$AAM?$AA?1?$AAd?$AAd?$AA?1?$AAy?$AAy?$AA?$AA@ 0000000180003188     libucrt:nlsdata.obj
 0001:000021a0       ??_C@_1CI@KNAKOEBC@?$AAd?$AAd?$AAd?$AAd?$AA?0?$AA?5?$AAM?$AAM?$AAM?$AAM?$AA?5?$AAd?$AAd?$AA?0?$AA?5?$AAy?$AAy?$AAy?$AAy?$AA?$AA@ 00000001800031a0     libucrt:nlsdata.obj
 0001:000021c8       ??_C@_1BC@GDGBMEMK@?$AAH?$AAH?$AA?3?$AAm?$AAm?$AA?3?$AAs?$AAs?$AA?$AA@ 00000001800031c8     libucrt:nlsdata.obj
 0001:000021e0       ??_C@_1M@BMHNFIME@?$AAe?$AAn?$AA?9?$AAU?$AAS?$AA?$AA@ 00000001800031e0     libucrt:nlsdata.obj
 0001:000021f0       __newctype                 00000001800031f0     libucrt:ctype.obj
 0001:000024f0       __newclmap                 00000001800034f0     libucrt:ctype.obj
 0001:00002670       __newcumap                 0000000180003670     libucrt:ctype.obj
 0001:00003630       ??_C@_15EMKDOKLE@?$AAa?$AAr?$AA?$AA@ 0000000180004630     libucrt:lcidtoname_downlevel.obj
 0001:00003638       ??_C@_15KNPADPLH@?$AAb?$AAg?$AA?$AA@ 0000000180004638     libucrt:lcidtoname_downlevel.obj
 0001:00003640       ??_C@_15EDMHLDMO@?$AAc?$AAa?$AA?$AA@ 0000000180004640     libucrt:lcidtoname_downlevel.obj
 0001:00003648       ??_C@_1O@BPEAJADD@?$AAz?$AAh?$AA?9?$AAC?$AAH?$AAS?$AA?$AA@ 0000000180004648     libucrt:lcidtoname_downlevel.obj
 0001:00003658       ??_C@_15LJNHCMNK@?$AAc?$AAs?$AA?$AA@ 0000000180004658     libucrt:lcidtoname_downlevel.obj
 0001:00003660       ??_C@_15FOMCIDHG@?$AAd?$AAa?$AA?$AA@ 0000000180004660     libucrt:lcidtoname_downlevel.obj
 0001:00003668       ??_C@_15NBKABECB@?$AAd?$AAe?$AA?$AA@ 0000000180004668     libucrt:lcidtoname_downlevel.obj
 0001:00003670       ??_C@_15GHPEIIAO@?$AAe?$AAl?$AA?$AA@ 0000000180004670     libucrt:lcidtoname_downlevel.obj
 0001:00003678       ??_C@_15MNPNEAIF@?$AAe?$AAn?$AA?$AA@ 0000000180004678     libucrt:lcidtoname_downlevel.obj
 0001:00003680       ??_C@_15GPIOMPMH@?$AAe?$AAs?$AA?$AA@ 0000000180004680     libucrt:lcidtoname_downlevel.obj
 0001:00003688       ??_C@_15NGLOAKJC@?$AAf?$AAi?$AA?$AA@ 0000000180004688     libucrt:lcidtoname_downlevel.obj
 0001:00003690       ??_C@_15FBKGNKAM@?$AAf?$AAr?$AA?$AA@ 0000000180004690     libucrt:lcidtoname_downlevel.obj
 0001:00003698       ??_C@_15KGGCNEFK@?$AAh?$AAe?$AA?$AA@ 0000000180004698     libucrt:lcidtoname_downlevel.obj
 0001:000036a0       ??_C@_15PGHLIDMF@?$AAh?$AAu?$AA?$AA@ 00000001800046a0     libucrt:lcidtoname_downlevel.obj
 0001:000036a8       ??_C@_15BIEMAPLM@?$AAi?$AAs?$AA?$AA@ 00000001800046a8     libucrt:lcidtoname_downlevel.obj
 0001:000036b0       ??_C@_15IFJLDHAF@?$AAi?$AAt?$AA?$AA@ 00000001800046b0     libucrt:lcidtoname_downlevel.obj
 0001:000036b8       ??_C@_15GEMIOCAG@?$AAj?$AAa?$AA?$AA@ 00000001800046b8     libucrt:lcidtoname_downlevel.obj
 0001:000036c0       ??_C@_15EPELEGJA@?$AAk?$AAo?$AA?$AA@ 00000001800046c0     libucrt:lcidtoname_downlevel.obj
 0001:000036c8       ??_C@_15NDDHIMN@?$AAn?$AAl?$AA?$AA@ 00000001800046c8     libucrt:lcidtoname_downlevel.obj
 0001:000036d0       ??_C@_15BPIGNHCD@?$AAn?$AAo?$AA?$AA@ 00000001800046d0     libucrt:lcidtoname_downlevel.obj
 0001:000036d8       ??_C@_15DEOPBLCG@?$AAp?$AAl?$AA?$AA@ 00000001800046d8     libucrt:lcidtoname_downlevel.obj
 0001:000036e0       ??_C@_15KBECGEFG@?$AAp?$AAt?$AA?$AA@ 00000001800046e0     libucrt:lcidtoname_downlevel.obj
 0001:000036e8       ??_C@_15GLJCBFMD@?$AAr?$AAo?$AA?$AA@ 00000001800046e8     libucrt:lcidtoname_downlevel.obj
 0001:000036f0       ??_C@_15FEDGKCDI@?$AAr?$AAu?$AA?$AA@ 00000001800046f0     libucrt:lcidtoname_downlevel.obj
 0001:000036f8       ??_C@_15GLKMLLHM@?$AAh?$AAr?$AA?$AA@ 00000001800046f8     libucrt:lcidtoname_downlevel.obj
 0001:00003700       ??_C@_15CPKMFBDB@?$AAs?$AAk?$AA?$AA@ 0000000180004700     libucrt:lcidtoname_downlevel.obj
 0001:00003708       ??_C@_15BAAIOGMK@?$AAs?$AAq?$AA?$AA@ 0000000180004708     libucrt:lcidtoname_downlevel.obj
 0001:00003710       ??_C@_15INNPNOHD@?$AAs?$AAv?$AA?$AA@ 0000000180004710     libucrt:lcidtoname_downlevel.obj
 0001:00003718       ??_C@_15CABMMOGH@?$AAt?$AAh?$AA?$AA@ 0000000180004718     libucrt:lcidtoname_downlevel.obj
 0001:00003720       ??_C@_15BPLIHJJM@?$AAt?$AAr?$AA?$AA@ 0000000180004720     libucrt:lcidtoname_downlevel.obj
 0001:00003728       ??_C@_15NEOEKKDJ@?$AAu?$AAr?$AA?$AA@ 0000000180004728     libucrt:lcidtoname_downlevel.obj
 0001:00003730       ??_C@_15NFICGAJK@?$AAi?$AAd?$AA?$AA@ 0000000180004730     libucrt:lcidtoname_downlevel.obj
 0001:00003738       ??_C@_15PJPFLCCM@?$AAu?$AAk?$AA?$AA@ 0000000180004738     libucrt:lcidtoname_downlevel.obj
 0001:00003740       ??_C@_15HPJPHDM@?$AAb?$AAe?$AA?$AA@ 0000000180004740     libucrt:lcidtoname_downlevel.obj
 0001:00003748       ??_C@_15LCHLGJII@?$AAs?$AAl?$AA?$AA@ 0000000180004748     libucrt:lcidtoname_downlevel.obj
 0001:00003750       ??_C@_15PCFJPHHO@?$AAe?$AAt?$AA?$AA@ 0000000180004750     libucrt:lcidtoname_downlevel.obj
 0001:00003758       ??_C@_15HPFPGODN@?$AAl?$AAv?$AA?$AA@ 0000000180004758     libucrt:lcidtoname_downlevel.obj
 0001:00003760       ??_C@_15NFFGKGLG@?$AAl?$AAt?$AA?$AA@ 0000000180004760     libucrt:lcidtoname_downlevel.obj
 0001:00003768       ??_C@_15BDAKCCHN@?$AAf?$AAa?$AA?$AA@ 0000000180004768     libucrt:lcidtoname_downlevel.obj
 0001:00003770       ??_C@_15NFGIAIAJ@?$AAv?$AAi?$AA?$AA@ 0000000180004770     libucrt:lcidtoname_downlevel.obj
 0001:00003778       ??_C@_15LMKNDMHN@?$AAh?$AAy?$AA?$AA@ 0000000180004778     libucrt:lcidtoname_downlevel.obj
 0001:00003780       ??_C@_15IJBHMCFL@?$AAa?$AAz?$AA?$AA@ 0000000180004780     libucrt:lcidtoname_downlevel.obj
 0001:00003788       ??_C@_15EKOFJABL@?$AAe?$AAu?$AA?$AA@ 0000000180004788     libucrt:lcidtoname_downlevel.obj
 0001:00003790       ??_C@_15BGHADCNK@?$AAm?$AAk?$AA?$AA@ 0000000180004790     libucrt:lcidtoname_downlevel.obj
 0001:00003798       ??_C@_15JDNICKHM@?$AAa?$AAf?$AA?$AA@ 0000000180004798     libucrt:lcidtoname_downlevel.obj
 0001:000037a0       ??_C@_15KPJEDBKD@?$AAk?$AAa?$AA?$AA@ 00000001800047a0     libucrt:lcidtoname_downlevel.obj
 0001:000037a8       ??_C@_15PDNFFFEO@?$AAf?$AAo?$AA?$AA@ 00000001800047a8     libucrt:lcidtoname_downlevel.obj
 0001:000037b0       ??_C@_15OMLEGLOC@?$AAh?$AAi?$AA?$AA@ 00000001800047b0     libucrt:lcidtoname_downlevel.obj
 0001:000037b8       ??_C@_15IDNNENKK@?$AAm?$AAs?$AA?$AA@ 00000001800047b8     libucrt:lcidtoname_downlevel.obj
 0001:000037c0       ??_C@_15MACJNBMH@?$AAk?$AAk?$AA?$AA@ 00000001800047c0     libucrt:lcidtoname_downlevel.obj
 0001:000037c8       ??_C@_15DKDJEOND@?$AAk?$AAy?$AA?$AA@ 00000001800047c8     libucrt:lcidtoname_downlevel.obj
 0001:000037d0       ??_C@_15DFGDLJBG@?$AAs?$AAw?$AA?$AA@ 00000001800047d0     libucrt:lcidtoname_downlevel.obj
 0001:000037d8       ??_C@_15BBFAICNG@?$AAu?$AAz?$AA?$AA@ 00000001800047d8     libucrt:lcidtoname_downlevel.obj
 0001:000037e0       ??_C@_15DKNDCGEA@?$AAt?$AAt?$AA?$AA@ 00000001800047e0     libucrt:lcidtoname_downlevel.obj
 0001:000037e8       ??_C@_15MGIFMDPL@?$AAp?$AAa?$AA?$AA@ 00000001800047e8     libucrt:lcidtoname_downlevel.obj
 0001:000037f0       ??_C@_15HCNDBBA@?$AAg?$AAu?$AA?$AA@ 00000001800047f0     libucrt:lcidtoname_downlevel.obj
 0001:000037f8       ??_C@_15FNBEIBON@?$AAt?$AAa?$AA?$AA@ 00000001800047f8     libucrt:lcidtoname_downlevel.obj
 0001:00003800       ??_C@_15NCHGBGLK@?$AAt?$AAe?$AA?$AA@ 0000000180004800     libucrt:lcidtoname_downlevel.obj
 0001:00003808       ??_C@_15PHPHCBPF@?$AAk?$AAn?$AA?$AA@ 0000000180004808     libucrt:lcidtoname_downlevel.obj
 0001:00003810       ??_C@_15DLGBCKMP@?$AAm?$AAr?$AA?$AA@ 0000000180004810     libucrt:lcidtoname_downlevel.obj
 0001:00003818       ??_C@_15EABBLBFF@?$AAs?$AAa?$AA?$AA@ 0000000180004818     libucrt:lcidtoname_downlevel.obj
 0001:00003820       ??_C@_15CBKOMCOI@?$AAm?$AAn?$AA?$AA@ 0000000180004820     libucrt:lcidtoname_downlevel.obj
 0001:00003828       ??_C@_15CKDMCJAF@?$AAg?$AAl?$AA?$AA@ 0000000180004828     libucrt:lcidtoname_downlevel.obj
 0001:00003830       ??_C@_17CNJFBPG@?$AAk?$AAo?$AAk?$AA?$AA@ 0000000180004830     libucrt:lcidtoname_downlevel.obj
 0001:00003838       ??_C@_17FFBJICPL@?$AAs?$AAy?$AAr?$AA?$AA@ 0000000180004838     libucrt:lcidtoname_downlevel.obj
 0001:00003840       ??_C@_17KPNDCPAF@?$AAd?$AAi?$AAv?$AA?$AA@ 0000000180004840     libucrt:lcidtoname_downlevel.obj
 0001:00003848       ??_C@_1M@OKAHONE@?$AAa?$AAr?$AA?9?$AAS?$AAA?$AA?$AA@ 0000000180004848     libucrt:lcidtoname_downlevel.obj
 0001:00003858       ??_C@_1M@FFFIGIGK@?$AAb?$AAg?$AA?9?$AAB?$AAG?$AA?$AA@ 0000000180004858     libucrt:lcidtoname_downlevel.obj
 0001:00003868       ??_C@_1M@BJNKEDC@?$AAc?$AAa?$AA?9?$AAE?$AAS?$AA?$AA@ 0000000180004868     libucrt:lcidtoname_downlevel.obj
 0001:00003878       ??_C@_1M@IJJHFJHA@?$AAc?$AAs?$AA?9?$AAC?$AAZ?$AA?$AA@ 0000000180004878     libucrt:lcidtoname_downlevel.obj
 0001:00003888       ??_C@_1M@CLPEOBGI@?$AAd?$AAa?$AA?9?$AAD?$AAK?$AA?$AA@ 0000000180004888     libucrt:lcidtoname_downlevel.obj
 0001:00003898       ??_C@_1M@MCMADGCB@?$AAd?$AAe?$AA?9?$AAD?$AAE?$AA?$AA@ 0000000180004898     libucrt:lcidtoname_downlevel.obj
 0001:000038a8       ??_C@_1M@OOCKEMAM@?$AAe?$AAl?$AA?9?$AAG?$AAR?$AA?$AA@ 00000001800048a8     libucrt:lcidtoname_downlevel.obj
 0001:000038b8       ??_C@_1M@DDNJFGID@?$AAf?$AAi?$AA?9?$AAF?$AAI?$AA?$AA@ 00000001800048b8     libucrt:lcidtoname_downlevel.obj
 0001:000038c8       ??_C@_1M@GLIPPMAC@?$AAf?$AAr?$AA?9?$AAF?$AAR?$AA?$AA@ 00000001800048c8     libucrt:lcidtoname_downlevel.obj
 0001:000038d8       ??_C@_1M@GFMCHPE@?$AAh?$AAe?$AA?9?$AAI?$AAL?$AA?$AA@ 00000001800048d8     libucrt:lcidtoname_downlevel.obj
 0001:000038e8       ??_C@_1M@MHLPGNKM@?$AAh?$AAu?$AA?9?$AAH?$AAU?$AA?$AA@ 00000001800048e8     libucrt:lcidtoname_downlevel.obj
 0001:000038f8       ??_C@_1M@LPDDNNPN@?$AAi?$AAs?$AA?9?$AAI?$AAS?$AA?$AA@ 00000001800048f8     libucrt:lcidtoname_downlevel.obj
 0001:00003908       ??_C@_1M@MADIPODN@?$AAi?$AAt?$AA?9?$AAI?$AAT?$AA?$AA@ 0000000180004908     libucrt:lcidtoname_downlevel.obj
 0001:00003918       ??_C@_1M@IHBJJGG@?$AAn?$AAl?$AA?9?$AAN?$AAL?$AA?$AA@ 0000000180004918     libucrt:lcidtoname_downlevel.obj
 0001:00003928       ??_C@_1M@EANAGDL@?$AAn?$AAb?$AA?9?$AAN?$AAO?$AA?$AA@ 0000000180004928     libucrt:lcidtoname_downlevel.obj
 0001:00003938       ??_C@_1M@NEIEMEGP@?$AAp?$AAl?$AA?9?$AAP?$AAL?$AA?$AA@ 0000000180004938     libucrt:lcidtoname_downlevel.obj
 0001:00003948       ??_C@_1M@BOCFIGEP@?$AAp?$AAt?$AA?9?$AAB?$AAR?$AA?$AA@ 0000000180004948     libucrt:lcidtoname_downlevel.obj
 0001:00003958       ??_C@_1M@IMPFOPBG@?$AAr?$AAo?$AA?9?$AAR?$AAO?$AA?$AA@ 0000000180004958     libucrt:lcidtoname_downlevel.obj
 0001:00003968       ??_C@_1M@IDNNEJMM@?$AAr?$AAu?$AA?9?$AAR?$AAU?$AA?$AA@ 0000000180004968     libucrt:lcidtoname_downlevel.obj
 0001:00003978       ??_C@_1M@LILEEOGM@?$AAh?$AAr?$AA?9?$AAH?$AAR?$AA?$AA@ 0000000180004978     libucrt:lcidtoname_downlevel.obj
 0001:00003988       ??_C@_1M@FKIFEHPB@?$AAs?$AAk?$AA?9?$AAS?$AAK?$AA?$AA@ 0000000180004988     libucrt:lcidtoname_downlevel.obj
 0001:00003998       ??_C@_1M@LJMAMNPJ@?$AAs?$AAq?$AA?9?$AAA?$AAL?$AA?$AA@ 0000000180004998     libucrt:lcidtoname_downlevel.obj
 0001:000039a8       ??_C@_1M@GIAKDKJK@?$AAs?$AAv?$AA?9?$AAS?$AAE?$AA?$AA@ 00000001800049a8     libucrt:lcidtoname_downlevel.obj
 0001:000039b8       ??_C@_1M@MKJKIKCL@?$AAt?$AAh?$AA?9?$AAT?$AAH?$AA?$AA@ 00000001800049b8     libucrt:lcidtoname_downlevel.obj
 0001:000039c8       ??_C@_1M@MFLCCMPB@?$AAt?$AAr?$AA?9?$AAT?$AAR?$AA?$AA@ 00000001800049c8     libucrt:lcidtoname_downlevel.obj
 0001:000039d8       ??_C@_1M@OIJHDKJN@?$AAu?$AAr?$AA?9?$AAP?$AAK?$AA?$AA@ 00000001800049d8     libucrt:lcidtoname_downlevel.obj
 0001:000039e8       ??_C@_1M@LHIPCIEK@?$AAi?$AAd?$AA?9?$AAI?$AAD?$AA?$AA@ 00000001800049e8     libucrt:lcidtoname_downlevel.obj
 0001:000039f8       ??_C@_1M@MFMOBGI@?$AAu?$AAk?$AA?9?$AAU?$AAA?$AA?$AA@ 00000001800049f8     libucrt:lcidtoname_downlevel.obj
 0001:00003a08       ??_C@_1M@OBGLJIPL@?$AAb?$AAe?$AA?9?$AAB?$AAY?$AA?$AA@ 0000000180004a08     libucrt:lcidtoname_downlevel.obj
 0001:00003a18       ??_C@_1M@BCFAJEAD@?$AAs?$AAl?$AA?9?$AAS?$AAI?$AA?$AA@ 0000000180004a18     libucrt:lcidtoname_downlevel.obj
 0001:00003a28       ??_C@_1M@FKFFEDDN@?$AAe?$AAt?$AA?9?$AAE?$AAE?$AA?$AA@ 0000000180004a28     libucrt:lcidtoname_downlevel.obj
 0001:00003a38       ??_C@_1M@KGKKAACI@?$AAl?$AAv?$AA?9?$AAL?$AAV?$AA?$AA@ 0000000180004a38     libucrt:lcidtoname_downlevel.obj
 0001:00003a48       ??_C@_1M@IFGBIJO@?$AAl?$AAt?$AA?9?$AAL?$AAT?$AA?$AA@ 0000000180004a48     libucrt:lcidtoname_downlevel.obj
 0001:00003a58       ??_C@_1M@FGEAHEDM@?$AAf?$AAa?$AA?9?$AAI?$AAR?$AA?$AA@ 0000000180004a58     libucrt:lcidtoname_downlevel.obj
 0001:00003a68       ??_C@_1M@KBMAIBFN@?$AAv?$AAi?$AA?9?$AAV?$AAN?$AA?$AA@ 0000000180004a68     libucrt:lcidtoname_downlevel.obj
 0001:00003a78       ??_C@_1M@GPCBKDJK@?$AAh?$AAy?$AA?9?$AAA?$AAM?$AA?$AA@ 0000000180004a78     libucrt:lcidtoname_downlevel.obj
 0001:00003a88       ??_C@_1BG@BECMDDJB@?$AAa?$AAz?$AA?9?$AAA?$AAZ?$AA?9?$AAL?$AAa?$AAt?$AAn?$AA?$AA@ 0000000180004a88     libucrt:lcidtoname_downlevel.obj
 0001:00003aa0       ??_C@_1M@MAOFCAEA@?$AAe?$AAu?$AA?9?$AAE?$AAS?$AA?$AA@ 0000000180004aa0     libucrt:lcidtoname_downlevel.obj
 0001:00003ab0       ??_C@_1M@IGHABKPI@?$AAm?$AAk?$AA?9?$AAM?$AAK?$AA?$AA@ 0000000180004ab0     libucrt:lcidtoname_downlevel.obj
 0001:00003ac0       ??_C@_1M@IAIGNEJG@?$AAt?$AAn?$AA?9?$AAZ?$AAA?$AA?$AA@ 0000000180004ac0     libucrt:lcidtoname_downlevel.obj
 0001:00003ad0       ??_C@_1M@IIJCOJFA@?$AAx?$AAh?$AA?9?$AAZ?$AAA?$AA?$AA@ 0000000180004ad0     libucrt:lcidtoname_downlevel.obj
 0001:00003ae0       ??_C@_1M@LGPJHNJH@?$AAz?$AAu?$AA?9?$AAZ?$AAA?$AA?$AA@ 0000000180004ae0     libucrt:lcidtoname_downlevel.obj
 0001:00003af0       ??_C@_1M@HOKAOIO@?$AAa?$AAf?$AA?9?$AAZ?$AAA?$AA?$AA@ 0000000180004af0     libucrt:lcidtoname_downlevel.obj
 0001:00003b00       ??_C@_1M@DPCLHLIE@?$AAk?$AAa?$AA?9?$AAG?$AAE?$AA?$AA@ 0000000180004b00     libucrt:lcidtoname_downlevel.obj
 0001:00003b10       ??_C@_1M@BLKMHJBI@?$AAf?$AAo?$AA?9?$AAF?$AAO?$AA?$AA@ 0000000180004b10     libucrt:lcidtoname_downlevel.obj
 0001:00003b20       ??_C@_1M@LGGJAPPB@?$AAh?$AAi?$AA?9?$AAI?$AAN?$AA?$AA@ 0000000180004b20     libucrt:lcidtoname_downlevel.obj
 0001:00003b30       ??_C@_1M@FIKPIHFE@?$AAm?$AAt?$AA?9?$AAM?$AAT?$AA?$AA@ 0000000180004b30     libucrt:lcidtoname_downlevel.obj
 0001:00003b40       ??_C@_1M@HEGGPBFA@?$AAs?$AAe?$AA?9?$AAN?$AAO?$AA?$AA@ 0000000180004b40     libucrt:lcidtoname_downlevel.obj
 0001:00003b50       ??_C@_1M@EIBJEEPA@?$AAm?$AAs?$AA?9?$AAM?$AAY?$AA?$AA@ 0000000180004b50     libucrt:lcidtoname_downlevel.obj
 0001:00003b60       ??_C@_1M@FHLBGMPP@?$AAk?$AAk?$AA?9?$AAK?$AAZ?$AA?$AA@ 0000000180004b60     libucrt:lcidtoname_downlevel.obj
 0001:00003b70       ??_C@_1M@NGJJLCGI@?$AAk?$AAy?$AA?9?$AAK?$AAG?$AA?$AA@ 0000000180004b70     libucrt:lcidtoname_downlevel.obj
 0001:00003b80       ??_C@_1M@GIENNBFC@?$AAs?$AAw?$AA?9?$AAK?$AAE?$AA?$AA@ 0000000180004b80     libucrt:lcidtoname_downlevel.obj
 0001:00003b90       ??_C@_1BG@NDGMJIMJ@?$AAu?$AAz?$AA?9?$AAU?$AAZ?$AA?9?$AAL?$AAa?$AAt?$AAn?$AA?$AA@ 0000000180004b90     libucrt:lcidtoname_downlevel.obj
 0001:00003ba8       ??_C@_1M@IDCCIHBC@?$AAt?$AAt?$AA?9?$AAR?$AAU?$AA?$AA@ 0000000180004ba8     libucrt:lcidtoname_downlevel.obj
 0001:00003bb8       ??_C@_1M@LOICPMOJ@?$AAb?$AAn?$AA?9?$AAI?$AAN?$AA?$AA@ 0000000180004bb8     libucrt:lcidtoname_downlevel.obj
 0001:00003bc8       ??_C@_1M@KPKKNEAH@?$AAp?$AAa?$AA?9?$AAI?$AAN?$AA?$AA@ 0000000180004bc8     libucrt:lcidtoname_downlevel.obj
 0001:00003bd8       ??_C@_1M@PJGPPBOG@?$AAg?$AAu?$AA?9?$AAI?$AAN?$AA?$AA@ 0000000180004bd8     libucrt:lcidtoname_downlevel.obj
 0001:00003be8       ??_C@_1M@KMKMOPHI@?$AAt?$AAa?$AA?9?$AAI?$AAN?$AA?$AA@ 0000000180004be8     libucrt:lcidtoname_downlevel.obj
 0001:00003bf8       ??_C@_1M@KFEHEPAC@?$AAt?$AAe?$AA?9?$AAI?$AAN?$AA?$AA@ 0000000180004bf8     libucrt:lcidtoname_downlevel.obj
 0001:00003c08       ??_C@_1M@CDCLMGHI@?$AAk?$AAn?$AA?9?$AAI?$AAN?$AA?$AA@ 0000000180004c08     libucrt:lcidtoname_downlevel.obj
 0001:00003c18       ??_C@_1M@MIODLDKF@?$AAm?$AAl?$AA?9?$AAI?$AAN?$AA?$AA@ 0000000180004c18     libucrt:lcidtoname_downlevel.obj
 0001:00003c28       ??_C@_1M@PBIEACPO@?$AAm?$AAr?$AA?9?$AAI?$AAN?$AA?$AA@ 0000000180004c28     libucrt:lcidtoname_downlevel.obj
 0001:00003c38       ??_C@_1M@NIDEAGPH@?$AAs?$AAa?$AA?9?$AAI?$AAN?$AA?$AA@ 0000000180004c38     libucrt:lcidtoname_downlevel.obj
 0001:00003c48       ??_C@_1M@FHIHCBIO@?$AAm?$AAn?$AA?9?$AAM?$AAN?$AA?$AA@ 0000000180004c48     libucrt:lcidtoname_downlevel.obj
 0001:00003c58       ??_C@_1M@JAIJPENP@?$AAc?$AAy?$AA?9?$AAG?$AAB?$AA?$AA@ 0000000180004c58     libucrt:lcidtoname_downlevel.obj
 0001:00003c68       ??_C@_1M@PHGFBEPN@?$AAg?$AAl?$AA?9?$AAE?$AAS?$AA?$AA@ 0000000180004c68     libucrt:lcidtoname_downlevel.obj
 0001:00003c78       ??_C@_1O@KPIPDNCP@?$AAk?$AAo?$AAk?$AA?9?$AAI?$AAN?$AA?$AA@ 0000000180004c78     libucrt:lcidtoname_downlevel.obj
 0001:00003c88       ??_C@_1O@KNHJLDJA@?$AAs?$AAy?$AAr?$AA?9?$AAS?$AAY?$AA?$AA@ 0000000180004c88     libucrt:lcidtoname_downlevel.obj
 0001:00003c98       ??_C@_1O@MKEKBLAH@?$AAd?$AAi?$AAv?$AA?9?$AAM?$AAV?$AA?$AA@ 0000000180004c98     libucrt:lcidtoname_downlevel.obj
 0001:00003ca8       ??_C@_1O@OHDCKDDF@?$AAq?$AAu?$AAz?$AA?9?$AAB?$AAO?$AA?$AA@ 0000000180004ca8     libucrt:lcidtoname_downlevel.obj
 0001:00003cb8       ??_C@_1M@LEPJNLFD@?$AAn?$AAs?$AA?9?$AAZ?$AAA?$AA?$AA@ 0000000180004cb8     libucrt:lcidtoname_downlevel.obj
 0001:00003cc8       ??_C@_1M@OMLEIIJB@?$AAm?$AAi?$AA?9?$AAN?$AAZ?$AA?$AA@ 0000000180004cc8     libucrt:lcidtoname_downlevel.obj
 0001:00003cd8       ??_C@_1M@PMPEAILG@?$AAa?$AAr?$AA?9?$AAI?$AAQ?$AA?$AA@ 0000000180004cd8     libucrt:lcidtoname_downlevel.obj
 0001:00003ce8       ??_C@_1M@CNKPNOEE@?$AAd?$AAe?$AA?9?$AAC?$AAH?$AA?$AA@ 0000000180004ce8     libucrt:lcidtoname_downlevel.obj
 0001:00003cf8       ??_C@_1M@LKMGMLKO@?$AAe?$AAn?$AA?9?$AAG?$AAB?$AA?$AA@ 0000000180004cf8     libucrt:lcidtoname_downlevel.obj
 0001:00003d08       ??_C@_1M@PGKJFFGL@?$AAe?$AAs?$AA?9?$AAM?$AAX?$AA?$AA@ 0000000180004d08     libucrt:lcidtoname_downlevel.obj
 0001:00003d18       ??_C@_1M@DNNANBDC@?$AAf?$AAr?$AA?9?$AAB?$AAE?$AA?$AA@ 0000000180004d18     libucrt:lcidtoname_downlevel.obj
 0001:00003d28       ??_C@_1M@HLGMDFHM@?$AAi?$AAt?$AA?9?$AAC?$AAH?$AA?$AA@ 0000000180004d28     libucrt:lcidtoname_downlevel.obj
 0001:00003d38       ??_C@_1M@CLLBGJH@?$AAn?$AAl?$AA?9?$AAB?$AAE?$AA?$AA@ 0000000180004d38     libucrt:lcidtoname_downlevel.obj
 0001:00003d48       ??_C@_1M@BODBOGLF@?$AAn?$AAn?$AA?9?$AAN?$AAO?$AA?$AA@ 0000000180004d48     libucrt:lcidtoname_downlevel.obj
 0001:00003d58       ??_C@_1M@HFFAHKAD@?$AAp?$AAt?$AA?9?$AAP?$AAT?$AA?$AA@ 0000000180004d58     libucrt:lcidtoname_downlevel.obj
 0001:00003d68       ??_C@_1BG@LNOAKHIE@?$AAs?$AAr?$AA?9?$AAS?$AAP?$AA?9?$AAL?$AAa?$AAt?$AAn?$AA?$AA@ 0000000180004d68     libucrt:lcidtoname_downlevel.obj
 0001:00003d80       ??_C@_1M@HBMHBGAK@?$AAs?$AAv?$AA?9?$AAF?$AAI?$AA?$AA@ 0000000180004d80     libucrt:lcidtoname_downlevel.obj
 0001:00003d90       ??_C@_1BG@DGCJGJBE@?$AAa?$AAz?$AA?9?$AAA?$AAZ?$AA?9?$AAC?$AAy?$AAr?$AAl?$AA?$AA@ 0000000180004d90     libucrt:lcidtoname_downlevel.obj
 0001:00003da8       ??_C@_1M@KEJDAAHB@?$AAs?$AAe?$AA?9?$AAS?$AAE?$AA?$AA@ 0000000180004da8     libucrt:lcidtoname_downlevel.obj
 0001:00003db8       ??_C@_1M@HEIBJJAD@?$AAm?$AAs?$AA?9?$AAB?$AAN?$AA?$AA@ 0000000180004db8     libucrt:lcidtoname_downlevel.obj
 0001:00003dc8       ??_C@_1BG@PBGJMCEM@?$AAu?$AAz?$AA?9?$AAU?$AAZ?$AA?9?$AAC?$AAy?$AAr?$AAl?$AA?$AA@ 0000000180004dc8     libucrt:lcidtoname_downlevel.obj
 0001:00003de0       ??_C@_1O@LAOBCMDF@?$AAq?$AAu?$AAz?$AA?9?$AAE?$AAC?$AA?$AA@ 0000000180004de0     libucrt:lcidtoname_downlevel.obj
 0001:00003df0       ??_C@_1M@POEEMAIO@?$AAa?$AAr?$AA?9?$AAE?$AAG?$AA?$AA@ 0000000180004df0     libucrt:lcidtoname_downlevel.obj
 0001:00003e00       ??_C@_1M@EFAKDEDL@?$AAz?$AAh?$AA?9?$AAH?$AAK?$AA?$AA@ 0000000180004e00     libucrt:lcidtoname_downlevel.obj
 0001:00003e10       ??_C@_1M@HKKIJHGI@?$AAd?$AAe?$AA?9?$AAA?$AAT?$AA?$AA@ 0000000180004e10     libucrt:lcidtoname_downlevel.obj
 0001:00003e20       ??_C@_1M@KBFBEHJF@?$AAe?$AAn?$AA?9?$AAA?$AAU?$AA?$AA@ 0000000180004e20     libucrt:lcidtoname_downlevel.obj
 0001:00003e30       ??_C@_1M@MNPLFAAH@?$AAe?$AAs?$AA?9?$AAE?$AAS?$AA?$AA@ 0000000180004e30     libucrt:lcidtoname_downlevel.obj
 0001:00003e40       ??_C@_1M@HJOOJFMA@?$AAf?$AAr?$AA?9?$AAC?$AAA?$AA?$AA@ 0000000180004e40     libucrt:lcidtoname_downlevel.obj
 0001:00003e50       ??_C@_1BG@JPOFPNAB@?$AAs?$AAr?$AA?9?$AAS?$AAP?$AA?9?$AAC?$AAy?$AAr?$AAl?$AA?$AA@ 0000000180004e50     libucrt:lcidtoname_downlevel.obj
 0001:00003e68       ??_C@_1M@LNFOCMOB@?$AAs?$AAe?$AA?9?$AAF?$AAI?$AA?$AA@ 0000000180004e68     libucrt:lcidtoname_downlevel.obj
 0001:00003e78       ??_C@_1O@MGJBOAMB@?$AAq?$AAu?$AAz?$AA?9?$AAP?$AAE?$AA?$AA@ 0000000180004e78     libucrt:lcidtoname_downlevel.obj
 0001:00003e88       ??_C@_1M@GJINLBOK@?$AAa?$AAr?$AA?9?$AAL?$AAY?$AA?$AA@ 0000000180004e88     libucrt:lcidtoname_downlevel.obj
 0001:00003e98       ??_C@_1M@GGMNHJNL@?$AAz?$AAh?$AA?9?$AAS?$AAG?$AA?$AA@ 0000000180004e98     libucrt:lcidtoname_downlevel.obj
 0001:00003ea8       ??_C@_1M@HOIKODND@?$AAd?$AAe?$AA?9?$AAL?$AAU?$AA?$AA@ 0000000180004ea8     libucrt:lcidtoname_downlevel.obj
 0001:00003eb8       ??_C@_1M@DDOCCGFG@?$AAe?$AAn?$AA?9?$AAC?$AAA?$AA?$AA@ 0000000180004eb8     libucrt:lcidtoname_downlevel.obj
 0001:00003ec8       ??_C@_1M@BNOEMJLF@?$AAe?$AAs?$AA?9?$AAG?$AAT?$AA?$AA@ 0000000180004ec8     libucrt:lcidtoname_downlevel.obj
 0001:00003ed8       ??_C@_1M@EOGNKEK@?$AAf?$AAr?$AA?9?$AAC?$AAH?$AA?$AA@ 0000000180004ed8     libucrt:lcidtoname_downlevel.obj
 0001:00003ee8       ??_C@_1M@FLIDJFHL@?$AAh?$AAr?$AA?9?$AAB?$AAA?$AA?$AA@ 0000000180004ee8     libucrt:lcidtoname_downlevel.obj
 0001:00003ef8       ??_C@_1O@FMCELNAJ@?$AAs?$AAm?$AAj?$AA?9?$AAN?$AAO?$AA?$AA@ 0000000180004ef8     libucrt:lcidtoname_downlevel.obj
 0001:00003f08       ??_C@_1M@JHGLJMGJ@?$AAa?$AAr?$AA?9?$AAD?$AAZ?$AA?$AA@ 0000000180004f08     libucrt:lcidtoname_downlevel.obj
 0001:00003f18       ??_C@_1M@JKKFDCNP@?$AAz?$AAh?$AA?9?$AAM?$AAO?$AA?$AA@ 0000000180004f18     libucrt:lcidtoname_downlevel.obj
 0001:00003f28       ??_C@_1M@GEEFALPE@?$AAd?$AAe?$AA?9?$AAL?$AAI?$AA?$AA@ 0000000180004f28     libucrt:lcidtoname_downlevel.obj
 0001:00003f38       ??_C@_1M@IGEOFBG@?$AAe?$AAn?$AA?9?$AAN?$AAZ?$AA?$AA@ 0000000180004f38     libucrt:lcidtoname_downlevel.obj
 0001:00003f48       ??_C@_1M@KDBONEHP@?$AAe?$AAs?$AA?9?$AAC?$AAR?$AA?$AA@ 0000000180004f48     libucrt:lcidtoname_downlevel.obj
 0001:00003f58       ??_C@_1M@FHMDOHNN@?$AAf?$AAr?$AA?9?$AAL?$AAU?$AA?$AA@ 0000000180004f58     libucrt:lcidtoname_downlevel.obj
 0001:00003f68       ??_C@_1BG@NFKKMAFG@?$AAb?$AAs?$AA?9?$AAB?$AAA?$AA?9?$AAL?$AAa?$AAt?$AAn?$AA?$AA@ 0000000180004f68     libucrt:lcidtoname_downlevel.obj
 0001:00003f80       ??_C@_1O@IMNBEMCI@?$AAs?$AAm?$AAj?$AA?9?$AAS?$AAE?$AA?$AA@ 0000000180004f80     libucrt:lcidtoname_downlevel.obj
 0001:00003f90       ??_C@_1M@DHHMBNDP@?$AAa?$AAr?$AA?9?$AAM?$AAA?$AA?$AA@ 0000000180004f90     libucrt:lcidtoname_downlevel.obj
 0001:00003fa0       ??_C@_1M@BNBLJCGH@?$AAe?$AAn?$AA?9?$AAI?$AAE?$AA?$AA@ 0000000180004fa0     libucrt:lcidtoname_downlevel.obj
 0001:00003fb0       ??_C@_1M@GEPAFMDL@?$AAe?$AAs?$AA?9?$AAP?$AAA?$AA?$AA@ 0000000180004fb0     libucrt:lcidtoname_downlevel.obj
 0001:00003fc0       ??_C@_1M@OJONDMDL@?$AAf?$AAr?$AA?9?$AAM?$AAC?$AA?$AA@ 0000000180004fc0     libucrt:lcidtoname_downlevel.obj
 0001:00003fd0       ??_C@_1BG@OBCNFJB@?$AAs?$AAr?$AA?9?$AAB?$AAA?$AA?9?$AAL?$AAa?$AAt?$AAn?$AA?$AA@ 0000000180004fd0     libucrt:lcidtoname_downlevel.obj
 0001:00003fe8       ??_C@_1O@KEMEEGPO@?$AAs?$AAm?$AAa?$AA?9?$AAN?$AAO?$AA?$AA@ 0000000180004fe8     libucrt:lcidtoname_downlevel.obj
 0001:00003ff8       ??_C@_1M@ELMGFODK@?$AAa?$AAr?$AA?9?$AAT?$AAN?$AA?$AA@ 0000000180004ff8     libucrt:lcidtoname_downlevel.obj
 0001:00004008       ??_C@_1M@BHDLHFAF@?$AAe?$AAn?$AA?9?$AAZ?$AAA?$AA?$AA@ 0000000180005008     libucrt:lcidtoname_downlevel.obj
 0001:00004018       ??_C@_1M@BMGIGLIF@?$AAe?$AAs?$AA?9?$AAD?$AAO?$AA?$AA@ 0000000180005018     libucrt:lcidtoname_downlevel.obj
 0001:00004028       ??_C@_1BG@CMBHIPBE@?$AAs?$AAr?$AA?9?$AAB?$AAA?$AA?9?$AAC?$AAy?$AAr?$AAl?$AA?$AA@ 0000000180005028     libucrt:lcidtoname_downlevel.obj
 0001:00004040       ??_C@_1O@HEDBLHNP@?$AAs?$AAm?$AAa?$AA?9?$AAS?$AAE?$AA?$AA@ 0000000180005040     libucrt:lcidtoname_downlevel.obj
 0001:00004050       ??_C@_1M@DAGCADIM@?$AAa?$AAr?$AA?9?$AAO?$AAM?$AA?$AA@ 0000000180005050     libucrt:lcidtoname_downlevel.obj
 0001:00004060       ??_C@_1M@FODLMICG@?$AAe?$AAn?$AA?9?$AAJ?$AAM?$AA?$AA@ 0000000180005060     libucrt:lcidtoname_downlevel.obj
 0001:00004070       ??_C@_1M@DNMLCIHB@?$AAe?$AAs?$AA?9?$AAV?$AAE?$AA?$AA@ 0000000180005070     libucrt:lcidtoname_downlevel.obj
 0001:00004080       ??_C@_1O@EOKHMKJK@?$AAs?$AAm?$AAs?$AA?9?$AAF?$AAI?$AA?$AA@ 0000000180005080     libucrt:lcidtoname_downlevel.obj
 0001:00004090       ??_C@_1M@CAFJMKOF@?$AAa?$AAr?$AA?9?$AAY?$AAE?$AA?$AA@ 0000000180005090     libucrt:lcidtoname_downlevel.obj
 0001:000040a0       ??_C@_1M@CBFHIJLI@?$AAe?$AAn?$AA?9?$AAC?$AAB?$AA?$AA@ 00000001800050a0     libucrt:lcidtoname_downlevel.obj
 0001:000040b0       ??_C@_1M@BGNFLDN@?$AAe?$AAs?$AA?9?$AAC?$AAO?$AA?$AA@ 00000001800050b0     libucrt:lcidtoname_downlevel.obj
 0001:000040c0       ??_C@_1O@JMPHMAMC@?$AAs?$AAm?$AAn?$AA?9?$AAF?$AAI?$AA?$AA@ 00000001800050c0     libucrt:lcidtoname_downlevel.obj
 0001:000040d0       ??_C@_1M@JLANABKE@?$AAa?$AAr?$AA?9?$AAS?$AAY?$AA?$AA@ 00000001800050d0     libucrt:lcidtoname_downlevel.obj
 0001:000040e0       ??_C@_1M@HPKGCFGN@?$AAe?$AAn?$AA?9?$AAB?$AAZ?$AA?$AA@ 00000001800050e0     libucrt:lcidtoname_downlevel.obj
 0001:000040f0       ??_C@_1M@OLJCMLGM@?$AAe?$AAs?$AA?9?$AAP?$AAE?$AA?$AA@ 00000001800050f0     libucrt:lcidtoname_downlevel.obj
 0001:00004100       ??_C@_1M@MKKGFKLE@?$AAa?$AAr?$AA?9?$AAJ?$AAO?$AA?$AA@ 0000000180005100     libucrt:lcidtoname_downlevel.obj
 0001:00004110       ??_C@_1M@EKPGLDNI@?$AAe?$AAn?$AA?9?$AAT?$AAT?$AA?$AA@ 0000000180005110     libucrt:lcidtoname_downlevel.obj
 0001:00004120       ??_C@_1M@OONGHFHE@?$AAe?$AAs?$AA?9?$AAA?$AAR?$AA?$AA@ 0000000180005120     libucrt:lcidtoname_downlevel.obj
 0001:00004130       ??_C@_1M@OOJFGBHE@?$AAa?$AAr?$AA?9?$AAL?$AAB?$AA?$AA@ 0000000180005130     libucrt:lcidtoname_downlevel.obj
 0001:00004140       ??_C@_1M@GCEJHNEG@?$AAe?$AAn?$AA?9?$AAZ?$AAW?$AA?$AA@ 0000000180005140     libucrt:lcidtoname_downlevel.obj
 0001:00004150       ??_C@_1M@JNOCAHJI@?$AAe?$AAs?$AA?9?$AAE?$AAC?$AA?$AA@ 0000000180005150     libucrt:lcidtoname_downlevel.obj
 0001:00004160       ??_C@_1M@JEFHPGGB@?$AAa?$AAr?$AA?9?$AAK?$AAW?$AA?$AA@ 0000000180005160     libucrt:lcidtoname_downlevel.obj
 0001:00004170       ??_C@_1M@MLKIBJOJ@?$AAe?$AAn?$AA?9?$AAP?$AAH?$AA?$AA@ 0000000180005170     libucrt:lcidtoname_downlevel.obj
 0001:00004180       ??_C@_1M@BDNIPEND@?$AAe?$AAs?$AA?9?$AAC?$AAL?$AA?$AA@ 0000000180005180     libucrt:lcidtoname_downlevel.obj
 0001:00004190       ??_C@_1M@MPNMEKBD@?$AAa?$AAr?$AA?9?$AAA?$AAE?$AA?$AA@ 0000000180005190     libucrt:lcidtoname_downlevel.obj
 0001:000041a0       ??_C@_1M@KBJALCPI@?$AAe?$AAs?$AA?9?$AAU?$AAY?$AA?$AA@ 00000001800051a0     libucrt:lcidtoname_downlevel.obj
 0001:000041b0       ??_C@_1M@LLCCOAGA@?$AAa?$AAr?$AA?9?$AAB?$AAH?$AA?$AA@ 00000001800051b0     libucrt:lcidtoname_downlevel.obj
 0001:000041c0       ??_C@_1M@PBFNCDEL@?$AAe?$AAs?$AA?9?$AAP?$AAY?$AA?$AA@ 00000001800051c0     libucrt:lcidtoname_downlevel.obj
 0001:000041d0       ??_C@_1M@EDGINPNP@?$AAa?$AAr?$AA?9?$AAQ?$AAA?$AA?$AA@ 00000001800051d0     libucrt:lcidtoname_downlevel.obj
 0001:000041e0       ??_C@_1M@MKDBIIJI@?$AAe?$AAs?$AA?9?$AAB?$AAO?$AA?$AA@ 00000001800051e0     libucrt:lcidtoname_downlevel.obj
 0001:000041f0       ??_C@_1M@CPKKEBLD@?$AAe?$AAs?$AA?9?$AAS?$AAV?$AA?$AA@ 00000001800051f0     libucrt:lcidtoname_downlevel.obj
 0001:00004200       ??_C@_1M@NDBGMMJL@?$AAe?$AAs?$AA?9?$AAH?$AAN?$AA?$AA@ 0000000180005200     libucrt:lcidtoname_downlevel.obj
 0001:00004210       ??_C@_1M@JIJIBHDP@?$AAe?$AAs?$AA?9?$AAN?$AAI?$AA?$AA@ 0000000180005210     libucrt:lcidtoname_downlevel.obj
 0001:00004220       ??_C@_1M@CGFMKEEK@?$AAe?$AAs?$AA?9?$AAP?$AAR?$AA?$AA@ 0000000180005220     libucrt:lcidtoname_downlevel.obj
 0001:00004230       ??_C@_1O@ICJHKIIK@?$AAz?$AAh?$AA?9?$AAC?$AAH?$AAT?$AA?$AA@ 0000000180005230     libucrt:lcidtoname_downlevel.obj
 0001:00004240       ??_C@_15CLNEJCE@?$AAs?$AAr?$AA?$AA@ 0000000180005240     libucrt:lcidtoname_downlevel.obj
 0001:00005090       ??_C@_1M@KAHEKEIG@?$AAa?$AAf?$AA?9?$AAz?$AAa?$AA?$AA@ 0000000180006090     libucrt:lcidtoname_downlevel.obj
 0001:000050a0       ??_C@_1M@GIECOABL@?$AAa?$AAr?$AA?9?$AAa?$AAe?$AA?$AA@ 00000001800060a0     libucrt:lcidtoname_downlevel.obj
 0001:000050b0       ??_C@_1M@BMLMEKGI@?$AAa?$AAr?$AA?9?$AAb?$AAh?$AA?$AA@ 00000001800060b0     libucrt:lcidtoname_downlevel.obj
 0001:000050c0       ??_C@_1M@DAPFDGGB@?$AAa?$AAr?$AA?9?$AAd?$AAz?$AA?$AA@ 00000001800060c0     libucrt:lcidtoname_downlevel.obj
 0001:000050d0       ??_C@_1M@FJNKGKIG@?$AAa?$AAr?$AA?9?$AAe?$AAg?$AA?$AA@ 00000001800060d0     libucrt:lcidtoname_downlevel.obj
 0001:000050e0       ??_C@_1M@FLGKKCLO@?$AAa?$AAr?$AA?9?$AAi?$AAq?$AA?$AA@ 00000001800060e0     libucrt:lcidtoname_downlevel.obj
 0001:000050f0       ??_C@_1M@GNDIPALM@?$AAa?$AAr?$AA?9?$AAj?$AAo?$AA?$AA@ 00000001800060f0     libucrt:lcidtoname_downlevel.obj
 0001:00005100       ??_C@_1M@DDMJFMGJ@?$AAa?$AAr?$AA?9?$AAk?$AAw?$AA?$AA@ 0000000180006100     libucrt:lcidtoname_downlevel.obj
 0001:00005110       ??_C@_1M@EJALMLHM@?$AAa?$AAr?$AA?9?$AAl?$AAb?$AA?$AA@ 0000000180006110     libucrt:lcidtoname_downlevel.obj
 0001:00005120       ??_C@_1M@MOBDBLOC@?$AAa?$AAr?$AA?9?$AAl?$AAy?$AA?$AA@ 0000000180006120     libucrt:lcidtoname_downlevel.obj
 0001:00005130       ??_C@_1M@JAOCLHDH@?$AAa?$AAr?$AA?9?$AAm?$AAa?$AA?$AA@ 0000000180006130     libucrt:lcidtoname_downlevel.obj
 0001:00005140       ??_C@_1M@JHPMKJIE@?$AAa?$AAr?$AA?9?$AAo?$AAm?$AA?$AA@ 0000000180006140     libucrt:lcidtoname_downlevel.obj
 0001:00005150       ??_C@_1M@OEPGHFNH@?$AAa?$AAr?$AA?9?$AAq?$AAa?$AA?$AA@ 0000000180006150     libucrt:lcidtoname_downlevel.obj
 0001:00005160       ??_C@_1M@KJDONENM@?$AAa?$AAr?$AA?9?$AAs?$AAa?$AA?$AA@ 0000000180006160     libucrt:lcidtoname_downlevel.obj
 0001:00005170       ??_C@_1M@DMJDKLKM@?$AAa?$AAr?$AA?9?$AAs?$AAy?$AA?$AA@ 0000000180006170     libucrt:lcidtoname_downlevel.obj
 0001:00005180       ??_C@_1M@OMFIPEDC@?$AAa?$AAr?$AA?9?$AAt?$AAn?$AA?$AA@ 0000000180006180     libucrt:lcidtoname_downlevel.obj
 0001:00005190       ??_C@_1M@IHMHGAON@?$AAa?$AAr?$AA?9?$AAy?$AAe?$AA?$AA@ 0000000180006190     libucrt:lcidtoname_downlevel.obj
 0001:000051a0       ??_C@_1BG@KDCPGJGB@?$AAa?$AAz?$AA?9?$AAa?$AAz?$AA?9?$AAc?$AAy?$AAr?$AAl?$AA?$AA@ 00000001800061a0     libucrt:lcidtoname_downlevel.obj
 0001:000051b8       ??_C@_1BG@IBCKDDOE@?$AAa?$AAz?$AA?9?$AAa?$AAz?$AA?9?$AAl?$AAa?$AAt?$AAn?$AA?$AA@ 00000001800061b8     libucrt:lcidtoname_downlevel.obj
 0001:000051d0       ??_C@_1M@EGPFDCPD@?$AAb?$AAe?$AA?9?$AAb?$AAy?$AA?$AA@ 00000001800061d0     libucrt:lcidtoname_downlevel.obj
 0001:000051e0       ??_C@_1M@PCMGMCGC@?$AAb?$AAg?$AA?9?$AAb?$AAg?$AA?$AA@ 00000001800061e0     libucrt:lcidtoname_downlevel.obj
 0001:000051f0       ??_C@_1M@BJBMFGOB@?$AAb?$AAn?$AA?9?$AAi?$AAn?$AA?$AA@ 00000001800061f0     libucrt:lcidtoname_downlevel.obj
 0001:00005200       ??_C@_1BG@EAKMMACD@?$AAb?$AAs?$AA?9?$AAb?$AAa?$AA?9?$AAl?$AAa?$AAt?$AAn?$AA?$AA@ 0000000180006200     libucrt:lcidtoname_downlevel.obj
 0001:00005218       ??_C@_1M@KGADAODK@?$AAc?$AAa?$AA?9?$AAe?$AAs?$AA?$AA@ 0000000180006218     libucrt:lcidtoname_downlevel.obj
 0001:00005228       ??_C@_1M@COAJPDHI@?$AAc?$AAs?$AA?9?$AAc?$AAz?$AA?$AA@ 0000000180006228     libucrt:lcidtoname_downlevel.obj
 0001:00005238       ??_C@_1M@DHBHFONH@?$AAc?$AAy?$AA?9?$AAg?$AAb?$AA?$AA@ 0000000180006238     libucrt:lcidtoname_downlevel.obj
 0001:00005248       ??_C@_1M@IMGKELGA@?$AAd?$AAa?$AA?9?$AAd?$AAk?$AA?$AA@ 0000000180006248     libucrt:lcidtoname_downlevel.obj
 0001:00005258       ??_C@_1M@NNDGDNGA@?$AAd?$AAe?$AA?9?$AAa?$AAt?$AA?$AA@ 0000000180006258     libucrt:lcidtoname_downlevel.obj
 0001:00005268       ??_C@_1M@IKDBHEEM@?$AAd?$AAe?$AA?9?$AAc?$AAh?$AA?$AA@ 0000000180006268     libucrt:lcidtoname_downlevel.obj
 0001:00005278       ??_C@_1M@GFFOJMCJ@?$AAd?$AAe?$AA?9?$AAd?$AAe?$AA?$AA@ 0000000180006278     libucrt:lcidtoname_downlevel.obj
 0001:00005288       ??_C@_1M@MDNLKBPM@?$AAd?$AAe?$AA?9?$AAl?$AAi?$AA?$AA@ 0000000180006288     libucrt:lcidtoname_downlevel.obj
 0001:00005298       ??_C@_1M@NJBEEJNL@?$AAd?$AAe?$AA?9?$AAl?$AAu?$AA?$AA@ 0000000180006298     libucrt:lcidtoname_downlevel.obj
 0001:000052a8       ??_C@_1O@GNNELBAP@?$AAd?$AAi?$AAv?$AA?9?$AAm?$AAv?$AA?$AA@ 00000001800062a8     libucrt:lcidtoname_downlevel.obj
 0001:000052b8       ??_C@_1M@EJLEOGAE@?$AAe?$AAl?$AA?9?$AAg?$AAr?$AA?$AA@ 00000001800062b8     libucrt:lcidtoname_downlevel.obj
 0001:000052c8       ??_C@_1M@GMPONJN@?$AAe?$AAn?$AA?9?$AAa?$AAu?$AA?$AA@ 00000001800062c8     libucrt:lcidtoname_downlevel.obj
 0001:000052d8       ??_C@_1M@NIDIIPGF@?$AAe?$AAn?$AA?9?$AAb?$AAz?$AA?$AA@ 00000001800062d8     libucrt:lcidtoname_downlevel.obj
 0001:000052e8       ??_C@_1M@JEHMIMFO@?$AAe?$AAn?$AA?9?$AAc?$AAa?$AA?$AA@ 00000001800062e8     libucrt:lcidtoname_downlevel.obj
 0001:000052f8       ??_C@_1M@IGMJCDLA@?$AAe?$AAn?$AA?9?$AAc?$AAb?$AA?$AA@ 00000001800062f8     libucrt:lcidtoname_downlevel.obj
 0001:00005308       ??_C@_1M@BNFIGBKG@?$AAe?$AAn?$AA?9?$AAg?$AAb?$AA?$AA@ 0000000180006308     libucrt:lcidtoname_downlevel.obj
 0001:00005318       ??_C@_1M@LKIFDIGP@?$AAe?$AAn?$AA?9?$AAi?$AAe?$AA?$AA@ 0000000180006318     libucrt:lcidtoname_downlevel.obj
 0001:00005328       ??_C@_1M@PJKFGCCO@?$AAe?$AAn?$AA?9?$AAj?$AAm?$AA?$AA@ 0000000180006328     libucrt:lcidtoname_downlevel.obj
 0001:00005338       ??_C@_1M@KPPKEPBO@?$AAe?$AAn?$AA?9?$AAn?$AAz?$AA?$AA@ 0000000180006338     libucrt:lcidtoname_downlevel.obj
 0001:00005348       ??_C@_1M@GMDGLDOB@?$AAe?$AAn?$AA?9?$AAp?$AAh?$AA?$AA@ 0000000180006348     libucrt:lcidtoname_downlevel.obj
 0001:00005358       ??_C@_1M@ONGIBJNA@?$AAe?$AAn?$AA?9?$AAt?$AAt?$AA?$AA@ 0000000180006358     libucrt:lcidtoname_downlevel.obj
 0001:00005368       ??_C@_1M@LLODPCMM@?$AAe?$AAn?$AA?9?$AAu?$AAs?$AA?$AA@ 0000000180006368     libucrt:lcidtoname_downlevel.obj
 0001:00005378       ??_C@_1M@LAKFNPAN@?$AAe?$AAn?$AA?9?$AAz?$AAa?$AA?$AA@ 0000000180006378     libucrt:lcidtoname_downlevel.obj
 0001:00005388       ??_C@_1M@MFNHNHEO@?$AAe?$AAn?$AA?9?$AAz?$AAw?$AA?$AA@ 0000000180006388     libucrt:lcidtoname_downlevel.obj
 0001:00005398       ??_C@_1M@EJEINPHM@?$AAe?$AAs?$AA?9?$AAa?$AAr?$AA?$AA@ 0000000180006398     libucrt:lcidtoname_downlevel.obj
 0001:000053a8       ??_C@_1M@GNKPCCJA@?$AAe?$AAs?$AA?9?$AAb?$AAo?$AA?$AA@ 00000001800063a8     libucrt:lcidtoname_downlevel.obj
 0001:000053b8       ??_C@_1M@LEEGFONL@?$AAe?$AAs?$AA?9?$AAc?$AAl?$AA?$AA@ 00000001800063b8     libucrt:lcidtoname_downlevel.obj
 0001:000053c8       ??_C@_1M@KGPDPBDF@?$AAe?$AAs?$AA?9?$AAc?$AAo?$AA?$AA@ 00000001800063c8     libucrt:lcidtoname_downlevel.obj
 0001:000053d8       ??_C@_1M@EIAHOHH@?$AAe?$AAs?$AA?9?$AAc?$AAr?$AA?$AA@ 00000001800063d8     libucrt:lcidtoname_downlevel.obj
 0001:000053e8       ??_C@_1M@LLPGMBIN@?$AAe?$AAs?$AA?9?$AAd?$AAo?$AA?$AA@ 00000001800063e8     libucrt:lcidtoname_downlevel.obj
 0001:000053f8       ??_C@_1M@DKHMKNJA@?$AAe?$AAs?$AA?9?$AAe?$AAc?$AA?$AA@ 00000001800063f8     libucrt:lcidtoname_downlevel.obj
 0001:00005408       ??_C@_1M@GKGFPKAP@?$AAe?$AAs?$AA?9?$AAe?$AAs?$AA?$AA@ 0000000180006408     libucrt:lcidtoname_downlevel.obj
 0001:00005418       ??_C@_1M@LKHKGDLN@?$AAe?$AAs?$AA?9?$AAg?$AAt?$AA?$AA@ 0000000180006418     libucrt:lcidtoname_downlevel.obj
 0001:00005428       ??_C@_1M@HEIIGGJD@?$AAe?$AAs?$AA?9?$AAh?$AAn?$AA?$AA@ 0000000180006428     libucrt:lcidtoname_downlevel.obj
 0001:00005438       ??_C@_1M@FBDHPPGD@?$AAe?$AAs?$AA?9?$AAm?$AAx?$AA?$AA@ 0000000180006438     libucrt:lcidtoname_downlevel.obj
 0001:00005448       ??_C@_1M@DPAGLNDH@?$AAe?$AAs?$AA?9?$AAn?$AAi?$AA?$AA@ 0000000180006448     libucrt:lcidtoname_downlevel.obj
 0001:00005458       ??_C@_1M@MDGOPGDD@?$AAe?$AAs?$AA?9?$AAp?$AAa?$AA?$AA@ 0000000180006458     libucrt:lcidtoname_downlevel.obj
 0001:00005468       ??_C@_1M@EMAMGBGE@?$AAe?$AAs?$AA?9?$AAp?$AAe?$AA?$AA@ 0000000180006468     libucrt:lcidtoname_downlevel.obj
 0001:00005478       ??_C@_1M@IBMCAOEC@?$AAe?$AAs?$AA?9?$AAp?$AAr?$AA?$AA@ 0000000180006478     libucrt:lcidtoname_downlevel.obj
 0001:00005488       ??_C@_1M@FGMDIJED@?$AAe?$AAs?$AA?9?$AAp?$AAy?$AA?$AA@ 0000000180006488     libucrt:lcidtoname_downlevel.obj
 0001:00005498       ??_C@_1M@IIDEOLLL@?$AAe?$AAs?$AA?9?$AAs?$AAv?$AA?$AA@ 0000000180006498     libucrt:lcidtoname_downlevel.obj
 0001:000054a8       ??_C@_1M@GAOBIPA@?$AAe?$AAs?$AA?9?$AAu?$AAy?$AA?$AA@ 00000001800064a8     libucrt:lcidtoname_downlevel.obj
 0001:000054b8       ??_C@_1M@JKFFICHJ@?$AAe?$AAs?$AA?9?$AAv?$AAe?$AA?$AA@ 00000001800064b8     libucrt:lcidtoname_downlevel.obj
 0001:000054c8       ??_C@_1M@PNMLOJDF@?$AAe?$AAt?$AA?9?$AAe?$AAe?$AA?$AA@ 00000001800064c8     libucrt:lcidtoname_downlevel.obj
 0001:000054d8       ??_C@_1M@GHHLIKEI@?$AAe?$AAu?$AA?9?$AAe?$AAs?$AA?$AA@ 00000001800064d8     libucrt:lcidtoname_downlevel.obj
 0001:000054e8       ??_C@_1M@PBNONODE@?$AAf?$AAa?$AA?9?$AAi?$AAr?$AA?$AA@ 00000001800064e8     libucrt:lcidtoname_downlevel.obj
 0001:000054f8       ??_C@_1M@JEEHPMIL@?$AAf?$AAi?$AA?9?$AAf?$AAi?$AA?$AA@ 00000001800064f8     libucrt:lcidtoname_downlevel.obj
 0001:00005508       ??_C@_1M@LMDCNDBA@?$AAf?$AAo?$AA?9?$AAf?$AAo?$AA?$AA@ 0000000180006508     libucrt:lcidtoname_downlevel.obj
 0001:00005518       ??_C@_1M@JKEOHLDK@?$AAf?$AAr?$AA?9?$AAb?$AAe?$AA?$AA@ 0000000180006518     libucrt:lcidtoname_downlevel.obj
 0001:00005528       ??_C@_1M@NOHADPMI@?$AAf?$AAr?$AA?9?$AAc?$AAa?$AA?$AA@ 0000000180006528     libucrt:lcidtoname_downlevel.obj
 0001:00005538       ??_C@_1M@KDHIHAEC@?$AAf?$AAr?$AA?9?$AAc?$AAh?$AA?$AA@ 0000000180006538     libucrt:lcidtoname_downlevel.obj
 0001:00005548       ??_C@_1M@MMBBFGAK@?$AAf?$AAr?$AA?9?$AAf?$AAr?$AA?$AA@ 0000000180006548     libucrt:lcidtoname_downlevel.obj
 0001:00005558       ??_C@_1M@PAFNENNF@?$AAf?$AAr?$AA?9?$AAl?$AAu?$AA?$AA@ 0000000180006558     libucrt:lcidtoname_downlevel.obj
 0001:00005568       ??_C@_1M@EOHDJGDD@?$AAf?$AAr?$AA?9?$AAm?$AAc?$AA?$AA@ 0000000180006568     libucrt:lcidtoname_downlevel.obj
 0001:00005578       ??_C@_1M@FAPLLOPF@?$AAg?$AAl?$AA?9?$AAe?$AAs?$AA?$AA@ 0000000180006578     libucrt:lcidtoname_downlevel.obj
 0001:00005588       ??_C@_1M@FOPBFLOO@?$AAg?$AAu?$AA?9?$AAi?$AAn?$AA?$AA@ 0000000180006588     libucrt:lcidtoname_downlevel.obj
 0001:00005598       ??_C@_1M@KBMCINPM@?$AAh?$AAe?$AA?9?$AAi?$AAl?$AA?$AA@ 0000000180006598     libucrt:lcidtoname_downlevel.obj
 0001:000055a8       ??_C@_1M@BBPHKFPJ@?$AAh?$AAi?$AA?9?$AAi?$AAn?$AA?$AA@ 00000001800065a8     libucrt:lcidtoname_downlevel.obj
 0001:000055b8       ??_C@_1M@PMBNDPHD@?$AAh?$AAr?$AA?9?$AAb?$AAa?$AA?$AA@ 00000001800065b8     libucrt:lcidtoname_downlevel.obj
 0001:000055c8       ??_C@_1M@BPCKOEGE@?$AAh?$AAr?$AA?9?$AAh?$AAr?$AA?$AA@ 00000001800065c8     libucrt:lcidtoname_downlevel.obj
 0001:000055d8       ??_C@_1M@GACBMHKE@?$AAh?$AAu?$AA?9?$AAh?$AAu?$AA?$AA@ 00000001800065d8     libucrt:lcidtoname_downlevel.obj
 0001:000055e8       ??_C@_1M@MILPAJJC@?$AAh?$AAy?$AA?9?$AAa?$AAm?$AA?$AA@ 00000001800065e8     libucrt:lcidtoname_downlevel.obj
 0001:000055f8       ??_C@_1M@BABBICEC@?$AAi?$AAd?$AA?9?$AAi?$AAd?$AA?$AA@ 00000001800065f8     libucrt:lcidtoname_downlevel.obj
 0001:00005608       ??_C@_1M@BIKNHHPF@?$AAi?$AAs?$AA?9?$AAi?$AAs?$AA?$AA@ 0000000180006608     libucrt:lcidtoname_downlevel.obj
 0001:00005618       ??_C@_1M@NMPCJPHE@?$AAi?$AAt?$AA?9?$AAc?$AAh?$AA?$AA@ 0000000180006618     libucrt:lcidtoname_downlevel.obj
 0001:00005628       ??_C@_1M@GHKGFEDF@?$AAi?$AAt?$AA?9?$AAi?$AAt?$AA?$AA@ 0000000180006628     libucrt:lcidtoname_downlevel.obj
 0001:00005638       ??_C@_1M@NIEJCJJA@?$AAj?$AAa?$AA?9?$AAj?$AAp?$AA?$AA@ 0000000180006638     libucrt:lcidtoname_downlevel.obj
 0001:00005648       ??_C@_1M@JILFNBIM@?$AAk?$AAa?$AA?9?$AAg?$AAe?$AA?$AA@ 0000000180006648     libucrt:lcidtoname_downlevel.obj
 0001:00005658       ??_C@_1M@PACPMGPH@?$AAk?$AAk?$AA?9?$AAk?$AAz?$AA?$AA@ 0000000180006658     libucrt:lcidtoname_downlevel.obj
 0001:00005668       ??_C@_1M@IELFGMHA@?$AAk?$AAn?$AA?9?$AAi?$AAn?$AA?$AA@ 0000000180006668     libucrt:lcidtoname_downlevel.obj
 0001:00005678       ??_C@_1O@IBBJHCH@?$AAk?$AAo?$AAk?$AA?9?$AAi?$AAn?$AA?$AA@ 0000000180006678     libucrt:lcidtoname_downlevel.obj
 0001:00005688       ??_C@_1M@DMHAEOGC@?$AAk?$AAo?$AA?9?$AAk?$AAr?$AA?$AA@ 0000000180006688     libucrt:lcidtoname_downlevel.obj
 0001:00005698       ??_C@_1M@HBAHBIGA@?$AAk?$AAy?$AA?9?$AAk?$AAg?$AA?$AA@ 0000000180006698     libucrt:lcidtoname_downlevel.obj
 0001:000056a8       ??_C@_1M@KPMILCJG@?$AAl?$AAt?$AA?9?$AAl?$AAt?$AA?$AA@ 00000001800066a8     libucrt:lcidtoname_downlevel.obj
 0001:000056b8       ??_C@_1M@BDEKKCA@?$AAl?$AAv?$AA?9?$AAl?$AAv?$AA?$AA@ 00000001800066b8     libucrt:lcidtoname_downlevel.obj
 0001:000056c8       ??_C@_1M@ELCKCCJJ@?$AAm?$AAi?$AA?9?$AAn?$AAz?$AA?$AA@ 00000001800066c8     libucrt:lcidtoname_downlevel.obj
 0001:000056d8       ??_C@_1M@CBOOLAPA@?$AAm?$AAk?$AA?9?$AAm?$AAk?$AA?$AA@ 00000001800066d8     libucrt:lcidtoname_downlevel.obj
 0001:000056e8       ??_C@_1M@GPHNBJKN@?$AAm?$AAl?$AA?9?$AAi?$AAn?$AA?$AA@ 00000001800066e8     libucrt:lcidtoname_downlevel.obj
 0001:000056f8       ??_C@_1M@PABJILIG@?$AAm?$AAn?$AA?9?$AAm?$AAn?$AA?$AA@ 00000001800066f8     libucrt:lcidtoname_downlevel.obj
 0001:00005708       ??_C@_1M@FGBKKIPG@?$AAm?$AAr?$AA?9?$AAi?$AAn?$AA?$AA@ 0000000180006708     libucrt:lcidtoname_downlevel.obj
 0001:00005718       ??_C@_1M@NDBPDDAL@?$AAm?$AAs?$AA?9?$AAb?$AAn?$AA?$AA@ 0000000180006718     libucrt:lcidtoname_downlevel.obj
 0001:00005728       ??_C@_1M@OPIHOOPI@?$AAm?$AAs?$AA?9?$AAm?$AAy?$AA?$AA@ 0000000180006728     libucrt:lcidtoname_downlevel.obj
 0001:00005738       ??_C@_1M@PPDBCNFM@?$AAm?$AAt?$AA?9?$AAm?$AAt?$AA?$AA@ 0000000180006738     libucrt:lcidtoname_downlevel.obj
 0001:00005748       ??_C@_1M@KDJDKMDD@?$AAn?$AAb?$AA?9?$AAn?$AAo?$AA?$AA@ 0000000180006748     libucrt:lcidtoname_downlevel.obj
 0001:00005758       ??_C@_1M@KFCFLMJP@?$AAn?$AAl?$AA?9?$AAb?$AAe?$AA?$AA@ 0000000180006758     libucrt:lcidtoname_downlevel.obj
 0001:00005768       ??_C@_1M@KPOPDDGO@?$AAn?$AAl?$AA?9?$AAn?$AAl?$AA?$AA@ 0000000180006768     libucrt:lcidtoname_downlevel.obj
 0001:00005778       ??_C@_1M@LJKPEMLN@?$AAn?$AAn?$AA?9?$AAn?$AAo?$AA?$AA@ 0000000180006778     libucrt:lcidtoname_downlevel.obj
 0001:00005788       ??_C@_1M@BDGHHBFL@?$AAn?$AAs?$AA?9?$AAz?$AAa?$AA?$AA@ 0000000180006788     libucrt:lcidtoname_downlevel.obj
 0001:00005798       ??_C@_1M@IDEHOAP@?$AAp?$AAa?$AA?9?$AAi?$AAn?$AA?$AA@ 0000000180006798     libucrt:lcidtoname_downlevel.obj
 0001:000057a8       ??_C@_1M@HDBKGOGH@?$AAp?$AAl?$AA?9?$AAp?$AAl?$AA?$AA@ 00000001800067a8     libucrt:lcidtoname_downlevel.obj
 0001:000057b8       ??_C@_1M@LJLLCMEH@?$AAp?$AAt?$AA?9?$AAb?$AAr?$AA?$AA@ 00000001800067b8     libucrt:lcidtoname_downlevel.obj
 0001:000057c8       ??_C@_1M@NCMONAAL@?$AAp?$AAt?$AA?9?$AAp?$AAt?$AA?$AA@ 00000001800067c8     libucrt:lcidtoname_downlevel.obj
 0001:000057d8       ??_C@_1O@EAKMAJDN@?$AAq?$AAu?$AAz?$AA?9?$AAb?$AAo?$AA?$AA@ 00000001800067d8     libucrt:lcidtoname_downlevel.obj
 0001:000057e8       ??_C@_1O@BHHPIGDN@?$AAq?$AAu?$AAz?$AA?9?$AAe?$AAc?$AA?$AA@ 00000001800067e8     libucrt:lcidtoname_downlevel.obj
 0001:000057f8       ??_C@_1O@GBAPEKMJ@?$AAq?$AAu?$AAz?$AA?9?$AAp?$AAe?$AA?$AA@ 00000001800067f8     libucrt:lcidtoname_downlevel.obj
 0001:00005808       ??_C@_1M@CLGLEFBO@?$AAr?$AAo?$AA?9?$AAr?$AAo?$AA?$AA@ 0000000180006808     libucrt:lcidtoname_downlevel.obj
 0001:00005818       ??_C@_1M@CEEDODME@?$AAr?$AAu?$AA?9?$AAr?$AAu?$AA?$AA@ 0000000180006818     libucrt:lcidtoname_downlevel.obj
 0001:00005828       ??_C@_1M@HPKKKMPP@?$AAs?$AAa?$AA?9?$AAi?$AAn?$AA?$AA@ 0000000180006828     libucrt:lcidtoname_downlevel.obj
 0001:00005838       ??_C@_1M@BKMAIGOJ@?$AAs?$AAe?$AA?9?$AAf?$AAi?$AA?$AA@ 0000000180006838     libucrt:lcidtoname_downlevel.obj
 0001:00005848       ??_C@_1M@NDPIFLFI@?$AAs?$AAe?$AA?9?$AAn?$AAo?$AA?$AA@ 0000000180006848     libucrt:lcidtoname_downlevel.obj
 0001:00005858       ??_C@_1M@DANKKHJ@?$AAs?$AAe?$AA?9?$AAs?$AAe?$AA?$AA@ 0000000180006858     libucrt:lcidtoname_downlevel.obj
 0001:00005868       ??_C@_1M@PNBLONPJ@?$AAs?$AAk?$AA?9?$AAs?$AAk?$AA?$AA@ 0000000180006868     libucrt:lcidtoname_downlevel.obj
 0001:00005878       ??_C@_1M@LFMODOAL@?$AAs?$AAl?$AA?9?$AAs?$AAi?$AA?$AA@ 0000000180006878     libucrt:lcidtoname_downlevel.obj
 0001:00005888       ??_C@_1O@DFKOMPG@?$AAs?$AAm?$AAa?$AA?9?$AAn?$AAo?$AA?$AA@ 0000000180006888     libucrt:lcidtoname_downlevel.obj
 0001:00005898       ??_C@_1O@NDKPBNNH@?$AAs?$AAm?$AAa?$AA?9?$AAs?$AAe?$AA?$AA@ 0000000180006898     libucrt:lcidtoname_downlevel.obj
 0001:000058a8       ??_C@_1O@PLLKBHAB@?$AAs?$AAm?$AAj?$AA?9?$AAn?$AAo?$AA?$AA@ 00000001800068a8     libucrt:lcidtoname_downlevel.obj
 0001:000058b8       ??_C@_1O@CLEPOGCA@?$AAs?$AAm?$AAj?$AA?9?$AAs?$AAe?$AA?$AA@ 00000001800068b8     libucrt:lcidtoname_downlevel.obj
 0001:000058c8       ??_C@_1O@DLGJGKMK@?$AAs?$AAm?$AAn?$AA?9?$AAf?$AAi?$AA?$AA@ 00000001800068c8     libucrt:lcidtoname_downlevel.obj
 0001:000058d8       ??_C@_1O@OJDJGAJC@?$AAs?$AAm?$AAs?$AA?9?$AAf?$AAi?$AA?$AA@ 00000001800068d8     libucrt:lcidtoname_downlevel.obj
 0001:000058e8       ??_C@_1M@BOFOGHPB@?$AAs?$AAq?$AA?9?$AAa?$AAl?$AA?$AA@ 00000001800068e8     libucrt:lcidtoname_downlevel.obj
 0001:000058f8       ??_C@_1BG@LJBBIPGB@?$AAs?$AAr?$AA?9?$AAb?$AAa?$AA?9?$AAc?$AAy?$AAr?$AAl?$AA?$AA@ 00000001800068f8     libucrt:lcidtoname_downlevel.obj
 0001:00005910       ??_C@_1BG@JLBENFOE@?$AAs?$AAr?$AA?9?$AAb?$AAa?$AA?9?$AAl?$AAa?$AAt?$AAn?$AA?$AA@ 0000000180006910     libucrt:lcidtoname_downlevel.obj
 0001:00005928       ??_C@_1BG@KODPNHE@?$AAs?$AAr?$AA?9?$AAs?$AAp?$AA?9?$AAc?$AAy?$AAr?$AAl?$AA?$AA@ 0000000180006928     libucrt:lcidtoname_downlevel.obj
 0001:00005940       ??_C@_1BG@CIOGKHPB@?$AAs?$AAr?$AA?9?$AAs?$AAp?$AA?9?$AAl?$AAa?$AAt?$AAn?$AA?$AA@ 0000000180006940     libucrt:lcidtoname_downlevel.obj
 0001:00005958       ??_C@_1M@NGFJLMAC@?$AAs?$AAv?$AA?9?$AAf?$AAi?$AA?$AA@ 0000000180006958     libucrt:lcidtoname_downlevel.obj
 0001:00005968       ??_C@_1M@MPJEJAJC@?$AAs?$AAv?$AA?9?$AAs?$AAe?$AA?$AA@ 0000000180006968     libucrt:lcidtoname_downlevel.obj
 0001:00005978       ??_C@_1M@MPNDHLFK@?$AAs?$AAw?$AA?9?$AAk?$AAe?$AA?$AA@ 0000000180006978     libucrt:lcidtoname_downlevel.obj
 0001:00005988       ??_C@_1O@KOHBJJI@?$AAs?$AAy?$AAr?$AA?9?$AAs?$AAy?$AA?$AA@ 0000000180006988     libucrt:lcidtoname_downlevel.obj
 0001:00005998       ??_C@_1M@LDCEFHA@?$AAt?$AAa?$AA?9?$AAi?$AAn?$AA?$AA@ 0000000180006998     libucrt:lcidtoname_downlevel.obj
 0001:000059a8       ??_C@_1M@CNJOFAK@?$AAt?$AAe?$AA?9?$AAi?$AAn?$AA?$AA@ 00000001800069a8     libucrt:lcidtoname_downlevel.obj
 0001:000059b8       ??_C@_1M@GNAECACD@?$AAt?$AAh?$AA?9?$AAt?$AAh?$AA?$AA@ 00000001800069b8     libucrt:lcidtoname_downlevel.obj
 0001:000059c8       ??_C@_1M@CHBIHOJO@?$AAt?$AAn?$AA?9?$AAz?$AAa?$AA?$AA@ 00000001800069c8     libucrt:lcidtoname_downlevel.obj
 0001:000059d8       ??_C@_1M@GCCMIGPJ@?$AAt?$AAr?$AA?9?$AAt?$AAr?$AA?$AA@ 00000001800069d8     libucrt:lcidtoname_downlevel.obj
 0001:000059e8       ??_C@_1M@CELMCNBK@?$AAt?$AAt?$AA?9?$AAr?$AAu?$AA?$AA@ 00000001800069e8     libucrt:lcidtoname_downlevel.obj
 0001:000059f8       ??_C@_1M@KLMCELGA@?$AAu?$AAk?$AA?9?$AAu?$AAa?$AA?$AA@ 00000001800069f8     libucrt:lcidtoname_downlevel.obj
 0001:00005a08       ??_C@_1M@EPAJJAJF@?$AAu?$AAr?$AA?9?$AAp?$AAk?$AA?$AA@ 0000000180006a08     libucrt:lcidtoname_downlevel.obj
 0001:00005a18       ??_C@_1BG@GEGPMCDJ@?$AAu?$AAz?$AA?9?$AAu?$AAz?$AA?9?$AAc?$AAy?$AAr?$AAl?$AA?$AA@ 0000000180006a18     libucrt:lcidtoname_downlevel.obj
 0001:00005a30       ??_C@_1BG@EGGKJILM@?$AAu?$AAz?$AA?9?$AAu?$AAz?$AA?9?$AAl?$AAa?$AAt?$AAn?$AA?$AA@ 0000000180006a30     libucrt:lcidtoname_downlevel.obj
 0001:00005a48       ??_C@_1M@GFOCLFF@?$AAv?$AAi?$AA?9?$AAv?$AAn?$AA?$AA@ 0000000180006a48     libucrt:lcidtoname_downlevel.obj
 0001:00005a58       ??_C@_1M@CPAMEDFI@?$AAx?$AAh?$AA?9?$AAz?$AAa?$AA?$AA@ 0000000180006a58     libucrt:lcidtoname_downlevel.obj
 0001:00005a68       ??_C@_1O@EBKIFIGN@?$AAz?$AAh?$AA?9?$AAc?$AAh?$AAs?$AA?$AA@ 0000000180006a68     libucrt:lcidtoname_downlevel.obj
 0001:00005a78       ??_C@_1O@NMHPGANE@?$AAz?$AAh?$AA?9?$AAc?$AAh?$AAt?$AA?$AA@ 0000000180006a78     libucrt:lcidtoname_downlevel.obj
 0001:00005a88       ??_C@_1M@LPINJOMC@?$AAz?$AAh?$AA?9?$AAc?$AAn?$AA?$AA@ 0000000180006a88     libucrt:lcidtoname_downlevel.obj
 0001:00005a98       ??_C@_1M@OCJEJODD@?$AAz?$AAh?$AA?9?$AAh?$AAk?$AA?$AA@ 0000000180006a98     libucrt:lcidtoname_downlevel.obj
 0001:00005aa8       ??_C@_1M@DNDLJINH@?$AAz?$AAh?$AA?9?$AAm?$AAo?$AA?$AA@ 0000000180006aa8     libucrt:lcidtoname_downlevel.obj
 0001:00005ab8       ??_C@_1M@MBFDNDND@?$AAz?$AAh?$AA?9?$AAs?$AAg?$AA?$AA@ 0000000180006ab8     libucrt:lcidtoname_downlevel.obj
 0001:00005ac8       ??_C@_1M@IMEPLEPE@?$AAz?$AAh?$AA?9?$AAt?$AAw?$AA?$AA@ 0000000180006ac8     libucrt:lcidtoname_downlevel.obj
 0001:00005ad8       ??_C@_1M@BBGHNHJP@?$AAz?$AAu?$AA?9?$AAz?$AAa?$AA?$AA@ 0000000180006ad8     libucrt:lcidtoname_downlevel.obj
 0001:00005d40       __log10_256_lead           0000000180006d40     libucrt:log10_256_lead_tail_table.obj
 0001:00006550       __log10_256_tail           0000000180007550     libucrt:log10_256_lead_tail_table.obj
 0001:00006d60       __log_F_inv_qword          0000000180007d60     libucrt:log_f_inv_qword_table.obj
 0001:00007570       ??_C@_05HGHHAHAP@log10?$AA@ 0000000180008570     libucrt:log_special.obj
 0001:00007578       ??_C@_1BA@BALFACEM@?$AAC?$AAO?$AAN?$AAO?$AAU?$AAT?$AA$?$AA?$AA@ 0000000180008578     libucrt:initcon.obj
 0001:000075d0       _load_config_used          00000001800085d0     LIBCMT:loadcfg.obj
 0001:00007668       ??_R4exception@std@@6B@    0000000180008668     LIBCMT:throw_bad_alloc.obj
 0001:00007690       ??_R3exception@std@@8      0000000180008690     LIBCMT:throw_bad_alloc.obj
 0001:000076a8       ??_R2exception@std@@8      00000001800086a8     LIBCMT:throw_bad_alloc.obj
 0001:000076b8       ??_R1A@?0A@EA@exception@std@@8 00000001800086b8     LIBCMT:throw_bad_alloc.obj
 0001:000076e0       ??_R4bad_alloc@std@@6B@    00000001800086e0     LIBCMT:throw_bad_alloc.obj
 0001:00007708       ??_R3bad_alloc@std@@8      0000000180008708     LIBCMT:throw_bad_alloc.obj
 0001:00007720       ??_R2bad_alloc@std@@8      0000000180008720     LIBCMT:throw_bad_alloc.obj
 0001:00007738       ??_R1A@?0A@EA@bad_alloc@std@@8 0000000180008738     LIBCMT:throw_bad_alloc.obj
 0001:00007760       ??_R4bad_array_new_length@std@@6B@ 0000000180008760     LIBCMT:throw_bad_alloc.obj
 0001:00007788       ??_R3bad_array_new_length@std@@8 0000000180008788     LIBCMT:throw_bad_alloc.obj
 0001:000077a0       ??_R2bad_array_new_length@std@@8 00000001800087a0     LIBCMT:throw_bad_alloc.obj
 0001:000077c0       ??_R1A@?0A@EA@bad_array_new_length@std@@8 00000001800087c0     LIBCMT:throw_bad_alloc.obj
 0001:000077e8       ??_R4type_info@@6B@        00000001800087e8     LIBCMT:std_type_info_static.obj
 0001:00007810       ??_R3type_info@@8          0000000180008810     LIBCMT:std_type_info_static.obj
 0001:00007828       ??_R2type_info@@8          0000000180008828     LIBCMT:std_type_info_static.obj
 0001:00007838       ??_R1A@?0A@EA@type_info@@8 0000000180008838     LIBCMT:std_type_info_static.obj
 0001:00007860       ?_TraceLoggingMetadata@?1??_TlgWrite@__vcrt_trace_logging_provider@@YAJPEBU_TlgProvider_t@2@PEFBXPEBU_GUID@@2IPEAU_EVENT_DATA_DESCRIPTOR@@@Z@4U_TraceLoggingMetadata_t@2@B 0000000180008860     libvcruntime:telemetry.obj
 0001:00007913       ?_TraceLoggingMetadataEnd@?1??_TlgWrite@__vcrt_trace_logging_provider@@YAJPEBU_TlgProvider_t@2@PEFBXPEBU_GUID@@2IPEAU_EVENT_DATA_DESCRIPTOR@@@Z@4EB 0000000180008913     libvcruntime:telemetry.obj
 0001:00007c60       __rtc_iaa                  0000000180008c60     LIBCMT:_initsect_.obj
 0001:00007c68       __rtc_izz                  0000000180008c68     LIBCMT:_initsect_.obj
 0001:00007c70       __rtc_taa                  0000000180008c70     LIBCMT:_initsect_.obj
 0001:00007c78       __rtc_tzz                  0000000180008c78     LIBCMT:_initsect_.obj
 0001:00007c80       ?TraceLoggingRegister@__vcrt_trace_logging_provider@@YAJPEBU_TlgProvider_t@1@PEBU_GUID@@P6AX1KE_K2PEAU_EVENT_FILTER_DESCRIPTOR@@PEAX@Z4@Z 0000000180008c80 f i libvcruntime:telemetry.obj
 0001:00007cfc       ?_TlgEnableCallback@__vcrt_trace_logging_provider@@YAXPEBU_GUID@@KE_K1PEAU_EVENT_FILTER_DESCRIPTOR@@PEAX@Z 0000000180008cfc f i libvcruntime:telemetry.obj
 0001:00007dc0       ?_TlgWrite@__vcrt_trace_logging_provider@@YAJPEBU_TlgProvider_t@1@PEFBXPEBU_GUID@@2IPEAU_EVENT_DATA_DESCRIPTOR@@@Z 0000000180008dc0 f i libvcruntime:telemetry.obj
 0001:00007e70       _alloca_probe              0000000180008e70 f   chkstk.obj
 0001:00007e70       __chkstk                   0000000180008e70 f   chkstk.obj
 0001:00007ed0       ConfigureW                 0000000180008ed0 f   EMenu.obj
 0001:00007ef0       ExitFARW                   0000000180008ef0 f   EMenu.obj
 0001:00007f40       GetGlobalInfoW             0000000180008f40 f   EMenu.obj
 0001:00007fc0       GetPluginInfoW             0000000180008fc0 f   EMenu.obj
 0001:00007fd0       OpenW                      0000000180008fd0 f   EMenu.obj
 0001:00007ff0       SetStartupInfoW            0000000180008ff0 f   EMenu.obj
 0001:00008040       ??0auto_sz@@QEAA@AEBU_STRRET@@PEFBU_ITEMIDLIST@@@Z 0000000180009040 f   auto_sz.obj
 0001:000080f0       ??0auto_sz@@QEAA@PEB_W@Z   00000001800090f0 f   auto_sz.obj
 0001:00008130       ??0auto_sz@@QEAA@PEB_W_K@Z 0000000180009130 f   auto_sz.obj
 0001:00008180       ??0auto_sz@@QEAA@XZ        0000000180009180 f   auto_sz.obj
 0001:00008190       ??1auto_sz@@QEAA@XZ        0000000180009190 f   auto_sz.obj
 0001:000081c0       ??4auto_sz@@QEAAAEAV0@AEBV0@@Z 00000001800091c0 f   auto_sz.obj
 0001:00008200       ??4auto_sz@@QEAAAEAV0@PEB_W@Z 0000000180009200 f   auto_sz.obj
 0001:00008260       ??9auto_sz@@QEAA_NPEB_W@Z  0000000180009260 f   auto_sz.obj
 0001:00008280       ??Aauto_sz@@QEAA_WH@Z      0000000180009280 f   auto_sz.obj
 0001:00008290       ??Bauto_sz@@QEAAPEB_WXZ    0000000180009290 f   auto_sz.obj
 0001:00008290       ??Bauto_sz@@QEAAPEA_WXZ    0000000180009290 f   auto_sz.obj
 0001:000082a0       ??Yauto_sz@@QEAAAEAV0@PEB_W@Z 00000001800092a0 f   auto_sz.obj
 0001:00008300       ?CompareExcluding@auto_sz@@QEAA_NPEB_W_W@Z 0000000180009300 f   auto_sz.obj
 0001:00008390       ?IsEmpty@auto_sz@@QEAA_NXZ 0000000180009390 f   auto_sz.obj
 0001:000083b0       ?Len@auto_sz@@QEBA_KXZ     00000001800093b0 f   auto_sz.obj
 0001:000083d0       ?Realloc@auto_sz@@QEAAX_K@Z 00000001800093d0 f   auto_sz.obj
 0001:00008480       ?RemoveTrailing@auto_sz@@QEAAX_W@Z 0000000180009480 f   auto_sz.obj
 0001:000084d0       ?Trunc@auto_sz@@QEAAX_K@Z  00000001800094d0 f   auto_sz.obj
 0001:000084e0       ??0CFarMenu@@QEAA@PEB_WPEBU_GUID@@I@Z 00000001800094e0 f   FarMenu.obj
 0001:00008580       ??1CFarMenu@@QEAA@XZ       0000000180009580 f   FarMenu.obj
 0001:00008600       ??ACFarMenu@@QEAAPEB_WI@Z  0000000180009600 f   FarMenu.obj
 0001:00008620       ?AddArrows@CFarMenu@@IEAAXXZ 0000000180009620 f   FarMenu.obj
 0001:00008810       ?AddItem@CFarMenu@@QEAAIPEB_W_NW4ECheck@1@1@Z 0000000180009810 f   FarMenu.obj
 0001:00008840       ?AddSeparator@CFarMenu@@QEAAXXZ 0000000180009840 f   FarMenu.obj
 0001:000088f0       ?GetCursorXY@CFarMenu@@QEAAXPEAH0@Z 00000001800098f0 f   FarMenu.obj
 0001:00008a10       ?InsertItem@CFarMenu@@QEAAIIPEB_W_NW4ECheck@1@1@Z 0000000180009a10 f   FarMenu.obj
 0001:00008b90       ?Show@CFarMenu@@QEAAHPEB_WH_N@Z 0000000180009b90 f   FarMenu.obj
 0001:00008e20       ?MenuDlgProc@@YAHPEAUHWND__@@I_K_J@Z 0000000180009e20 f   MenuDlg.obj
 0001:00008f00       ?Cleanup@OleThread@@YAXXZ  0000000180009f00 f   OleThread.obj
 0001:00009030       ?EnsureThreadStarted@OleThread@@YA_NXZ 000000018000a030 f   OleThread.obj
 0001:000091c0       ?OpenPlugin@OleThread@@YA?AW4EDoMenu@CPlugin@@H_J@Z 000000018000a1c0 f   OleThread.obj
 0001:00009290       ?ShowMenu@OleThread@@YAHAEAVCFarMenu@@PEB_WH_N@Z 000000018000a290 f   OleThread.obj
 0001:000092f0       ?Startup@OleThread@@YAXXZ  000000018000a2f0 f   OleThread.obj
 0001:000093c0       ?Stop@OleThread@@YAXXZ     000000018000a3c0 f   OleThread.obj
 0001:000093e0       ?ThreadProc@OleThread@@YAKPEAX@Z 000000018000a3e0 f   OleThread.obj
 0001:00009510       ??0CPidl@@QEAA@XZ          000000018000a510 f   Pidl.obj
 0001:00009520       ??1CPidl@@QEAA@XZ          000000018000a520 f   Pidl.obj
 0001:00009570       ??BCPidl@@QEAAPEFAU_ITEMIDLIST@@XZ 000000018000a570 f   Pidl.obj
 0001:00009580       ??ICPidl@@QEAAPEAPEFAU_ITEMIDLIST@@XZ 000000018000a580 f   Pidl.obj
 0001:00009580       ?GetArray@CPidl@@QEAAPEAPEFBU_ITEMIDLIST@@XZ 000000018000a580 f   Pidl.obj
 0001:000095b0       ?Add@CPidl@@QEAAXPEFAU_ITEMIDLIST@@@Z 000000018000a5b0 f   Pidl.obj
 0001:00009620       ?Count@CPidl@@QEAAIXZ      000000018000a620 f   Pidl.obj
 0001:00009630       ?EnsureSpace@CPidl@@QEAAXXZ 000000018000a630 f   Pidl.obj
 0001:000096b0       ?GetAt@CPidl@@QEAAPEFAU_ITEMIDLIST@@I@Z 000000018000a6b0 f   Pidl.obj
 0001:000096d0       ?Insert@CPidl@@QEAAXIPEFAU_ITEMIDLIST@@@Z 000000018000a6d0 f   Pidl.obj
 0001:00009740       ??0CPlugin@@QEAA@PEBUPluginStartupInfo@@@Z 000000018000a740 f   Plugin.obj
 0001:000098f0       ??0PluginIntEditFieldBinding@@QEAA@AEBUPluginStartupInfo@@PEAPEAXHPEAHH@Z 000000018000a8f0 f i Plugin.obj
 0001:000099b0       ??0PluginUIntEditFieldBinding@@QEAA@AEBUPluginStartupInfo@@PEAPEAXHPEAIH@Z 000000018000a9b0 f i Plugin.obj
 0001:00009a70       ??1?$DialogBuilderBase@UFarDialogItem@@@@MEAA@XZ 000000018000aa70 f i Plugin.obj
 0001:00009af0       ??_E?$DialogBuilderBase@UFarDialogItem@@@@MEAAPEAXI@Z 000000018000aaf0 f i Plugin.obj
 0001:00009af0       ??_G?$DialogBuilderBase@UFarDialogItem@@@@MEAAPEAXI@Z 000000018000aaf0 f i Plugin.obj
 0001:00009b30       ??_G?$DialogItemBinding@UFarDialogItem@@@@UEAAPEAXI@Z 000000018000ab30 f i Plugin.obj
 0001:00009b30       ??_E?$DialogItemBinding@UFarDialogItem@@@@UEAAPEAXI@Z 000000018000ab30 f i Plugin.obj
 0001:00009b60       ??_GPluginCheckBoxBinding@@UEAAPEAXI@Z 000000018000ab60 f i Plugin.obj
 0001:00009b60       ??_EPluginCheckBoxBinding@@UEAAPEAXI@Z 000000018000ab60 f i Plugin.obj
 0001:00009b90       ??_EPluginDialogBuilder@@UEAAPEAXI@Z 000000018000ab90 f i Plugin.obj
 0001:00009b90       ??_GPluginDialogBuilder@@UEAAPEAXI@Z 000000018000ab90 f i Plugin.obj
 0001:00009be0       ??_EPluginRadioButtonBinding@@UEAAPEAXI@Z 000000018000abe0 f i Plugin.obj
 0001:00009be0       ??_GPluginRadioButtonBinding@@UEAAPEAXI@Z 000000018000abe0 f i Plugin.obj
 0001:00009c10       ??_GPluginIntEditFieldBinding@@UEAAPEAXI@Z 000000018000ac10 f i Plugin.obj
 0001:00009c10       ??_EPluginUIntEditFieldBinding@@UEAAPEAXI@Z 000000018000ac10 f i Plugin.obj
 0001:00009c10       ??_EPluginIntEditFieldBinding@@UEAAPEAXI@Z 000000018000ac10 f i Plugin.obj
 0001:00009c10       ??_GPluginUIntEditFieldBinding@@UEAAPEAXI@Z 000000018000ac10 f i Plugin.obj
 0001:00009c40       ?AddButtons@?$DialogBuilderBase@UFarDialogItem@@@@QEAAXHPEBHHH@Z 000000018000ac40 f i Plugin.obj
 0001:00009da0       ?AddIntEditField@PluginDialogBuilder@@UEAAPEAUFarDialogItem@@PEAHH@Z 000000018000ada0 f i Plugin.obj
 0001:00009eb0       ?AddUIntEditField@PluginDialogBuilder@@UEAAPEAUFarDialogItem@@PEAIH@Z 000000018000aeb0 f i Plugin.obj
 0001:00009fc0       ?CfgDlgProc@CPlugin@@IEAAXPEAX_J10@Z 000000018000afc0 f   Plugin.obj
 0001:0000a0e0       ?CfgDlgProcStatic@CPlugin@@KA_JPEAX_J10@Z 000000018000b0e0 f   Plugin.obj
 0001:0000a160       ?Configure@CPlugin@@QEAAHXZ 000000018000b160 f   Plugin.obj
 0001:0000b390       ?GetLangString@?$DialogBuilderBase@UFarDialogItem@@@@MEAAPEB_WH@Z 000000018000c390 f i Plugin.obj
 0001:0000b390       ?AddIntEditField@?$DialogBuilderBase@UFarDialogItem@@@@UEAAPEAUFarDialogItem@@PEAHH@Z 000000018000c390 f i Plugin.obj
 0001:0000b390       ?CreateRadioButtonBinding@?$DialogBuilderBase@UFarDialogItem@@@@MEAAPEAU?$DialogItemBinding@UFarDialogItem@@@@PEAH@Z 000000018000c390 f i Plugin.obj
 0001:0000b390       ?CreateCheckBoxBinding@?$DialogBuilderBase@UFarDialogItem@@@@MEAAPEAU?$DialogItemBinding@UFarDialogItem@@@@PEAHH@Z 000000018000c390 f i Plugin.obj
 0001:0000b390       ?AddUIntEditField@?$DialogBuilderBase@UFarDialogItem@@@@UEAAPEAUFarDialogItem@@PEAIH@Z 000000018000c390 f i Plugin.obj
 0001:0000b3a0       ?CreateCheckBoxBinding@PluginDialogBuilder@@MEAAPEAU?$DialogItemBinding@UFarDialogItem@@@@PEAHH@Z 000000018000c3a0 f i Plugin.obj
 0001:0000b420       ?CreateRadioButtonBinding@PluginDialogBuilder@@MEAAPEAU?$DialogItemBinding@UFarDialogItem@@@@PEAH@Z 000000018000c420 f i Plugin.obj
 0001:0000b490       ?DoMenu@CPlugin@@IEAA?AW4EDoMenu@1@PEAUIShellFolder@@PEAPEFBU_ITEMIDLIST@@QEAPEB_WIIPEB_WW4EAutoItem@1@@Z 000000018000c490 f   Plugin.obj
 0001:0000bd90       ?DoMenu@CPlugin@@IEAA?AW4EDoMenu@1@PEA_WW4CallMode@1@@Z 000000018000cd90 f   Plugin.obj
 0001:0000c020       ?DoShowDialog@?$DialogBuilderBase@UFarDialogItem@@@@MEAA_JXZ 000000018000d020 f i Plugin.obj
 0001:0000c030       ?DoShowDialog@PluginDialogBuilder@@MEAA_JXZ 000000018000d030 f i Plugin.obj
 0001:0000c0e0       ?ExitFAR@CPlugin@@QEAAXXZ  000000018000d0e0 f   Plugin.obj
 0001:0000c0f0       ?GetAdditionalString@CPlugin@@IEAA_NPEAUIContextMenu@@IW4EAdditionalStr@1@PEAVauto_sz@@@Z 000000018000d0f0 f   Plugin.obj
 0001:0000c1e0       ?GetFilesFromPanel@CPlugin@@IEAA_NPEAPEAPEB_WPEAI1PEAVauto_sz@@@Z 000000018000d1e0 f   Plugin.obj
 0001:0000c5d0       ?GetFilesFromParams@CPlugin@@IEAA_NPEA_WPEAPEAPEB_WPEAI2PEAVauto_sz@@_N@Z 000000018000d5d0 f   Plugin.obj
 0001:0000c7f0       ?GetLangString@PluginDialogBuilder@@MEAAPEB_WH@Z 000000018000d7f0 f i Plugin.obj
 0001:0000c800       ?GetPluginInfo@CPlugin@@QEAAXPEAUPluginInfo@@@Z 000000018000d800 f   Plugin.obj
 0001:0000c870       ?SaveValue@?$DialogItemBinding@UFarDialogItem@@@@UEAAXPEAUFarDialogItem@@H@Z 000000018000d870 f i Plugin.obj
 0001:0000c870       ?InitDialogItem@?$DialogBuilderBase@UFarDialogItem@@@@MEAAXPEAUFarDialogItem@@PEB_W@Z 000000018000d870 f i Plugin.obj
 0001:0000c870       ??1CPlugin@@QEAA@XZ        000000018000d870 f i Plugin.obj
 0001:0000c870       _guard_check_icall_nop     000000018000d870 f i LIBCMT:guard_support.obj
 0001:0000c870       __except_validate_context_record 000000018000d870 f i libvcruntime:jbcxrval.obj
 0001:0000c880       ?InitDialogItem@PluginDialogBuilder@@MEAAXPEAUFarDialogItem@@PEB_W@Z 000000018000d880 f i Plugin.obj
 0001:0000c8b0       ?IsWindowsVersionOrGreater@@YA_NGGG@Z 000000018000d8b0 f i Plugin.obj
 0001:0000c970       ?ItemWidth@?$DialogBuilderBase@UFarDialogItem@@@@IEAA_JAEBUFarDialogItem@@@Z 000000018000d970 f i Plugin.obj
 0001:0000ca10       ?MaxTextWidth@?$DialogBuilderBase@UFarDialogItem@@@@IEAA_JXZ 000000018000da10 f i Plugin.obj
 0001:0000cb40       ?MenuForPanelOrCmdLine@CPlugin@@IEAA?AW4EDoMenu@1@PEA_WW4EAutoItem@1@@Z 000000018000db40 f   Plugin.obj
 0001:0000cfb0       ?OpenPlugin@CPlugin@@QEAAPEAXH_J@Z 000000018000dfb0 f   Plugin.obj
 0001:0000d1d0       ?OpenPluginBkg@CPlugin@@QEAA?AW4EDoMenu@1@H_J@Z 000000018000e1d0 f   Plugin.obj
 0001:0000d300       ?ReadRegValues@CPlugin@@IEAAXXZ 000000018000e300 f   Plugin.obj
 0001:0000d5d0       ?ReallocDialogItems@?$DialogBuilderBase@UFarDialogItem@@@@IEAAXXZ 000000018000e5d0 f i Plugin.obj
 0001:0000d730       ?SaveValue@PluginCheckBoxBinding@@UEAAXPEAUFarDialogItem@@H@Z 000000018000e730 f i Plugin.obj
 0001:0000d790       ?SaveValue@PluginIntEditFieldBinding@@UEAAXPEAUFarDialogItem@@H@Z 000000018000e790 f i Plugin.obj
 0001:0000d7e0       ?SaveValue@PluginRadioButtonBinding@@UEAAXPEAUFarDialogItem@@H@Z 000000018000e7e0 f i Plugin.obj
 0001:0000d830       ?SaveValue@PluginUIntEditFieldBinding@@UEAAXPEAUFarDialogItem@@H@Z 000000018000e830 f i Plugin.obj
 0001:0000d880       ?SaveValues@?$DialogBuilderBase@UFarDialogItem@@@@IEAAXXZ 000000018000e880 f i Plugin.obj
 0001:0000d910       ?SelectDrive@CPlugin@@IEAA?AW4EDoMenu@1@XZ 000000018000e910 f   Plugin.obj
 0001:0000dd20       ?ShowFolder@CPlugin@@IEAA_NPEAUIShellFolder@@PEFBU_ITEMIDLIST@@PEAHPEB_WPEAPEAUIDropTarget@@@Z 000000018000ed20 f   Plugin.obj
 0001:0000e0a0       ?ShowGuiMenu@CPlugin@@IEAA_NPEAUHMENU__@@PEAUIContextMenu@@PEAUIContextMenu2@@PEAUIContextMenu3@@PEAH@Z 000000018000f0a0 f   Plugin.obj
 0001:0000e220       ?ShowTextMenu@CPlugin@@IEAA_NPEAUHMENU__@@PEAUIContextMenu@@PEAUIContextMenu2@@PEAUIContextMenu3@@PEAHPEB_WPEAUIShellFolder@@PEAPEFBU_ITEMIDLIST@@I@Z 000000018000f220 f   Plugin.obj
 0001:0000e810       ?TextWidth@?$DialogBuilderBase@UFarDialogItem@@@@MEAAHAEBUFarDialogItem@@@Z 000000018000f810 f i Plugin.obj
 0001:0000e820       ?TextWidth@PluginDialogBuilder@@MEAAHAEBUFarDialogItem@@@Z 000000018000f820 f i Plugin.obj
 0001:0000e830       ?UpdateBorderSize@?$DialogBuilderBase@UFarDialogItem@@@@IEAAXXZ 000000018000f830 f i Plugin.obj
 0001:0000e8e4       ??2@YAPEAX_K@Z             000000018000f8e4 f   LIBCMT:new_scalar.obj
 0001:0000e920       ??_U@YAPEAX_K@Z            000000018000f920 f   LIBCMT:new_array.obj
 0001:0000e928       ??_V@YAXPEAX@Z             000000018000f928 f   LIBCMT:delete_array.obj
 0001:0000e928       ??3@YAXPEAX_K@Z            000000018000f928 f   LIBCMT:delete_scalar_size.obj
 0001:0000eca0       _DllMainCRTStartup         000000018000fca0 f   LIBCMT:dll_dllmain.obj
 0001:0000ece0       ??0bad_alloc@std@@QEAA@AEBV01@@Z 000000018000fce0 f i LIBCMT:throw_bad_alloc.obj
 0001:0000ed20       ??0bad_alloc@std@@QEAA@XZ  000000018000fd20 f i LIBCMT:throw_bad_alloc.obj
 0001:0000ed40       ??0bad_array_new_length@std@@QEAA@AEBV01@@Z 000000018000fd40 f i LIBCMT:throw_bad_alloc.obj
 0001:0000ed80       ??0bad_array_new_length@std@@QEAA@XZ 000000018000fd80 f i LIBCMT:throw_bad_alloc.obj
 0001:0000eda0       ??0exception@std@@QEAA@AEBV01@@Z 000000018000fda0 f i LIBCMT:throw_bad_alloc.obj
 0001:0000edd8       ??1bad_alloc@std@@UEAA@XZ  000000018000fdd8 f i LIBCMT:throw_bad_alloc.obj
 0001:0000edd8       ??1bad_array_new_length@std@@UEAA@XZ 000000018000fdd8 f i LIBCMT:throw_bad_alloc.obj
 0001:0000edec       ??_Gbad_array_new_length@std@@UEAAPEAXI@Z 000000018000fdec f i LIBCMT:throw_bad_alloc.obj
 0001:0000edec       ??_Gexception@std@@UEAAPEAXI@Z 000000018000fdec f i LIBCMT:throw_bad_alloc.obj
 0001:0000edec       ??_Gbad_alloc@std@@UEAAPEAXI@Z 000000018000fdec f i LIBCMT:throw_bad_alloc.obj
 0001:0000edec       ??_Ebad_alloc@std@@UEAAPEAXI@Z 000000018000fdec f i LIBCMT:throw_bad_alloc.obj
 0001:0000edec       ??_Eexception@std@@UEAAPEAXI@Z 000000018000fdec f i LIBCMT:throw_bad_alloc.obj
 0001:0000edec       ??_Ebad_array_new_length@std@@UEAAPEAXI@Z 000000018000fdec f i LIBCMT:throw_bad_alloc.obj
 0001:0000ee30       ?__scrt_throw_std_bad_alloc@@YAXXZ 000000018000fe30 f   LIBCMT:throw_bad_alloc.obj
 0001:0000ee50       ?__scrt_throw_std_bad_array_new_length@@YAXXZ 000000018000fe50 f   LIBCMT:throw_bad_alloc.obj
 0001:0000ee70       ?what@exception@std@@UEBAPEBDXZ 000000018000fe70 f i LIBCMT:throw_bad_alloc.obj
 0001:0000ee84       ??3@YAXPEAX@Z              000000018000fe84 f   LIBCMT:delete_scalar.obj
 0001:0000ee8c       __scrt_acquire_startup_lock 000000018000fe8c f   LIBCMT:utility.obj
 0001:0000eec8       __scrt_dllmain_after_initialize_c 000000018000fec8 f   LIBCMT:utility.obj
 0001:0000eefc       __scrt_dllmain_before_initialize_c 000000018000fefc f   LIBCMT:utility.obj
 0001:0000ef14       __scrt_dllmain_crt_thread_attach 000000018000ff14 f   LIBCMT:utility.obj
 0001:0000ef3c       __scrt_dllmain_crt_thread_detach 000000018000ff3c f   LIBCMT:utility.obj
 0001:0000ef54       __scrt_dllmain_exception_filter 000000018000ff54 f   LIBCMT:utility.obj
 0001:0000efb8       __scrt_dllmain_uninitialize_c 000000018000ffb8 f   LIBCMT:utility.obj
 0001:0000efe8       __scrt_dllmain_uninitialize_critical 000000018000ffe8 f   LIBCMT:utility.obj
 0001:0000effc       __scrt_initialize_crt      000000018000fffc f   LIBCMT:utility.obj
 0001:0000f048       __scrt_initialize_onexit_tables 0000000180010048 f   LIBCMT:utility.obj
 0001:0000f114       __scrt_is_nonwritable_in_current_image 0000000180010114 f   LIBCMT:utility.obj
 0001:0000f1b0       __scrt_release_startup_lock 00000001800101b0 f   LIBCMT:utility.obj
 0001:0000f1d4       __scrt_uninitialize_crt    00000001800101d4 f   LIBCMT:utility.obj
 0001:0000f200       _onexit                    0000000180010200 f   LIBCMT:utility.obj
 0001:0000f250       atexit                     0000000180010250 f   LIBCMT:utility.obj
 0001:0000f268       __security_init_cookie     0000000180010268 f   LIBCMT:gs_support.obj
 0001:0000f314       ?__scrt_initialize_type_info@@YAXXZ 0000000180010314 f   LIBCMT:tncleanup.obj
 0001:0000f324       ?__scrt_uninitialize_type_info@@YAXXZ 0000000180010324 f   LIBCMT:tncleanup.obj
 0001:0000f330       __local_stdio_printf_options 0000000180010330 f i LIBCMT:default_local_stdio_options.obj
 0001:0000f338       __local_stdio_scanf_options 0000000180010338 f i LIBCMT:default_local_stdio_options.obj
 0001:0000f340       __scrt_initialize_default_local_stdio_options 0000000180010340 f   LIBCMT:default_local_stdio_options.obj
 0001:0000f35c       __scrt_get_dyn_tls_init_callback 000000018001035c f   LIBCMT:dyn_tls_init.obj
 0001:0000f364       __crt_debugger_hook        0000000180010364 f   LIBCMT:utility_desktop.obj
 0001:0000f36c       __scrt_fastfail            000000018001036c f   LIBCMT:utility_desktop.obj
 0001:0000f4b4       _RTC_Initialize            00000001800104b4 f   LIBCMT:_initsect_.obj
 0001:0000f500       _RTC_Terminate             0000000180010500 f   LIBCMT:_initsect_.obj
 0001:0000f54c       _guard_check_icall         000000018001054c f i LIBCMT:checkcfg.obj
 0001:0000f554       ??_Etype_info@@UEAAPEAXI@Z 0000000180010554 f i LIBCMT:std_type_info_static.obj
 0001:0000f554       ??_Gtype_info@@UEAAPEAXI@Z 0000000180010554 f i LIBCMT:std_type_info_static.obj
 0001:0000f580       __isa_available_init       0000000180010580 f   LIBCMT:_cpu_disp_.obj
 0001:0000f744       _get_startup_argv_mode     0000000180010744 f   LIBCMT:argv_mode.obj
 0001:0000f744       DllMain                    0000000180010744 f   LIBCMT:dll_dllmain_stub.obj
 0001:0000f74c       __scrt_is_ucrt_dll_in_use  000000018001074c f   LIBCMT:ucrt_detection.obj
 0001:0000f760       ?_com_issue_error@@YAXJ@Z  0000000180010760 f   comsuppw:comsupp.obj
 0001:0000f790       ??0_com_error@@QEAA@AEBV0@@Z 0000000180010790 f i comsuppw:comraise.obj
 0001:0000f800       ??0_com_error@@QEAA@JPEAUIErrorInfo@@_N@Z 0000000180010800 f i comsuppw:comraise.obj
 0001:0000f870       ??1_com_error@@UEAA@XZ     0000000180010870 f i comsuppw:comraise.obj
 0001:0000f8e0       ??_G_com_error@@UEAAPEAXI@Z 00000001800108e0 f i comsuppw:comraise.obj
 0001:0000f8e0       ??_E_com_error@@UEAAPEAXI@Z 00000001800108e0 f i comsuppw:comraise.obj
 0001:0000f920       ?_com_raise_error@@YAXJPEAUIErrorInfo@@@Z 0000000180010920 f   comsuppw:comraise.obj
 0001:0000f960       memcpy                     0000000180010960 f   libvcruntime:memcpy.obj
 0001:0000f960       memmove                    0000000180010960 f   libvcruntime:memcpy.obj
 0001:0000fd98       __C_specific_handler       0000000180010d98 f   libvcruntime:_chandler_.obj
 0001:0000ffb0       memset                     0000000180010fb0 f   libvcruntime:memset.obj
 0001:00010154       __telemetry_main_invoke_trigger 0000000180011154 f   libvcruntime:telemetry.obj
 0001:0001026c       __telemetry_main_return_trigger 000000018001126c f   libvcruntime:telemetry.obj
 0001:00010384       __vcrt_initialize_telemetry_provider 0000000180011384 f   libvcruntime:telemetry.obj
 0001:00010398       __vcrt_uninitialize_telemetry_provider 0000000180011398 f   libvcruntime:telemetry.obj
 0001:000103b8       __std_exception_copy       00000001800113b8 f   libvcruntime:std_exception.obj
 0001:00010448       __std_exception_destroy    0000000180011448 f   libvcruntime:std_exception.obj
 0001:00010470       _CxxThrowException         0000000180011470 f   libvcruntime:throw.obj
 0001:00010548       __vcrt_initialize          0000000180011548 f   libvcruntime:initialization.obj
 0001:00010580       __vcrt_thread_attach       0000000180011580 f   libvcruntime:initialization.obj
 0001:00010594       __vcrt_thread_detach       0000000180011594 f   libvcruntime:initialization.obj
 0001:000105a8       __vcrt_uninitialize        00000001800115a8 f   libvcruntime:initialization.obj
 0001:000105d4       __vcrt_uninitialize_critical 00000001800115d4 f   libvcruntime:initialization.obj
 0001:000105e4       __std_type_info_destroy_list 00000001800115e4 f   libvcruntime:std_type_info.obj
 0001:00010620       _local_unwind              0000000180011620 f   libvcruntime:_jmpuwind_.obj
 0001:00010650       _NLG_Notify                0000000180011650 f   libvcruntime:_jmpuwind_.obj
 0001:00010670       __NLG_Dispatch2            0000000180011670 f   libvcruntime:_jmpuwind_.obj
 0001:00010680       __NLG_Return2              0000000180011680 f   libvcruntime:_jmpuwind_.obj
 0001:0001084c       __vcrt_EventRegister       000000018001184c f   libvcruntime:winapi_downlevel.obj
 0001:000108d0       __vcrt_EventSetInformation 00000001800118d0 f   libvcruntime:winapi_downlevel.obj
 0001:00010954       __vcrt_EventUnregister     0000000180011954 f   libvcruntime:winapi_downlevel.obj
 0001:000109a8       __vcrt_EventWriteTransfer  00000001800119a8 f   libvcruntime:winapi_downlevel.obj
 0001:00010a40       __vcrt_FlsAlloc            0000000180011a40 f   libvcruntime:winapi_downlevel.obj
 0001:00010a94       __vcrt_FlsFree             0000000180011a94 f   libvcruntime:winapi_downlevel.obj
 0001:00010ae8       __vcrt_FlsGetValue         0000000180011ae8 f   libvcruntime:winapi_downlevel.obj
 0001:00010b3c       __vcrt_FlsSetValue         0000000180011b3c f   libvcruntime:winapi_downlevel.obj
 0001:00010ba4       __vcrt_InitializeCriticalSectionEx 0000000180011ba4 f   libvcruntime:winapi_downlevel.obj
 0001:00010c1c       __vcrt_initialize_winapi_thunks 0000000180011c1c f   libvcruntime:winapi_downlevel.obj
 0001:00010c54       __vcrt_uninitialize_winapi_thunks 0000000180011c54 f   libvcruntime:winapi_downlevel.obj
 0001:00010c94       __vcrt_freefls             0000000180011c94 f   libvcruntime:per_thread_data.obj
 0001:00010cb4       __vcrt_freeptd             0000000180011cb4 f   libvcruntime:per_thread_data.obj
 0001:00010d04       __vcrt_getptd_noexit       0000000180011d04 f   libvcruntime:per_thread_data.obj
 0001:00010dbc       __vcrt_initialize_ptd      0000000180011dbc f   libvcruntime:per_thread_data.obj
 0001:00010dfc       __vcrt_uninitialize_ptd    0000000180011dfc f   libvcruntime:per_thread_data.obj
 0001:00010e20       __vcrt_initialize_locks    0000000180011e20 f   libvcruntime:locks.obj
 0001:00010e68       __vcrt_uninitialize_locks  0000000180011e68 f   libvcruntime:locks.obj
 0001:00010ea0       __vcrt_initialize_pure_virtual_call_handler 0000000180011ea0 f   libvcruntime:purevirt_data.obj
 0001:00010ec4       __acrt_initialize_new_handler 0000000180011ec4 f   libucrt:new_handler.obj
 0001:00010ecc       _callnewh                  0000000180011ecc f   libucrt:new_handler.obj
 0001:00010f0c       _query_new_handler         0000000180011f0c f   libucrt:new_handler.obj
 0001:00010f40       malloc                     0000000180011f40 f   libucrt:malloc.obj
 0001:00010f48       _initterm                  0000000180011f48 f   libucrt:initterm.obj
 0001:00010fc0       _initterm_e                0000000180011fc0 f   libucrt:initterm.obj
 0001:0001100c       free                       000000018001200c f   libucrt:free.obj
 0001:00011014       _seh_filter_dll            0000000180012014 f   libucrt:exception_filter.obj
 0001:00011028       _seh_filter_exe            0000000180012028 f   libucrt:exception_filter.obj
 0001:000113e8       __acrt_initialize_thread_local_exit_callback 00000001800123e8 f   libucrt:exit.obj
 0001:000113f0       _cexit                     00000001800123f0 f   libucrt:exit.obj
 0001:00011400       _exit                      0000000180012400 f   libucrt:exit.obj
 0001:0001140c       _is_c_termination_complete 000000018001240c f   libucrt:exit.obj
 0001:000115d0       __acrt_allocate_buffer_for_argv 00000001800125d0 f   libucrt:argv_parsing.obj
 0001:00011634       _configure_narrow_argv     0000000180012634 f   libucrt:argv_parsing.obj
 0001:00011990       __dcrt_uninitialize_environments_nolock 0000000180012990 f   libucrt:environment_initialization.obj
 0001:000119c8       _initialize_narrow_environment 00000001800129c8 f   libucrt:environment_initialization.obj
 0001:000119d0       ??$?RV<lambda_b8c45f8f788dd370798f47cfe8ac3a86>@@AEAV<lambda_4e60a939b0d047cfe11ddc22648dfba9>@@V<lambda_332c3edc96d0294ec56c57d38c1cdfd5>@@@?$__crt_seh_guarded_call@H@@QEAAH$$QEAV<lambda_b8c45f8f788dd370798f47cfe8ac3a86>@@AEAV<lambda_4e60a939b0d047cfe11ddc22648dfba9>@@$$QEAV<lambda_332c3edc96d0294ec56c57d38c1cdfd5>@@@Z 00000001800129d0 f i libucrt:onexit.obj
 0001:00011a0c       ??$?RV<lambda_e24bbb7b643b32fcea6fa61b31d4c984>@@AEAV<lambda_275893d493268fdec8709772e3fcec0e>@@V<lambda_9d71df4d7cf3f480f8d633942495c3b0>@@@?$__crt_seh_guarded_call@H@@QEAAH$$QEAV<lambda_e24bbb7b643b32fcea6fa61b31d4c984>@@AEAV<lambda_275893d493268fdec8709772e3fcec0e>@@$$QEAV<lambda_9d71df4d7cf3f480f8d633942495c3b0>@@@Z 0000000180012a0c f i libucrt:onexit.obj
 0001:00011d88       _crt_atexit                0000000180012d88 f   libucrt:onexit.obj
 0001:00011d98       _execute_onexit_table      0000000180012d98 f   libucrt:onexit.obj
 0001:00011dd4       _initialize_onexit_table   0000000180012dd4 f   libucrt:onexit.obj
 0001:00011e14       _register_onexit_function  0000000180012e14 f   libucrt:onexit.obj
 0001:00011ea4       __acrt_uninitialize_command_line 0000000180012ea4 f   libucrt:argv_data.obj
 0001:00011f94       __acrt_initialize          0000000180012f94 f   libucrt:initialization.obj
 0001:00011fa8       __acrt_thread_attach       0000000180012fa8 f   libucrt:initialization.obj
 0001:00011fbc       __acrt_thread_detach       0000000180012fbc f   libucrt:initialization.obj
 0001:00011fcc       __acrt_uninitialize        0000000180012fcc f   libucrt:initialization.obj
 0001:00011fe0       __acrt_uninitialize_critical 0000000180012fe0 f   libucrt:initialization.obj
 0001:00011ff0       terminate                  0000000180012ff0 f   libucrt:terminate.obj
 0001:00012018       strcpy_s                   0000000180013018 f   libucrt:strcpy_s.obj
 0001:00012078       _free_base                 0000000180013078 f   libucrt:free_base.obj
 0001:000120b8       _malloc_base               00000001800130b8 f   libucrt:malloc_base.obj
 0001:00012118       abort                      0000000180013118 f   libucrt:abort.obj
 0001:00012170       _calloc_base               0000000180013170 f   libucrt:calloc_base.obj
 0001:000121e8       ??0_LocaleUpdate@@QEAA@QEAU__crt_locale_pointers@@@Z 00000001800131e8 f i libucrt:output.obj
 0001:00012278       __acrt_initialize_locks    0000000180013278 f   libucrt:locks.obj
 0001:000122c0       __acrt_lock                00000001800132c0 f   libucrt:locks.obj
 0001:000122dc       __acrt_uninitialize_locks  00000001800132dc f   libucrt:locks.obj
 0001:00012314       __acrt_unlock              0000000180013314 f   libucrt:locks.obj
 0001:00012330       ??$?RV<lambda_46352004c1216016012b18bd6f87e700>@@AEAV<lambda_3bd07e1a1191394380780325891bf33f>@@V<lambda_334532d3f185bcaa59b5be82d7d22bff>@@@?$__crt_seh_guarded_call@X@@QEAAX$$QEAV<lambda_46352004c1216016012b18bd6f87e700>@@AEAV<lambda_3bd07e1a1191394380780325891bf33f>@@$$QEAV<lambda_334532d3f185bcaa59b5be82d7d22bff>@@@Z 0000000180013330 f i libucrt:per_thread_data.obj
 0001:00012390       ??$?RV<lambda_5e887d1dcbef67a5eb4283622ba103bf>@@AEAV<lambda_4466841279450cc726390878d4a41900>@@V<lambda_341c25c0346d94847f1f3c463c57e077>@@@?$__crt_seh_guarded_call@X@@QEAAX$$QEAV<lambda_5e887d1dcbef67a5eb4283622ba103bf>@@AEAV<lambda_4466841279450cc726390878d4a41900>@@$$QEAV<lambda_341c25c0346d94847f1f3c463c57e077>@@@Z 0000000180013390 f i libucrt:per_thread_data.obj
 0001:000123d8       ??$?RV<lambda_72d1df2b273a38828b1ce30cbf4cdab5>@@AEAV<lambda_876a65b173b8412d3a47c70a915b0cf4>@@V<lambda_41932305e351933ebe8f8be3ed8bb5dc>@@@?$__crt_seh_guarded_call@X@@QEAAX$$QEAV<lambda_72d1df2b273a38828b1ce30cbf4cdab5>@@AEAV<lambda_876a65b173b8412d3a47c70a915b0cf4>@@$$QEAV<lambda_41932305e351933ebe8f8be3ed8bb5dc>@@@Z 00000001800133d8 f i libucrt:per_thread_data.obj
 0001:00012418       ??$?RV<lambda_fb3a7dec4e47f37f22dae91bb15c9095>@@AEAV<lambda_698284760c8add0bfb0756c19673e34b>@@V<lambda_dfb8eca1e75fef3034a8fb18dd509707>@@@?$__crt_seh_guarded_call@X@@QEAAX$$QEAV<lambda_fb3a7dec4e47f37f22dae91bb15c9095>@@AEAV<lambda_698284760c8add0bfb0756c19673e34b>@@$$QEAV<lambda_dfb8eca1e75fef3034a8fb18dd509707>@@@Z 0000000180013418 f i libucrt:per_thread_data.obj
 0001:000126a8       __acrt_freeptd             00000001800136a8 f   libucrt:per_thread_data.obj
 0001:000126ec       __acrt_getptd              00000001800136ec f   libucrt:per_thread_data.obj
 0001:00012780       __acrt_getptd_noexit       0000000180013780 f   libucrt:per_thread_data.obj
 0001:00012820       __acrt_initialize_ptd      0000000180013820 f   libucrt:per_thread_data.obj
 0001:0001285c       __acrt_uninitialize_ptd    000000018001385c f   libucrt:per_thread_data.obj
 0001:00012a20       __acrt_FlsAlloc            0000000180013a20 f   libucrt:winapi_thunks.obj
 0001:00012a78       __acrt_FlsFree             0000000180013a78 f   libucrt:winapi_thunks.obj
 0001:00012ad0       __acrt_FlsGetValue         0000000180013ad0 f   libucrt:winapi_thunks.obj
 0001:00012b28       __acrt_FlsSetValue         0000000180013b28 f   libucrt:winapi_thunks.obj
 0001:00012b90       __acrt_InitializeCriticalSectionEx 0000000180013b90 f   libucrt:winapi_thunks.obj
 0001:00012c08       __acrt_LCMapStringEx       0000000180013c08 f   libucrt:winapi_thunks.obj
 0001:00012cf8       __acrt_LocaleNameToLCID    0000000180013cf8 f   libucrt:winapi_thunks.obj
 0001:00012d60       __acrt_initialize_winapi_thunks 0000000180013d60 f   libucrt:winapi_thunks.obj
 0001:00012d98       __acrt_is_packaged_app     0000000180013d98 f   libucrt:winapi_thunks.obj
 0001:00012e20       __acrt_uninitialize_winapi_thunks 0000000180013e20 f   libucrt:winapi_thunks.obj
 0001:00012e64       __acrt_call_reportfault    0000000180013e64 f   libucrt:invalid_parameter.obj
 0001:00012fc0       __acrt_initialize_invalid_parameter_handler 0000000180013fc0 f   libucrt:invalid_parameter.obj
 0001:00012fc8       _invalid_parameter         0000000180013fc8 f   libucrt:invalid_parameter.obj
 0001:00013070       _invalid_parameter_noinfo  0000000180014070 f   libucrt:invalid_parameter.obj
 0001:00013090       _invoke_watson             0000000180014090 f   libucrt:invalid_parameter.obj
 0001:000130d8       __acrt_errno_from_os_error 00000001800140d8 f   libucrt:errno.obj
 0001:00013120       __acrt_errno_map_os_error  0000000180014120 f   libucrt:errno.obj
 0001:00013170       __doserrno                 0000000180014170 f   libucrt:errno.obj
 0001:00013190       _errno                     0000000180014190 f   libucrt:errno.obj
 0001:0001368c       ?expand_if_necessary@?$argument_list@D@?A0xca0879c4@@AEAAHXZ 000000018001468c f i libucrt:argv_wildcards.obj
 0001:00013754       __acrt_expand_narrow_argv_wildcards 0000000180014754 f   libucrt:argv_wildcards.obj
 0001:0001375c       ??$?RV<lambda_99476a1ad63dd22509b5d3e65b0ffc95>@@AEAV<lambda_ad1ced32f4ac17aa236e5ef05d6b3b7c>@@V<lambda_f7424dd8d45958661754dc4f2697e9c3>@@@?$__crt_seh_guarded_call@X@@QEAAX$$QEAV<lambda_99476a1ad63dd22509b5d3e65b0ffc95>@@AEAV<lambda_ad1ced32f4ac17aa236e5ef05d6b3b7c>@@$$QEAV<lambda_f7424dd8d45958661754dc4f2697e9c3>@@@Z 000000018001475c f i libucrt:mbctype.obj
 0001:00013e58       __acrt_initialize_multibyte 0000000180014e58 f   libucrt:mbctype.obj
 0001:00013e80       __acrt_update_thread_multibyte_data 0000000180014e80 f   libucrt:mbctype.obj
 0001:00013f40       _setmbcp_nolock            0000000180014f40 f   libucrt:mbctype.obj
 0001:00014260       _ismbblead                 0000000180015260 f   libucrt:ismbbyte.obj
 0001:00014274       __acrt_initialize_command_line 0000000180015274 f   libucrt:argv_data.obj
 0001:0001429c       __dcrt_get_narrow_environment_from_os 000000018001529c f   libucrt:get_environment_from_os.obj
 0001:000143a0       _recalloc                  00000001800153a0 f   libucrt:recalloc.obj
 0001:000143a8       _recalloc_base             00000001800153a8 f   libucrt:recalloc.obj
 0001:00014440       __acrt_initialize_heap     0000000180015440 f   libucrt:heap_handle.obj
 0001:0001445c       __acrt_uninitialize_heap   000000018001545c f   libucrt:heap_handle.obj
 0001:00014650       __acrt_initialize_lowio    0000000180015650 f   libucrt:ioinit.obj
 0001:0001468c       __acrt_uninitialize_lowio  000000018001568c f   libucrt:ioinit.obj
 0001:000146cc       __acrt_execute_initializers 00000001800156cc f   libucrt:shared_initialization.obj
 0001:00014760       __acrt_execute_uninitializers 0000000180015760 f   libucrt:shared_initialization.obj
 0001:000147b0       ??$?RV<lambda_c36588078e9f5dfd39652860aa6b3aaf>@@AEAV<lambda_ec61778202f4f5fc7e7711acc23c3bca>@@V<lambda_dc9d2797ccde5d239b4a0efae8ebd7db>@@@?$__crt_seh_guarded_call@P6AXH@Z@@QEAAP6AXH@Z$$QEAV<lambda_c36588078e9f5dfd39652860aa6b3aaf>@@AEAV<lambda_ec61778202f4f5fc7e7711acc23c3bca>@@$$QEAV<lambda_dc9d2797ccde5d239b4a0efae8ebd7db>@@@Z 00000001800157b0 f i libucrt:signal.obj
 0001:000147f8       __acrt_get_sigabrt_handler 00000001800157f8 f   libucrt:signal.obj
 0001:00014828       __acrt_initialize_signal_handlers 0000000180015828 f   libucrt:signal.obj
 0001:00014848       raise                      0000000180015848 f   libucrt:signal.obj
 0001:00014ae4       __acrt_has_user_matherr    0000000180015ae4 f   libucrt:matherr.obj
 0001:00014b04       __acrt_initialize_user_matherr 0000000180015b04 f   libucrt:matherr.obj
 0001:00014b0c       __acrt_invoke_user_matherr 0000000180015b0c f   libucrt:matherr.obj
 0001:00014b54       _query_new_mode            0000000180015b54 f   libucrt:new_mode.obj
 0001:00014b5c       _mbtowc_l                  0000000180015b5c f   libucrt:mbtowc.obj
 0001:00014ca4       mbtowc                     0000000180015ca4 f   libucrt:mbtowc.obj
 0001:00014cac       __acrt_update_locale_info  0000000180015cac f   libucrt:locale_update.obj
 0001:00014ce0       __acrt_update_multibyte_info 0000000180015ce0 f   libucrt:locale_update.obj
 0001:00014d14       _fileno                    0000000180015d14 f   libucrt:fileno.obj
 0001:00014d3c       __acrt_initialize_stdio    0000000180015d3c f   libucrt:_file.obj
 0001:00014e5c       __acrt_uninitialize_stdio  0000000180015e5c f   libucrt:_file.obj
 0001:00014eb8       _lock_file                 0000000180015eb8 f   libucrt:_file.obj
 0001:00014ec4       _unlock_file               0000000180015ec4 f   libucrt:_file.obj
 0001:00014ed0       __acrt_set_locale_changed  0000000180015ed0 f   libucrt:wsetlocale.obj
 0001:00014edc       __acrt_uninitialize_locale 0000000180015edc f   libucrt:wsetlocale.obj
 0001:00014f24       __pctype_func              0000000180015f24 f   libucrt:ctype.obj
 0001:00014f54       __acrt_add_locale_ref      0000000180015f54 f   libucrt:locale_refcounting.obj
 0001:00014fe0       __acrt_free_locale         0000000180015fe0 f   libucrt:locale_refcounting.obj
 0001:00015158       __acrt_locale_add_lc_time_reference 0000000180016158 f   libucrt:locale_refcounting.obj
 0001:00015180       __acrt_locale_free_lc_time_if_unreferenced 0000000180016180 f   libucrt:locale_refcounting.obj
 0001:000151b8       __acrt_locale_release_lc_time_reference 00000001800161b8 f   libucrt:locale_refcounting.obj
 0001:000151e0       __acrt_release_locale_ref  00000001800161e0 f   libucrt:locale_refcounting.obj
 0001:00015288       __acrt_update_thread_locale_data 0000000180016288 f   libucrt:locale_refcounting.obj
 0001:000152f8       _updatetlocinfoEx_nolock   00000001800162f8 f   libucrt:locale_refcounting.obj
 0001:00015428       __acrt_DownlevelLocaleNameToLCID 0000000180016428 f   libucrt:lcidtoname_downlevel.obj
 0001:00015530       qsort                      0000000180016530 f   libucrt:qsort.obj
 0001:00015864       strncpy_s                  0000000180016864 f   libucrt:strncpy_s.obj
 0001:00015938       strpbrk                    0000000180016938 f   libucrt:strpbrk.obj
 0001:000159d8       _mbsdec                    00000001800169d8 f   libucrt:mbsdec.obj
 0001:000159e0       _mbsdec_l                  00000001800169e0 f   libucrt:mbsdec.obj
 0001:00015a90       __acrt_GetStringTypeA      0000000180016a90 f   libucrt:getstringtypea.obj
 0001:00015fa0       __acrt_LCMapStringA        0000000180016fa0 f   libucrt:lcmapstringa.obj
 0001:00016038       _msize                     0000000180017038 f   libucrt:msize.obj
 0001:00016074       _realloc_base              0000000180017074 f   libucrt:realloc_base.obj
 0001:000160f8       __acrt_lowio_create_handle_array 00000001800170f8 f   libucrt:osfinfo.obj
 0001:00016190       __acrt_lowio_destroy_handle_array 0000000180017190 f   libucrt:osfinfo.obj
 0001:000161e0       __acrt_lowio_ensure_fh_exists 00000001800171e0 f   libucrt:osfinfo.obj
 0001:00016298       __acrt_lowio_lock_fh       0000000180017298 f   libucrt:osfinfo.obj
 0001:000162bc       __acrt_lowio_unlock_fh     00000001800172bc f   libucrt:osfinfo.obj
 0001:000162e0       _free_osfhnd               00000001800172e0 f   libucrt:osfinfo.obj
 0001:0001639c       _get_osfhandle             000000018001739c f   libucrt:osfinfo.obj
 0001:00016414       _isatty                    0000000180017414 f   libucrt:isatty.obj
 0001:00016474       __acrt_stdio_flush_nolock  0000000180017474 f   libucrt:fflush.obj
 0001:000164ec       _fflush_nolock             00000001800174ec f   libucrt:fflush.obj
 0001:00016538       _flushall                  0000000180017538 f   libucrt:fflush.obj
 0001:00016628       _isleadbyte_l              0000000180017628 f i libucrt:_wctype.obj
 0001:00016668       _fcloseall                 0000000180017668 f   libucrt:closeall.obj
 0001:0001671c       __acrt_stdio_free_buffer_nolock 000000018001771c f   libucrt:_freebuf.obj
 0001:0001675c       __acrt_locale_free_monetary 000000018001775c f   libucrt:initmon.obj
 0001:00016868       __acrt_locale_free_numeric 0000000180017868 f   libucrt:initnum.obj
 0001:0001692c       __acrt_locale_free_time    000000018001792c f   libucrt:inittime.obj
 0001:00016a34       __strncnt                  0000000180017a34 f   libucrt:strncnt.obj
 0001:00016a4c       _query_app_type            0000000180017a4c f   libucrt:report_runtime_error.obj
 0001:00016a54       ??$?RV<lambda_b521505b218e5242e90febf6bfebc422>@@AEAV<lambda_6978c1fb23f02e42e1d9e99668cc68aa>@@V<lambda_314360699dd331753a4119843814e9a7>@@@?$__crt_seh_guarded_call@H@@QEAAH$$QEAV<lambda_b521505b218e5242e90febf6bfebc422>@@AEAV<lambda_6978c1fb23f02e42e1d9e99668cc68aa>@@$$QEAV<lambda_314360699dd331753a4119843814e9a7>@@@Z 0000000180017a54 f i libucrt:commit.obj
 0001:00016ae0       _commit                    0000000180017ae0 f   libucrt:commit.obj
 0001:00017114       _write                     0000000180018114 f   libucrt:write.obj
 0001:00017200       _write_nolock              0000000180018200 f   libucrt:write.obj
 0001:000174f0       log10                      00000001800184f0 f   libucrt:log10.obj
 0001:00017b38       _lseeki64_nolock           0000000180018b38 f   libucrt:lseek.obj
 0001:00017b40       _fclose_nolock             0000000180018b40 f   libucrt:fclose.obj
 0001:00017bc4       fclose                     0000000180018bc4 f   libucrt:fclose.obj
 0001:00017c30       _putwch_nolock             0000000180018c30 f   libucrt:putwch.obj
 0001:00017db0       _handle_error              0000000180018db0 f   libucrt:libm_error.obj
 0001:00017ee0       __acrt_initialize_fma3     0000000180018ee0 f   libucrt:fma3_available.obj
 0001:00017f50       _log10_special             0000000180018f50 f   libucrt:log_special.obj
 0001:00018008       ??$?RV<lambda_bfedae4ebbf01fab1bb6dcc6a9e276e0>@@AEAV<lambda_2fe9b910cf3cbf4a0ab98a02ba45b3ec>@@V<lambda_237c231691f317818eb88cc1d5d642d6>@@@?$__crt_seh_guarded_call@H@@QEAAH$$QEAV<lambda_bfedae4ebbf01fab1bb6dcc6a9e276e0>@@AEAV<lambda_2fe9b910cf3cbf4a0ab98a02ba45b3ec>@@$$QEAV<lambda_237c231691f317818eb88cc1d5d642d6>@@@Z 0000000180019008 f i libucrt:close.obj
 0001:0001807c       _close                     000000018001907c f   libucrt:close.obj
 0001:00018120       _close_nolock              0000000180019120 f   libucrt:close.obj
 0001:000181dc       ?__acrt_stdio_free_stream@@YAXV__crt_stdio_stream@@@Z 00000001800191dc f   libucrt:stream.obj
 0001:00018220       __dcrt_lowio_initialize_console_output 0000000180019220 f   libucrt:initcon.obj
 0001:0001825c       __dcrt_terminate_console_output 000000018001925c f   libucrt:initcon.obj
 0001:00018290       _get_fpsr                  0000000180019290 f   libucrt:fpsr.obj
 0001:000182a0       _set_fpsr                  00000001800192a0 f   libucrt:fpsr.obj
 0001:000182aa       _fclrf                     00000001800192aa f   libucrt:fpsr.obj
 0001:000182be       _frnd                      00000001800192be f   libucrt:fpsr.obj
 0001:000182e0       _raise_exc                 00000001800192e0 f   libucrt:fpexcept.obj
 0001:00018308       _raise_exc_ex              0000000180019308 f   libucrt:fpexcept.obj
 0001:00018610       _set_errno_from_matherr    0000000180019610 f   libucrt:fpexcept.obj
 0001:00018640       _clrfp                     0000000180019640 f   libucrt:fpctrl.obj
 0001:00018660       _ctrlfp                    0000000180019660 f   libucrt:fpctrl.obj
 0001:000186dc       _set_statfp                00000001800196dc f   libucrt:fpctrl.obj
 0001:000186fc       _statfp                    00000001800196fc f   libucrt:fpctrl.obj
 0001:0001870e       IsProcessorFeaturePresent  000000018001970e f   kernel32:KERNEL32.dll
 0001:00018714       RtlUnwindEx                0000000180019714 f   kernel32:KERNEL32.dll
 0001:0001871a       SystemFunction036          000000018001971a f   advapi32:ADVAPI32.dll
 0001:00018730       __security_check_cookie    0000000180019730 f   LIBCMT:_amdsecgs_.obj
 0001:00018760       _FindPESection             0000000180019760 f   LIBCMT:pesect.obj
 0001:000187b0       _IsNonwritableInCurrentImage 00000001800197b0 f   LIBCMT:pesect.obj
 0001:00018800       _ValidateImageBase         0000000180019800 f   LIBCMT:pesect.obj
 0001:00018830       __GSHandlerCheck           0000000180019830 f   LIBCMT:_gshandler_.obj
 0001:00018850       __GSHandlerCheckCommon     0000000180019850 f   LIBCMT:_gshandler_.obj
 0001:000188ac       __raise_securityfailure    00000001800198ac f   LIBCMT:gs_report.obj
 0001:000188e0       __report_gsfailure         00000001800198e0 f   LIBCMT:gs_report.obj
 0001:000189b4       __report_rangecheckfailure 00000001800199b4 f   LIBCMT:gs_report.obj
 0001:000189c8       __report_securityfailure   00000001800199c8 f   LIBCMT:gs_report.obj
 0001:00018b60       memcmp                     0000000180019b60 f   libvcruntime:memcmp.obj
 0001:00018c40       _guard_dispatch_icall_nop  0000000180019c40 f   LIBCMT:_guard_dispatch_.obj
 0001:00019f00       _TI2?AVbad_alloc@std@@     000000018001af00     LIBCMT:throw_bad_alloc.obj
 0001:00019f20       _CTA2?AVbad_alloc@std@@    000000018001af20     LIBCMT:throw_bad_alloc.obj
 0001:00019f38       _CT??_R0?AVbad_alloc@std@@@8??0bad_alloc@std@@QEAA@AEBV01@@Z24 000000018001af38     LIBCMT:throw_bad_alloc.obj
 0001:00019f60       _CT??_R0?AVexception@std@@@8??0exception@std@@QEAA@AEBV01@@Z24 000000018001af60     LIBCMT:throw_bad_alloc.obj
 0001:00019f88       _TI3?AVbad_array_new_length@std@@ 000000018001af88     LIBCMT:throw_bad_alloc.obj
 0001:00019fa8       _CTA3?AVbad_array_new_length@std@@ 000000018001afa8     LIBCMT:throw_bad_alloc.obj
 0001:00019fc8       _CT??_R0?AVbad_array_new_length@std@@@8??0bad_array_new_length@std@@QEAA@AEBV01@@Z24 000000018001afc8     LIBCMT:throw_bad_alloc.obj
 0001:00019ff0       _TI1?AV_com_error@@        000000018001aff0     comsuppw:comraise.obj
 0001:0001a010       _CTA1?AV_com_error@@       000000018001b010     comsuppw:comraise.obj
 0001:0001a020       _CT??_R0?AV_com_error@@@8??0_com_error@@QEAA@AEBV0@@Z32 000000018001b020     comsuppw:comraise.obj
 0002:00000000       ?g_szTopicMain@@3PEB_WEB   000000018001c000     Plugin.obj
 0002:00000008       ?g_szTopicConfig@@3PEB_WEB 000000018001c008     Plugin.obj
 0002:00000010       ?g_szTopicChooseMenuType@@3PEB_WEB 000000018001c010     Plugin.obj
 0002:00000018       ?g_szTopicContextMenu@@3PEB_WEB 000000018001c018     Plugin.obj
 0002:00000020       ?g_szTopicMyComp@@3PEB_WEB 000000018001c020     Plugin.obj
 0002:00000028       ?g_szTopicError0@@3PEB_WEB 000000018001c028     Plugin.obj
 0002:00000030       ?g_szTopicError1@@3PEB_WEB 000000018001c030     Plugin.obj
 0002:00000038       ?g_szTopicError2@@3PEB_WEB 000000018001c038     Plugin.obj
 0002:00000040       ?g_szTopicClose@@3PEB_WEB  000000018001c040     Plugin.obj
 0002:00000048       __scrt_native_dllmain_reason 000000018001c048     LIBCMT:utility.obj
 0002:00000050       __isa_available            000000018001c050     LIBCMT:_cpu_disp_.obj
 0002:00000054       __isa_enabled              000000018001c054     LIBCMT:_cpu_disp_.obj
 0002:00000058       __memcpy_nt_iters          000000018001c058     LIBCMT:_cpu_disp_.obj
 0002:00000060       __security_cookie          000000018001c060     LIBCMT:gs_cookie.obj
 0002:00000068       __security_cookie_complement 000000018001c068     LIBCMT:gs_cookie.obj
 0002:00000070       ?__errorPfn@@3P6AXJPEAUIErrorInfo@@@ZEA 000000018001c070     comsuppw:comsupp.obj
 0002:000000d4       __abort_behavior           000000018001c0d4     libucrt:abort.obj
 0002:000000f0       __acrt_initial_multibyte_data 000000018001c0f0     libucrt:mbctype.obj
 0002:00000318       __acrt_current_multibyte_data 000000018001c318     libucrt:mbctype.obj
 0002:00000420       _mbctype                   000000018001c420     libucrt:mbctype.obj
 0002:00000530       _mbcasemap                 000000018001c530     libucrt:mbctype.obj
 0002:00000630       __acrt_initial_locale_data 000000018001c630     libucrt:nlsdata.obj
 0002:00000788       __acrt_initial_locale_pointers 000000018001c788     libucrt:nlsdata.obj
 0002:00000798       __acrt_wide_c_locale_string 000000018001c798     libucrt:nlsdata.obj
 0002:000007a0       _iob                       000000018001c7a0     libucrt:_file.obj
 0002:000008a8       __globallocalestatus       000000018001c8a8     libucrt:glstatus.obj
 0002:000008b0       __acrt_lconv_c             000000018001c8b0     libucrt:localeconv.obj
 0002:00000948       __acrt_lconv_static_decimal 000000018001c948     libucrt:localeconv.obj
 0002:0000094c       __acrt_lconv_static_W_decimal 000000018001c94c     libucrt:localeconv.obj
 0002:00000950       __dcrt_lowio_console_output_handle 000000018001c950     libucrt:initcon.obj
 0002:00000970       _fltused                   000000018001c970     LIBCMT:fltused.obj
 0002:00000980       ??_R0?AVbad_alloc@std@@@8  000000018001c980     LIBCMT:throw_bad_alloc.obj
 0002:000009a8       ??_R0?AVexception@std@@@8  000000018001c9a8     LIBCMT:throw_bad_alloc.obj
 0002:000009d0       ??_R0?AVbad_array_new_length@std@@@8 000000018001c9d0     LIBCMT:throw_bad_alloc.obj
 0002:00000a00       ??_R0?AVtype_info@@@8      000000018001ca00     LIBCMT:std_type_info_static.obj
 0002:00000a20       ??_R0?AV_com_error@@@8     000000018001ca20     comsuppw:comraise.obj
 0002:00000a50       ?thePlug@@3PEAVCPlugin@@EA 000000018001ca50     EMenu.obj
 0002:00000a58       ?hNeedInvoke@OleThread@@3PEAVCHandle@@EA 000000018001ca58     OleThread.obj
 0002:00000a60       ?hInvokeDone@OleThread@@3PEAVCHandle@@EA 000000018001ca60     OleThread.obj
 0002:00000a68       ?hStop@OleThread@@3PEAVCHandle@@EA 000000018001ca68     OleThread.obj
 0002:00000a70       ?hShowMenu@OleThread@@3PEAVCHandle@@EA 000000018001ca70     OleThread.obj
 0002:00000a78       ?hMenuDone@OleThread@@3PEAVCHandle@@EA 000000018001ca78     OleThread.obj
 0002:00000a80       ?hTerminator@OleThread@@3PEAVCThreadTerminator@1@EA 000000018001ca80     OleThread.obj
 0002:00000a88       ?nOpenFrom@OpenPluginArgs@OleThread@@3HA 000000018001ca88     OleThread.obj
 0002:00000a8c       ?enRes@OpenPluginArgs@OleThread@@3W4EDoMenu@CPlugin@@A 000000018001ca8c     OleThread.obj
 0002:00000a90       ?nItem@OpenPluginArgs@OleThread@@3_JA 000000018001ca90     OleThread.obj
 0002:00000a98       ?Menu@ShowMenuArgs@OleThread@@3PEAVCFarMenu@@EA 000000018001ca98     OleThread.obj
 0002:00000aa0       ?szTitle@ShowMenuArgs@OleThread@@3PEB_WEB 000000018001caa0     OleThread.obj
 0002:00000aa8       ?nSelItem@ShowMenuArgs@OleThread@@3HA 000000018001caa8     OleThread.obj
 0002:00000aac       ?bAtCursorPos@ShowMenuArgs@OleThread@@3_NA 000000018001caac     OleThread.obj
 0002:00000ab0       ?Res@ShowMenuArgs@OleThread@@3HA 000000018001cab0     OleThread.obj
 0002:00000ab8       ?hThread@OleThread@@3PEAXEA 000000018001cab8     OleThread.obj
 0002:000012d8       __scrt_current_native_startup_state 000000018001d2d8     LIBCMT:utility.obj
 0002:000012e0       __scrt_native_startup_lock 000000018001d2e0     LIBCMT:utility.obj
 0002:00001320       ?__type_info_root_node@@3U__type_info_node@@A 000000018001d320     LIBCMT:tncleanup.obj
 0002:00001330       ?_OptionsStorage@?1??__local_stdio_printf_options@@9@4_KA 000000018001d330     LIBCMT:default_local_stdio_options.obj
 0002:00001338       ?_OptionsStorage@?1??__local_stdio_scanf_options@@9@4_KA 000000018001d338     LIBCMT:default_local_stdio_options.obj
 0002:00001340       __scrt_debugger_hook_flag  000000018001d340     LIBCMT:utility_desktop.obj
 0002:00001344       __favor                    000000018001d344     LIBCMT:_cpu_disp_.obj
 0002:00001468       __pPurecall                000000018001d468     libvcruntime:purevirt_data.obj
 0002:00001470       ?pArgList@UnDecorator@@0PEAVReplicator@@EA 000000018001d470     libvcruntime:undname.obj
 0002:00001478       ?pZNameList@UnDecorator@@0PEAVReplicator@@EA 000000018001d478     libvcruntime:undname.obj
 0002:00001480       ?pTemplateArgList@UnDecorator@@0PEAVReplicator@@EA 000000018001d480     libvcruntime:undname.obj
 0002:00001488       ?gName@UnDecorator@@0PEBDEB 000000018001d488     libvcruntime:undname.obj
 0002:00001490       ?name@UnDecorator@@0PEBDEB 000000018001d490     libvcruntime:undname.obj
 0002:00001498       ?outputString@UnDecorator@@0PEADEA 000000018001d498     libvcruntime:undname.obj
 0002:000014a0       ?maxStringLength@UnDecorator@@0HA 000000018001d4a0     libvcruntime:undname.obj
 0002:000014a4       ?disableFlags@UnDecorator@@0KA 000000018001d4a4     libvcruntime:undname.obj
 0002:000014a8       ?fExplicitTemplateParams@UnDecorator@@0_NA 000000018001d4a8     libvcruntime:undname.obj
 0002:000014a9       ?fGetTemplateArgumentList@UnDecorator@@0_NA 000000018001d4a9     libvcruntime:undname.obj
 0002:000014b0       ?m_pGetParameter@UnDecorator@@0P6APEADJ@ZEA 000000018001d4b0     libvcruntime:undname.obj
 0002:00001608       _environ_table             000000018001d608     libucrt:environment_initialization.obj
 0002:00001610       _wenviron_table            000000018001d610     libucrt:environment_initialization.obj
 0002:00001618       __dcrt_initial_wide_environment 000000018001d618     libucrt:environment_initialization.obj
 0002:00001620       __dcrt_initial_narrow_environment 000000018001d620     libucrt:environment_initialization.obj
 0002:00001628       __acrt_atexit_table        000000018001d628     libucrt:onexit.obj
 0002:00001640       __acrt_at_quick_exit_table 000000018001d640     libucrt:onexit.obj
 0002:00001a20       __mbcodepage               000000018001da20     libucrt:mbctype.obj
 0002:00001a24       __ismbcodepage             000000018001da24     libucrt:mbctype.obj
 0002:00001a28       __mbulinfo                 000000018001da28     libucrt:mbctype.obj
 0002:00001a38       __mblocalename             000000018001da38     libucrt:mbctype.obj
 0002:00001a44       __argc                     000000018001da44     libucrt:argv_data.obj
 0002:00001a48       __argv                     000000018001da48     libucrt:argv_data.obj
 0002:00001a50       __wargv                    000000018001da50     libucrt:argv_data.obj
 0002:00001a58       _acmdln                    000000018001da58     libucrt:argv_data.obj
 0002:00001a60       _wcmdln                    000000018001da60     libucrt:argv_data.obj
 0002:00001a68       _pgmptr                    000000018001da68     libucrt:argv_data.obj
 0002:00001a70       __acrt_heap                000000018001da70     libucrt:heap_handle.obj
 0002:00001a80       __pioinfo                  000000018001da80     libucrt:ioinit.obj
 0002:00001e80       _nhandle                   000000018001de80     libucrt:ioinit.obj
 0002:00001eb0       __acrt_current_locale_data 000000018001deb0     libucrt:nlsdata.obj
 0002:00001eb8       __acrt_stdout_buffer       000000018001deb8     libucrt:_sftbuf.obj
 0002:00001ec0       __acrt_stderr_buffer       000000018001dec0     libucrt:_sftbuf.obj
 0002:00001ed0       _nstream                   000000018001ded0     libucrt:_file.obj
 0002:00001ed8       __piob                     000000018001ded8     libucrt:_file.obj
 0002:00001ee0       __acrt_locale_changed_data 000000018001dee0     libucrt:wsetlocale.obj
 0002:00001ee4       __acrt_lconv_static_null   000000018001dee4     libucrt:localeconv.obj
 0002:00001ee8       __acrt_lconv_static_W_null 000000018001dee8     libucrt:localeconv.obj
 0002:00001ef0       __fma3_is_available        000000018001def0     libucrt:fma3_available.obj
 0002:00001ef4       __use_fma3_lib             000000018001def4     libucrt:fma3_available.obj
 0002:00002470       __scrt_ucrt_dll_is_in_use  000000018001e470     <common>
 0002:00002478       __dyn_tls_init_callback    000000018001e478     <common>
 0002:00002480       _pDestructExceptionObject  000000018001e480     <common>
 0004:00000000       __imp_SystemFunction036    0000000180021000     advapi32:ADVAPI32.dll
 0004:00000008       \177ADVAPI32_NULL_THUNK_DATA 0000000180021008     advapi32:ADVAPI32.dll
 0004:00000010       __imp_lstrcpynW            0000000180021010     kernel32:KERNEL32.dll
 0004:00000018       __imp_lstrcpyW             0000000180021018     kernel32:KERNEL32.dll
 0004:00000020       __imp_lstrcatW             0000000180021020     kernel32:KERNEL32.dll
 0004:00000028       __imp_lstrlenA             0000000180021028     kernel32:KERNEL32.dll
 0004:00000030       __imp_lstrlenW             0000000180021030     kernel32:KERNEL32.dll
 0004:00000038       __imp_CompareStringW       0000000180021038     kernel32:KERNEL32.dll
 0004:00000040       __imp_MultiByteToWideChar  0000000180021040     kernel32:KERNEL32.dll
 0004:00000048       __imp_CloseHandle          0000000180021048     kernel32:KERNEL32.dll
 0004:00000050       __imp_SetEvent             0000000180021050     kernel32:KERNEL32.dll
 0004:00000058       __imp_WaitForSingleObject  0000000180021058     kernel32:KERNEL32.dll
 0004:00000060       __imp_CreateThread         0000000180021060     kernel32:KERNEL32.dll
 0004:00000068       __imp_TerminateThread      0000000180021068     kernel32:KERNEL32.dll
 0004:00000070       __imp_GetExitCodeThread    0000000180021070     kernel32:KERNEL32.dll
 0004:00000078       __imp_WaitForMultipleObjects 0000000180021078     kernel32:KERNEL32.dll
 0004:00000080       __imp_VerSetConditionMask  0000000180021080     kernel32:KERNEL32.dll
 0004:00000088       __imp_ExpandEnvironmentStringsW 0000000180021088     kernel32:KERNEL32.dll
 0004:00000090       __imp_GetFileAttributesW   0000000180021090     kernel32:KERNEL32.dll
 0004:00000098       __imp_GetModuleHandleW     0000000180021098     kernel32:KERNEL32.dll
 0004:000000a0       __imp_lstrcmpA             00000001800210a0     kernel32:KERNEL32.dll
 0004:000000a8       __imp_VerifyVersionInfoW   00000001800210a8     kernel32:KERNEL32.dll
 0004:000000b0       __imp_CreateEventW         00000001800210b0     kernel32:KERNEL32.dll
 0004:000000b8       __imp_lstrcmpW             00000001800210b8     kernel32:KERNEL32.dll
 0004:000000c0       __imp_CreateFileW          00000001800210c0     kernel32:KERNEL32.dll
 0004:000000c8       __imp_WriteConsoleW        00000001800210c8     kernel32:KERNEL32.dll
 0004:000000d0       __imp_SetFilePointerEx     00000001800210d0     kernel32:KERNEL32.dll
 0004:000000d8       __imp_GetConsoleMode       00000001800210d8     kernel32:KERNEL32.dll
 0004:000000e0       __imp_GetConsoleCP         00000001800210e0     kernel32:KERNEL32.dll
 0004:000000e8       __imp_FlushFileBuffers     00000001800210e8     kernel32:KERNEL32.dll
 0004:000000f0       __imp_WriteFile            00000001800210f0     kernel32:KERNEL32.dll
 0004:000000f8       __imp_SetStdHandle         00000001800210f8     kernel32:KERNEL32.dll
 0004:00000100       __imp_HeapReAlloc          0000000180021100     kernel32:KERNEL32.dll
 0004:00000108       __imp_HeapSize             0000000180021108     kernel32:KERNEL32.dll
 0004:00000110       __imp_GetStringTypeW       0000000180021110     kernel32:KERNEL32.dll
 0004:00000118       __imp_GetFileType          0000000180021118     kernel32:KERNEL32.dll
 0004:00000120       __imp_GetStdHandle         0000000180021120     kernel32:KERNEL32.dll
 0004:00000128       __imp_GetProcessHeap       0000000180021128     kernel32:KERNEL32.dll
 0004:00000130       __imp_FreeEnvironmentStringsW 0000000180021130     kernel32:KERNEL32.dll
 0004:00000138       __imp_GetEnvironmentStringsW 0000000180021138     kernel32:KERNEL32.dll
 0004:00000140       __imp_GetCommandLineW      0000000180021140     kernel32:KERNEL32.dll
 0004:00000148       __imp_GetCommandLineA      0000000180021148     kernel32:KERNEL32.dll
 0004:00000150       __imp_GetCPInfo            0000000180021150     kernel32:KERNEL32.dll
 0004:00000158       __imp_GetOEMCP             0000000180021158     kernel32:KERNEL32.dll
 0004:00000160       __imp_GetACP               0000000180021160     kernel32:KERNEL32.dll
 0004:00000168       __imp_QueryPerformanceCounter 0000000180021168     kernel32:KERNEL32.dll
 0004:00000170       __imp_GetCurrentProcessId  0000000180021170     kernel32:KERNEL32.dll
 0004:00000178       __imp_GetCurrentThreadId   0000000180021178     kernel32:KERNEL32.dll
 0004:00000180       __imp_GetSystemTimeAsFileTime 0000000180021180     kernel32:KERNEL32.dll
 0004:00000188       __imp_InitializeSListHead  0000000180021188     kernel32:KERNEL32.dll
 0004:00000190       __imp_RtlCaptureContext    0000000180021190     kernel32:KERNEL32.dll
 0004:00000198       __imp_RtlLookupFunctionEntry 0000000180021198     kernel32:KERNEL32.dll
 0004:000001a0       __imp_RtlVirtualUnwind     00000001800211a0     kernel32:KERNEL32.dll
 0004:000001a8       __imp_IsDebuggerPresent    00000001800211a8     kernel32:KERNEL32.dll
 0004:000001b0       __imp_UnhandledExceptionFilter 00000001800211b0     kernel32:KERNEL32.dll
 0004:000001b8       __imp_SetUnhandledExceptionFilter 00000001800211b8     kernel32:KERNEL32.dll
 0004:000001c0       __imp_GetStartupInfoW      00000001800211c0     kernel32:KERNEL32.dll
 0004:000001c8       __imp_IsProcessorFeaturePresent 00000001800211c8     kernel32:KERNEL32.dll
 0004:000001d0       __imp_LocalFree            00000001800211d0     kernel32:KERNEL32.dll
 0004:000001d8       __imp_GetLastError         00000001800211d8     kernel32:KERNEL32.dll
 0004:000001e0       __imp_RtlUnwindEx          00000001800211e0     kernel32:KERNEL32.dll
 0004:000001e8       __imp_GetModuleFileNameW   00000001800211e8     kernel32:KERNEL32.dll
 0004:000001f0       __imp_RtlPcToFileHeader    00000001800211f0     kernel32:KERNEL32.dll
 0004:000001f8       __imp_RaiseException       00000001800211f8     kernel32:KERNEL32.dll
 0004:00000200       __imp_InterlockedFlushSList 0000000180021200     kernel32:KERNEL32.dll
 0004:00000208       __imp_InitializeCriticalSectionAndSpinCount 0000000180021208     kernel32:KERNEL32.dll
 0004:00000210       __imp_TlsAlloc             0000000180021210     kernel32:KERNEL32.dll
 0004:00000218       __imp_TlsGetValue          0000000180021218     kernel32:KERNEL32.dll
 0004:00000220       __imp_TlsSetValue          0000000180021220     kernel32:KERNEL32.dll
 0004:00000228       __imp_TlsFree              0000000180021228     kernel32:KERNEL32.dll
 0004:00000230       __imp_FreeLibrary          0000000180021230     kernel32:KERNEL32.dll
 0004:00000238       __imp_GetProcAddress       0000000180021238     kernel32:KERNEL32.dll
 0004:00000240       __imp_LoadLibraryExW       0000000180021240     kernel32:KERNEL32.dll
 0004:00000248       __imp_SetLastError         0000000180021248     kernel32:KERNEL32.dll
 0004:00000250       __imp_EnterCriticalSection 0000000180021250     kernel32:KERNEL32.dll
 0004:00000258       __imp_LeaveCriticalSection 0000000180021258     kernel32:KERNEL32.dll
 0004:00000260       __imp_DeleteCriticalSection 0000000180021260     kernel32:KERNEL32.dll
 0004:00000268       __imp_GetCurrentProcess    0000000180021268     kernel32:KERNEL32.dll
 0004:00000270       __imp_ExitProcess          0000000180021270     kernel32:KERNEL32.dll
 0004:00000278       __imp_TerminateProcess     0000000180021278     kernel32:KERNEL32.dll
 0004:00000280       __imp_GetModuleHandleExW   0000000180021280     kernel32:KERNEL32.dll
 0004:00000288       __imp_GetModuleFileNameA   0000000180021288     kernel32:KERNEL32.dll
 0004:00000290       __imp_WideCharToMultiByte  0000000180021290     kernel32:KERNEL32.dll
 0004:00000298       __imp_HeapFree             0000000180021298     kernel32:KERNEL32.dll
 0004:000002a0       __imp_HeapAlloc            00000001800212a0     kernel32:KERNEL32.dll
 0004:000002a8       __imp_LCMapStringW         00000001800212a8     kernel32:KERNEL32.dll
 0004:000002b0       __imp_FindClose            00000001800212b0     kernel32:KERNEL32.dll
 0004:000002b8       __imp_FindFirstFileExA     00000001800212b8     kernel32:KERNEL32.dll
 0004:000002c0       __imp_FindNextFileA        00000001800212c0     kernel32:KERNEL32.dll
 0004:000002c8       __imp_IsValidCodePage      00000001800212c8     kernel32:KERNEL32.dll
 0004:000002d0       \177KERNEL32_NULL_THUNK_DATA 00000001800212d0     kernel32:KERNEL32.dll
 0004:000002d8       __imp_SHGetSpecialFolderLocation 00000001800212d8     shell32:SHELL32.dll
 0004:000002e0       __imp_SHGetDesktopFolder   00000001800212e0     shell32:SHELL32.dll
 0004:000002e8       \177SHELL32_NULL_THUNK_DATA 00000001800212e8     shell32:SHELL32.dll
 0004:000002f0       __imp_GetMenuItemCount     00000001800212f0     user32:USER32.dll
 0004:000002f8       __imp_DestroyMenu          00000001800212f8     user32:USER32.dll
 0004:00000300       __imp_CreatePopupMenu      0000000180021300     user32:USER32.dll
 0004:00000308       __imp_GetMenuStringW       0000000180021308     user32:USER32.dll
 0004:00000310       __imp_GetKeyState          0000000180021310     user32:USER32.dll
 0004:00000318       __imp_SetWindowPos         0000000180021318     user32:USER32.dll
 0004:00000320       __imp_DestroyWindow        0000000180021320     user32:USER32.dll
 0004:00000328       __imp_TrackPopupMenu       0000000180021328     user32:USER32.dll
 0004:00000330       __imp_ReplyMessage         0000000180021330     user32:USER32.dll
 0004:00000338       __imp_PeekMessageW         0000000180021338     user32:USER32.dll
 0004:00000340       __imp_DispatchMessageW     0000000180021340     user32:USER32.dll
 0004:00000348       __imp_GetMessageW          0000000180021348     user32:USER32.dll
 0004:00000350       __imp_SetWindowLongPtrW    0000000180021350     user32:USER32.dll
 0004:00000358       __imp_GetWindowLongPtrW    0000000180021358     user32:USER32.dll
 0004:00000360       __imp_ScreenToClient       0000000180021360     user32:USER32.dll
 0004:00000368       __imp_GetCursorPos         0000000180021368     user32:USER32.dll
 0004:00000370       __imp_GetClientRect        0000000180021370     user32:USER32.dll
 0004:00000378       __imp_GetMenuItemInfoW     0000000180021378     user32:USER32.dll
 0004:00000380       __imp_wsprintfW            0000000180021380     user32:USER32.dll
 0004:00000388       __imp_GetWindowRect        0000000180021388     user32:USER32.dll
 0004:00000390       __imp_CreateDialogParamW   0000000180021390     user32:USER32.dll
 0004:00000398       \177USER32_NULL_THUNK_DATA 0000000180021398     user32:USER32.dll
 0004:000003a0       __imp_CoTaskMemFree        00000001800213a0     ole32:ole32.dll
 0004:000003a8       __imp_OleFlushClipboard    00000001800213a8     ole32:ole32.dll
 0004:000003b0       __imp_OleInitialize        00000001800213b0     ole32:ole32.dll
 0004:000003b8       \177ole32_NULL_THUNK_DATA  00000001800213b8     ole32:ole32.dll
 0004:000003c0       __IMPORT_DESCRIPTOR_KERNEL32 00000001800213c0     kernel32:KERNEL32.dll
 0004:000003d4       __IMPORT_DESCRIPTOR_USER32 00000001800213d4     user32:USER32.dll
 0004:000003e8       __IMPORT_DESCRIPTOR_SHELL32 00000001800213e8     shell32:SHELL32.dll
 0004:000003fc       __IMPORT_DESCRIPTOR_ole32  00000001800213fc     ole32:ole32.dll
 0004:00000410       __IMPORT_DESCRIPTOR_ADVAPI32 0000000180021410     advapi32:ADVAPI32.dll
 0004:00000424       __NULL_IMPORT_DESCRIPTOR   0000000180021424     kernel32:KERNEL32.dll

 entry point at        0001:0000eca0

 Static symbols

 0004:fffdf000       .idata$6                   0000000180000000     oleaut32:OLEAUT32.dll
 0001:00000144       ?empty_wstr@@3QB_WB        0000000180001144     FarMenu.obj
 0001:00000690       ?ExceptionTemplate@?1??_CxxThrowException@@9@4UEHExceptionRecord@@B 0000000180001690     libvcruntime:throw.obj
 0001:000006d0       ?module_names@?A0x49c8dc86@@3QBQEB_WB 00000001800016d0     libvcruntime:winapi_downlevel.obj
 0001:0000079c       ?candidate_modules@?1??try_get_EventRegister@@YAP6AKPEBU_GUID@@P6AX0KE_K1PEAU_EVENT_FILTER_DESCRIPTOR@@PEAX@Z3PEA_K@ZXZ@4QBW4module_id@?A0x49c8dc86@@B 000000018000179c     libvcruntime:winapi_downlevel.obj
 0001:000007b0       ?candidate_modules@?1??try_get_EventSetInformation@@YAP6AK_KW4_EVENT_INFO_CLASS@@PEAXK@ZXZ@4QBW4module_id@?A0x49c8dc86@@B 00000001800017b0     libvcruntime:winapi_downlevel.obj
 0001:000007cc       ?candidate_modules@?1??try_get_EventUnregister@@YAP6AK_K@ZXZ@4QBW4module_id@?A0x49c8dc86@@B 00000001800017cc     libvcruntime:winapi_downlevel.obj
 0001:000007e0       ?candidate_modules@?1??try_get_EventWriteTransfer@@YAP6AK_KPEBU_EVENT_DESCRIPTOR@@PEBU_GUID@@2KPEAU_EVENT_DATA_DESCRIPTOR@@@ZXZ@4QBW4module_id@?A0x49c8dc86@@B 00000001800017e0     libvcruntime:winapi_downlevel.obj
 0001:00000800       ?candidate_modules@?1??try_get_FlsAlloc@@YAP6AKP6AXPEAX@Z@ZXZ@4QBW4module_id@?A0x49c8dc86@@B 0000000180001800     libvcruntime:winapi_downlevel.obj
 0001:00000818       ?candidate_modules@?1??try_get_FlsFree@@YAP6AHK@ZXZ@4QBW4module_id@?A0x49c8dc86@@B 0000000180001818     libvcruntime:winapi_downlevel.obj
 0001:00000828       ?candidate_modules@?1??try_get_FlsGetValue@@YAP6APEAXK@ZXZ@4QBW4module_id@?A0x49c8dc86@@B 0000000180001828     libvcruntime:winapi_downlevel.obj
 0001:00000840       ?candidate_modules@?1??try_get_FlsSetValue@@YAP6AHKPEAX@ZXZ@4QBW4module_id@?A0x49c8dc86@@B 0000000180001840     libvcruntime:winapi_downlevel.obj
 0001:00000858       ?candidate_modules@?1??try_get_InitializeCriticalSectionEx@@YAP6AHPEAU_RTL_CRITICAL_SECTION@@KK@ZXZ@4QBW4module_id@?A0x49c8dc86@@B 0000000180001858     libvcruntime:winapi_downlevel.obj
 0001:00000880       ?tokenTable@@3QBQEBDB      0000000180001880     libvcruntime:undname.obj
 0001:000008f0       ?nameTable@@3QBQEBDB       00000001800018f0     libvcruntime:undname.obj
 0001:00000b78       ?rttiTable@@3QBQEBDB       0000000180001b78     libvcruntime:undname.obj
 0001:00001300       __acrt_initializers        0000000180002300     libucrt:initialization.obj
 0001:000013f0       module_names               00000001800023f0     libucrt:winapi_thunks.obj
 0001:00001920       ?candidate_modules@?1??try_get_FlsAlloc@@YAP6AKP6AXPEAX@Z@ZXZ@4QBW4module_id@?A0x63058377@@B 0000000180002920     libucrt:winapi_thunks.obj
 0001:00001928       ?candidate_modules@?1??try_get_FlsFree@@YAP6AHK@ZXZ@4QBW4module_id@?A0x63058377@@B 0000000180002928     libucrt:winapi_thunks.obj
 0001:00001930       ?candidate_modules@?1??try_get_FlsGetValue@@YAP6APEAXK@ZXZ@4QBW4module_id@?A0x63058377@@B 0000000180002930     libucrt:winapi_thunks.obj
 0001:00001938       ?candidate_modules@?1??try_get_FlsSetValue@@YAP6AHKPEAX@ZXZ@4QBW4module_id@?A0x63058377@@B 0000000180002938     libucrt:winapi_thunks.obj
 0001:00001940       ?candidate_modules@?1??try_get_GetCurrentPackageId@@YAP6AJPEAIPEAE@ZXZ@4QBW4module_id@?A0x63058377@@B 0000000180002940     libucrt:winapi_thunks.obj
 0001:00001960       ?candidate_modules@?1??try_get_InitializeCriticalSectionEx@@YAP6AHPEAU_RTL_CRITICAL_SECTION@@KK@ZXZ@4QBW4module_id@?A0x63058377@@B 0000000180002960     libucrt:winapi_thunks.obj
 0001:00001968       ?candidate_modules@?1??try_get_LCMapStringEx@@YAP6AHPEB_WK0HPEA_WHPEAU_nlsversioninfo@@PEAX_J@ZXZ@4QBW4module_id@?A0x63058377@@B 0000000180002968     libucrt:winapi_thunks.obj
 0001:00001980       ?candidate_modules@?1??try_get_LocaleNameToLCID@@YAP6AKPEB_WK@ZXZ@4QBW4module_id@?A0x63058377@@B 0000000180002980     libucrt:winapi_thunks.obj
 0001:000019a0       errtable                   00000001800029a0     libucrt:errno.obj
 0001:00001b08       _mb_locale_names           0000000180002b08     libucrt:mbctype.obj
 0001:000027f0       LcidToLocaleNameTable      00000001800037f0     libucrt:lcidtoname_downlevel.obj
 0001:00004250       LocaleNameToIndexTable     0000000180005250     libucrt:lcidtoname_downlevel.obj
 0001:00005af0       __real_ninf                0000000180006af0     libucrt:log10.obj
 0001:00005b00       __real_inf                 0000000180006b00     libucrt:log10.obj
 0001:00005b10       __real_neg_qnan            0000000180006b10     libucrt:log10.obj
 0001:00005b20       __real_qnanbit             0000000180006b20     libucrt:log10.obj
 0001:00005b30       __int_1023                 0000000180006b30     libucrt:log10.obj
 0001:00005b40       __mask_001                 0000000180006b40     libucrt:log10.obj
 0001:00005b50       __mask_mant                0000000180006b50     libucrt:log10.obj
 0001:00005b60       __mask_mant_top8           0000000180006b60     libucrt:log10.obj
 0001:00005b70       __mask_mant9               0000000180006b70     libucrt:log10.obj
 0001:00005b80       __real_log10_e             0000000180006b80     libucrt:log10.obj
 0001:00005b90       __real_log10_e_lead        0000000180006b90     libucrt:log10.obj
 0001:00005ba0       __real_log10_e_tail        0000000180006ba0     libucrt:log10.obj
 0001:00005bb0       __real_log10_2_lead        0000000180006bb0     libucrt:log10.obj
 0001:00005bc0       __real_log10_2_tail        0000000180006bc0     libucrt:log10.obj
 0001:00005bd0       __real_two                 0000000180006bd0     libucrt:log10.obj
 0001:00005be0       __real_one                 0000000180006be0     libucrt:log10.obj
 0001:00005bf0       __real_half                0000000180006bf0     libucrt:log10.obj
 0001:00005c00       __mask_100                 0000000180006c00     libucrt:log10.obj
 0001:00005c10       __real_1_over_512          0000000180006c10     libucrt:log10.obj
 0001:00005c20       __real_1_over_2            0000000180006c20     libucrt:log10.obj
 0001:00005c30       __real_1_over_3            0000000180006c30     libucrt:log10.obj
 0001:00005c40       __real_1_over_4            0000000180006c40     libucrt:log10.obj
 0001:00005c50       __real_1_over_5            0000000180006c50     libucrt:log10.obj
 0001:00005c60       __real_1_over_6            0000000180006c60     libucrt:log10.obj
 0001:00005c70       __real_neg_1023            0000000180006c70     libucrt:log10.obj
 0001:00005c80       __mask_2045                0000000180006c80     libucrt:log10.obj
 0001:00005c90       __real_threshold           0000000180006c90     libucrt:log10.obj
 0001:00005ca0       __real_near_one_lt         0000000180006ca0     libucrt:log10.obj
 0001:00005cb0       __real_near_one_gt         0000000180006cb0     libucrt:log10.obj
 0001:00005cc0       __real_min_norm            0000000180006cc0     libucrt:log10.obj
 0001:00005cd0       __real_notsign             0000000180006cd0     libucrt:log10.obj
 0001:00005ce0       __real_ca1                 0000000180006ce0     libucrt:log10.obj
 0001:00005cf0       __real_ca2                 0000000180006cf0     libucrt:log10.obj
 0001:00005d00       __real_ca3                 0000000180006d00     libucrt:log10.obj
 0001:00005d10       __real_ca4                 0000000180006d10     libucrt:log10.obj
 0001:00005d20       __mask_lower               0000000180006d20     libucrt:log10.obj
 0001:00005d30       __flag_x_zero              0000000180006d30     libucrt:log10.obj
 0001:00005d34       __flag_x_neg               0000000180006d34     libucrt:log10.obj
 0001:00005d38       __flag_x_nan               0000000180006d38     libucrt:log10.obj
 0001:00007590       __real@433fffffffffffff    0000000180008590     libucrt:fpsr.obj
 0001:00007598       __real@c33fffffffffffff    0000000180008598     libucrt:fpsr.obj
 0001:000075a0       GS_ExceptionPointers       00000001800085a0     LIBCMT:gs_report.obj
 0001:00007870       ?_TlgEvent@?3??__telemetry_main_invoke_trigger@@9@4U<unnamed-type-_TlgEvent>@?3??1@YAXQEAUHINSTANCE__@@@Z@B 0000000180008870     libvcruntime:telemetry.obj
 0001:000078ac       ?_TlgEvent@?3??__telemetry_main_return_trigger@@9@4U<unnamed-type-_TlgEvent>@?3??1@YAXQEAUHINSTANCE__@@@Z@B 00000001800088ac     libvcruntime:telemetry.obj
 0001:000078e7       ?_Tlg_Microsoft_CRTProviderProv_Meta@@3U<unnamed-type-_Tlg_Microsoft_CRTProviderProv_Meta>@@B 00000001800088e7     libvcruntime:telemetry.obj
 0001:00007e60       $$000000                   0000000180008e60     chkstk.obj
 0001:00008d8c       $LN32                      0000000180009d8c     FarMenu.obj
 0001:00008da0       $LN31                      0000000180009da0     FarMenu.obj
 0001:0000b208       $LN331                     000000018000c208     Plugin.obj
 0001:0000b238       $LN330                     000000018000c238     Plugin.obj
 0001:0000b268       $LN329                     000000018000c268     Plugin.obj
 0001:0000b298       $LN328                     000000018000c298     Plugin.obj
 0001:0000b2c8       $LN327                     000000018000c2c8     Plugin.obj
 0001:0000b2f8       $LN326                     000000018000c2f8     Plugin.obj
 0001:0000b328       $LN325                     000000018000c328     Plugin.obj
 0001:0000b358       $LN324                     000000018000c358     Plugin.obj
 0001:0000c9d4       $LN10                      000000018000d9d4     Plugin.obj
 0001:0000cb08       $LN22                      000000018000db08     Plugin.obj
 0001:0000e930       ?dllmain_crt_dispatch@@YAHQEAUHINSTANCE__@@KQEAX@Z 000000018000f930 f   LIBCMT:dll_dllmain.obj
 0001:0000e980       ?dllmain_crt_process_attach@@YAHQEAUHINSTANCE__@@QEAX@Z 000000018000f980 f   LIBCMT:dll_dllmain.obj
 0001:0000eaac       ?dllmain_crt_process_detach@@YAH_N@Z 000000018000faac f   LIBCMT:dll_dllmain.obj
 0001:0000eb30       ?dllmain_dispatch@@YAHQEAUHINSTANCE__@@KQEAX@Z 000000018000fb30 f   LIBCMT:dll_dllmain.obj
 0001:0000ec4c       ?dllmain_raw@@YAHQEAUHINSTANCE__@@KQEAX@Z 000000018000fc4c f   LIBCMT:dll_dllmain.obj
 0001:0000f950       $$000000                   0000000180010950     libvcruntime:memcpy.obj
 0001:0000f9f7       MoveSmall                  00000001800109f7     libvcruntime:memcpy.obj
 0001:0000ffa0       $$000000                   0000000180010fa0     libvcruntime:memset.obj
 0001:0001008c       MsetTab                    000000018001108c     libvcruntime:memset.obj
 0001:00010150       _TlgDefineProvider_annotation__Tlg_Microsoft_CRTProviderProv 0000000180011150 f   libvcruntime:telemetry.obj
 0001:00010610       $$000000                   0000000180011610     libvcruntime:_jmpuwind_.obj
 0001:00010684       ?try_get_function@@YAPEAXW4function_id@?A0x49c8dc86@@QEBDQEBW4module_id@2@2@Z 0000000180011684 f   libvcruntime:winapi_downlevel.obj
 0001:000111b8       ?atexit_exception_filter@@YAHK@Z 00000001800121b8 f   libucrt:exit.obj
 0001:000111c4       ?common_exit@@YAXHW4_crt_exit_cleanup_mode@@W4_crt_exit_return_mode@@@Z 00000001800121c4 f   libucrt:exit.obj
 0001:00011330       ?exit_or_terminate_process@@YAXI@Z 0000000180012330 f   libucrt:exit.obj
 0001:0001137c       ?try_cor_exit_process@@YAXI@Z 000000018001237c f   libucrt:exit.obj
 0001:00011414       ??$parse_command_line@D@@YAXPEADPEAPEAD0PEA_K2@Z 0000000180012414 f   libucrt:argv_parsing.obj
 0001:000117ac       ??$common_initialize_environment_nolock@D@@YAHXZ 00000001800127ac f   libucrt:environment_initialization.obj
 0001:00011818       ??$create_environment@D@@YAQEAPEADQEAD@Z 0000000180012818 f   libucrt:environment_initialization.obj
 0001:00011914       ??$free_environment@D@@YAXQEAPEAD@Z 0000000180012914 f   libucrt:environment_initialization.obj
 0001:00011914       ??$free_environment@_W@@YAXQEAPEA_W@Z 0000000180012914 f   libucrt:environment_initialization.obj
 0001:00011958       ??$uninitialize_environment_internal@D@@YAXAEAPEAPEAD@Z 0000000180012958 f   libucrt:environment_initialization.obj
 0001:00011974       ??$uninitialize_environment_internal@_W@@YAXAEAPEAPEA_W@Z 0000000180012974 f   libucrt:environment_initialization.obj
 0001:00011bac       ??R<lambda_4e60a939b0d047cfe11ddc22648dfba9>@@QEBAHXZ 0000000180012bac f   libucrt:onexit.obj
 0001:00011e5c       initialize_global_variables 0000000180012e5c f   libucrt:initialization.obj
 0001:00011e70       initialize_c               0000000180012e70 f   libucrt:initialization.obj
 0001:00011e94       uninitialize_environment   0000000180012e94 f   libucrt:initialization.obj
 0001:00011ea4       initialize_global_state_isolation 0000000180012ea4 f   libucrt:initialization.obj
 0001:00011ea4       uninitialize_c             0000000180012ea4 f   libucrt:initialization.obj
 0001:00011ea4       initialize_environment     0000000180012ea4 f   libucrt:initialization.obj
 0001:00011ea4       report_memory_leaks        0000000180012ea4 f   libucrt:initialization.obj
 0001:00011ea4       uninitialize_global_state_isolation 0000000180012ea4 f   libucrt:initialization.obj
 0001:00011ea8       initialize_pointers        0000000180012ea8 f   libucrt:initialization.obj
 0001:00011efc       uninitialize_vcruntime     0000000180012efc f   libucrt:initialization.obj
 0001:00011f04       uninitialize_allocated_memory 0000000180012f04 f   libucrt:initialization.obj
 0001:00012458       ?construct_ptd_array@@YAXQEAU__acrt_ptd@@@Z 0000000180013458 f   libucrt:per_thread_data.obj
 0001:00012528       ?destroy_fls@@YAXPEAX@Z    0000000180013528 f   libucrt:per_thread_data.obj
 0001:00012548       ?destroy_ptd_array@@YAXQEAU__acrt_ptd@@@Z 0000000180013548 f   libucrt:per_thread_data.obj
 0001:00012640       ?replace_current_thread_locale_nolock@@YAXQEAU__acrt_ptd@@QEAU__crt_locale_data@@@Z 0000000180013640 f   libucrt:per_thread_data.obj
 0001:00012880       ?try_get_function@@YAPEAXW4function_id@?A0x63058377@@QEBDQEBW4module_id@2@2@Z 0000000180013880 f   libucrt:winapi_thunks.obj
 0001:000131b0       ?<helper_func_cdecl>@<lambda_2feae5270eb4d0d5532525f423405775>@@CAHPEBX0@Z 00000001800141b0 f   libucrt:argv_wildcards.obj
 0001:000131c4       ??$common_expand_argv_wildcards@D@@YAHQEAPEADQEAPEAPEAD@Z 00000001800141c4 f   libucrt:argv_wildcards.obj
 0001:000133d0       ??$copy_and_add_argument_to_buffer@D@@YAHQEBD0_KAEAV?$argument_list@D@?A0xca0879c4@@@Z 00000001800143d0 f   libucrt:argv_wildcards.obj
 0001:000134e0       ??$expand_argument_wildcards@D@@YAHQEAD0AEAV?$argument_list@D@?A0xca0879c4@@@Z 00000001800144e0 f   libucrt:argv_wildcards.obj
 0001:00013794       ??R<lambda_ad1ced32f4ac17aa236e5ef05d6b3b7c>@@QEBAXXZ 0000000180014794 f   libucrt:mbctype.obj
 0001:000139ac       ?getSystemCP@@YAHH@Z       00000001800149ac f   libucrt:mbctype.obj
 0001:00013a2c       ?setSBCS@@YAXPEAU__crt_multibyte_data@@@Z 0000000180014a2c f   libucrt:mbctype.obj
 0001:00013abc       ?setSBUpLow@@YAXPEAU__crt_multibyte_data@@@Z 0000000180014abc f   libucrt:mbctype.obj
 0001:00013ca0       ?setmbcp_internal@@YAHH_N@Z 0000000180014ca0 f   libucrt:mbctype.obj
 0001:000141e8       ?x_ismbbtype_l@@YAHPEAU__crt_locale_pointers@@IHH@Z 00000001800151e8 f   libucrt:ismbbyte.obj
 0001:00014468       ?initialize_inherited_file_handles_nolock@@YAXXZ 0000000180015468 f   libucrt:ioinit.obj
 0001:00014554       ?initialize_stdio_handles_nolock@@YAXXZ 0000000180015554 f   libucrt:ioinit.obj
 0001:00015360       ?GetTableIndexFromLocaleName@@YAHPEB_W@Z 0000000180016360 f   libucrt:lcidtoname_downlevel.obj
 0001:00015460       ?shortsort@@YAXPEAD0_KP6AHPEBX2@Z@Z 0000000180016460 f   libucrt:qsort.obj
 0001:00015a78       ?initialize_multibyte@@YAHXZ 0000000180016a78 f   libucrt:multibyte_initializer.obj
 0001:00015c44       ?__acrt_LCMapStringA_stat@@YAHPEAU__crt_locale_pointers@@PEB_WKPEBDHPEADHHH@Z 0000000180016c44 f   libucrt:lcmapstringa.obj
 0001:00016544       common_flush_all           0000000180017544 f   libucrt:fflush.obj
 0001:000168d4       ?free_crt_array_internal@@YAXQEAPEBX_K@Z 00000001800178d4 f   libucrt:inittime.obj
 0001:00016b74       ?write_double_translated_ansi_nolock@@YA?AUwrite_result@?A0x9c548279@@HQEBDI@Z 0000000180017b74 f   libucrt:write.obj
 0001:00016d7c       ?write_text_ansi_nolock@@YA?AUwrite_result@?A0x9c548279@@HQEBDI@Z 0000000180017d7c f   libucrt:write.obj
 0001:00016e84       ?write_text_utf16le_nolock@@YA?AUwrite_result@?A0x9c548279@@HQEBDI@Z 0000000180017e84 f   libucrt:write.obj
 0001:00016fa0       ?write_text_utf8_nolock@@YA?AUwrite_result@?A0x9c548279@@HQEBDI@Z 0000000180017fa0 f   libucrt:write.obj
 0001:000174f0       $$000000                   00000001800184f0     libucrt:log10.obj
 0001:00017a9c       ??$common_lseek_nolock@_J@@YA_JH_JH@Z 0000000180018a9c f   libucrt:lseek.obj
 0001:00017c8c       _call_matherr              0000000180018c8c f   libucrt:libm_error.obj
 0001:00017cf4       _exception_enabled         0000000180018cf4 f   libucrt:libm_error.obj
 0001:00017f70       _log_special_common        0000000180018f70 f   libucrt:log_special.obj
 0001:00018280       $$000000                   0000000180019280     libucrt:fpsr.obj
 0001:00018720       $$000000                   0000000180019720     LIBCMT:_amdsecgs_.obj
 0001:00018a64       capture_current_context    0000000180019a64 f   LIBCMT:gs_report.obj
 0001:00018ad4       capture_previous_context   0000000180019ad4 f   LIBCMT:gs_report.obj
 0001:00018b50       $$000000                   0000000180019b50     libvcruntime:memcmp.obj
 0001:00018c30       $$000000                   0000000180019c30     LIBCMT:_guard_dispatch_.obj
 0001:00018c50       ?fin$0@?0??dllmain_crt_process_attach@@YAHQEAUHINSTANCE__@@QEAX@Z@4HA 0000000180019c50 f   LIBCMT:dll_dllmain.obj
 0001:00018c67       ?fin$0@?0??dllmain_crt_process_detach@@YAH_N@Z@4HA 0000000180019c67 f   LIBCMT:dll_dllmain.obj
 0001:00018c83       ?filt$0@?0??dllmain_dispatch@@YAHQEAUHINSTANCE__@@KQEAX@Z@4HA 0000000180019c83 f   LIBCMT:dll_dllmain.obj
 0001:00018cb9       __scrt_is_nonwritable_in_current_image$filt$0 0000000180019cb9 f   LIBCMT:utility.obj
 0001:00018cd1       _query_new_handler$fin$0   0000000180019cd1 f   libucrt:new_handler.obj
 0001:00018ce7       ?filt$0@?0??common_exit@@YAXHW4_crt_exit_cleanup_mode@@W4_crt_exit_return_mode@@@Z@4HA 0000000180019ce7 f   libucrt:exit.obj
 0001:00018d02       ?fin$1@?0??common_exit@@YAXHW4_crt_exit_cleanup_mode@@W4_crt_exit_return_mode@@@Z@4HA 0000000180019d02 f   libucrt:exit.obj
 0001:00018d1b       ?fin$0@?0???$?RV<lambda_e24bbb7b643b32fcea6fa61b31d4c984>@@AEAV<lambda_275893d493268fdec8709772e3fcec0e>@@V<lambda_9d71df4d7cf3f480f8d633942495c3b0>@@@?$__crt_seh_guarded_call@H@@QEAAH$$QEAV<lambda_e24bbb7b643b32fcea6fa61b31d4c984>@@AEAV<lambda_275893d493268fdec8709772e3fcec0e>@@$$QEAV<lambda_9d71df4d7cf3f480f8d633942495c3b0>@@@Z@4HA 0000000180019d1b f   libucrt:onexit.obj
 0001:00018d38       ?fin$0@?0???$?RV<lambda_46352004c1216016012b18bd6f87e700>@@AEAV<lambda_3bd07e1a1191394380780325891bf33f>@@V<lambda_334532d3f185bcaa59b5be82d7d22bff>@@@?$__crt_seh_guarded_call@X@@QEAAX$$QEAV<lambda_46352004c1216016012b18bd6f87e700>@@AEAV<lambda_3bd07e1a1191394380780325891bf33f>@@$$QEAV<lambda_334532d3f185bcaa59b5be82d7d22bff>@@@Z@4HA 0000000180019d38 f   libucrt:per_thread_data.obj
 0001:00018d38       ?fin$0@?0???$?RV<lambda_fb3a7dec4e47f37f22dae91bb15c9095>@@AEAV<lambda_698284760c8add0bfb0756c19673e34b>@@V<lambda_dfb8eca1e75fef3034a8fb18dd509707>@@@?$__crt_seh_guarded_call@X@@QEAAX$$QEAV<lambda_fb3a7dec4e47f37f22dae91bb15c9095>@@AEAV<lambda_698284760c8add0bfb0756c19673e34b>@@$$QEAV<lambda_dfb8eca1e75fef3034a8fb18dd509707>@@@Z@4HA 0000000180019d38 f   libucrt:per_thread_data.obj
 0001:00018d38       ?fin$0@?0???$?RV<lambda_b8c45f8f788dd370798f47cfe8ac3a86>@@AEAV<lambda_4e60a939b0d047cfe11ddc22648dfba9>@@V<lambda_332c3edc96d0294ec56c57d38c1cdfd5>@@@?$__crt_seh_guarded_call@H@@QEAAH$$QEAV<lambda_b8c45f8f788dd370798f47cfe8ac3a86>@@AEAV<lambda_4e60a939b0d047cfe11ddc22648dfba9>@@$$QEAV<lambda_332c3edc96d0294ec56c57d38c1cdfd5>@@@Z@4HA 0000000180019d38 f   libucrt:onexit.obj
 0001:00018d38       ?fin$0@?0???$?RV<lambda_c36588078e9f5dfd39652860aa6b3aaf>@@AEAV<lambda_ec61778202f4f5fc7e7711acc23c3bca>@@V<lambda_dc9d2797ccde5d239b4a0efae8ebd7db>@@@?$__crt_seh_guarded_call@P6AXH@Z@@QEAAP6AXH@Z$$QEAV<lambda_c36588078e9f5dfd39652860aa6b3aaf>@@AEAV<lambda_ec61778202f4f5fc7e7711acc23c3bca>@@$$QEAV<lambda_dc9d2797ccde5d239b4a0efae8ebd7db>@@@Z@4HA 0000000180019d38 f   libucrt:signal.obj
 0001:00018d38       ?fin$0@?0???$?RV<lambda_72d1df2b273a38828b1ce30cbf4cdab5>@@AEAV<lambda_876a65b173b8412d3a47c70a915b0cf4>@@V<lambda_41932305e351933ebe8f8be3ed8bb5dc>@@@?$__crt_seh_guarded_call@X@@QEAAX$$QEAV<lambda_72d1df2b273a38828b1ce30cbf4cdab5>@@AEAV<lambda_876a65b173b8412d3a47c70a915b0cf4>@@$$QEAV<lambda_41932305e351933ebe8f8be3ed8bb5dc>@@@Z@4HA 0000000180019d38 f   libucrt:per_thread_data.obj
 0001:00018d38       ?fin$0@?0???$?RV<lambda_99476a1ad63dd22509b5d3e65b0ffc95>@@AEAV<lambda_ad1ced32f4ac17aa236e5ef05d6b3b7c>@@V<lambda_f7424dd8d45958661754dc4f2697e9c3>@@@?$__crt_seh_guarded_call@X@@QEAAX$$QEAV<lambda_99476a1ad63dd22509b5d3e65b0ffc95>@@AEAV<lambda_ad1ced32f4ac17aa236e5ef05d6b3b7c>@@$$QEAV<lambda_f7424dd8d45958661754dc4f2697e9c3>@@@Z@4HA 0000000180019d38 f   libucrt:mbctype.obj
 0001:00018d38       ?fin$0@?0???$?RV<lambda_5e887d1dcbef67a5eb4283622ba103bf>@@AEAV<lambda_4466841279450cc726390878d4a41900>@@V<lambda_341c25c0346d94847f1f3c463c57e077>@@@?$__crt_seh_guarded_call@X@@QEAAX$$QEAV<lambda_5e887d1dcbef67a5eb4283622ba103bf>@@AEAV<lambda_4466841279450cc726390878d4a41900>@@$$QEAV<lambda_341c25c0346d94847f1f3c463c57e077>@@@Z@4HA 0000000180019d38 f   libucrt:per_thread_data.obj
 0001:00018d52       __acrt_update_thread_multibyte_data$fin$0 0000000180019d52 f   libucrt:mbctype.obj
 0001:00018d6b       raise$fin$0                0000000180019d6b f   libucrt:signal.obj
 0001:00018d8f       __acrt_update_thread_locale_data$fin$0 0000000180019d8f f   libucrt:locale_refcounting.obj
 0001:00018d8f       __acrt_uninitialize_locale$fin$0 0000000180019d8f f   libucrt:wsetlocale.obj
 0001:00018da8       __acrt_lowio_ensure_fh_exists$fin$0 0000000180019da8 f   libucrt:osfinfo.obj
 0001:00018da8       __acrt_initialize_lowio$fin$0 0000000180019da8 f   libucrt:ioinit.obj
 0001:00018dc1       common_flush_all$fin$0     0000000180019dc1 f   libucrt:fflush.obj
 0001:00018ddb       common_flush_all$fin$1     0000000180019ddb f   libucrt:fflush.obj
 0001:00018df4       _fcloseall$fin$0           0000000180019df4 f   libucrt:closeall.obj
 0001:00018e0d       _write$fin$0               0000000180019e0d f   libucrt:write.obj
 0001:00018e24       fclose$fin$0               0000000180019e24 f   libucrt:fclose.obj
 0001:00018e3c       ?fin$0@?0???$?RV<lambda_bfedae4ebbf01fab1bb6dcc6a9e276e0>@@AEAV<lambda_2fe9b910cf3cbf4a0ab98a02ba45b3ec>@@V<lambda_237c231691f317818eb88cc1d5d642d6>@@@?$__crt_seh_guarded_call@H@@QEAAH$$QEAV<lambda_bfedae4ebbf01fab1bb6dcc6a9e276e0>@@AEAV<lambda_2fe9b910cf3cbf4a0ab98a02ba45b3ec>@@$$QEAV<lambda_237c231691f317818eb88cc1d5d642d6>@@@Z@4HA 0000000180019e3c f   libucrt:close.obj
 0001:00018e3c       ?fin$0@?0???$?RV<lambda_b521505b218e5242e90febf6bfebc422>@@AEAV<lambda_6978c1fb23f02e42e1d9e99668cc68aa>@@V<lambda_314360699dd331753a4119843814e9a7>@@@?$__crt_seh_guarded_call@H@@QEAAH$$QEAV<lambda_b521505b218e5242e90febf6bfebc422>@@AEAV<lambda_6978c1fb23f02e42e1d9e99668cc68aa>@@$$QEAV<lambda_314360699dd331753a4119843814e9a7>@@@Z@4HA 0000000180019e3c f   libucrt:commit.obj
 0001:00018e56       _ctrlfp$filt$0             0000000180019e56 f   libucrt:fpctrl.obj
 0001:00018e90       _IsNonwritableInCurrentImage$filt$0 0000000180019e90 f   LIBCMT:pesect.obj
 0001:00018eb0       $xdatasym                  0000000180019eb0     chkstk.obj
 0001:00018eb8       $unwind$__acrt_uninitialize_ptd 0000000180019eb8     libucrt:per_thread_data.obj
 0001:00018eb8       $unwind$?ItemWidth@?$DialogBuilderBase@UFarDialogItem@@@@IEAA_JAEBUFarDialogItem@@@Z 0000000180019eb8     Plugin.obj
 0001:00018eb8       $unwind$__scrt_dllmain_crt_thread_detach 0000000180019eb8     LIBCMT:utility.obj
 0001:00018eb8       $unwind$__vcrt_initialize  0000000180019eb8     libvcruntime:initialization.obj
 0001:00018eb8       $unwind$__vcrt_uninitialize_critical 0000000180019eb8     libvcruntime:initialization.obj
 0001:00018eb8       $unwind$__doserrno         0000000180019eb8     libucrt:errno.obj
 0001:00018eb8       $unwind$__scrt_initialize_default_local_stdio_options 0000000180019eb8     LIBCMT:default_local_stdio_options.obj
 0001:00018eb8       $unwind$_set_errno_from_matherr 0000000180019eb8     libucrt:fpexcept.obj
 0001:00018eb8       $unwind$__scrt_acquire_startup_lock 0000000180019eb8     LIBCMT:utility.obj
 0001:00018eb8       $unwind$__acrt_thread_detach 0000000180019eb8     libucrt:initialization.obj
 0001:00018eb8       $unwind$__vcrt_thread_attach 0000000180019eb8     libvcruntime:initialization.obj
 0001:00018eb8       $unwind$__vcrt_uninitialize_telemetry_provider 0000000180019eb8     libvcruntime:telemetry.obj
 0001:00018eb8       $unwind$__acrt_initialize_ptd 0000000180019eb8     libucrt:per_thread_data.obj
 0001:00018eb8       $unwind$__acrt_DownlevelLocaleNameToLCID 0000000180019eb8     libucrt:lcidtoname_downlevel.obj
 0001:00018eb8       $unwind$__pctype_func      0000000180019eb8     libucrt:ctype.obj
 0001:00018eb8       $unwind$?dllmain_crt_dispatch@@YAHQEAUHINSTANCE__@@KQEAX@Z 0000000180019eb8     LIBCMT:dll_dllmain.obj
 0001:00018eb8       $unwind$?initialize_multibyte@@YAHXZ 0000000180019eb8     libucrt:multibyte_initializer.obj
 0001:00018eb8       $unwind$ConfigureW         0000000180019eb8     EMenu.obj
 0001:00018eb8       $unwind$__vcrt_thread_detach 0000000180019eb8     libvcruntime:initialization.obj
 0001:00018eb8       $unwind$_invoke_watson     0000000180019eb8     libucrt:invalid_parameter.obj
 0001:00018eb8       $unwind$__acrt_release_locale_ref 0000000180019eb8     libucrt:locale_refcounting.obj
 0001:00018eb8       $unwind$__scrt_dllmain_uninitialize_critical 0000000180019eb8     LIBCMT:utility.obj
 0001:00018eb8       $unwind$_errno             0000000180019eb8     libucrt:errno.obj
 0001:00018eb8       $unwind$_get_osfhandle     0000000180019eb8     libucrt:osfinfo.obj
 0001:00018eb8       $unwind$__scrt_dllmain_crt_thread_attach 0000000180019eb8     LIBCMT:utility.obj
 0001:00018eb8       $unwind$__acrt_initialize_multibyte 0000000180019eb8     libucrt:mbctype.obj
 0001:00018eb8       $unwind$__scrt_dllmain_before_initialize_c 0000000180019eb8     LIBCMT:utility.obj
 0001:00018eb8       $unwind$??1_com_error@@UEAA@XZ 0000000180019eb8     comsuppw:comraise.obj
 0001:00018eb8       $unwind$_msize             0000000180019eb8     libucrt:msize.obj
 0001:00018eb8       $unwind$??9auto_sz@@QEAA_NPEB_W@Z 0000000180019eb8     auto_sz.obj
 0001:00018eb8       $unwind$atexit             0000000180019eb8     LIBCMT:utility.obj
 0001:00018eb8       $unwind$uninitialize_environment 0000000180019eb8     libucrt:initialization.obj
 0001:00018eb8       $unwind$__vcrt_initialize_ptd 0000000180019eb8     libvcruntime:per_thread_data.obj
 0001:00018eb8       $unwind$?Len@auto_sz@@QEBA_KXZ 0000000180019eb8     auto_sz.obj
 0001:00018eb8       $unwind$__vcrt_uninitialize_ptd 0000000180019eb8     libvcruntime:per_thread_data.obj
 0001:00018eb8       $unwind$_statfp            0000000180019eb8     libucrt:fpctrl.obj
 0001:00018eb8       $unwind$__acrt_initialize_command_line 0000000180019eb8     libucrt:argv_data.obj
 0001:00018eb8       $unwind$__acrt_thread_attach 0000000180019eb8     libucrt:initialization.obj
 0001:00018eb8       $unwind$__scrt_dllmain_after_initialize_c 0000000180019eb8     LIBCMT:utility.obj
 0001:00018eb8       $unwind$initialize_c       0000000180019eb8     libucrt:initialization.obj
 0001:00018eb8       $unwind$abort              0000000180019eb8     libucrt:abort.obj
 0001:00018eb8       $unwind$_fileno            0000000180019eb8     libucrt:fileno.obj
 0001:00018eb8       $unwind$GetGlobalInfoW     0000000180019eb8     EMenu.obj
 0001:00018eb8       $unwind$?ShowMenu@OleThread@@YAHAEAVCFarMenu@@PEB_WH_N@Z 0000000180019eb8     OleThread.obj
 0001:00018eb8       $unwind$_isatty            0000000180019eb8     libucrt:isatty.obj
 0001:00018eb8       $unwind$__scrt_dllmain_uninitialize_c 0000000180019eb8     LIBCMT:utility.obj
 0001:00018eb8       $unwind$__dcrt_terminate_console_output 0000000180019eb8     libucrt:initcon.obj
 0001:00018eb8       $unwind$__report_rangecheckfailure 0000000180019eb8     LIBCMT:gs_report.obj
 0001:00018eb8       $unwind$__acrt_initialize_heap 0000000180019eb8     libucrt:heap_handle.obj
 0001:00018eb8       $unwind$__acrt_uninitialize_critical 0000000180019eb8     libucrt:initialization.obj
 0001:00018eb8       $unwind$??$uninitialize_environment_internal@_W@@YAXAEAPEAPEA_W@Z 0000000180019eb8     libucrt:environment_initialization.obj
 0001:00018eb8       $unwind$__GSHandlerCheck   0000000180019eb8     LIBCMT:_gshandler_.obj
 0001:00018eb8       $unwind$??$uninitialize_environment_internal@D@@YAXAEAPEAPEAD@Z 0000000180019eb8     libucrt:environment_initialization.obj
 0001:00018eb8       $unwind$__dcrt_uninitialize_environments_nolock 0000000180019eb8     libucrt:environment_initialization.obj
 0001:00018eb8       $unwind$__vcrt_freefls     0000000180019eb8     libvcruntime:per_thread_data.obj
 0001:00018ec0       $unwind$??0auto_sz@@QEAA@AEBU_STRRET@@PEFBU_ITEMIDLIST@@@Z 0000000180019ec0     auto_sz.obj
 0001:00018ec8       $chain$1$??0auto_sz@@QEAA@AEBU_STRRET@@PEFBU_ITEMIDLIST@@@Z 0000000180019ec8     auto_sz.obj
 0001:00018ee0       $chain$2$??0auto_sz@@QEAA@AEBU_STRRET@@PEFBU_ITEMIDLIST@@@Z 0000000180019ee0     auto_sz.obj
 0001:00018ef0       $unwind$?Realloc@auto_sz@@QEAAX_K@Z 0000000180019ef0     auto_sz.obj
 0001:00018f00       $chain$0$??1CFarMenu@@QEAA@XZ 0000000180019f00     FarMenu.obj
 0001:00018f14       $chain$1$??1CFarMenu@@QEAA@XZ 0000000180019f14     FarMenu.obj
 0001:00018f24       $unwind$?InsertItem@CFarMenu@@QEAAIIPEB_W_NW4ECheck@1@1@Z 0000000180019f24     FarMenu.obj
 0001:00018f34       $chain$1$?InsertItem@CFarMenu@@QEAAIIPEB_W_NW4ECheck@1@1@Z 0000000180019f34     FarMenu.obj
 0001:00018f4c       $chain$2$?InsertItem@CFarMenu@@QEAAIIPEB_W_NW4ECheck@1@1@Z 0000000180019f4c     FarMenu.obj
 0001:00018f60       $chain$3$?InsertItem@CFarMenu@@QEAAIIPEB_W_NW4ECheck@1@1@Z 0000000180019f60     FarMenu.obj
 0001:00018f70       $unwind$?AddSeparator@CFarMenu@@QEAAXXZ 0000000180019f70     FarMenu.obj
 0001:00018f7c       $chain$1$?AddSeparator@CFarMenu@@QEAAXXZ 0000000180019f7c     FarMenu.obj
 0001:00018f94       $chain$2$?AddSeparator@CFarMenu@@QEAAXXZ 0000000180019f94     FarMenu.obj
 0001:00018fa4       $unwind$?Show@CFarMenu@@QEAAHPEB_WH_N@Z 0000000180019fa4     FarMenu.obj
 0001:00018fc0       $unwind$?GetCursorXY@CFarMenu@@QEAAXPEAH0@Z 0000000180019fc0     FarMenu.obj
 0001:00018fcc       $chain$0$?GetCursorXY@CFarMenu@@QEAAXPEAH0@Z 0000000180019fcc     FarMenu.obj
 0001:00018fe0       $chain$1$?GetCursorXY@CFarMenu@@QEAAXPEAH0@Z 0000000180019fe0     FarMenu.obj
 0001:00018ff0       $unwind$?AddArrows@CFarMenu@@IEAAXXZ 0000000180019ff0     FarMenu.obj
 0001:00018ff8       $chain$3$?AddArrows@CFarMenu@@IEAAXXZ 0000000180019ff8     FarMenu.obj
 0001:00019018       $chain$6$?AddArrows@CFarMenu@@IEAAXXZ 000000018001a018     FarMenu.obj
 0001:00019034       $chain$7$?AddArrows@CFarMenu@@IEAAXXZ 000000018001a034     FarMenu.obj
 0001:00019044       $chain$8$?AddArrows@CFarMenu@@IEAAXXZ 000000018001a044     FarMenu.obj
 0001:00019054       $unwind$?MenuDlgProc@@YAHPEAUHWND__@@I_K_J@Z 000000018001a054     MenuDlg.obj
 0001:00019068       $unwind$_invalid_parameter_noinfo 000000018001a068     libucrt:invalid_parameter.obj
 0001:00019068       $unwind$_log10_special     000000018001a068     libucrt:log_special.obj
 0001:00019068       $unwind$?AddItem@CFarMenu@@QEAAIPEB_W_NW4ECheck@1@1@Z 000000018001a068     FarMenu.obj
 0001:00019068       $unwind$?OpenPlugin@OleThread@@YA?AW4EDoMenu@CPlugin@@H_J@Z 000000018001a068     OleThread.obj
 0001:00019068       $unwind$?EnsureThreadStarted@OleThread@@YA_NXZ 000000018001a068     OleThread.obj
 0001:00019070       $unwind$?ThreadProc@OleThread@@YAKPEAX@Z 000000018001a070     OleThread.obj
 0001:00019078       $chain$0$?ThreadProc@OleThread@@YAKPEAX@Z 000000018001a078     OleThread.obj
 0001:0001908c       $chain$1$?ThreadProc@OleThread@@YAKPEAX@Z 000000018001a08c     OleThread.obj
 0001:0001909c       $chain$0$?EnsureThreadStarted@OleThread@@YA_NXZ 000000018001a09c     OleThread.obj
 0001:000190b0       $chain$1$?EnsureThreadStarted@OleThread@@YA_NXZ 000000018001a0b0     OleThread.obj
 0001:000190c0       $chain$0$?EnsureSpace@CPidl@@QEAAXXZ 000000018001a0c0     Pidl.obj
 0001:000190d4       $chain$1$?EnsureSpace@CPidl@@QEAAXXZ 000000018001a0d4     Pidl.obj
 0001:000190e4       $chain$0$?Add@CPidl@@QEAAXPEFAU_ITEMIDLIST@@@Z 000000018001a0e4     Pidl.obj
 0001:000190f8       $chain$1$?Add@CPidl@@QEAAXPEFAU_ITEMIDLIST@@@Z 000000018001a0f8     Pidl.obj
 0001:00019108       $unwind$?Add@CPidl@@QEAAXPEFAU_ITEMIDLIST@@@Z 000000018001a108     Pidl.obj
 0001:00019108       $unwind$?Insert@CPidl@@QEAAXIPEFAU_ITEMIDLIST@@@Z 000000018001a108     Pidl.obj
 0001:00019118       $chain$0$?Insert@CPidl@@QEAAXIPEFAU_ITEMIDLIST@@@Z 000000018001a118     Pidl.obj
 0001:0001912c       $chain$1$?Insert@CPidl@@QEAAXIPEFAU_ITEMIDLIST@@@Z 000000018001a12c     Pidl.obj
 0001:0001913c       $unwind$?OpenPlugin@CPlugin@@QEAAPEAXH_J@Z 000000018001a13c     Plugin.obj
 0001:0001914c       $unwind$?OpenPluginBkg@CPlugin@@QEAA?AW4EDoMenu@1@H_J@Z 000000018001a14c     Plugin.obj
 0001:00019164       $unwind$?Configure@CPlugin@@QEAAHXZ 000000018001a164     Plugin.obj
 0001:00019180       $unwind$?DoMenu@CPlugin@@IEAA?AW4EDoMenu@1@PEA_WW4CallMode@1@@Z 000000018001a180     Plugin.obj
 0001:00019188       $chain$2$?DoMenu@CPlugin@@IEAA?AW4EDoMenu@1@PEA_WW4CallMode@1@@Z 000000018001a188     Plugin.obj
 0001:000191a4       $chain$4$?DoMenu@CPlugin@@IEAA?AW4EDoMenu@1@PEA_WW4CallMode@1@@Z 000000018001a1a4     Plugin.obj
 0001:000191bc       $chain$5$?DoMenu@CPlugin@@IEAA?AW4EDoMenu@1@PEA_WW4CallMode@1@@Z 000000018001a1bc     Plugin.obj
 0001:000191cc       $chain$6$?DoMenu@CPlugin@@IEAA?AW4EDoMenu@1@PEA_WW4CallMode@1@@Z 000000018001a1cc     Plugin.obj
 0001:000191dc       $unwind$?SelectDrive@CPlugin@@IEAA?AW4EDoMenu@1@XZ 000000018001a1dc     Plugin.obj
 0001:000191f0       $chain$0$?SelectDrive@CPlugin@@IEAA?AW4EDoMenu@1@XZ 000000018001a1f0     Plugin.obj
 0001:00019204       $chain$1$?SelectDrive@CPlugin@@IEAA?AW4EDoMenu@1@XZ 000000018001a204     Plugin.obj
 0001:00019214       $unwind$?MenuForPanelOrCmdLine@CPlugin@@IEAA?AW4EDoMenu@1@PEA_WW4EAutoItem@1@@Z 000000018001a214     Plugin.obj
 0001:00019230       $unwind$?DoMenu@CPlugin@@IEAA?AW4EDoMenu@1@PEAUIShellFolder@@PEAPEFBU_ITEMIDLIST@@QEAPEB_WIIPEB_WW4EAutoItem@1@@Z 000000018001a230     Plugin.obj
 0001:0001924c       $unwind$?ShowGuiMenu@CPlugin@@IEAA_NPEAUHMENU__@@PEAUIContextMenu@@PEAUIContextMenu2@@PEAUIContextMenu3@@PEAH@Z 000000018001a24c     Plugin.obj
 0001:0001925c       $unwind$?ShowTextMenu@CPlugin@@IEAA_NPEAUHMENU__@@PEAUIContextMenu@@PEAUIContextMenu2@@PEAUIContextMenu3@@PEAHPEB_WPEAUIShellFolder@@PEAPEFBU_ITEMIDLIST@@I@Z 000000018001a25c     Plugin.obj
 0001:0001926c       $chain$0$?ShowTextMenu@CPlugin@@IEAA_NPEAUHMENU__@@PEAUIContextMenu@@PEAUIContextMenu2@@PEAUIContextMenu3@@PEAHPEB_WPEAUIShellFolder@@PEAPEFBU_ITEMIDLIST@@I@Z 000000018001a26c     Plugin.obj
 0001:00019280       $chain$2$?ShowTextMenu@CPlugin@@IEAA_NPEAUHMENU__@@PEAUIContextMenu@@PEAUIContextMenu2@@PEAUIContextMenu3@@PEAHPEB_WPEAUIShellFolder@@PEAPEFBU_ITEMIDLIST@@I@Z 000000018001a280     Plugin.obj
 0001:00019294       $unwind$?ShowFolder@CPlugin@@IEAA_NPEAUIShellFolder@@PEFBU_ITEMIDLIST@@PEAHPEB_WPEAPEAUIDropTarget@@@Z 000000018001a294     Plugin.obj
 0001:000192a8       $unwind$?GetFilesFromParams@CPlugin@@IEAA_NPEA_WPEAPEAPEB_WPEAI2PEAVauto_sz@@_N@Z 000000018001a2a8     Plugin.obj
 0001:000192c4       $unwind$?GetFilesFromPanel@CPlugin@@IEAA_NPEAPEAPEB_WPEAI1PEAVauto_sz@@@Z 000000018001a2c4     Plugin.obj
 0001:000192e4       $unwind$?ReadRegValues@CPlugin@@IEAAXXZ 000000018001a2e4     Plugin.obj
 0001:000192fc       $unwind$?CfgDlgProcStatic@CPlugin@@KA_JPEAX_J10@Z 000000018001a2fc     Plugin.obj
 0001:000192fc       $unwind$?CompareExcluding@auto_sz@@QEAA_NPEB_W_W@Z 000000018001a2fc     auto_sz.obj
 0001:00019310       $unwind$?GetAdditionalString@CPlugin@@IEAA_NPEAUIContextMenu@@IW4EAdditionalStr@1@PEAVauto_sz@@@Z 000000018001a310     Plugin.obj
 0001:00019340       $unwind$__raise_securityfailure 000000018001a340     LIBCMT:gs_report.obj
 0001:00019340       $unwind$?GetPluginInfo@CPlugin@@QEAAXPEAUPluginInfo@@@Z 000000018001a340     Plugin.obj
 0001:00019340       $unwind$_onexit            000000018001a340     LIBCMT:utility.obj
 0001:00019340       $unwind$__acrt_stdio_free_buffer_nolock 000000018001a340     libucrt:_freebuf.obj
 0001:00019340       $unwind$__vcrt_uninitialize_locks 000000018001a340     libvcruntime:locks.obj
 0001:00019340       $unwind$__acrt_uninitialize_locks 000000018001a340     libucrt:locks.obj
 0001:00019340       $unwind$??_GPluginCheckBoxBinding@@UEAAPEAXI@Z 000000018001a340     Plugin.obj
 0001:00019340       $unwind$__scrt_uninitialize_crt 000000018001a340     LIBCMT:utility.obj
 0001:00019340       $unwind$?exit_or_terminate_process@@YAXI@Z 000000018001a340     libucrt:exit.obj
 0001:00019340       $unwind$__acrt_update_multibyte_info 000000018001a340     libucrt:locale_update.obj
 0001:00019340       $unwind$__acrt_update_locale_info 000000018001a340     libucrt:locale_update.obj
 0001:00019340       $unwind$__scrt_release_startup_lock 000000018001a340     LIBCMT:utility.obj
 0001:00019340       $unwind$??_Gtype_info@@UEAAPEAXI@Z 000000018001a340     LIBCMT:std_type_info_static.obj
 0001:00019340       $unwind$uninitialize_allocated_memory 000000018001a340     libucrt:initialization.obj
 0001:00019340       $unwind$__vcrt_uninitialize 000000018001a340     libvcruntime:initialization.obj
 0001:00019340       $unwind$??2@YAPEAX_K@Z     000000018001a340     LIBCMT:new_scalar.obj
 0001:00019340       $unwind$strcpy_s           000000018001a340     libucrt:strcpy_s.obj
 0001:00019340       $unwind$??0exception@std@@QEAA@AEBV01@@Z 000000018001a340     LIBCMT:throw_bad_alloc.obj
 0001:00019340       $unwind$?Cleanup@OleThread@@YAXXZ 000000018001a340     OleThread.obj
 0001:00019340       $unwind$??ICPidl@@QEAAPEAPEFAU_ITEMIDLIST@@XZ 000000018001a340     Pidl.obj
 0001:00019340       $unwind$_malloc_base       000000018001a340     libucrt:malloc_base.obj
 0001:00019340       $unwind$??0bad_alloc@std@@QEAA@AEBV01@@Z 000000018001a340     LIBCMT:throw_bad_alloc.obj
 0001:00019340       $unwind$__std_type_info_destroy_list 000000018001a340     libvcruntime:std_type_info.obj
 0001:00019340       $unwind$__std_exception_destroy 000000018001a340     libvcruntime:std_exception.obj
 0001:00019340       $unwind$?GetArray@CPidl@@QEAAPEAPEFBU_ITEMIDLIST@@XZ 000000018001a340     Pidl.obj
 0001:00019340       $unwind$??0bad_array_new_length@std@@QEAA@AEBV01@@Z 000000018001a340     LIBCMT:throw_bad_alloc.obj
 0001:00019340       $unwind$??_GPluginRadioButtonBinding@@UEAAPEAXI@Z 000000018001a340     Plugin.obj
 0001:00019340       $unwind$__acrt_initialize_locks 000000018001a340     libucrt:locks.obj
 0001:00019340       $unwind$?SaveValue@PluginCheckBoxBinding@@UEAAXPEAUFarDialogItem@@H@Z 000000018001a340     Plugin.obj
 0001:00019340       $unwind$__acrt_uninitialize_stdio 000000018001a340     libucrt:_file.obj
 0001:00019340       $unwind$??0auto_sz@@QEAA@PEB_W@Z 000000018001a340     auto_sz.obj
 0001:00019340       $unwind$__acrt_allocate_buffer_for_argv 000000018001a340     libucrt:argv_parsing.obj
 0001:00019340       $unwind$__acrt_uninitialize_winapi_thunks 000000018001a340     libucrt:winapi_thunks.obj
 0001:00019340       $unwind$?SaveValue@PluginIntEditFieldBinding@@UEAAXPEAUFarDialogItem@@H@Z 000000018001a340     Plugin.obj
 0001:00019340       $unwind$__acrt_freeptd     000000018001a340     libucrt:per_thread_data.obj
 0001:00019340       $unwind$??1auto_sz@@QEAA@XZ 000000018001a340     auto_sz.obj
 0001:00019340       $unwind$??_GPluginUIntEditFieldBinding@@UEAAPEAXI@Z 000000018001a340     Plugin.obj
 0001:00019340       $unwind$__scrt_initialize_crt 000000018001a340     LIBCMT:utility.obj
 0001:00019340       $unwind$_set_statfp        000000018001a340     libucrt:fpctrl.obj
 0001:00019340       $unwind$??_G?$DialogItemBinding@UFarDialogItem@@@@UEAAPEAXI@Z 000000018001a340     Plugin.obj
 0001:00019340       $unwind$_clrfp             000000018001a340     libucrt:fpctrl.obj
 0001:00019340       $unwind$ExitFARW           000000018001a340     EMenu.obj
 0001:00019340       $unwind$SetStartupInfoW    000000018001a340     EMenu.obj
 0001:00019340       $unwind$_calloc_base       000000018001a340     libucrt:calloc_base.obj
 0001:00019340       $unwind$??_GPluginIntEditFieldBinding@@UEAAPEAXI@Z 000000018001a340     Plugin.obj
 0001:00019340       $unwind$initialize_pointers 000000018001a340     libucrt:initialization.obj
 0001:00019340       $unwind$_fflush_nolock     000000018001a340     libucrt:fflush.obj
 0001:00019340       $unwind$__vcrt_freeptd     000000018001a340     libvcruntime:per_thread_data.obj
 0001:00019340       $unwind$__vcrt_initialize_locks 000000018001a340     libvcruntime:locks.obj
 0001:00019340       $unwind$?SaveValue@PluginUIntEditFieldBinding@@UEAAXPEAUFarDialogItem@@H@Z 000000018001a340     Plugin.obj
 0001:00019340       $unwind$?Startup@OleThread@@YAXXZ 000000018001a340     OleThread.obj
 0001:00019348       $unwind$?ReallocDialogItems@?$DialogBuilderBase@UFarDialogItem@@@@IEAAXXZ 000000018001a348     Plugin.obj
 0001:00019358       $unwind$?MaxTextWidth@?$DialogBuilderBase@UFarDialogItem@@@@IEAA_JXZ 000000018001a358     Plugin.obj
 0001:00019368       $chain$1$?MaxTextWidth@?$DialogBuilderBase@UFarDialogItem@@@@IEAA_JXZ 000000018001a368     Plugin.obj
 0001:00019380       $chain$2$?MaxTextWidth@?$DialogBuilderBase@UFarDialogItem@@@@IEAA_JXZ 000000018001a380     Plugin.obj
 0001:00019390       $unwind$?SaveValues@?$DialogBuilderBase@UFarDialogItem@@@@IEAAXXZ 000000018001a390     Plugin.obj
 0001:000193a0       $chain$1$?SaveValues@?$DialogBuilderBase@UFarDialogItem@@@@IEAAXXZ 000000018001a3a0     Plugin.obj
 0001:000193b8       $chain$2$?SaveValues@?$DialogBuilderBase@UFarDialogItem@@@@IEAAXXZ 000000018001a3b8     Plugin.obj
 0001:000193c8       $chain$0$??1?$DialogBuilderBase@UFarDialogItem@@@@MEAA@XZ 000000018001a3c8     Plugin.obj
 0001:000193dc       $chain$1$??1?$DialogBuilderBase@UFarDialogItem@@@@MEAA@XZ 000000018001a3dc     Plugin.obj
 0001:000193ec       $unwind$?AddButtons@?$DialogBuilderBase@UFarDialogItem@@@@QEAAXHPEBHHH@Z 000000018001a3ec     Plugin.obj
 0001:000193fc       $chain$3$?AddButtons@?$DialogBuilderBase@UFarDialogItem@@@@QEAAXHPEBHHH@Z 000000018001a3fc     Plugin.obj
 0001:0001941c       $chain$4$?AddButtons@?$DialogBuilderBase@UFarDialogItem@@@@QEAAXHPEBHHH@Z 000000018001a41c     Plugin.obj
 0001:0001942c       $unwind$?DoShowDialog@PluginDialogBuilder@@MEAA_JXZ 000000018001a42c     Plugin.obj
 0001:00019438       $unwind$?IsWindowsVersionOrGreater@@YA_NGGG@Z 000000018001a438     Plugin.obj
 0001:00019450       $unwind$?dllmain_crt_process_attach@@YAHQEAUHINSTANCE__@@QEAX@Z 000000018001a450     LIBCMT:dll_dllmain.obj
 0001:0001947c       $unwind$?dllmain_crt_process_detach@@YAH_N@Z 000000018001a47c     LIBCMT:dll_dllmain.obj
 0001:000194a4       $unwind$?dllmain_dispatch@@YAHQEAUHINSTANCE__@@KQEAX@Z 000000018001a4a4     LIBCMT:dll_dllmain.obj
 0001:000194cc       $unwind$?filt$0@?0??dllmain_dispatch@@YAHQEAUHINSTANCE__@@KQEAX@Z@4HA 000000018001a4cc     LIBCMT:dll_dllmain.obj
 0001:000194d4       $unwind$__scrt_is_nonwritable_in_current_image 000000018001a4d4     LIBCMT:utility.obj
 0001:000194f4       $unwind$__scrt_is_nonwritable_in_current_image$filt$0 000000018001a4f4     LIBCMT:utility.obj
 0001:000194fc       $unwind$__scrt_initialize_onexit_tables 000000018001a4fc     LIBCMT:utility.obj
 0001:00019508       $unwind$__security_init_cookie 000000018001a508     LIBCMT:gs_support.obj
 0001:00019514       $unwind$__scrt_fastfail    000000018001a514     LIBCMT:utility_desktop.obj
 0001:00019524       $unwind$__isa_available_init 000000018001a524     LIBCMT:_cpu_disp_.obj
 0001:00019530       $xdatasym                  000000018001a530     LIBCMT:_guard_dispatch_.obj
 0001:00019534       $chain$0$??0_com_error@@QEAA@JPEAUIErrorInfo@@_N@Z 000000018001a534     comsuppw:comraise.obj
 0001:00019548       $chain$1$??0_com_error@@QEAA@JPEAUIErrorInfo@@_N@Z 000000018001a548     comsuppw:comraise.obj
 0001:00019558       $unwind$??0_com_error@@QEAA@JPEAUIErrorInfo@@_N@Z 000000018001a558     comsuppw:comraise.obj
 0001:00019558       $unwind$??0_com_error@@QEAA@AEBV0@@Z 000000018001a558     comsuppw:comraise.obj
 0001:00019558       $unwind$?EnsureSpace@CPidl@@QEAAXXZ 000000018001a558     Pidl.obj
 0001:00019564       $chain$0$??0_com_error@@QEAA@AEBV0@@Z 000000018001a564     comsuppw:comraise.obj
 0001:00019578       $chain$1$??0_com_error@@QEAA@AEBV0@@Z 000000018001a578     comsuppw:comraise.obj
 0001:00019588       $chain$1$??1_com_error@@UEAA@XZ 000000018001a588     comsuppw:comraise.obj
 0001:000195a0       $chain$2$??1_com_error@@UEAA@XZ 000000018001a5a0     comsuppw:comraise.obj
 0001:000195b4       $chain$3$??1_com_error@@UEAA@XZ 000000018001a5b4     comsuppw:comraise.obj
 0001:000195c4       $chain$4$??1_com_error@@UEAA@XZ 000000018001a5c4     comsuppw:comraise.obj
 0001:000195d8       $xdatasym                  000000018001a5d8     libvcruntime:memcpy.obj
 0001:000195dc       $unwind$__C_specific_handler 000000018001a5dc     libvcruntime:_chandler_.obj
 0001:000195f8       $xdatasym                  000000018001a5f8     libvcruntime:memset.obj
 0001:000195fc       $unwind$__telemetry_main_invoke_trigger 000000018001a5fc     libvcruntime:telemetry.obj
 0001:000195fc       $unwind$__telemetry_main_return_trigger 000000018001a5fc     libvcruntime:telemetry.obj
 0001:00019614       $unwind$?_TlgEnableCallback@__vcrt_trace_logging_provider@@YAXPEBU_GUID@@KE_K1PEAU_EVENT_FILTER_DESCRIPTOR@@PEAX@Z 000000018001a614     libvcruntime:telemetry.obj
 0001:00019630       $unwind$_CxxThrowException 000000018001a630     libvcruntime:throw.obj
 0001:00019648       $xdatasym                  000000018001a648     libvcruntime:_jmpuwind_.obj
 0001:0001965c       $unwind$_invalid_parameter 000000018001a65c     libucrt:invalid_parameter.obj
 0001:0001965c       $unwind$__vcrt_EventWriteTransfer 000000018001a65c     libvcruntime:winapi_downlevel.obj
 0001:00019674       $unwind$__vcrt_initialize_winapi_thunks 000000018001a674     libvcruntime:winapi_downlevel.obj
 0001:00019674       $unwind$__acrt_initialize_winapi_thunks 000000018001a674     libucrt:winapi_thunks.obj
 0001:0001967c       $unwind$__vcrt_uninitialize_winapi_thunks 000000018001a67c     libvcruntime:winapi_downlevel.obj
 0001:00019684       $unwind$?replace_current_thread_locale_nolock@@YAXQEAU__acrt_ptd@@QEAU__crt_locale_data@@@Z 000000018001a684     libucrt:per_thread_data.obj
 0001:00019684       $unwind$??0_LocaleUpdate@@QEAA@QEAU__crt_locale_pointers@@@Z 000000018001a684     libucrt:output.obj
 0001:00019684       $unwind$??4auto_sz@@QEAAAEAV0@AEBV0@@Z 000000018001a684     auto_sz.obj
 0001:00019684       $unwind$?RemoveTrailing@auto_sz@@QEAAX_W@Z 000000018001a684     auto_sz.obj
 0001:00019684       $unwind$?CreateRadioButtonBinding@PluginDialogBuilder@@MEAAPEAU?$DialogItemBinding@UFarDialogItem@@@@PEAH@Z 000000018001a684     Plugin.obj
 0001:00019684       $unwind$_realloc_base      000000018001a684     libucrt:realloc_base.obj
 0001:00019684       $unwind$__acrt_getptd      000000018001a684     libucrt:per_thread_data.obj
 0001:00019684       $unwind$__acrt_invoke_user_matherr 000000018001a684     libucrt:matherr.obj
 0001:00019684       $unwind$__acrt_uninitialize_lowio 000000018001a684     libucrt:ioinit.obj
 0001:00019684       $unwind$??_G?$DialogBuilderBase@UFarDialogItem@@@@MEAAPEAXI@Z 000000018001a684     Plugin.obj
 0001:00019684       $unwind$??_GPluginDialogBuilder@@UEAAPEAXI@Z 000000018001a684     Plugin.obj
 0001:00019684       $unwind$??4auto_sz@@QEAAAEAV0@PEB_W@Z 000000018001a684     auto_sz.obj
 0001:00019684       $unwind$??0PluginUIntEditFieldBinding@@QEAA@AEBUPluginStartupInfo@@PEAPEAXHPEAIH@Z 000000018001a684     Plugin.obj
 0001:00019684       $unwind$__acrt_FlsFree     000000018001a684     libucrt:winapi_thunks.obj
 0001:00019684       $unwind$??$common_initialize_environment_nolock@D@@YAHXZ 000000018001a684     libucrt:environment_initialization.obj
 0001:00019684       $unwind$?SaveValue@PluginRadioButtonBinding@@UEAAXPEAUFarDialogItem@@H@Z 000000018001a684     Plugin.obj
 0001:00019684       $unwind$_updatetlocinfoEx_nolock 000000018001a684     libucrt:locale_refcounting.obj
 0001:00019684       $unwind$__vcrt_FlsGetValue 000000018001a684     libvcruntime:winapi_downlevel.obj
 0001:00019684       $unwind$__vcrt_FlsFree     000000018001a684     libvcruntime:winapi_downlevel.obj
 0001:00019684       $unwind$?UpdateBorderSize@?$DialogBuilderBase@UFarDialogItem@@@@IEAAXXZ 000000018001a684     Plugin.obj
 0001:00019684       $unwind$__vcrt_FlsAlloc    000000018001a684     libvcruntime:winapi_downlevel.obj
 0001:00019684       $unwind$??0PluginIntEditFieldBinding@@QEAA@AEBUPluginStartupInfo@@PEAPEAXHPEAHH@Z 000000018001a684     Plugin.obj
 0001:00019684       $unwind$?InitDialogItem@PluginDialogBuilder@@MEAAXPEAUFarDialogItem@@PEB_W@Z 000000018001a684     Plugin.obj
 0001:00019684       $unwind$__acrt_errno_map_os_error 000000018001a684     libucrt:errno.obj
 0001:00019684       $unwind$__vcrt_EventUnregister 000000018001a684     libvcruntime:winapi_downlevel.obj
 0001:00019684       $unwind$_close_nolock      000000018001a684     libucrt:close.obj
 0001:00019684       $unwind$??0CPlugin@@QEAA@PEBUPluginStartupInfo@@@Z 000000018001a684     Plugin.obj
 0001:00019684       $unwind$??_G_com_error@@UEAAPEAXI@Z 000000018001a684     comsuppw:comraise.obj
 0001:00019684       $unwind$_callnewh          000000018001a684     libucrt:new_handler.obj
 0001:00019684       $unwind$?try_cor_exit_process@@YAXI@Z 000000018001a684     libucrt:exit.obj
 0001:00019684       $unwind$??_Gexception@std@@UEAAPEAXI@Z 000000018001a684     LIBCMT:throw_bad_alloc.obj
 0001:00019684       $unwind$?_com_issue_error@@YAXJ@Z 000000018001a684     comsuppw:comsupp.obj
 0001:00019684       $unwind$_fclose_nolock     000000018001a684     libucrt:fclose.obj
 0001:00019684       $unwind$strncpy_s          000000018001a684     libucrt:strncpy_s.obj
 0001:00019684       $unwind$??_Gbad_alloc@std@@UEAAPEAXI@Z 000000018001a684     LIBCMT:throw_bad_alloc.obj
 0001:00019684       $unwind$__acrt_FlsGetValue 000000018001a684     libucrt:winapi_thunks.obj
 0001:00019684       $unwind$__acrt_FlsAlloc    000000018001a684     libucrt:winapi_thunks.obj
 0001:00019684       $unwind$??1CPidl@@QEAA@XZ  000000018001a684     Pidl.obj
 0001:00019684       $unwind$??_Gbad_array_new_length@std@@UEAAPEAXI@Z 000000018001a684     LIBCMT:throw_bad_alloc.obj
 0001:00019690       $unwind$_query_new_handler 000000018001a690     libucrt:new_handler.obj
 0001:000196b0       $unwind$__vcrt_InitializeCriticalSectionEx 000000018001a6b0     libvcruntime:winapi_downlevel.obj
 0001:000196b0       $unwind$_seh_filter_exe    000000018001a6b0     libucrt:exception_filter.obj
 0001:000196b0       $unwind$_recalloc_base     000000018001a6b0     libucrt:recalloc.obj
 0001:000196b0       $unwind$__acrt_InitializeCriticalSectionEx 000000018001a6b0     libucrt:winapi_thunks.obj
 0001:000196b0       $unwind$__scrt_dllmain_exception_filter 000000018001a6b0     LIBCMT:utility.obj
 0001:000196b0       $unwind$?setSBCS@@YAXPEAU__crt_multibyte_data@@@Z 000000018001a6b0     libucrt:mbctype.obj
 0001:000196b0       $unwind$__acrt_execute_initializers 000000018001a6b0     libucrt:shared_initialization.obj
 0001:000196b0       $unwind$__acrt_lowio_create_handle_array 000000018001a6b0     libucrt:osfinfo.obj
 0001:000196b0       $unwind$?expand_if_necessary@?$argument_list@D@?A0xca0879c4@@AEAAHXZ 000000018001a6b0     libucrt:argv_wildcards.obj
 0001:000196b0       $unwind$__acrt_free_locale 000000018001a6b0     libucrt:locale_refcounting.obj
 0001:000196b0       $unwind$?CfgDlgProc@CPlugin@@IEAAXPEAX_J10@Z 000000018001a6b0     Plugin.obj
 0001:000196b0       $unwind$?dllmain_raw@@YAHQEAUHINSTANCE__@@KQEAX@Z 000000018001a6b0     LIBCMT:dll_dllmain.obj
 0001:000196c4       $unwind$?common_exit@@YAXHW4_crt_exit_cleanup_mode@@W4_crt_exit_return_mode@@@Z 000000018001a6c4     libucrt:exit.obj
 0001:00019704       $unwind$_configure_narrow_argv 000000018001a704     libucrt:argv_parsing.obj
 0001:00019718       $unwind$??$free_environment@D@@YAXQEAPEAD@Z 000000018001a718     libucrt:environment_initialization.obj
 0001:00019718       $unwind$??$free_environment@_W@@YAXQEAPEA_W@Z 000000018001a718     libucrt:environment_initialization.obj
 0001:00019724       $unwind$??$create_environment@D@@YAQEAPEADQEAD@Z 000000018001a724     libucrt:environment_initialization.obj
 0001:00019724       $unwind$?AddUIntEditField@PluginDialogBuilder@@UEAAPEAUFarDialogItem@@PEAIH@Z 000000018001a724     Plugin.obj
 0001:00019724       $unwind$?AddIntEditField@PluginDialogBuilder@@UEAAPEAUFarDialogItem@@PEAHH@Z 000000018001a724     Plugin.obj
 0001:0001973c       $unwind$_register_onexit_function 000000018001a73c     libucrt:onexit.obj
 0001:00019744       $unwind$_execute_onexit_table 000000018001a744     libucrt:onexit.obj
 0001:0001974c       $unwind$??$parse_command_line@D@@YAXPEADPEAPEAD0PEA_K2@Z 000000018001a74c     libucrt:argv_parsing.obj
 0001:0001974c       $unwind$??R<lambda_4e60a939b0d047cfe11ddc22648dfba9>@@QEBAHXZ 000000018001a74c     libucrt:onexit.obj
 0001:00019768       $unwind$??$?RV<lambda_b8c45f8f788dd370798f47cfe8ac3a86>@@AEAV<lambda_4e60a939b0d047cfe11ddc22648dfba9>@@V<lambda_332c3edc96d0294ec56c57d38c1cdfd5>@@@?$__crt_seh_guarded_call@H@@QEAAH$$QEAV<lambda_b8c45f8f788dd370798f47cfe8ac3a86>@@AEAV<lambda_4e60a939b0d047cfe11ddc22648dfba9>@@$$QEAV<lambda_332c3edc96d0294ec56c57d38c1cdfd5>@@@Z 000000018001a768     libucrt:onexit.obj
 0001:0001978c       $unwind$??$?RV<lambda_e24bbb7b643b32fcea6fa61b31d4c984>@@AEAV<lambda_275893d493268fdec8709772e3fcec0e>@@V<lambda_9d71df4d7cf3f480f8d633942495c3b0>@@@?$__crt_seh_guarded_call@H@@QEAAH$$QEAV<lambda_e24bbb7b643b32fcea6fa61b31d4c984>@@AEAV<lambda_275893d493268fdec8709772e3fcec0e>@@$$QEAV<lambda_9d71df4d7cf3f480f8d633942495c3b0>@@@Z 000000018001a78c     libucrt:onexit.obj
 0001:000197bc       $unwind$terminate          000000018001a7bc     libucrt:terminate.obj
 0001:000197dc       $unwind$?construct_ptd_array@@YAXQEAU__acrt_ptd@@@Z 000000018001a7dc     libucrt:per_thread_data.obj
 0001:000197e4       $unwind$?destroy_ptd_array@@YAXQEAU__acrt_ptd@@@Z 000000018001a7e4     libucrt:per_thread_data.obj
 0001:000197ec       $unwind$??$?RV<lambda_72d1df2b273a38828b1ce30cbf4cdab5>@@AEAV<lambda_876a65b173b8412d3a47c70a915b0cf4>@@V<lambda_41932305e351933ebe8f8be3ed8bb5dc>@@@?$__crt_seh_guarded_call@X@@QEAAX$$QEAV<lambda_72d1df2b273a38828b1ce30cbf4cdab5>@@AEAV<lambda_876a65b173b8412d3a47c70a915b0cf4>@@$$QEAV<lambda_41932305e351933ebe8f8be3ed8bb5dc>@@@Z 000000018001a7ec     libucrt:per_thread_data.obj
 0001:00019810       $unwind$??$?RV<lambda_5e887d1dcbef67a5eb4283622ba103bf>@@AEAV<lambda_4466841279450cc726390878d4a41900>@@V<lambda_341c25c0346d94847f1f3c463c57e077>@@@?$__crt_seh_guarded_call@X@@QEAAX$$QEAV<lambda_5e887d1dcbef67a5eb4283622ba103bf>@@AEAV<lambda_4466841279450cc726390878d4a41900>@@$$QEAV<lambda_341c25c0346d94847f1f3c463c57e077>@@@Z 000000018001a810     libucrt:per_thread_data.obj
 0001:00019834       $unwind$??$?RV<lambda_46352004c1216016012b18bd6f87e700>@@AEAV<lambda_3bd07e1a1191394380780325891bf33f>@@V<lambda_334532d3f185bcaa59b5be82d7d22bff>@@@?$__crt_seh_guarded_call@X@@QEAAX$$QEAV<lambda_46352004c1216016012b18bd6f87e700>@@AEAV<lambda_3bd07e1a1191394380780325891bf33f>@@$$QEAV<lambda_334532d3f185bcaa59b5be82d7d22bff>@@@Z 000000018001a834     libucrt:per_thread_data.obj
 0001:00019858       $unwind$??$?RV<lambda_fb3a7dec4e47f37f22dae91bb15c9095>@@AEAV<lambda_698284760c8add0bfb0756c19673e34b>@@V<lambda_dfb8eca1e75fef3034a8fb18dd509707>@@@?$__crt_seh_guarded_call@X@@QEAAX$$QEAV<lambda_fb3a7dec4e47f37f22dae91bb15c9095>@@AEAV<lambda_698284760c8add0bfb0756c19673e34b>@@$$QEAV<lambda_dfb8eca1e75fef3034a8fb18dd509707>@@@Z 000000018001a858     libucrt:per_thread_data.obj
 0001:0001987c       $unwind$??1?$DialogBuilderBase@UFarDialogItem@@@@MEAA@XZ 000000018001a87c     Plugin.obj
 0001:0001987c       $unwind$??1CFarMenu@@QEAA@XZ 000000018001a87c     FarMenu.obj
 0001:0001987c       $unwind$__acrt_is_packaged_app 000000018001a87c     libucrt:winapi_thunks.obj
 0001:00019888       $unwind$?try_get_function@@YAPEAXW4function_id@?A0x49c8dc86@@QEBDQEBW4module_id@2@2@Z 000000018001a888     libvcruntime:winapi_downlevel.obj
 0001:00019888       $unwind$?try_get_function@@YAPEAXW4function_id@?A0x63058377@@QEBDQEBW4module_id@2@2@Z 000000018001a888     libucrt:winapi_thunks.obj
 0001:000198a4       $unwind$__acrt_call_reportfault 000000018001a8a4     libucrt:invalid_parameter.obj
 0001:000198c4       $unwind$??$common_expand_argv_wildcards@D@@YAHQEAPEADQEAPEAPEAD@Z 000000018001a8c4     libucrt:argv_wildcards.obj
 0001:000198dc       $unwind$??$copy_and_add_argument_to_buffer@D@@YAHQEBD0_KAEAV?$argument_list@D@?A0xca0879c4@@@Z 000000018001a8dc     libucrt:argv_wildcards.obj
 0001:000198f8       $unwind$??$expand_argument_wildcards@D@@YAHQEAD0AEAV?$argument_list@D@?A0xca0879c4@@@Z 000000018001a8f8     libucrt:argv_wildcards.obj
 0001:00019918       $unwind$__acrt_update_thread_multibyte_data 000000018001a918     libucrt:mbctype.obj
 0001:0001993c       $unwind$_setmbcp_nolock    000000018001a93c     libucrt:mbctype.obj
 0001:0001995c       $unwind$?setSBUpLow@@YAXPEAU__crt_multibyte_data@@@Z 000000018001a95c     libucrt:mbctype.obj
 0001:00019978       $unwind$?setmbcp_internal@@YAHH_N@Z 000000018001a978     libucrt:mbctype.obj
 0001:00019988       $unwind$_initterm_e        000000018001a988     libucrt:initterm.obj
 0001:00019988       $unwind$__acrt_FlsSetValue 000000018001a988     libucrt:winapi_thunks.obj
 0001:00019988       $unwind$_exception_enabled 000000018001a988     libucrt:libm_error.obj
 0001:00019988       $unwind$?CreateCheckBoxBinding@PluginDialogBuilder@@MEAAPEAU?$DialogItemBinding@UFarDialogItem@@@@PEAHH@Z 000000018001a988     Plugin.obj
 0001:00019988       $unwind$_DllMainCRTStartup 000000018001a988     LIBCMT:dll_dllmain.obj
 0001:00019988       $unwind$??Yauto_sz@@QEAAAEAV0@PEB_W@Z 000000018001a988     auto_sz.obj
 0001:00019988       $unwind$__acrt_getptd_noexit 000000018001a988     libucrt:per_thread_data.obj
 0001:00019988       $unwind$__acrt_stdio_flush_nolock 000000018001a988     libucrt:fflush.obj
 0001:00019988       $unwind$??$common_lseek_nolock@_J@@YA_JH_JH@Z 000000018001a988     libucrt:lseek.obj
 0001:00019988       $unwind$??0auto_sz@@QEAA@PEB_W_K@Z 000000018001a988     auto_sz.obj
 0001:00019988       $unwind$_RTC_Initialize    000000018001a988     LIBCMT:_initsect_.obj
 0001:00019988       $unwind$??R<lambda_ad1ced32f4ac17aa236e5ef05d6b3b7c>@@QEBAXXZ 000000018001a988     libucrt:mbctype.obj
 0001:00019988       $unwind$__acrt_LocaleNameToLCID 000000018001a988     libucrt:winapi_thunks.obj
 0001:00019988       $unwind$??0CFarMenu@@QEAA@PEB_WPEBU_GUID@@I@Z 000000018001a988     FarMenu.obj
 0001:00019988       $unwind$__vcrt_FlsSetValue 000000018001a988     libvcruntime:winapi_downlevel.obj
 0001:00019988       $unwind$__vcrt_getptd_noexit 000000018001a988     libvcruntime:per_thread_data.obj
 0001:00019988       $unwind$?free_crt_array_internal@@YAXQEAPEBX_K@Z 000000018001a988     libucrt:inittime.obj
 0001:00019988       $unwind$_RTC_Terminate     000000018001a988     LIBCMT:_initsect_.obj
 0001:00019988       $unwind$?TraceLoggingRegister@__vcrt_trace_logging_provider@@YAJPEBU_TlgProvider_t@1@PEBU_GUID@@P6AX1KE_K2PEAU_EVENT_FILTER_DESCRIPTOR@@PEAX@Z4@Z 000000018001a988     libvcruntime:telemetry.obj
 0001:00019988       $unwind$__acrt_execute_uninitializers 000000018001a988     libucrt:shared_initialization.obj
 0001:00019998       $unwind$??$?RV<lambda_99476a1ad63dd22509b5d3e65b0ffc95>@@AEAV<lambda_ad1ced32f4ac17aa236e5ef05d6b3b7c>@@V<lambda_f7424dd8d45958661754dc4f2697e9c3>@@@?$__crt_seh_guarded_call@X@@QEAAX$$QEAV<lambda_99476a1ad63dd22509b5d3e65b0ffc95>@@AEAV<lambda_ad1ced32f4ac17aa236e5ef05d6b3b7c>@@$$QEAV<lambda_f7424dd8d45958661754dc4f2697e9c3>@@@Z 000000018001a998     libucrt:mbctype.obj
 0001:000199bc       $unwind$?x_ismbbtype_l@@YAHPEAU__crt_locale_pointers@@IHH@Z 000000018001a9bc     libucrt:ismbbyte.obj
 0001:000199cc       $unwind$__dcrt_get_narrow_environment_from_os 000000018001a9cc     libucrt:get_environment_from_os.obj
 0001:000199e4       $unwind$__acrt_initialize_lowio 000000018001a9e4     libucrt:ioinit.obj
 0001:00019a04       $unwind$?initialize_inherited_file_handles_nolock@@YAXXZ 000000018001aa04     libucrt:ioinit.obj
 0001:00019a20       $unwind$_free_osfhnd       000000018001aa20     libucrt:osfinfo.obj
 0001:00019a20       $unwind$?initialize_stdio_handles_nolock@@YAXXZ 000000018001aa20     libucrt:ioinit.obj
 0001:00019a20       $unwind$__std_exception_copy 000000018001aa20     libvcruntime:std_exception.obj
 0001:00019a34       $unwind$__acrt_get_sigabrt_handler 000000018001aa34     libucrt:signal.obj
 0001:00019a3c       $unwind$raise              000000018001aa3c     libucrt:signal.obj
 0001:00019a68       $unwind$??$?RV<lambda_c36588078e9f5dfd39652860aa6b3aaf>@@AEAV<lambda_ec61778202f4f5fc7e7711acc23c3bca>@@V<lambda_dc9d2797ccde5d239b4a0efae8ebd7db>@@@?$__crt_seh_guarded_call@P6AXH@Z@@QEAAP6AXH@Z$$QEAV<lambda_c36588078e9f5dfd39652860aa6b3aaf>@@AEAV<lambda_ec61778202f4f5fc7e7711acc23c3bca>@@$$QEAV<lambda_dc9d2797ccde5d239b4a0efae8ebd7db>@@@Z 000000018001aa68     libucrt:signal.obj
 0001:00019a8c       $unwind$__acrt_LCMapStringEx 000000018001aa8c     libucrt:winapi_thunks.obj
 0001:00019a8c       $unwind$_mbtowc_l          000000018001aa8c     libucrt:mbtowc.obj
 0001:00019aa4       $unwind$__vcrt_EventSetInformation 000000018001aaa4     libvcruntime:winapi_downlevel.obj
 0001:00019aa4       $unwind$_initterm          000000018001aaa4     libucrt:initterm.obj
 0001:00019aa4       $unwind$__acrt_initialize_stdio 000000018001aaa4     libucrt:_file.obj
 0001:00019aa4       $unwind$__vcrt_EventRegister 000000018001aaa4     libvcruntime:winapi_downlevel.obj
 0001:00019abc       $unwind$__acrt_uninitialize_locale 000000018001aabc     libucrt:wsetlocale.obj
 0001:00019adc       $unwind$?destroy_fls@@YAXPEAX@Z 000000018001aadc     libucrt:per_thread_data.obj
 0001:00019adc       $unwind$_free_base         000000018001aadc     libucrt:free_base.obj
 0001:00019adc       $unwind$__acrt_locale_free_numeric 000000018001aadc     libucrt:initnum.obj
 0001:00019adc       $unwind$__acrt_locale_free_lc_time_if_unreferenced 000000018001aadc     libucrt:locale_refcounting.obj
 0001:00019ae4       $unwind$__acrt_update_thread_locale_data 000000018001aae4     libucrt:locale_refcounting.obj
 0001:00019b08       $unwind$?GetTableIndexFromLocaleName@@YAHPEB_W@Z 000000018001ab08     libucrt:lcidtoname_downlevel.obj
 0001:00019b20       $unwind$qsort              000000018001ab20     libucrt:qsort.obj
 0001:00019b38       $chain$4$qsort             000000018001ab38     libucrt:qsort.obj
 0001:00019b5c       $chain$5$qsort             000000018001ab5c     libucrt:qsort.obj
 0001:00019b6c       $unwind$?shortsort@@YAXPEAD0_KP6AHPEBX2@Z@Z 000000018001ab6c     libucrt:qsort.obj
 0001:00019b7c       $chain$2$?shortsort@@YAXPEAD0_KP6AHPEBX2@Z@Z 000000018001ab7c     libucrt:qsort.obj
 0001:00019b98       $chain$3$?shortsort@@YAXPEAD0_KP6AHPEBX2@Z@Z 000000018001ab98     libucrt:qsort.obj
 0001:00019ba8       $unwind$strpbrk            000000018001aba8     libucrt:strpbrk.obj
 0001:00019bb8       $unwind$_mbsdec_l          000000018001abb8     libucrt:mbsdec.obj
 0001:00019bc4       $unwind$__acrt_GetStringTypeA 000000018001abc4     libucrt:getstringtypea.obj
 0001:00019bec       $unwind$__acrt_LCMapStringA 000000018001abec     libucrt:lcmapstringa.obj
 0001:00019bfc       $unwind$?__acrt_LCMapStringA_stat@@YAHPEAU__crt_locale_pointers@@PEB_WKPEBDHPEADHHH@Z 000000018001abfc     libucrt:lcmapstringa.obj
 0001:00019c24       $unwind$__acrt_lowio_destroy_handle_array 000000018001ac24     libucrt:osfinfo.obj
 0001:00019c34       $unwind$__acrt_lowio_ensure_fh_exists 000000018001ac34     libucrt:osfinfo.obj
 0001:00019c60       $unwind$_IsNonwritableInCurrentImage$filt$0 000000018001ac60     LIBCMT:pesect.obj
 0001:00019c60       $unwind$?fin$0@?0??dllmain_crt_process_attach@@YAHQEAUHINSTANCE__@@QEAX@Z@4HA 000000018001ac60     LIBCMT:dll_dllmain.obj
 0001:00019c60       $unwind$__acrt_update_thread_multibyte_data$fin$0 000000018001ac60     libucrt:mbctype.obj
 0001:00019c60       $unwind$?fin$0@?0???$?RV<lambda_5e887d1dcbef67a5eb4283622ba103bf>@@AEAV<lambda_4466841279450cc726390878d4a41900>@@V<lambda_341c25c0346d94847f1f3c463c57e077>@@@?$__crt_seh_guarded_call@X@@QEAAX$$QEAV<lambda_5e887d1dcbef67a5eb4283622ba103bf>@@AEAV<lambda_4466841279450cc726390878d4a41900>@@$$QEAV<lambda_341c25c0346d94847f1f3c463c57e077>@@@Z@4HA 000000018001ac60     libucrt:per_thread_data.obj
 0001:00019c60       $unwind$?filt$0@?0??common_exit@@YAXHW4_crt_exit_cleanup_mode@@W4_crt_exit_return_mode@@@Z@4HA 000000018001ac60     libucrt:exit.obj
 0001:00019c60       $unwind$__acrt_update_thread_locale_data$fin$0 000000018001ac60     libucrt:locale_refcounting.obj
 0001:00019c60       $unwind$common_flush_all$fin$1 000000018001ac60     libucrt:fflush.obj
 0001:00019c60       $unwind$__acrt_lowio_ensure_fh_exists$fin$0 000000018001ac60     libucrt:osfinfo.obj
 0001:00019c60       $unwind$__acrt_initialize_lowio$fin$0 000000018001ac60     libucrt:ioinit.obj
 0001:00019c60       $unwind$common_flush_all$fin$0 000000018001ac60     libucrt:fflush.obj
 0001:00019c60       $unwind$_query_new_handler$fin$0 000000018001ac60     libucrt:new_handler.obj
 0001:00019c60       $unwind$?fin$0@?0???$?RV<lambda_b521505b218e5242e90febf6bfebc422>@@AEAV<lambda_6978c1fb23f02e42e1d9e99668cc68aa>@@V<lambda_314360699dd331753a4119843814e9a7>@@@?$__crt_seh_guarded_call@H@@QEAAH$$QEAV<lambda_b521505b218e5242e90febf6bfebc422>@@AEAV<lambda_6978c1fb23f02e42e1d9e99668cc68aa>@@$$QEAV<lambda_314360699dd331753a4119843814e9a7>@@@Z@4HA 000000018001ac60     libucrt:commit.obj
 0001:00019c60       $unwind$_ctrlfp$filt$0     000000018001ac60     libucrt:fpctrl.obj
 0001:00019c60       $unwind$__acrt_uninitialize_locale$fin$0 000000018001ac60     libucrt:wsetlocale.obj
 0001:00019c60       $unwind$?fin$0@?0???$?RV<lambda_e24bbb7b643b32fcea6fa61b31d4c984>@@AEAV<lambda_275893d493268fdec8709772e3fcec0e>@@V<lambda_9d71df4d7cf3f480f8d633942495c3b0>@@@?$__crt_seh_guarded_call@H@@QEAAH$$QEAV<lambda_e24bbb7b643b32fcea6fa61b31d4c984>@@AEAV<lambda_275893d493268fdec8709772e3fcec0e>@@$$QEAV<lambda_9d71df4d7cf3f480f8d633942495c3b0>@@@Z@4HA 000000018001ac60     libucrt:onexit.obj
 0001:00019c60       $unwind$?fin$0@?0???$?RV<lambda_fb3a7dec4e47f37f22dae91bb15c9095>@@AEAV<lambda_698284760c8add0bfb0756c19673e34b>@@V<lambda_dfb8eca1e75fef3034a8fb18dd509707>@@@?$__crt_seh_guarded_call@X@@QEAAX$$QEAV<lambda_fb3a7dec4e47f37f22dae91bb15c9095>@@AEAV<lambda_698284760c8add0bfb0756c19673e34b>@@$$QEAV<lambda_dfb8eca1e75fef3034a8fb18dd509707>@@@Z@4HA 000000018001ac60     libucrt:per_thread_data.obj
 0001:00019c60       $unwind$_write$fin$0       000000018001ac60     libucrt:write.obj
 0001:00019c60       $unwind$?fin$0@?0???$?RV<lambda_b8c45f8f788dd370798f47cfe8ac3a86>@@AEAV<lambda_4e60a939b0d047cfe11ddc22648dfba9>@@V<lambda_332c3edc96d0294ec56c57d38c1cdfd5>@@@?$__crt_seh_guarded_call@H@@QEAAH$$QEAV<lambda_b8c45f8f788dd370798f47cfe8ac3a86>@@AEAV<lambda_4e60a939b0d047cfe11ddc22648dfba9>@@$$QEAV<lambda_332c3edc96d0294ec56c57d38c1cdfd5>@@@Z@4HA 000000018001ac60     libucrt:onexit.obj
 0001:00019c60       $unwind$?fin$0@?0???$?RV<lambda_c36588078e9f5dfd39652860aa6b3aaf>@@AEAV<lambda_ec61778202f4f5fc7e7711acc23c3bca>@@V<lambda_dc9d2797ccde5d239b4a0efae8ebd7db>@@@?$__crt_seh_guarded_call@P6AXH@Z@@QEAAP6AXH@Z$$QEAV<lambda_c36588078e9f5dfd39652860aa6b3aaf>@@AEAV<lambda_ec61778202f4f5fc7e7711acc23c3bca>@@$$QEAV<lambda_dc9d2797ccde5d239b4a0efae8ebd7db>@@@Z@4HA 000000018001ac60     libucrt:signal.obj
 0001:00019c60       $unwind$?fin$0@?0???$?RV<lambda_bfedae4ebbf01fab1bb6dcc6a9e276e0>@@AEAV<lambda_2fe9b910cf3cbf4a0ab98a02ba45b3ec>@@V<lambda_237c231691f317818eb88cc1d5d642d6>@@@?$__crt_seh_guarded_call@H@@QEAAH$$QEAV<lambda_bfedae4ebbf01fab1bb6dcc6a9e276e0>@@AEAV<lambda_2fe9b910cf3cbf4a0ab98a02ba45b3ec>@@$$QEAV<lambda_237c231691f317818eb88cc1d5d642d6>@@@Z@4HA 000000018001ac60     libucrt:close.obj
 0001:00019c60       $unwind$fclose$fin$0       000000018001ac60     libucrt:fclose.obj
 0001:00019c60       $unwind$?fin$0@?0???$?RV<lambda_72d1df2b273a38828b1ce30cbf4cdab5>@@AEAV<lambda_876a65b173b8412d3a47c70a915b0cf4>@@V<lambda_41932305e351933ebe8f8be3ed8bb5dc>@@@?$__crt_seh_guarded_call@X@@QEAAX$$QEAV<lambda_72d1df2b273a38828b1ce30cbf4cdab5>@@AEAV<lambda_876a65b173b8412d3a47c70a915b0cf4>@@$$QEAV<lambda_41932305e351933ebe8f8be3ed8bb5dc>@@@Z@4HA 000000018001ac60     libucrt:per_thread_data.obj
 0001:00019c60       $unwind$?fin$1@?0??common_exit@@YAXHW4_crt_exit_cleanup_mode@@W4_crt_exit_return_mode@@@Z@4HA 000000018001ac60     libucrt:exit.obj
 0001:00019c60       $unwind$_fcloseall$fin$0   000000018001ac60     libucrt:closeall.obj
 0001:00019c60       $unwind$?fin$0@?0???$?RV<lambda_99476a1ad63dd22509b5d3e65b0ffc95>@@AEAV<lambda_ad1ced32f4ac17aa236e5ef05d6b3b7c>@@V<lambda_f7424dd8d45958661754dc4f2697e9c3>@@@?$__crt_seh_guarded_call@X@@QEAAX$$QEAV<lambda_99476a1ad63dd22509b5d3e65b0ffc95>@@AEAV<lambda_ad1ced32f4ac17aa236e5ef05d6b3b7c>@@$$QEAV<lambda_f7424dd8d45958661754dc4f2697e9c3>@@@Z@4HA 000000018001ac60     libucrt:mbctype.obj
 0001:00019c60       $unwind$?fin$0@?0??dllmain_crt_process_detach@@YAH_N@Z@4HA 000000018001ac60     LIBCMT:dll_dllmain.obj
 0001:00019c60       $unwind$raise$fin$0        000000018001ac60     libucrt:signal.obj
 0001:00019c60       $unwind$?fin$0@?0???$?RV<lambda_46352004c1216016012b18bd6f87e700>@@AEAV<lambda_3bd07e1a1191394380780325891bf33f>@@V<lambda_334532d3f185bcaa59b5be82d7d22bff>@@@?$__crt_seh_guarded_call@X@@QEAAX$$QEAV<lambda_46352004c1216016012b18bd6f87e700>@@AEAV<lambda_3bd07e1a1191394380780325891bf33f>@@$$QEAV<lambda_334532d3f185bcaa59b5be82d7d22bff>@@@Z@4HA 000000018001ac60     libucrt:per_thread_data.obj
 0001:00019c68       $unwind$common_flush_all   000000018001ac68     libucrt:fflush.obj
 0001:00019ca4       $unwind$?_TlgWrite@__vcrt_trace_logging_provider@@YAJPEBU_TlgProvider_t@1@PEFBXPEBU_GUID@@2IPEAU_EVENT_DATA_DESCRIPTOR@@@Z 000000018001aca4     libvcruntime:telemetry.obj
 0001:00019ca4       $unwind$?getSystemCP@@YAHH@Z 000000018001aca4     libucrt:mbctype.obj
 0001:00019ca4       $unwind$_isleadbyte_l      000000018001aca4     libucrt:_wctype.obj
 0001:00019cac       $unwind$_fcloseall         000000018001acac     libucrt:closeall.obj
 0001:00019cd0       $unwind$__acrt_locale_free_monetary 000000018001acd0     libucrt:initmon.obj
 0001:00019cd8       $unwind$__acrt_locale_free_time 000000018001acd8     libucrt:inittime.obj
 0001:00019ce8       $unwind$_commit            000000018001ace8     libucrt:commit.obj
 0001:00019ce8       $unwind$_close             000000018001ace8     libucrt:close.obj
 0001:00019cf0       $unwind$??$?RV<lambda_b521505b218e5242e90febf6bfebc422>@@AEAV<lambda_6978c1fb23f02e42e1d9e99668cc68aa>@@V<lambda_314360699dd331753a4119843814e9a7>@@@?$__crt_seh_guarded_call@H@@QEAAH$$QEAV<lambda_b521505b218e5242e90febf6bfebc422>@@AEAV<lambda_6978c1fb23f02e42e1d9e99668cc68aa>@@$$QEAV<lambda_314360699dd331753a4119843814e9a7>@@@Z 000000018001acf0     libucrt:commit.obj
 0001:00019d14       $unwind$_write             000000018001ad14     libucrt:write.obj
 0001:00019d44       $unwind$_write_nolock      000000018001ad44     libucrt:write.obj
 0001:00019d5c       $unwind$?write_double_translated_ansi_nolock@@YA?AUwrite_result@?A0x9c548279@@HQEBDI@Z 000000018001ad5c     libucrt:write.obj
 0001:00019d7c       $unwind$?write_text_ansi_nolock@@YA?AUwrite_result@?A0x9c548279@@HQEBDI@Z 000000018001ad7c     libucrt:write.obj
 0001:00019d7c       $unwind$?write_text_utf16le_nolock@@YA?AUwrite_result@?A0x9c548279@@HQEBDI@Z 000000018001ad7c     libucrt:write.obj
 0001:00019d9c       $unwind$?write_text_utf8_nolock@@YA?AUwrite_result@?A0x9c548279@@HQEBDI@Z 000000018001ad9c     libucrt:write.obj
 0001:00019dc0       $xdatasym                  000000018001adc0     libucrt:log10.obj
 0001:00019dcc       $unwind$fclose             000000018001adcc     libucrt:fclose.obj
 0001:00019df0       $unwind$_call_matherr      000000018001adf0     libucrt:libm_error.obj
 0001:00019df8       $unwind$_handle_error      000000018001adf8     libucrt:libm_error.obj
 0001:00019e18       $unwind$__acrt_initialize_fma3 000000018001ae18     libucrt:fma3_available.obj
 0001:00019e20       $unwind$_log_special_common 000000018001ae20     libucrt:log_special.obj
 0001:00019e2c       $unwind$??$?RV<lambda_bfedae4ebbf01fab1bb6dcc6a9e276e0>@@AEAV<lambda_2fe9b910cf3cbf4a0ab98a02ba45b3ec>@@V<lambda_237c231691f317818eb88cc1d5d642d6>@@@?$__crt_seh_guarded_call@H@@QEAAH$$QEAV<lambda_bfedae4ebbf01fab1bb6dcc6a9e276e0>@@AEAV<lambda_2fe9b910cf3cbf4a0ab98a02ba45b3ec>@@$$QEAV<lambda_237c231691f317818eb88cc1d5d642d6>@@@Z 000000018001ae2c     libucrt:close.obj
 0001:00019e50       $xdatasym                  000000018001ae50     libucrt:fpsr.obj
 0001:00019e58       $unwind$?_com_raise_error@@YAXJPEAUIErrorInfo@@@Z 000000018001ae58     comsuppw:comraise.obj
 0001:00019e58       $unwind$?__scrt_throw_std_bad_alloc@@YAXXZ 000000018001ae58     LIBCMT:throw_bad_alloc.obj
 0001:00019e58       $unwind$__dcrt_lowio_initialize_console_output 000000018001ae58     libucrt:initcon.obj
 0001:00019e58       $unwind$?__scrt_throw_std_bad_array_new_length@@YAXXZ 000000018001ae58     LIBCMT:throw_bad_alloc.obj
 0001:00019e58       $unwind$_raise_exc         000000018001ae58     libucrt:fpexcept.obj
 0001:00019e60       $unwind$_raise_exc_ex      000000018001ae60     libucrt:fpexcept.obj
 0001:00019e74       $unwind$_ctrlfp            000000018001ae74     libucrt:fpctrl.obj
 0001:00019ea0       $xdatasym                  000000018001aea0     LIBCMT:_amdsecgs_.obj
 0001:00019ea4       $unwind$_IsNonwritableInCurrentImage 000000018001aea4     LIBCMT:pesect.obj
 0001:00019ec8       $unwind$__GSHandlerCheckCommon 000000018001aec8     LIBCMT:_gshandler_.obj
 0001:00019ed0       $unwind$__report_securityfailure 000000018001aed0     LIBCMT:gs_report.obj
 0001:00019ed8       $unwind$_putwch_nolock     000000018001aed8     libucrt:putwch.obj
 0001:00019ed8       $unwind$__report_gsfailure 000000018001aed8     LIBCMT:gs_report.obj
 0001:00019ee0       $unwind$capture_current_context 000000018001aee0     LIBCMT:gs_report.obj
 0001:00019eec       $unwind$capture_previous_context 000000018001aeec     LIBCMT:gs_report.obj
 0001:00019ef8       $xdatasym                  000000018001aef8     libvcruntime:memcmp.obj
 0001:0001a050       .edata                     000000018001b050     EMenu.exp
 0001:0001a078       rgpv                       000000018001b078     EMenu.exp
 0001:0001a090       rgszName                   000000018001b090     EMenu.exp
 0001:0001a0a8       rgwOrd                     000000018001b0a8     EMenu.exp
 0001:0001a0b4       szName                     000000018001b0b4     EMenu.exp
 0001:0001a0be       $N00001                    000000018001b0be     EMenu.exp
 0001:0001a0c9       $N00002                    000000018001b0c9     EMenu.exp
 0001:0001a0d2       $N00003                    000000018001b0d2     EMenu.exp
 0001:0001a0e1       $N00004                    000000018001b0e1     EMenu.exp
 0001:0001a0f0       $N00005                    000000018001b0f0     EMenu.exp
 0001:0001a0f6       $N00006                    000000018001b0f6     EMenu.exp
 0002:00000080       ?_Tlg_Microsoft_CRTProviderProv@@3U_TlgProvider_t@__vcrt_trace_logging_provider@@A 000000018001c080     libvcruntime:telemetry.obj
 0002:000000d0       ?__vcrt_flsindex@@3KA      000000018001c0d0     libvcruntime:per_thread_data.obj
 0002:000000d8       __acrt_flsindex            000000018001c0d8     libucrt:per_thread_data.obj
 0002:000000dc       errno_no_memory            000000018001c0dc     libucrt:errno.obj
 0002:000000e0       doserrno_no_memory         000000018001c0e0     libucrt:errno.obj
 0002:00000320       __rgctypeflag              000000018001c320     libucrt:mbctype.obj
 0002:00000330       __rgcode_page_info         000000018001c330     libucrt:mbctype.obj
 0002:00000960       ?dazSupported@?1??_ctrlfp@@9@9 000000018001c960     libucrt:fpctrl.obj
 0002:00000ac0       ?PluginMenuStrings@?1??GetPluginInfo@CPlugin@@QEAAXPEAUPluginInfo@@@Z@4PAPEB_WA 000000018001cac0     Plugin.obj
 0002:00000ac8       ?pThis@?1??CfgDlgProcStatic@CPlugin@@KA_JPEAX_J10@Z@4PEAV2@EA 000000018001cac8     Plugin.obj
 0002:00000ad0       ?szFNameTmp@?BH@??GetFilesFromPanel@CPlugin@@IEAA_NPEAPEAPEB_WPEAI1PEAVauto_sz@@@Z@4PA_WA 000000018001cad0     Plugin.obj
 0002:000012d0       ?__proc_attached@@3HA      000000018001d2d0     LIBCMT:dll_dllmain.obj
 0002:000012e8       ?module_local_atexit_table@@3U_onexit_table_t@@A 000000018001d2e8     LIBCMT:utility.obj
 0002:00001300       ?module_local_at_quick_exit_table@@3U_onexit_table_t@@A 000000018001d300     LIBCMT:utility.obj
 0002:00001318       ?is_initialized_as_dll@@3_NA 000000018001d318     LIBCMT:utility.obj
 0002:00001350       ?module_handles@@3PAPEAUHINSTANCE__@@A 000000018001d350     libvcruntime:winapi_downlevel.obj
 0002:00001370       ?encoded_function_pointers@@3PAPEAXA 000000018001d370     libvcruntime:winapi_downlevel.obj
 0002:000013c0       ?__vcrt_startup_thread_ptd@@3U__vcrt_ptd@@A 000000018001d3c0     libvcruntime:per_thread_data.obj
 0002:00001438       __vcrt_lock_table          000000018001d438     libvcruntime:locks.obj
 0002:00001460       __vcrt_locks_initialized   000000018001d460     libvcruntime:locks.obj
 0002:000014b8       ?heap@@3V_HeapManager@@A   000000018001d4b8     libvcruntime:undname.obj
 0002:000014e0       __acrt_new_handler         000000018001d4e0     libucrt:new_handler.obj
 0002:000014e8       c_termination_complete     000000018001d4e8     libucrt:exit.obj
 0002:000014f0       thread_local_exit_callback_func 000000018001d4f0     libucrt:exit.obj
 0002:000014f8       ?c_exit_complete@?5??common_exit@@YAXHW4_crt_exit_cleanup_mode@@W4_crt_exit_return_mode@@@Z@4_NA 000000018001d4f8     libucrt:exit.obj
 0002:00001500       ?program_name@?5???$common_configure_argv@D@@YAHW4_crt_argv_mode@@@Z@4PADA 000000018001d500     libucrt:argv_parsing.obj
 0002:00001660       __acrt_lock_table          000000018001d660     libucrt:locks.obj
 0002:00001868       __acrt_locks_initialized   000000018001d868     libucrt:locks.obj
 0002:00001870       module_handles             000000018001d870     libucrt:winapi_thunks.obj
 0002:00001910       encoded_function_pointers  000000018001d910     libucrt:winapi_thunks.obj
 0002:00001a10       ?state_cache@?1??__acrt_is_packaged_app@@9@4JA 000000018001da10     libucrt:winapi_thunks.obj
 0002:00001a18       __acrt_invalid_parameter_handler 000000018001da18     libucrt:invalid_parameter.obj
 0002:00001a34       fSystemSet                 000000018001da34     libucrt:mbctype.obj
 0002:00001a40       ?initialized@?1??__acrt_initialize_multibyte@@9@4_NA 000000018001da40     libucrt:mbctype.obj
 0002:00001e88       ctrlc_action               000000018001de88     libucrt:signal.obj
 0002:00001e90       ctrlbreak_action           000000018001de90     libucrt:signal.obj
 0002:00001e98       abort_action               000000018001de98     libucrt:signal.obj
 0002:00001ea0       term_action                000000018001dea0     libucrt:signal.obj
 0002:00001ea8       user_matherr               000000018001dea8     libucrt:matherr.obj
 0002:00001ec8       __acrt_global_new_mode     000000018001dec8     libucrt:new_mode.obj
 0002:00001eec       __acrt_app_type            000000018001deec     libucrt:report_runtime_error.obj
 0002:00001f00       GS_ExceptionRecord         000000018001df00     LIBCMT:gs_report.obj
 0002:00001fa0       GS_ContextRecord           000000018001dfa0     LIBCMT:gs_report.obj
 0003:00000000       $pdata$?TraceLoggingRegister@__vcrt_trace_logging_provider@@YAJPEBU_TlgProvider_t@1@PEBU_GUID@@P6AX1KE_K2PEAU_EVENT_FILTER_DESCRIPTOR@@PEAX@Z4@Z 000000018001f000     libvcruntime:telemetry.obj
 0003:0000000c       $pdata$?_TlgEnableCallback@__vcrt_trace_logging_provider@@YAXPEBU_GUID@@KE_K1PEAU_EVENT_FILTER_DESCRIPTOR@@PEAX@Z 000000018001f00c     libvcruntime:telemetry.obj
 0003:00000018       $pdata$?_TlgWrite@__vcrt_trace_logging_provider@@YAJPEBU_TlgProvider_t@1@PEFBXPEBU_GUID@@2IPEAU_EVENT_DATA_DESCRIPTOR@@@Z 000000018001f018     libvcruntime:telemetry.obj
 0003:00000030       $pdata$ConfigureW          000000018001f030     EMenu.obj
 0003:0000003c       $pdata$ExitFARW            000000018001f03c     EMenu.obj
 0003:00000048       $pdata$GetGlobalInfoW      000000018001f048     EMenu.obj
 0003:00000054       $pdata$SetStartupInfoW     000000018001f054     EMenu.obj
 0003:00000060       $pdata$??0auto_sz@@QEAA@AEBU_STRRET@@PEFBU_ITEMIDLIST@@@Z 000000018001f060     auto_sz.obj
 0003:0000006c       $pdata$1$??0auto_sz@@QEAA@AEBU_STRRET@@PEFBU_ITEMIDLIST@@@Z 000000018001f06c     auto_sz.obj
 0003:00000078       $pdata$2$??0auto_sz@@QEAA@AEBU_STRRET@@PEFBU_ITEMIDLIST@@@Z 000000018001f078     auto_sz.obj
 0003:00000084       $pdata$??0auto_sz@@QEAA@PEB_W@Z 000000018001f084     auto_sz.obj
 0003:00000090       $pdata$??0auto_sz@@QEAA@PEB_W_K@Z 000000018001f090     auto_sz.obj
 0003:0000009c       $pdata$??1auto_sz@@QEAA@XZ 000000018001f09c     auto_sz.obj
 0003:000000a8       $pdata$??4auto_sz@@QEAAAEAV0@AEBV0@@Z 000000018001f0a8     auto_sz.obj
 0003:000000b4       $pdata$??4auto_sz@@QEAAAEAV0@PEB_W@Z 000000018001f0b4     auto_sz.obj
 0003:000000c0       $pdata$??9auto_sz@@QEAA_NPEB_W@Z 000000018001f0c0     auto_sz.obj
 0003:000000cc       $pdata$??Yauto_sz@@QEAAAEAV0@PEB_W@Z 000000018001f0cc     auto_sz.obj
 0003:000000d8       $pdata$?CompareExcluding@auto_sz@@QEAA_NPEB_W_W@Z 000000018001f0d8     auto_sz.obj
 0003:000000e4       $pdata$?Len@auto_sz@@QEBA_KXZ 000000018001f0e4     auto_sz.obj
 0003:000000f0       $pdata$?Realloc@auto_sz@@QEAAX_K@Z 000000018001f0f0     auto_sz.obj
 0003:000000fc       $pdata$?RemoveTrailing@auto_sz@@QEAAX_W@Z 000000018001f0fc     auto_sz.obj
 0003:00000108       $pdata$??0CFarMenu@@QEAA@PEB_WPEBU_GUID@@I@Z 000000018001f108     FarMenu.obj
 0003:00000114       $pdata$??1CFarMenu@@QEAA@XZ 000000018001f114     FarMenu.obj
 0003:00000120       $pdata$0$??1CFarMenu@@QEAA@XZ 000000018001f120     FarMenu.obj
 0003:0000012c       $pdata$1$??1CFarMenu@@QEAA@XZ 000000018001f12c     FarMenu.obj
 0003:00000138       $pdata$?AddArrows@CFarMenu@@IEAAXXZ 000000018001f138     FarMenu.obj
 0003:00000144       $pdata$3$?AddArrows@CFarMenu@@IEAAXXZ 000000018001f144     FarMenu.obj
 0003:00000150       $pdata$6$?AddArrows@CFarMenu@@IEAAXXZ 000000018001f150     FarMenu.obj
 0003:0000015c       $pdata$7$?AddArrows@CFarMenu@@IEAAXXZ 000000018001f15c     FarMenu.obj
 0003:00000168       $pdata$8$?AddArrows@CFarMenu@@IEAAXXZ 000000018001f168     FarMenu.obj
 0003:00000174       $pdata$?AddItem@CFarMenu@@QEAAIPEB_W_NW4ECheck@1@1@Z 000000018001f174     FarMenu.obj
 0003:00000180       $pdata$?AddSeparator@CFarMenu@@QEAAXXZ 000000018001f180     FarMenu.obj
 0003:0000018c       $pdata$1$?AddSeparator@CFarMenu@@QEAAXXZ 000000018001f18c     FarMenu.obj
 0003:00000198       $pdata$2$?AddSeparator@CFarMenu@@QEAAXXZ 000000018001f198     FarMenu.obj
 0003:000001a4       $pdata$?GetCursorXY@CFarMenu@@QEAAXPEAH0@Z 000000018001f1a4     FarMenu.obj
 0003:000001b0       $pdata$0$?GetCursorXY@CFarMenu@@QEAAXPEAH0@Z 000000018001f1b0     FarMenu.obj
 0003:000001bc       $pdata$1$?GetCursorXY@CFarMenu@@QEAAXPEAH0@Z 000000018001f1bc     FarMenu.obj
 0003:000001c8       $pdata$?InsertItem@CFarMenu@@QEAAIIPEB_W_NW4ECheck@1@1@Z 000000018001f1c8     FarMenu.obj
 0003:000001d4       $pdata$1$?InsertItem@CFarMenu@@QEAAIIPEB_W_NW4ECheck@1@1@Z 000000018001f1d4     FarMenu.obj
 0003:000001e0       $pdata$2$?InsertItem@CFarMenu@@QEAAIIPEB_W_NW4ECheck@1@1@Z 000000018001f1e0     FarMenu.obj
 0003:000001ec       $pdata$3$?InsertItem@CFarMenu@@QEAAIIPEB_W_NW4ECheck@1@1@Z 000000018001f1ec     FarMenu.obj
 0003:000001f8       $pdata$?Show@CFarMenu@@QEAAHPEB_WH_N@Z 000000018001f1f8     FarMenu.obj
 0003:00000204       $pdata$?MenuDlgProc@@YAHPEAUHWND__@@I_K_J@Z 000000018001f204     MenuDlg.obj
 0003:00000210       $pdata$?Cleanup@OleThread@@YAXXZ 000000018001f210     OleThread.obj
 0003:0000021c       $pdata$?EnsureThreadStarted@OleThread@@YA_NXZ 000000018001f21c     OleThread.obj
 0003:00000228       $pdata$0$?EnsureThreadStarted@OleThread@@YA_NXZ 000000018001f228     OleThread.obj
 0003:00000234       $pdata$1$?EnsureThreadStarted@OleThread@@YA_NXZ 000000018001f234     OleThread.obj
 0003:00000240       $pdata$?OpenPlugin@OleThread@@YA?AW4EDoMenu@CPlugin@@H_J@Z 000000018001f240     OleThread.obj
 0003:0000024c       $pdata$?ShowMenu@OleThread@@YAHAEAVCFarMenu@@PEB_WH_N@Z 000000018001f24c     OleThread.obj
 0003:00000258       $pdata$?Startup@OleThread@@YAXXZ 000000018001f258     OleThread.obj
 0003:00000264       $pdata$?ThreadProc@OleThread@@YAKPEAX@Z 000000018001f264     OleThread.obj
 0003:00000270       $pdata$0$?ThreadProc@OleThread@@YAKPEAX@Z 000000018001f270     OleThread.obj
 0003:0000027c       $pdata$1$?ThreadProc@OleThread@@YAKPEAX@Z 000000018001f27c     OleThread.obj
 0003:00000288       $pdata$??1CPidl@@QEAA@XZ   000000018001f288     Pidl.obj
 0003:00000294       $pdata$?GetArray@CPidl@@QEAAPEAPEFBU_ITEMIDLIST@@XZ 000000018001f294     Pidl.obj
 0003:00000294       $pdata$??ICPidl@@QEAAPEAPEFAU_ITEMIDLIST@@XZ 000000018001f294     Pidl.obj
 0003:000002a0       $pdata$?Add@CPidl@@QEAAXPEFAU_ITEMIDLIST@@@Z 000000018001f2a0     Pidl.obj
 0003:000002ac       $pdata$0$?Add@CPidl@@QEAAXPEFAU_ITEMIDLIST@@@Z 000000018001f2ac     Pidl.obj
 0003:000002b8       $pdata$1$?Add@CPidl@@QEAAXPEFAU_ITEMIDLIST@@@Z 000000018001f2b8     Pidl.obj
 0003:000002c4       $pdata$?EnsureSpace@CPidl@@QEAAXXZ 000000018001f2c4     Pidl.obj
 0003:000002d0       $pdata$0$?EnsureSpace@CPidl@@QEAAXXZ 000000018001f2d0     Pidl.obj
 0003:000002dc       $pdata$1$?EnsureSpace@CPidl@@QEAAXXZ 000000018001f2dc     Pidl.obj
 0003:000002e8       $pdata$?Insert@CPidl@@QEAAXIPEFAU_ITEMIDLIST@@@Z 000000018001f2e8     Pidl.obj
 0003:000002f4       $pdata$0$?Insert@CPidl@@QEAAXIPEFAU_ITEMIDLIST@@@Z 000000018001f2f4     Pidl.obj
 0003:00000300       $pdata$1$?Insert@CPidl@@QEAAXIPEFAU_ITEMIDLIST@@@Z 000000018001f300     Pidl.obj
 0003:0000030c       $pdata$??0CPlugin@@QEAA@PEBUPluginStartupInfo@@@Z 000000018001f30c     Plugin.obj
 0003:00000318       $pdata$??0PluginIntEditFieldBinding@@QEAA@AEBUPluginStartupInfo@@PEAPEAXHPEAHH@Z 000000018001f318     Plugin.obj
 0003:00000324       $pdata$??0PluginUIntEditFieldBinding@@QEAA@AEBUPluginStartupInfo@@PEAPEAXHPEAIH@Z 000000018001f324     Plugin.obj
 0003:00000330       $pdata$??1?$DialogBuilderBase@UFarDialogItem@@@@MEAA@XZ 000000018001f330     Plugin.obj
 0003:0000033c       $pdata$0$??1?$DialogBuilderBase@UFarDialogItem@@@@MEAA@XZ 000000018001f33c     Plugin.obj
 0003:00000348       $pdata$1$??1?$DialogBuilderBase@UFarDialogItem@@@@MEAA@XZ 000000018001f348     Plugin.obj
 0003:00000354       $pdata$??_G?$DialogBuilderBase@UFarDialogItem@@@@MEAAPEAXI@Z 000000018001f354     Plugin.obj
 0003:00000360       $pdata$??_G?$DialogItemBinding@UFarDialogItem@@@@UEAAPEAXI@Z 000000018001f360     Plugin.obj
 0003:0000036c       $pdata$??_GPluginCheckBoxBinding@@UEAAPEAXI@Z 000000018001f36c     Plugin.obj
 0003:00000378       $pdata$??_GPluginDialogBuilder@@UEAAPEAXI@Z 000000018001f378     Plugin.obj
 0003:00000384       $pdata$??_GPluginRadioButtonBinding@@UEAAPEAXI@Z 000000018001f384     Plugin.obj
 0003:00000390       $pdata$??_GPluginUIntEditFieldBinding@@UEAAPEAXI@Z 000000018001f390     Plugin.obj
 0003:00000390       $pdata$??_GPluginIntEditFieldBinding@@UEAAPEAXI@Z 000000018001f390     Plugin.obj
 0003:0000039c       $pdata$?AddButtons@?$DialogBuilderBase@UFarDialogItem@@@@QEAAXHPEBHHH@Z 000000018001f39c     Plugin.obj
 0003:000003a8       $pdata$3$?AddButtons@?$DialogBuilderBase@UFarDialogItem@@@@QEAAXHPEBHHH@Z 000000018001f3a8     Plugin.obj
 0003:000003b4       $pdata$4$?AddButtons@?$DialogBuilderBase@UFarDialogItem@@@@QEAAXHPEBHHH@Z 000000018001f3b4     Plugin.obj
 0003:000003c0       $pdata$?AddIntEditField@PluginDialogBuilder@@UEAAPEAUFarDialogItem@@PEAHH@Z 000000018001f3c0     Plugin.obj
 0003:000003cc       $pdata$?AddUIntEditField@PluginDialogBuilder@@UEAAPEAUFarDialogItem@@PEAIH@Z 000000018001f3cc     Plugin.obj
 0003:000003d8       $pdata$?CfgDlgProc@CPlugin@@IEAAXPEAX_J10@Z 000000018001f3d8     Plugin.obj
 0003:000003e4       $pdata$?CfgDlgProcStatic@CPlugin@@KA_JPEAX_J10@Z 000000018001f3e4     Plugin.obj
 0003:000003f0       $pdata$?Configure@CPlugin@@QEAAHXZ 000000018001f3f0     Plugin.obj
 0003:000003fc       $pdata$?CreateCheckBoxBinding@PluginDialogBuilder@@MEAAPEAU?$DialogItemBinding@UFarDialogItem@@@@PEAHH@Z 000000018001f3fc     Plugin.obj
 0003:00000408       $pdata$?CreateRadioButtonBinding@PluginDialogBuilder@@MEAAPEAU?$DialogItemBinding@UFarDialogItem@@@@PEAH@Z 000000018001f408     Plugin.obj
 0003:00000414       $pdata$?DoMenu@CPlugin@@IEAA?AW4EDoMenu@1@PEAUIShellFolder@@PEAPEFBU_ITEMIDLIST@@QEAPEB_WIIPEB_WW4EAutoItem@1@@Z 000000018001f414     Plugin.obj
 0003:00000420       $pdata$?DoMenu@CPlugin@@IEAA?AW4EDoMenu@1@PEA_WW4CallMode@1@@Z 000000018001f420     Plugin.obj
 0003:0000042c       $pdata$2$?DoMenu@CPlugin@@IEAA?AW4EDoMenu@1@PEA_WW4CallMode@1@@Z 000000018001f42c     Plugin.obj
 0003:00000438       $pdata$4$?DoMenu@CPlugin@@IEAA?AW4EDoMenu@1@PEA_WW4CallMode@1@@Z 000000018001f438     Plugin.obj
 0003:00000444       $pdata$5$?DoMenu@CPlugin@@IEAA?AW4EDoMenu@1@PEA_WW4CallMode@1@@Z 000000018001f444     Plugin.obj
 0003:00000450       $pdata$6$?DoMenu@CPlugin@@IEAA?AW4EDoMenu@1@PEA_WW4CallMode@1@@Z 000000018001f450     Plugin.obj
 0003:0000045c       $pdata$?DoShowDialog@PluginDialogBuilder@@MEAA_JXZ 000000018001f45c     Plugin.obj
 0003:00000468       $pdata$?GetAdditionalString@CPlugin@@IEAA_NPEAUIContextMenu@@IW4EAdditionalStr@1@PEAVauto_sz@@@Z 000000018001f468     Plugin.obj
 0003:00000474       $pdata$?GetFilesFromPanel@CPlugin@@IEAA_NPEAPEAPEB_WPEAI1PEAVauto_sz@@@Z 000000018001f474     Plugin.obj
 0003:00000480       $pdata$?GetFilesFromParams@CPlugin@@IEAA_NPEA_WPEAPEAPEB_WPEAI2PEAVauto_sz@@_N@Z 000000018001f480     Plugin.obj
 0003:0000048c       $pdata$?GetPluginInfo@CPlugin@@QEAAXPEAUPluginInfo@@@Z 000000018001f48c     Plugin.obj
 0003:00000498       $pdata$?InitDialogItem@PluginDialogBuilder@@MEAAXPEAUFarDialogItem@@PEB_W@Z 000000018001f498     Plugin.obj
 0003:000004a4       $pdata$?IsWindowsVersionOrGreater@@YA_NGGG@Z 000000018001f4a4     Plugin.obj
 0003:000004b0       $pdata$?ItemWidth@?$DialogBuilderBase@UFarDialogItem@@@@IEAA_JAEBUFarDialogItem@@@Z 000000018001f4b0     Plugin.obj
 0003:000004bc       $pdata$?MaxTextWidth@?$DialogBuilderBase@UFarDialogItem@@@@IEAA_JXZ 000000018001f4bc     Plugin.obj
 0003:000004c8       $pdata$1$?MaxTextWidth@?$DialogBuilderBase@UFarDialogItem@@@@IEAA_JXZ 000000018001f4c8     Plugin.obj
 0003:000004d4       $pdata$2$?MaxTextWidth@?$DialogBuilderBase@UFarDialogItem@@@@IEAA_JXZ 000000018001f4d4     Plugin.obj
 0003:000004e0       $pdata$?MenuForPanelOrCmdLine@CPlugin@@IEAA?AW4EDoMenu@1@PEA_WW4EAutoItem@1@@Z 000000018001f4e0     Plugin.obj
 0003:000004ec       $pdata$?OpenPlugin@CPlugin@@QEAAPEAXH_J@Z 000000018001f4ec     Plugin.obj
 0003:000004f8       $pdata$?OpenPluginBkg@CPlugin@@QEAA?AW4EDoMenu@1@H_J@Z 000000018001f4f8     Plugin.obj
 0003:00000504       $pdata$?ReadRegValues@CPlugin@@IEAAXXZ 000000018001f504     Plugin.obj
 0003:00000510       $pdata$?ReallocDialogItems@?$DialogBuilderBase@UFarDialogItem@@@@IEAAXXZ 000000018001f510     Plugin.obj
 0003:0000051c       $pdata$?SaveValue@PluginCheckBoxBinding@@UEAAXPEAUFarDialogItem@@H@Z 000000018001f51c     Plugin.obj
 0003:00000528       $pdata$?SaveValue@PluginIntEditFieldBinding@@UEAAXPEAUFarDialogItem@@H@Z 000000018001f528     Plugin.obj
 0003:00000534       $pdata$?SaveValue@PluginRadioButtonBinding@@UEAAXPEAUFarDialogItem@@H@Z 000000018001f534     Plugin.obj
 0003:00000540       $pdata$?SaveValue@PluginUIntEditFieldBinding@@UEAAXPEAUFarDialogItem@@H@Z 000000018001f540     Plugin.obj
 0003:0000054c       $pdata$?SaveValues@?$DialogBuilderBase@UFarDialogItem@@@@IEAAXXZ 000000018001f54c     Plugin.obj
 0003:00000558       $pdata$1$?SaveValues@?$DialogBuilderBase@UFarDialogItem@@@@IEAAXXZ 000000018001f558     Plugin.obj
 0003:00000564       $pdata$2$?SaveValues@?$DialogBuilderBase@UFarDialogItem@@@@IEAAXXZ 000000018001f564     Plugin.obj
 0003:00000570       $pdata$?SelectDrive@CPlugin@@IEAA?AW4EDoMenu@1@XZ 000000018001f570     Plugin.obj
 0003:0000057c       $pdata$0$?SelectDrive@CPlugin@@IEAA?AW4EDoMenu@1@XZ 000000018001f57c     Plugin.obj
 0003:00000588       $pdata$1$?SelectDrive@CPlugin@@IEAA?AW4EDoMenu@1@XZ 000000018001f588     Plugin.obj
 0003:00000594       $pdata$?ShowFolder@CPlugin@@IEAA_NPEAUIShellFolder@@PEFBU_ITEMIDLIST@@PEAHPEB_WPEAPEAUIDropTarget@@@Z 000000018001f594     Plugin.obj
 0003:000005a0       $pdata$?ShowGuiMenu@CPlugin@@IEAA_NPEAUHMENU__@@PEAUIContextMenu@@PEAUIContextMenu2@@PEAUIContextMenu3@@PEAH@Z 000000018001f5a0     Plugin.obj
 0003:000005ac       $pdata$?ShowTextMenu@CPlugin@@IEAA_NPEAUHMENU__@@PEAUIContextMenu@@PEAUIContextMenu2@@PEAUIContextMenu3@@PEAHPEB_WPEAUIShellFolder@@PEAPEFBU_ITEMIDLIST@@I@Z 000000018001f5ac     Plugin.obj
 0003:000005b8       $pdata$0$?ShowTextMenu@CPlugin@@IEAA_NPEAUHMENU__@@PEAUIContextMenu@@PEAUIContextMenu2@@PEAUIContextMenu3@@PEAHPEB_WPEAUIShellFolder@@PEAPEFBU_ITEMIDLIST@@I@Z 000000018001f5b8     Plugin.obj
 0003:000005c4       $pdata$2$?ShowTextMenu@CPlugin@@IEAA_NPEAUHMENU__@@PEAUIContextMenu@@PEAUIContextMenu2@@PEAUIContextMenu3@@PEAHPEB_WPEAUIShellFolder@@PEAPEFBU_ITEMIDLIST@@I@Z 000000018001f5c4     Plugin.obj
 0003:000005d0       $pdata$?UpdateBorderSize@?$DialogBuilderBase@UFarDialogItem@@@@IEAAXXZ 000000018001f5d0     Plugin.obj
 0003:000005dc       $pdata$??2@YAPEAX_K@Z      000000018001f5dc     LIBCMT:new_scalar.obj
 0003:000005e8       $pdata$?dllmain_crt_dispatch@@YAHQEAUHINSTANCE__@@KQEAX@Z 000000018001f5e8     LIBCMT:dll_dllmain.obj
 0003:000005f4       $pdata$?dllmain_crt_process_attach@@YAHQEAUHINSTANCE__@@QEAX@Z 000000018001f5f4     LIBCMT:dll_dllmain.obj
 0003:00000600       $pdata$?dllmain_crt_process_detach@@YAH_N@Z 000000018001f600     LIBCMT:dll_dllmain.obj
 0003:0000060c       $pdata$?dllmain_dispatch@@YAHQEAUHINSTANCE__@@KQEAX@Z 000000018001f60c     LIBCMT:dll_dllmain.obj
 0003:00000618       $pdata$?dllmain_raw@@YAHQEAUHINSTANCE__@@KQEAX@Z 000000018001f618     LIBCMT:dll_dllmain.obj
 0003:00000624       $pdata$_DllMainCRTStartup  000000018001f624     LIBCMT:dll_dllmain.obj
 0003:00000630       $pdata$??0bad_alloc@std@@QEAA@AEBV01@@Z 000000018001f630     LIBCMT:throw_bad_alloc.obj
 0003:0000063c       $pdata$??0bad_array_new_length@std@@QEAA@AEBV01@@Z 000000018001f63c     LIBCMT:throw_bad_alloc.obj
 0003:00000648       $pdata$??0exception@std@@QEAA@AEBV01@@Z 000000018001f648     LIBCMT:throw_bad_alloc.obj
 0003:00000654       $pdata$??_Gbad_alloc@std@@UEAAPEAXI@Z 000000018001f654     LIBCMT:throw_bad_alloc.obj
 0003:00000654       $pdata$??_Gexception@std@@UEAAPEAXI@Z 000000018001f654     LIBCMT:throw_bad_alloc.obj
 0003:00000654       $pdata$??_Gbad_array_new_length@std@@UEAAPEAXI@Z 000000018001f654     LIBCMT:throw_bad_alloc.obj
 0003:00000660       $pdata$?__scrt_throw_std_bad_alloc@@YAXXZ 000000018001f660     LIBCMT:throw_bad_alloc.obj
 0003:0000066c       $pdata$?__scrt_throw_std_bad_array_new_length@@YAXXZ 000000018001f66c     LIBCMT:throw_bad_alloc.obj
 0003:00000678       $pdata$__scrt_acquire_startup_lock 000000018001f678     LIBCMT:utility.obj
 0003:00000684       $pdata$__scrt_dllmain_after_initialize_c 000000018001f684     LIBCMT:utility.obj
 0003:00000690       $pdata$__scrt_dllmain_before_initialize_c 000000018001f690     LIBCMT:utility.obj
 0003:0000069c       $pdata$__scrt_dllmain_crt_thread_attach 000000018001f69c     LIBCMT:utility.obj
 0003:000006a8       $pdata$__scrt_dllmain_crt_thread_detach 000000018001f6a8     LIBCMT:utility.obj
 0003:000006b4       $pdata$__scrt_dllmain_exception_filter 000000018001f6b4     LIBCMT:utility.obj
 0003:000006c0       $pdata$__scrt_dllmain_uninitialize_c 000000018001f6c0     LIBCMT:utility.obj
 0003:000006cc       $pdata$__scrt_dllmain_uninitialize_critical 000000018001f6cc     LIBCMT:utility.obj
 0003:000006d8       $pdata$__scrt_initialize_crt 000000018001f6d8     LIBCMT:utility.obj
 0003:000006e4       $pdata$__scrt_initialize_onexit_tables 000000018001f6e4     LIBCMT:utility.obj
 0003:000006f0       $pdata$__scrt_is_nonwritable_in_current_image 000000018001f6f0     LIBCMT:utility.obj
 0003:000006fc       $pdata$__scrt_release_startup_lock 000000018001f6fc     LIBCMT:utility.obj
 0003:00000708       $pdata$__scrt_uninitialize_crt 000000018001f708     LIBCMT:utility.obj
 0003:00000714       $pdata$_onexit             000000018001f714     LIBCMT:utility.obj
 0003:00000720       $pdata$atexit              000000018001f720     LIBCMT:utility.obj
 0003:0000072c       $pdata$__security_init_cookie 000000018001f72c     LIBCMT:gs_support.obj
 0003:00000738       $pdata$__scrt_initialize_default_local_stdio_options 000000018001f738     LIBCMT:default_local_stdio_options.obj
 0003:00000744       $pdata$__scrt_fastfail     000000018001f744     LIBCMT:utility_desktop.obj
 0003:00000750       $pdata$_RTC_Initialize     000000018001f750     LIBCMT:_initsect_.obj
 0003:0000075c       $pdata$_RTC_Terminate      000000018001f75c     LIBCMT:_initsect_.obj
 0003:00000768       $pdata$??_Gtype_info@@UEAAPEAXI@Z 000000018001f768     LIBCMT:std_type_info_static.obj
 0003:00000774       $pdata$__isa_available_init 000000018001f774     LIBCMT:_cpu_disp_.obj
 0003:00000780       $pdata$?_com_issue_error@@YAXJ@Z 000000018001f780     comsuppw:comsupp.obj
 0003:0000078c       $pdata$??0_com_error@@QEAA@AEBV0@@Z 000000018001f78c     comsuppw:comraise.obj
 0003:00000798       $pdata$0$??0_com_error@@QEAA@AEBV0@@Z 000000018001f798     comsuppw:comraise.obj
 0003:000007a4       $pdata$1$??0_com_error@@QEAA@AEBV0@@Z 000000018001f7a4     comsuppw:comraise.obj
 0003:000007b0       $pdata$??0_com_error@@QEAA@JPEAUIErrorInfo@@_N@Z 000000018001f7b0     comsuppw:comraise.obj
 0003:000007bc       $pdata$0$??0_com_error@@QEAA@JPEAUIErrorInfo@@_N@Z 000000018001f7bc     comsuppw:comraise.obj
 0003:000007c8       $pdata$1$??0_com_error@@QEAA@JPEAUIErrorInfo@@_N@Z 000000018001f7c8     comsuppw:comraise.obj
 0003:000007d4       $pdata$??1_com_error@@UEAA@XZ 000000018001f7d4     comsuppw:comraise.obj
 0003:000007e0       $pdata$1$??1_com_error@@UEAA@XZ 000000018001f7e0     comsuppw:comraise.obj
 0003:000007ec       $pdata$2$??1_com_error@@UEAA@XZ 000000018001f7ec     comsuppw:comraise.obj
 0003:000007f8       $pdata$3$??1_com_error@@UEAA@XZ 000000018001f7f8     comsuppw:comraise.obj
 0003:00000804       $pdata$4$??1_com_error@@UEAA@XZ 000000018001f804     comsuppw:comraise.obj
 0003:00000810       $pdata$??_G_com_error@@UEAAPEAXI@Z 000000018001f810     comsuppw:comraise.obj
 0003:0000081c       $pdata$?_com_raise_error@@YAXJPEAUIErrorInfo@@@Z 000000018001f81c     comsuppw:comraise.obj
 0003:00000834       $pdata$__C_specific_handler 000000018001f834     libvcruntime:_chandler_.obj
 0003:0000084c       $pdata$__telemetry_main_invoke_trigger 000000018001f84c     libvcruntime:telemetry.obj
 0003:00000858       $pdata$__telemetry_main_return_trigger 000000018001f858     libvcruntime:telemetry.obj
 0003:00000864       $pdata$__vcrt_uninitialize_telemetry_provider 000000018001f864     libvcruntime:telemetry.obj
 0003:00000870       $pdata$__std_exception_copy 000000018001f870     libvcruntime:std_exception.obj
 0003:0000087c       $pdata$__std_exception_destroy 000000018001f87c     libvcruntime:std_exception.obj
 0003:00000888       $pdata$_CxxThrowException  000000018001f888     libvcruntime:throw.obj
 0003:00000894       $pdata$__vcrt_initialize   000000018001f894     libvcruntime:initialization.obj
 0003:000008a0       $pdata$__vcrt_thread_attach 000000018001f8a0     libvcruntime:initialization.obj
 0003:000008ac       $pdata$__vcrt_thread_detach 000000018001f8ac     libvcruntime:initialization.obj
 0003:000008b8       $pdata$__vcrt_uninitialize 000000018001f8b8     libvcruntime:initialization.obj
 0003:000008c4       $pdata$__vcrt_uninitialize_critical 000000018001f8c4     libvcruntime:initialization.obj
 0003:000008d0       $pdata$__std_type_info_destroy_list 000000018001f8d0     libvcruntime:std_type_info.obj
 0003:0000090c       $pdata$?try_get_function@@YAPEAXW4function_id@?A0x49c8dc86@@QEBDQEBW4module_id@2@2@Z 000000018001f90c     libvcruntime:winapi_downlevel.obj
 0003:00000918       $pdata$__vcrt_EventRegister 000000018001f918     libvcruntime:winapi_downlevel.obj
 0003:00000924       $pdata$__vcrt_EventSetInformation 000000018001f924     libvcruntime:winapi_downlevel.obj
 0003:00000930       $pdata$__vcrt_EventUnregister 000000018001f930     libvcruntime:winapi_downlevel.obj
 0003:0000093c       $pdata$__vcrt_EventWriteTransfer 000000018001f93c     libvcruntime:winapi_downlevel.obj
 0003:00000948       $pdata$__vcrt_FlsAlloc     000000018001f948     libvcruntime:winapi_downlevel.obj
 0003:00000954       $pdata$__vcrt_FlsFree      000000018001f954     libvcruntime:winapi_downlevel.obj
 0003:00000960       $pdata$__vcrt_FlsGetValue  000000018001f960     libvcruntime:winapi_downlevel.obj
 0003:0000096c       $pdata$__vcrt_FlsSetValue  000000018001f96c     libvcruntime:winapi_downlevel.obj
 0003:00000978       $pdata$__vcrt_InitializeCriticalSectionEx 000000018001f978     libvcruntime:winapi_downlevel.obj
 0003:00000984       $pdata$__vcrt_initialize_winapi_thunks 000000018001f984     libvcruntime:winapi_downlevel.obj
 0003:00000990       $pdata$__vcrt_uninitialize_winapi_thunks 000000018001f990     libvcruntime:winapi_downlevel.obj
 0003:0000099c       $pdata$__vcrt_freefls      000000018001f99c     libvcruntime:per_thread_data.obj
 0003:000009a8       $pdata$__vcrt_freeptd      000000018001f9a8     libvcruntime:per_thread_data.obj
 0003:000009b4       $pdata$__vcrt_getptd_noexit 000000018001f9b4     libvcruntime:per_thread_data.obj
 0003:000009c0       $pdata$__vcrt_initialize_ptd 000000018001f9c0     libvcruntime:per_thread_data.obj
 0003:000009cc       $pdata$__vcrt_uninitialize_ptd 000000018001f9cc     libvcruntime:per_thread_data.obj
 0003:000009d8       $pdata$__vcrt_initialize_locks 000000018001f9d8     libvcruntime:locks.obj
 0003:000009e4       $pdata$__vcrt_uninitialize_locks 000000018001f9e4     libvcruntime:locks.obj
 0003:000009f0       $pdata$_callnewh           000000018001f9f0     libucrt:new_handler.obj
 0003:000009fc       $pdata$_query_new_handler  000000018001f9fc     libucrt:new_handler.obj
 0003:00000a08       $pdata$_initterm           000000018001fa08     libucrt:initterm.obj
 0003:00000a14       $pdata$_initterm_e         000000018001fa14     libucrt:initterm.obj
 0003:00000a20       $pdata$_seh_filter_exe     000000018001fa20     libucrt:exception_filter.obj
 0003:00000a2c       $pdata$?common_exit@@YAXHW4_crt_exit_cleanup_mode@@W4_crt_exit_return_mode@@@Z 000000018001fa2c     libucrt:exit.obj
 0003:00000a38       $pdata$?exit_or_terminate_process@@YAXI@Z 000000018001fa38     libucrt:exit.obj
 0003:00000a44       $pdata$?try_cor_exit_process@@YAXI@Z 000000018001fa44     libucrt:exit.obj
 0003:00000a50       $pdata$??$parse_command_line@D@@YAXPEADPEAPEAD0PEA_K2@Z 000000018001fa50     libucrt:argv_parsing.obj
 0003:00000a5c       $pdata$__acrt_allocate_buffer_for_argv 000000018001fa5c     libucrt:argv_parsing.obj
 0003:00000a68       $pdata$_configure_narrow_argv 000000018001fa68     libucrt:argv_parsing.obj
 0003:00000a74       $pdata$??$common_initialize_environment_nolock@D@@YAHXZ 000000018001fa74     libucrt:environment_initialization.obj
 0003:00000a80       $pdata$??$create_environment@D@@YAQEAPEADQEAD@Z 000000018001fa80     libucrt:environment_initialization.obj
 0003:00000a8c       $pdata$??$free_environment@D@@YAXQEAPEAD@Z 000000018001fa8c     libucrt:environment_initialization.obj
 0003:00000a8c       $pdata$??$free_environment@_W@@YAXQEAPEA_W@Z 000000018001fa8c     libucrt:environment_initialization.obj
 0003:00000a98       $pdata$??$uninitialize_environment_internal@D@@YAXAEAPEAPEAD@Z 000000018001fa98     libucrt:environment_initialization.obj
 0003:00000aa4       $pdata$??$uninitialize_environment_internal@_W@@YAXAEAPEAPEA_W@Z 000000018001faa4     libucrt:environment_initialization.obj
 0003:00000ab0       $pdata$__dcrt_uninitialize_environments_nolock 000000018001fab0     libucrt:environment_initialization.obj
 0003:00000abc       $pdata$??$?RV<lambda_b8c45f8f788dd370798f47cfe8ac3a86>@@AEAV<lambda_4e60a939b0d047cfe11ddc22648dfba9>@@V<lambda_332c3edc96d0294ec56c57d38c1cdfd5>@@@?$__crt_seh_guarded_call@H@@QEAAH$$QEAV<lambda_b8c45f8f788dd370798f47cfe8ac3a86>@@AEAV<lambda_4e60a939b0d047cfe11ddc22648dfba9>@@$$QEAV<lambda_332c3edc96d0294ec56c57d38c1cdfd5>@@@Z 000000018001fabc     libucrt:onexit.obj
 0003:00000ac8       $pdata$??$?RV<lambda_e24bbb7b643b32fcea6fa61b31d4c984>@@AEAV<lambda_275893d493268fdec8709772e3fcec0e>@@V<lambda_9d71df4d7cf3f480f8d633942495c3b0>@@@?$__crt_seh_guarded_call@H@@QEAAH$$QEAV<lambda_e24bbb7b643b32fcea6fa61b31d4c984>@@AEAV<lambda_275893d493268fdec8709772e3fcec0e>@@$$QEAV<lambda_9d71df4d7cf3f480f8d633942495c3b0>@@@Z 000000018001fac8     libucrt:onexit.obj
 0003:00000ad4       $pdata$??R<lambda_4e60a939b0d047cfe11ddc22648dfba9>@@QEBAHXZ 000000018001fad4     libucrt:onexit.obj
 0003:00000ae0       $pdata$_execute_onexit_table 000000018001fae0     libucrt:onexit.obj
 0003:00000aec       $pdata$_register_onexit_function 000000018001faec     libucrt:onexit.obj
 0003:00000af8       $pdata$initialize_c        000000018001faf8     libucrt:initialization.obj
 0003:00000b04       $pdata$uninitialize_environment 000000018001fb04     libucrt:initialization.obj
 0003:00000b10       $pdata$initialize_pointers 000000018001fb10     libucrt:initialization.obj
 0003:00000b1c       $pdata$uninitialize_allocated_memory 000000018001fb1c     libucrt:initialization.obj
 0003:00000b28       $pdata$__acrt_thread_attach 000000018001fb28     libucrt:initialization.obj
 0003:00000b34       $pdata$__acrt_thread_detach 000000018001fb34     libucrt:initialization.obj
 0003:00000b40       $pdata$__acrt_uninitialize_critical 000000018001fb40     libucrt:initialization.obj
 0003:00000b4c       $pdata$terminate           000000018001fb4c     libucrt:terminate.obj
 0003:00000b58       $pdata$strcpy_s            000000018001fb58     libucrt:strcpy_s.obj
 0003:00000b64       $pdata$_free_base          000000018001fb64     libucrt:free_base.obj
 0003:00000b70       $pdata$_malloc_base        000000018001fb70     libucrt:malloc_base.obj
 0003:00000b7c       $pdata$abort               000000018001fb7c     libucrt:abort.obj
 0003:00000b88       $pdata$_calloc_base        000000018001fb88     libucrt:calloc_base.obj
 0003:00000b94       $pdata$??0_LocaleUpdate@@QEAA@QEAU__crt_locale_pointers@@@Z 000000018001fb94     libucrt:output.obj
 0003:00000ba0       $pdata$__acrt_initialize_locks 000000018001fba0     libucrt:locks.obj
 0003:00000bac       $pdata$__acrt_uninitialize_locks 000000018001fbac     libucrt:locks.obj
 0003:00000bb8       $pdata$??$?RV<lambda_46352004c1216016012b18bd6f87e700>@@AEAV<lambda_3bd07e1a1191394380780325891bf33f>@@V<lambda_334532d3f185bcaa59b5be82d7d22bff>@@@?$__crt_seh_guarded_call@X@@QEAAX$$QEAV<lambda_46352004c1216016012b18bd6f87e700>@@AEAV<lambda_3bd07e1a1191394380780325891bf33f>@@$$QEAV<lambda_334532d3f185bcaa59b5be82d7d22bff>@@@Z 000000018001fbb8     libucrt:per_thread_data.obj
 0003:00000bc4       $pdata$??$?RV<lambda_5e887d1dcbef67a5eb4283622ba103bf>@@AEAV<lambda_4466841279450cc726390878d4a41900>@@V<lambda_341c25c0346d94847f1f3c463c57e077>@@@?$__crt_seh_guarded_call@X@@QEAAX$$QEAV<lambda_5e887d1dcbef67a5eb4283622ba103bf>@@AEAV<lambda_4466841279450cc726390878d4a41900>@@$$QEAV<lambda_341c25c0346d94847f1f3c463c57e077>@@@Z 000000018001fbc4     libucrt:per_thread_data.obj
 0003:00000bd0       $pdata$??$?RV<lambda_72d1df2b273a38828b1ce30cbf4cdab5>@@AEAV<lambda_876a65b173b8412d3a47c70a915b0cf4>@@V<lambda_41932305e351933ebe8f8be3ed8bb5dc>@@@?$__crt_seh_guarded_call@X@@QEAAX$$QEAV<lambda_72d1df2b273a38828b1ce30cbf4cdab5>@@AEAV<lambda_876a65b173b8412d3a47c70a915b0cf4>@@$$QEAV<lambda_41932305e351933ebe8f8be3ed8bb5dc>@@@Z 000000018001fbd0     libucrt:per_thread_data.obj
 0003:00000bdc       $pdata$??$?RV<lambda_fb3a7dec4e47f37f22dae91bb15c9095>@@AEAV<lambda_698284760c8add0bfb0756c19673e34b>@@V<lambda_dfb8eca1e75fef3034a8fb18dd509707>@@@?$__crt_seh_guarded_call@X@@QEAAX$$QEAV<lambda_fb3a7dec4e47f37f22dae91bb15c9095>@@AEAV<lambda_698284760c8add0bfb0756c19673e34b>@@$$QEAV<lambda_dfb8eca1e75fef3034a8fb18dd509707>@@@Z 000000018001fbdc     libucrt:per_thread_data.obj
 0003:00000be8       $pdata$?construct_ptd_array@@YAXQEAU__acrt_ptd@@@Z 000000018001fbe8     libucrt:per_thread_data.obj
 0003:00000bf4       $pdata$?destroy_fls@@YAXPEAX@Z 000000018001fbf4     libucrt:per_thread_data.obj
 0003:00000c00       $pdata$?destroy_ptd_array@@YAXQEAU__acrt_ptd@@@Z 000000018001fc00     libucrt:per_thread_data.obj
 0003:00000c0c       $pdata$?replace_current_thread_locale_nolock@@YAXQEAU__acrt_ptd@@QEAU__crt_locale_data@@@Z 000000018001fc0c     libucrt:per_thread_data.obj
 0003:00000c18       $pdata$__acrt_freeptd      000000018001fc18     libucrt:per_thread_data.obj
 0003:00000c24       $pdata$__acrt_getptd       000000018001fc24     libucrt:per_thread_data.obj
 0003:00000c30       $pdata$__acrt_getptd_noexit 000000018001fc30     libucrt:per_thread_data.obj
 0003:00000c3c       $pdata$__acrt_initialize_ptd 000000018001fc3c     libucrt:per_thread_data.obj
 0003:00000c48       $pdata$__acrt_uninitialize_ptd 000000018001fc48     libucrt:per_thread_data.obj
 0003:00000c54       $pdata$?try_get_function@@YAPEAXW4function_id@?A0x63058377@@QEBDQEBW4module_id@2@2@Z 000000018001fc54     libucrt:winapi_thunks.obj
 0003:00000c60       $pdata$__acrt_FlsAlloc     000000018001fc60     libucrt:winapi_thunks.obj
 0003:00000c6c       $pdata$__acrt_FlsFree      000000018001fc6c     libucrt:winapi_thunks.obj
 0003:00000c78       $pdata$__acrt_FlsGetValue  000000018001fc78     libucrt:winapi_thunks.obj
 0003:00000c84       $pdata$__acrt_FlsSetValue  000000018001fc84     libucrt:winapi_thunks.obj
 0003:00000c90       $pdata$__acrt_InitializeCriticalSectionEx 000000018001fc90     libucrt:winapi_thunks.obj
 0003:00000c9c       $pdata$__acrt_LCMapStringEx 000000018001fc9c     libucrt:winapi_thunks.obj
 0003:00000ca8       $pdata$__acrt_LocaleNameToLCID 000000018001fca8     libucrt:winapi_thunks.obj
 0003:00000cb4       $pdata$__acrt_initialize_winapi_thunks 000000018001fcb4     libucrt:winapi_thunks.obj
 0003:00000cc0       $pdata$__acrt_is_packaged_app 000000018001fcc0     libucrt:winapi_thunks.obj
 0003:00000ccc       $pdata$__acrt_uninitialize_winapi_thunks 000000018001fccc     libucrt:winapi_thunks.obj
 0003:00000cd8       $pdata$__acrt_call_reportfault 000000018001fcd8     libucrt:invalid_parameter.obj
 0003:00000ce4       $pdata$_invalid_parameter  000000018001fce4     libucrt:invalid_parameter.obj
 0003:00000cf0       $pdata$_invalid_parameter_noinfo 000000018001fcf0     libucrt:invalid_parameter.obj
 0003:00000cfc       $pdata$_invoke_watson      000000018001fcfc     libucrt:invalid_parameter.obj
 0003:00000d08       $pdata$__acrt_errno_map_os_error 000000018001fd08     libucrt:errno.obj
 0003:00000d14       $pdata$__doserrno          000000018001fd14     libucrt:errno.obj
 0003:00000d20       $pdata$_errno              000000018001fd20     libucrt:errno.obj
 0003:00000d2c       $pdata$??$common_expand_argv_wildcards@D@@YAHQEAPEADQEAPEAPEAD@Z 000000018001fd2c     libucrt:argv_wildcards.obj
 0003:00000d38       $pdata$??$copy_and_add_argument_to_buffer@D@@YAHQEBD0_KAEAV?$argument_list@D@?A0xca0879c4@@@Z 000000018001fd38     libucrt:argv_wildcards.obj
 0003:00000d44       $pdata$??$expand_argument_wildcards@D@@YAHQEAD0AEAV?$argument_list@D@?A0xca0879c4@@@Z 000000018001fd44     libucrt:argv_wildcards.obj
 0003:00000d50       $pdata$?expand_if_necessary@?$argument_list@D@?A0xca0879c4@@AEAAHXZ 000000018001fd50     libucrt:argv_wildcards.obj
 0003:00000d5c       $pdata$??$?RV<lambda_99476a1ad63dd22509b5d3e65b0ffc95>@@AEAV<lambda_ad1ced32f4ac17aa236e5ef05d6b3b7c>@@V<lambda_f7424dd8d45958661754dc4f2697e9c3>@@@?$__crt_seh_guarded_call@X@@QEAAX$$QEAV<lambda_99476a1ad63dd22509b5d3e65b0ffc95>@@AEAV<lambda_ad1ced32f4ac17aa236e5ef05d6b3b7c>@@$$QEAV<lambda_f7424dd8d45958661754dc4f2697e9c3>@@@Z 000000018001fd5c     libucrt:mbctype.obj
 0003:00000d68       $pdata$??R<lambda_ad1ced32f4ac17aa236e5ef05d6b3b7c>@@QEBAXXZ 000000018001fd68     libucrt:mbctype.obj
 0003:00000d74       $pdata$?getSystemCP@@YAHH@Z 000000018001fd74     libucrt:mbctype.obj
 0003:00000d80       $pdata$?setSBCS@@YAXPEAU__crt_multibyte_data@@@Z 000000018001fd80     libucrt:mbctype.obj
 0003:00000d8c       $pdata$?setSBUpLow@@YAXPEAU__crt_multibyte_data@@@Z 000000018001fd8c     libucrt:mbctype.obj
 0003:00000d98       $pdata$?setmbcp_internal@@YAHH_N@Z 000000018001fd98     libucrt:mbctype.obj
 0003:00000da4       $pdata$__acrt_initialize_multibyte 000000018001fda4     libucrt:mbctype.obj
 0003:00000db0       $pdata$__acrt_update_thread_multibyte_data 000000018001fdb0     libucrt:mbctype.obj
 0003:00000dbc       $pdata$_setmbcp_nolock     000000018001fdbc     libucrt:mbctype.obj
 0003:00000dc8       $pdata$?x_ismbbtype_l@@YAHPEAU__crt_locale_pointers@@IHH@Z 000000018001fdc8     libucrt:ismbbyte.obj
 0003:00000dd4       $pdata$__acrt_initialize_command_line 000000018001fdd4     libucrt:argv_data.obj
 0003:00000de0       $pdata$__dcrt_get_narrow_environment_from_os 000000018001fde0     libucrt:get_environment_from_os.obj
 0003:00000dec       $pdata$_recalloc_base      000000018001fdec     libucrt:recalloc.obj
 0003:00000df8       $pdata$__acrt_initialize_heap 000000018001fdf8     libucrt:heap_handle.obj
 0003:00000e04       $pdata$?initialize_inherited_file_handles_nolock@@YAXXZ 000000018001fe04     libucrt:ioinit.obj
 0003:00000e10       $pdata$?initialize_stdio_handles_nolock@@YAXXZ 000000018001fe10     libucrt:ioinit.obj
 0003:00000e1c       $pdata$__acrt_initialize_lowio 000000018001fe1c     libucrt:ioinit.obj
 0003:00000e28       $pdata$__acrt_uninitialize_lowio 000000018001fe28     libucrt:ioinit.obj
 0003:00000e34       $pdata$__acrt_execute_initializers 000000018001fe34     libucrt:shared_initialization.obj
 0003:00000e40       $pdata$__acrt_execute_uninitializers 000000018001fe40     libucrt:shared_initialization.obj
 0003:00000e4c       $pdata$??$?RV<lambda_c36588078e9f5dfd39652860aa6b3aaf>@@AEAV<lambda_ec61778202f4f5fc7e7711acc23c3bca>@@V<lambda_dc9d2797ccde5d239b4a0efae8ebd7db>@@@?$__crt_seh_guarded_call@P6AXH@Z@@QEAAP6AXH@Z$$QEAV<lambda_c36588078e9f5dfd39652860aa6b3aaf>@@AEAV<lambda_ec61778202f4f5fc7e7711acc23c3bca>@@$$QEAV<lambda_dc9d2797ccde5d239b4a0efae8ebd7db>@@@Z 000000018001fe4c     libucrt:signal.obj
 0003:00000e58       $pdata$__acrt_get_sigabrt_handler 000000018001fe58     libucrt:signal.obj
 0003:00000e64       $pdata$raise               000000018001fe64     libucrt:signal.obj
 0003:00000e70       $pdata$__acrt_invoke_user_matherr 000000018001fe70     libucrt:matherr.obj
 0003:00000e7c       $pdata$_mbtowc_l           000000018001fe7c     libucrt:mbtowc.obj
 0003:00000e88       $pdata$__acrt_update_locale_info 000000018001fe88     libucrt:locale_update.obj
 0003:00000e94       $pdata$__acrt_update_multibyte_info 000000018001fe94     libucrt:locale_update.obj
 0003:00000ea0       $pdata$_fileno             000000018001fea0     libucrt:fileno.obj
 0003:00000eac       $pdata$__acrt_initialize_stdio 000000018001feac     libucrt:_file.obj
 0003:00000eb8       $pdata$__acrt_uninitialize_stdio 000000018001feb8     libucrt:_file.obj
 0003:00000ec4       $pdata$__acrt_uninitialize_locale 000000018001fec4     libucrt:wsetlocale.obj
 0003:00000ed0       $pdata$__pctype_func       000000018001fed0     libucrt:ctype.obj
 0003:00000edc       $pdata$__acrt_free_locale  000000018001fedc     libucrt:locale_refcounting.obj
 0003:00000ee8       $pdata$__acrt_locale_free_lc_time_if_unreferenced 000000018001fee8     libucrt:locale_refcounting.obj
 0003:00000ef4       $pdata$__acrt_release_locale_ref 000000018001fef4     libucrt:locale_refcounting.obj
 0003:00000f00       $pdata$__acrt_update_thread_locale_data 000000018001ff00     libucrt:locale_refcounting.obj
 0003:00000f0c       $pdata$_updatetlocinfoEx_nolock 000000018001ff0c     libucrt:locale_refcounting.obj
 0003:00000f18       $pdata$?GetTableIndexFromLocaleName@@YAHPEB_W@Z 000000018001ff18     libucrt:lcidtoname_downlevel.obj
 0003:00000f24       $pdata$__acrt_DownlevelLocaleNameToLCID 000000018001ff24     libucrt:lcidtoname_downlevel.obj
 0003:00000f30       $pdata$?shortsort@@YAXPEAD0_KP6AHPEBX2@Z@Z 000000018001ff30     libucrt:qsort.obj
 0003:00000f3c       $pdata$2$?shortsort@@YAXPEAD0_KP6AHPEBX2@Z@Z 000000018001ff3c     libucrt:qsort.obj
 0003:00000f48       $pdata$3$?shortsort@@YAXPEAD0_KP6AHPEBX2@Z@Z 000000018001ff48     libucrt:qsort.obj
 0003:00000f54       $pdata$qsort               000000018001ff54     libucrt:qsort.obj
 0003:00000f60       $pdata$4$qsort             000000018001ff60     libucrt:qsort.obj
 0003:00000f6c       $pdata$5$qsort             000000018001ff6c     libucrt:qsort.obj
 0003:00000f78       $pdata$strncpy_s           000000018001ff78     libucrt:strncpy_s.obj
 0003:00000f84       $pdata$strpbrk             000000018001ff84     libucrt:strpbrk.obj
 0003:00000f90       $pdata$_mbsdec_l           000000018001ff90     libucrt:mbsdec.obj
 0003:00000f9c       $pdata$?initialize_multibyte@@YAHXZ 000000018001ff9c     libucrt:multibyte_initializer.obj
 0003:00000fa8       $pdata$__acrt_GetStringTypeA 000000018001ffa8     libucrt:getstringtypea.obj
 0003:00000fb4       $pdata$?__acrt_LCMapStringA_stat@@YAHPEAU__crt_locale_pointers@@PEB_WKPEBDHPEADHHH@Z 000000018001ffb4     libucrt:lcmapstringa.obj
 0003:00000fc0       $pdata$__acrt_LCMapStringA 000000018001ffc0     libucrt:lcmapstringa.obj
 0003:00000fcc       $pdata$_msize              000000018001ffcc     libucrt:msize.obj
 0003:00000fd8       $pdata$_realloc_base       000000018001ffd8     libucrt:realloc_base.obj
 0003:00000fe4       $pdata$__acrt_lowio_create_handle_array 000000018001ffe4     libucrt:osfinfo.obj
 0003:00000ff0       $pdata$__acrt_lowio_destroy_handle_array 000000018001fff0     libucrt:osfinfo.obj
 0003:00000ffc       $pdata$__acrt_lowio_ensure_fh_exists 000000018001fffc     libucrt:osfinfo.obj
 0003:00001008       $pdata$_free_osfhnd        0000000180020008     libucrt:osfinfo.obj
 0003:00001014       $pdata$_get_osfhandle      0000000180020014     libucrt:osfinfo.obj
 0003:00001020       $pdata$_isatty             0000000180020020     libucrt:isatty.obj
 0003:0000102c       $pdata$__acrt_stdio_flush_nolock 000000018002002c     libucrt:fflush.obj
 0003:00001038       $pdata$_fflush_nolock      0000000180020038     libucrt:fflush.obj
 0003:00001044       $pdata$common_flush_all    0000000180020044     libucrt:fflush.obj
 0003:00001050       $pdata$_isleadbyte_l       0000000180020050     libucrt:_wctype.obj
 0003:0000105c       $pdata$_fcloseall          000000018002005c     libucrt:closeall.obj
 0003:00001068       $pdata$__acrt_stdio_free_buffer_nolock 0000000180020068     libucrt:_freebuf.obj
 0003:00001074       $pdata$__acrt_locale_free_monetary 0000000180020074     libucrt:initmon.obj
 0003:00001080       $pdata$__acrt_locale_free_numeric 0000000180020080     libucrt:initnum.obj
 0003:0000108c       $pdata$?free_crt_array_internal@@YAXQEAPEBX_K@Z 000000018002008c     libucrt:inittime.obj
 0003:00001098       $pdata$__acrt_locale_free_time 0000000180020098     libucrt:inittime.obj
 0003:000010a4       $pdata$??$?RV<lambda_b521505b218e5242e90febf6bfebc422>@@AEAV<lambda_6978c1fb23f02e42e1d9e99668cc68aa>@@V<lambda_314360699dd331753a4119843814e9a7>@@@?$__crt_seh_guarded_call@H@@QEAAH$$QEAV<lambda_b521505b218e5242e90febf6bfebc422>@@AEAV<lambda_6978c1fb23f02e42e1d9e99668cc68aa>@@$$QEAV<lambda_314360699dd331753a4119843814e9a7>@@@Z 00000001800200a4     libucrt:commit.obj
 0003:000010b0       $pdata$_commit             00000001800200b0     libucrt:commit.obj
 0003:000010bc       $pdata$?write_double_translated_ansi_nolock@@YA?AUwrite_result@?A0x9c548279@@HQEBDI@Z 00000001800200bc     libucrt:write.obj
 0003:000010c8       $pdata$?write_text_ansi_nolock@@YA?AUwrite_result@?A0x9c548279@@HQEBDI@Z 00000001800200c8     libucrt:write.obj
 0003:000010d4       $pdata$?write_text_utf16le_nolock@@YA?AUwrite_result@?A0x9c548279@@HQEBDI@Z 00000001800200d4     libucrt:write.obj
 0003:000010e0       $pdata$?write_text_utf8_nolock@@YA?AUwrite_result@?A0x9c548279@@HQEBDI@Z 00000001800200e0     libucrt:write.obj
 0003:000010ec       $pdata$_write              00000001800200ec     libucrt:write.obj
 0003:000010f8       $pdata$_write_nolock       00000001800200f8     libucrt:write.obj
 0003:00001110       $pdata$??$common_lseek_nolock@_J@@YA_JH_JH@Z 0000000180020110     libucrt:lseek.obj
 0003:0000111c       $pdata$_fclose_nolock      000000018002011c     libucrt:fclose.obj
 0003:00001128       $pdata$fclose              0000000180020128     libucrt:fclose.obj
 0003:00001134       $pdata$_putwch_nolock      0000000180020134     libucrt:putwch.obj
 0003:00001140       $pdata$_call_matherr       0000000180020140     libucrt:libm_error.obj
 0003:0000114c       $pdata$_exception_enabled  000000018002014c     libucrt:libm_error.obj
 0003:00001158       $pdata$_handle_error       0000000180020158     libucrt:libm_error.obj
 0003:00001164       $pdata$__acrt_initialize_fma3 0000000180020164     libucrt:fma3_available.obj
 0003:00001170       $pdata$_log10_special      0000000180020170     libucrt:log_special.obj
 0003:0000117c       $pdata$_log_special_common 000000018002017c     libucrt:log_special.obj
 0003:00001188       $pdata$??$?RV<lambda_bfedae4ebbf01fab1bb6dcc6a9e276e0>@@AEAV<lambda_2fe9b910cf3cbf4a0ab98a02ba45b3ec>@@V<lambda_237c231691f317818eb88cc1d5d642d6>@@@?$__crt_seh_guarded_call@H@@QEAAH$$QEAV<lambda_bfedae4ebbf01fab1bb6dcc6a9e276e0>@@AEAV<lambda_2fe9b910cf3cbf4a0ab98a02ba45b3ec>@@$$QEAV<lambda_237c231691f317818eb88cc1d5d642d6>@@@Z 0000000180020188     libucrt:close.obj
 0003:00001194       $pdata$_close              0000000180020194     libucrt:close.obj
 0003:000011a0       $pdata$_close_nolock       00000001800201a0     libucrt:close.obj
 0003:000011ac       $pdata$__dcrt_lowio_initialize_console_output 00000001800201ac     libucrt:initcon.obj
 0003:000011b8       $pdata$__dcrt_terminate_console_output 00000001800201b8     libucrt:initcon.obj
 0003:000011d0       $pdata$_raise_exc          00000001800201d0     libucrt:fpexcept.obj
 0003:000011dc       $pdata$_raise_exc_ex       00000001800201dc     libucrt:fpexcept.obj
 0003:000011e8       $pdata$_set_errno_from_matherr 00000001800201e8     libucrt:fpexcept.obj
 0003:000011f4       $pdata$_clrfp              00000001800201f4     libucrt:fpctrl.obj
 0003:00001200       $pdata$_ctrlfp             0000000180020200     libucrt:fpctrl.obj
 0003:0000120c       $pdata$_set_statfp         000000018002020c     libucrt:fpctrl.obj
 0003:00001218       $pdata$_statfp             0000000180020218     libucrt:fpctrl.obj
 0003:00001230       $pdata$_IsNonwritableInCurrentImage 0000000180020230     LIBCMT:pesect.obj
 0003:0000123c       $pdata$__GSHandlerCheck    000000018002023c     LIBCMT:_gshandler_.obj
 0003:00001248       $pdata$__GSHandlerCheckCommon 0000000180020248     LIBCMT:_gshandler_.obj
 0003:00001254       $pdata$__raise_securityfailure 0000000180020254     LIBCMT:gs_report.obj
 0003:00001260       $pdata$__report_gsfailure  0000000180020260     LIBCMT:gs_report.obj
 0003:0000126c       $pdata$__report_rangecheckfailure 000000018002026c     LIBCMT:gs_report.obj
 0003:00001278       $pdata$__report_securityfailure 0000000180020278     LIBCMT:gs_report.obj
 0003:00001284       $pdata$capture_current_context 0000000180020284     LIBCMT:gs_report.obj
 0003:00001290       $pdata$capture_previous_context 0000000180020290     LIBCMT:gs_report.obj
 0003:000012b4       $pdata$?fin$0@?0??dllmain_crt_process_attach@@YAHQEAUHINSTANCE__@@QEAX@Z@4HA 00000001800202b4     LIBCMT:dll_dllmain.obj
 0003:000012c0       $pdata$?fin$0@?0??dllmain_crt_process_detach@@YAH_N@Z@4HA 00000001800202c0     LIBCMT:dll_dllmain.obj
 0003:000012cc       $pdata$?filt$0@?0??dllmain_dispatch@@YAHQEAUHINSTANCE__@@KQEAX@Z@4HA 00000001800202cc     LIBCMT:dll_dllmain.obj
 0003:000012d8       $pdata$__scrt_is_nonwritable_in_current_image$filt$0 00000001800202d8     LIBCMT:utility.obj
 0003:000012e4       $pdata$_query_new_handler$fin$0 00000001800202e4     libucrt:new_handler.obj
 0003:000012f0       $pdata$?filt$0@?0??common_exit@@YAXHW4_crt_exit_cleanup_mode@@W4_crt_exit_return_mode@@@Z@4HA 00000001800202f0     libucrt:exit.obj
 0003:000012fc       $pdata$?fin$1@?0??common_exit@@YAXHW4_crt_exit_cleanup_mode@@W4_crt_exit_return_mode@@@Z@4HA 00000001800202fc     libucrt:exit.obj
 0003:00001308       $pdata$?fin$0@?0???$?RV<lambda_e24bbb7b643b32fcea6fa61b31d4c984>@@AEAV<lambda_275893d493268fdec8709772e3fcec0e>@@V<lambda_9d71df4d7cf3f480f8d633942495c3b0>@@@?$__crt_seh_guarded_call@H@@QEAAH$$QEAV<lambda_e24bbb7b643b32fcea6fa61b31d4c984>@@AEAV<lambda_275893d493268fdec8709772e3fcec0e>@@$$QEAV<lambda_9d71df4d7cf3f480f8d633942495c3b0>@@@Z@4HA 0000000180020308     libucrt:onexit.obj
 0003:00001314       $pdata$?fin$0@?0???$?RV<lambda_72d1df2b273a38828b1ce30cbf4cdab5>@@AEAV<lambda_876a65b173b8412d3a47c70a915b0cf4>@@V<lambda_41932305e351933ebe8f8be3ed8bb5dc>@@@?$__crt_seh_guarded_call@X@@QEAAX$$QEAV<lambda_72d1df2b273a38828b1ce30cbf4cdab5>@@AEAV<lambda_876a65b173b8412d3a47c70a915b0cf4>@@$$QEAV<lambda_41932305e351933ebe8f8be3ed8bb5dc>@@@Z@4HA 0000000180020314     libucrt:per_thread_data.obj
 0003:00001314       $pdata$?fin$0@?0???$?RV<lambda_99476a1ad63dd22509b5d3e65b0ffc95>@@AEAV<lambda_ad1ced32f4ac17aa236e5ef05d6b3b7c>@@V<lambda_f7424dd8d45958661754dc4f2697e9c3>@@@?$__crt_seh_guarded_call@X@@QEAAX$$QEAV<lambda_99476a1ad63dd22509b5d3e65b0ffc95>@@AEAV<lambda_ad1ced32f4ac17aa236e5ef05d6b3b7c>@@$$QEAV<lambda_f7424dd8d45958661754dc4f2697e9c3>@@@Z@4HA 0000000180020314     libucrt:mbctype.obj
 0003:00001314       $pdata$?fin$0@?0???$?RV<lambda_5e887d1dcbef67a5eb4283622ba103bf>@@AEAV<lambda_4466841279450cc726390878d4a41900>@@V<lambda_341c25c0346d94847f1f3c463c57e077>@@@?$__crt_seh_guarded_call@X@@QEAAX$$QEAV<lambda_5e887d1dcbef67a5eb4283622ba103bf>@@AEAV<lambda_4466841279450cc726390878d4a41900>@@$$QEAV<lambda_341c25c0346d94847f1f3c463c57e077>@@@Z@4HA 0000000180020314     libucrt:per_thread_data.obj
 0003:00001314       $pdata$?fin$0@?0???$?RV<lambda_fb3a7dec4e47f37f22dae91bb15c9095>@@AEAV<lambda_698284760c8add0bfb0756c19673e34b>@@V<lambda_dfb8eca1e75fef3034a8fb18dd509707>@@@?$__crt_seh_guarded_call@X@@QEAAX$$QEAV<lambda_fb3a7dec4e47f37f22dae91bb15c9095>@@AEAV<lambda_698284760c8add0bfb0756c19673e34b>@@$$QEAV<lambda_dfb8eca1e75fef3034a8fb18dd509707>@@@Z@4HA 0000000180020314     libucrt:per_thread_data.obj
 0003:00001314       $pdata$?fin$0@?0???$?RV<lambda_b8c45f8f788dd370798f47cfe8ac3a86>@@AEAV<lambda_4e60a939b0d047cfe11ddc22648dfba9>@@V<lambda_332c3edc96d0294ec56c57d38c1cdfd5>@@@?$__crt_seh_guarded_call@H@@QEAAH$$QEAV<lambda_b8c45f8f788dd370798f47cfe8ac3a86>@@AEAV<lambda_4e60a939b0d047cfe11ddc22648dfba9>@@$$QEAV<lambda_332c3edc96d0294ec56c57d38c1cdfd5>@@@Z@4HA 0000000180020314     libucrt:onexit.obj
 0003:00001314       $pdata$?fin$0@?0???$?RV<lambda_c36588078e9f5dfd39652860aa6b3aaf>@@AEAV<lambda_ec61778202f4f5fc7e7711acc23c3bca>@@V<lambda_dc9d2797ccde5d239b4a0efae8ebd7db>@@@?$__crt_seh_guarded_call@P6AXH@Z@@QEAAP6AXH@Z$$QEAV<lambda_c36588078e9f5dfd39652860aa6b3aaf>@@AEAV<lambda_ec61778202f4f5fc7e7711acc23c3bca>@@$$QEAV<lambda_dc9d2797ccde5d239b4a0efae8ebd7db>@@@Z@4HA 0000000180020314     libucrt:signal.obj
 0003:00001314       $pdata$?fin$0@?0???$?RV<lambda_46352004c1216016012b18bd6f87e700>@@AEAV<lambda_3bd07e1a1191394380780325891bf33f>@@V<lambda_334532d3f185bcaa59b5be82d7d22bff>@@@?$__crt_seh_guarded_call@X@@QEAAX$$QEAV<lambda_46352004c1216016012b18bd6f87e700>@@AEAV<lambda_3bd07e1a1191394380780325891bf33f>@@$$QEAV<lambda_334532d3f185bcaa59b5be82d7d22bff>@@@Z@4HA 0000000180020314     libucrt:per_thread_data.obj
 0003:00001320       $pdata$__acrt_update_thread_multibyte_data$fin$0 0000000180020320     libucrt:mbctype.obj
 0003:0000132c       $pdata$raise$fin$0         000000018002032c     libucrt:signal.obj
 0003:00001338       $pdata$__acrt_uninitialize_locale$fin$0 0000000180020338     libucrt:wsetlocale.obj
 0003:00001338       $pdata$__acrt_update_thread_locale_data$fin$0 0000000180020338     libucrt:locale_refcounting.obj
 0003:00001344       $pdata$__acrt_initialize_lowio$fin$0 0000000180020344     libucrt:ioinit.obj
 0003:00001344       $pdata$__acrt_lowio_ensure_fh_exists$fin$0 0000000180020344     libucrt:osfinfo.obj
 0003:00001350       $pdata$common_flush_all$fin$0 0000000180020350     libucrt:fflush.obj
 0003:0000135c       $pdata$common_flush_all$fin$1 000000018002035c     libucrt:fflush.obj
 0003:00001368       $pdata$_fcloseall$fin$0    0000000180020368     libucrt:closeall.obj
 0003:00001374       $pdata$_write$fin$0        0000000180020374     libucrt:write.obj
 0003:00001380       $pdata$fclose$fin$0        0000000180020380     libucrt:fclose.obj
 0003:0000138c       $pdata$?fin$0@?0???$?RV<lambda_bfedae4ebbf01fab1bb6dcc6a9e276e0>@@AEAV<lambda_2fe9b910cf3cbf4a0ab98a02ba45b3ec>@@V<lambda_237c231691f317818eb88cc1d5d642d6>@@@?$__crt_seh_guarded_call@H@@QEAAH$$QEAV<lambda_bfedae4ebbf01fab1bb6dcc6a9e276e0>@@AEAV<lambda_2fe9b910cf3cbf4a0ab98a02ba45b3ec>@@$$QEAV<lambda_237c231691f317818eb88cc1d5d642d6>@@@Z@4HA 000000018002038c     libucrt:close.obj
 0003:0000138c       $pdata$?fin$0@?0???$?RV<lambda_b521505b218e5242e90febf6bfebc422>@@AEAV<lambda_6978c1fb23f02e42e1d9e99668cc68aa>@@V<lambda_314360699dd331753a4119843814e9a7>@@@?$__crt_seh_guarded_call@H@@QEAAH$$QEAV<lambda_b521505b218e5242e90febf6bfebc422>@@AEAV<lambda_6978c1fb23f02e42e1d9e99668cc68aa>@@$$QEAV<lambda_314360699dd331753a4119843814e9a7>@@@Z@4HA 000000018002038c     libucrt:commit.obj
 0003:00001398       $pdata$_ctrlfp$filt$0      0000000180020398     libucrt:fpctrl.obj
 0003:000013a4       $pdata$_IsNonwritableInCurrentImage$filt$0 00000001800203a4     LIBCMT:pesect.obj
 0004:00000976       .idata$6                   0000000180021976     kernel32:KERNEL32.dll
 0004:00000aec       .idata$6                   0000000180021aec     user32:USER32.dll
 0004:00000b2c       .idata$6                   0000000180021b2c     shell32:SHELL32.dll
 0004:00000b6c       .idata$6                   0000000180021b6c     ole32:ole32.dll
 0004:0000105c       .idata$6                   000000018002205c     advapi32:ADVAPI32.dll
 0005:00000000       __guard_fids__             0000000180023000     libucrt:initialization.obj
 0005:00000060       __guard_fids___acrt_initialize_ptd 0000000180023060     libucrt:per_thread_data.obj
 0005:00000064       __guard_fids_??$expand_argument_wildcards@D@@YAHQEAD0AEAV?$argument_list@D@?A0xca0879c4@@@Z 0000000180023064     libucrt:argv_wildcards.obj
 0005:00000068       __guard_fids__             0000000180023068     libucrt:multibyte_initializer.obj
 0005:0000006c       __guard_fids__             000000018002306c     libucrt:stdio_initializer.obj
 0005:00000070       __guard_fids__             0000000180023070     libucrt:stdio_initializer.obj
 0005:00000074       __guard_fids__             0000000180023074     libucrt:locale_initializer.obj
 0005:00000078       __guard_fids__             0000000180023078     libucrt:fma3_initializer.obj
 0005:0000007c       __guard_fids__             000000018002307c     libucrt:console_output_initializer.obj
 0005:00000080       __guard_fids_?dllmain_crt_process_attach@@YAHQEAUHINSTANCE__@@QEAX@Z 0000000180023080     LIBCMT:dll_dllmain.obj
 0005:00000088       __guard_fids_?dllmain_dispatch@@YAHQEAUHINSTANCE__@@KQEAX@Z 0000000180023088     LIBCMT:dll_dllmain.obj
 0005:0000008c       __guard_fids__             000000018002308c     LIBCMT:throw_bad_alloc.obj
 0005:00000094       __guard_fids__             0000000180023094     LIBCMT:throw_bad_alloc.obj
 0005:0000009c       __guard_fids__             000000018002309c     LIBCMT:throw_bad_alloc.obj
 0005:000000a4       __guard_fids__             00000001800230a4     LIBCMT:std_type_info_static.obj
 0005:000000a8       __guard_fids__             00000001800230a8     LIBCMT:guard_support.obj
 0005:000000ac       __guard_fids__             00000001800230ac     comsuppw:comsupp.obj
 0005:000000b0       __guard_fids__             00000001800230b0     comsuppw:comraise.obj
 0005:000000b4       __guard_fids__             00000001800230b4     libvcruntime:telemetry.obj
 0005:000000b8       __guard_fids_?TraceLoggingRegister@__vcrt_trace_logging_provider@@YAJPEBU_TlgProvider_t@1@PEBU_GUID@@P6AX1KE_K2PEAU_EVENT_FILTER_DESCRIPTOR@@PEAX@Z4@Z 00000001800230b8     libvcruntime:telemetry.obj
 0005:000000bc       __guard_fids___vcrt_initialize_ptd 00000001800230bc     libvcruntime:per_thread_data.obj
 0006:000000a0       $R000000                   00000001800240a0     EMenu.res
 0006:00000408       $R000368                   0000000180024408     EMenu.res
